Microchip Technology Inc, vš_

Tool Name:
  c:\program files (x86)\microchip\xc16\v1.20\bin\bin\..\bin/elf-ld.exe

Command:
  -p24EP512GU810 \
  -o \
  dist/XC16-EX16_MRF24WB/production/MPLAB.X.production.elf \
  -Lc:/program files (x86)/microchip/xc16/v1.20/bin/bin/.. \
  -Lc:/program files (x86)/microchip/xc16/v1.20/bin/bin/../../lib \
  -Lc:/program files (x86)/microchip/xc16/v1.20/bin/bin/../../lib/PIC24E \
  -Lc:/program files (x86)/microchip/xc16/v1.20/bin/bin/../../support/PIC24E/gld \
  -Lc:/program files (x86)/microchip/xc16/v1.20/bin/bin/../../lib/PIC24F \
  -Lc:/program files (x86)/microchip/xc16/v1.20/bin/bin/../../support/PIC24F/gld \
  -Lc:/program files (x86)/microchip/xc16/v1.20/bin/bin/../../lib/PIC24H \
  -Lc:/program files (x86)/microchip/xc16/v1.20/bin/bin/../../support/PIC24H/gld \
  -Lc:/program files (x86)/microchip/xc16/v1.20/bin/bin/../../lib/dsPIC30F \
  -Lc:/program files (x86)/microchip/xc16/v1.20/bin/bin/../../support/dsPIC30F/gld \
  -Lc:/program files (x86)/microchip/xc16/v1.20/bin/bin/../../lib/dsPIC33E \
  -Lc:/program files (x86)/microchip/xc16/v1.20/bin/bin/../../support/dsPIC33E/gld \
  -Lc:/program files (x86)/microchip/xc16/v1.20/bin/bin/../../lib/dsPIC33F \
  -Lc:/program files (x86)/microchip/xc16/v1.20/bin/bin/../../support/dsPIC33F/gld \
  build/XC16-EX16_MRF24WB/production/_ext/1954962658/ARP.o \
  build/XC16-EX16_MRF24WB/production/_ext/1954962658/Announce.o \
  build/XC16-EX16_MRF24WB/production/_ext/1954962658/AutoIP.o \
  build/XC16-EX16_MRF24WB/production/_ext/1954962658/BerkeleyAPI.o \
  build/XC16-EX16_MRF24WB/production/_ext/1954962658/DHCP.o \
  build/XC16-EX16_MRF24WB/production/_ext/1954962658/DHCPs.o \
  build/XC16-EX16_MRF24WB/production/_ext/1954962658/DNS.o \
  build/XC16-EX16_MRF24WB/production/_ext/1954962658/DNSs.o \
  build/XC16-EX16_MRF24WB/production/_ext/1954962658/Delay.o \
  build/XC16-EX16_MRF24WB/production/_ext/1954962658/DynDNS.o \
  build/XC16-EX16_MRF24WB/production/_ext/1954962658/ENC28J60.o \
  build/XC16-EX16_MRF24WB/production/_ext/1954962658/ENCX24J600.o \
  build/XC16-EX16_MRF24WB/production/_ext/1954962658/FTP.o \
  build/XC16-EX16_MRF24WB/production/_ext/1954962658/Hashes.o \
  build/XC16-EX16_MRF24WB/production/_ext/1954962658/Helpers.o \
  build/XC16-EX16_MRF24WB/production/_ext/1954962658/ICMP.o \
  build/XC16-EX16_MRF24WB/production/_ext/1954962658/IP.o \
  build/XC16-EX16_MRF24WB/production/_ext/1954962658/LCDBlocking.o \
  build/XC16-EX16_MRF24WB/production/_ext/1954962658/NBNS.o \
  build/XC16-EX16_MRF24WB/production/_ext/1954962658/Reboot.o \
  build/XC16-EX16_MRF24WB/production/_ext/1954962658/SMTP.o \
  build/XC16-EX16_MRF24WB/production/_ext/1954962658/SNMP.o \
  build/XC16-EX16_MRF24WB/production/_ext/1954962658/SNTP.o \
  build/XC16-EX16_MRF24WB/production/_ext/1954962658/SPIEEPROM.o \
  build/XC16-EX16_MRF24WB/production/_ext/1954962658/SPIFlash.o \
  build/XC16-EX16_MRF24WB/production/_ext/1954962658/SPIRAM.o \
  build/XC16-EX16_MRF24WB/production/_ext/1954962658/StackTsk.o \
  build/XC16-EX16_MRF24WB/production/_ext/1954962658/TCP.o \
  build/XC16-EX16_MRF24WB/production/_ext/1954962658/TCPPerformanceTest.o \
  build/XC16-EX16_MRF24WB/production/_ext/1954962658/TFTPc.o \
  build/XC16-EX16_MRF24WB/production/_ext/1954962658/Telnet.o \
  build/XC16-EX16_MRF24WB/production/_ext/1954962658/Tick.o \
  build/XC16-EX16_MRF24WB/production/_ext/1954962658/UART.o \
  build/XC16-EX16_MRF24WB/production/_ext/1954962658/UART2TCPBridge.o \
  build/XC16-EX16_MRF24WB/production/_ext/1954962658/UDP.o \
  build/XC16-EX16_MRF24WB/production/_ext/1954962658/UDPPerformanceTest.o \
  build/XC16-EX16_MRF24WB/production/_ext/1954962658/ZeroconfHelper.o \
  build/XC16-EX16_MRF24WB/production/_ext/1954962658/ZeroconfLinkLocal.o \
  build/XC16-EX16_MRF24WB/production/_ext/1954962658/ZeroconfMulticastDNS.o \
  build/XC16-EX16_MRF24WB/production/_ext/243675038/WFConnectionAlgorithm.o \
  build/XC16-EX16_MRF24WB/production/_ext/243675038/WFConnectionManager.o \
  build/XC16-EX16_MRF24WB/production/_ext/243675038/WFConnectionProfile.o \
  build/XC16-EX16_MRF24WB/production/_ext/243675038/WFConsole.o \
  build/XC16-EX16_MRF24WB/production/_ext/243675038/WFConsoleIfconfig.o \
  build/XC16-EX16_MRF24WB/production/_ext/243675038/WFConsoleIwconfig.o \
  build/XC16-EX16_MRF24WB/production/_ext/243675038/WFConsoleIwpriv.o \
  build/XC16-EX16_MRF24WB/production/_ext/243675038/WFConsoleMsgHandler.o \
  build/XC16-EX16_MRF24WB/production/_ext/243675038/WFConsoleMsgs.o \
  build/XC16-EX16_MRF24WB/production/_ext/243675038/WFDataTxRx.o \
  build/XC16-EX16_MRF24WB/production/_ext/243675038/WFDriverCom.o \
  build/XC16-EX16_MRF24WB/production/_ext/243675038/WFDriverRaw.o \
  build/XC16-EX16_MRF24WB/production/_ext/243675038/WFEasyConfig.o \
  build/XC16-EX16_MRF24WB/production/_ext/243675038/WFEventHandler.o \
  build/XC16-EX16_MRF24WB/production/_ext/243675038/WFInit.o \
  build/XC16-EX16_MRF24WB/production/_ext/243675038/WFMac.o \
  build/XC16-EX16_MRF24WB/production/_ext/243675038/WFMgmtMsg.o \
  build/XC16-EX16_MRF24WB/production/_ext/243675038/WFParamMsg.o \
  build/XC16-EX16_MRF24WB/production/_ext/243675038/WFPowerSave.o \
  build/XC16-EX16_MRF24WB/production/_ext/243675038/WFScan.o \
  build/XC16-EX16_MRF24WB/production/_ext/243675038/WFTxPower.o \
  build/XC16-EX16_MRF24WB/production/_ext/243675038/WF_Eint.o \
  build/XC16-EX16_MRF24WB/production/_ext/243675038/WF_Spi.o \
  build/XC16-EX16_MRF24WB/production/_ext/243675038/WFDebugStrings.o \
  build/XC16-EX16_MRF24WB/production/_ext/243675038/WF_pbkdf2.o \
  build/XC16-EX16_MRF24WB/production/_ext/1472/UARTConfig.o \
  build/XC16-EX16_MRF24WB/production/_ext/1472/WF_Config.o \
  build/XC16-EX16_MRF24WB/production/_ext/1472/HTTP2.o \
  build/XC16-EX16_MRF24WB/production/_ext/1472/MPFS2.o \
  build/XC16-EX16_MRF24WB/production/_ext/1472/WiSteerHTTP.o \
  build/XC16-EX16_MRF24WB/production/_ext/1472/WiSteerMain.o \
  build/XC16-EX16_MRF24WB/production/_ext/1472/WiSteerHTTPtools.o \
  build/XC16-EX16_MRF24WB/production/_ext/1472/WiSteerUpdate.o \
  build/XC16-EX16_MRF24WB/production/WiSteerUpdateHlp.o \
  build/XC16-EX16_MRF24WB/production/_ext/1472/WiSteerLog.o \
  build/XC16-EX16_MRF24WB/production/_ext/1472/WiSteerTime.o \
  build/XC16-EX16_MRF24WB/production/_ext/1472/WiSteerCom.o \
  build/XC16-EX16_MRF24WB/production/_ext/1472/WiSteerAction.o \
  build/XC16-EX16_MRF24WB/production/_ext/1472/WiSteerMpfsSource.o \
  build/XC16-EX16_MRF24WB/production/_ext/1472/WiSteerStructSizeCheck.o \
  build/XC16-EX16_MRF24WB/production/_ext/1472/pic32helpers.o \
  --local-stack \
  --defsym=__MPLAB_BUILD=1 \
  -Tp24EP512GU810.gld.00 \
  --heap=1000 \
  --no-check-sections \
  --data-init \
  --pack-data \
  --handles \
  --isr \
  --no-gc-sections \
  --fill-upper=0 \
  --stackguard=16 \
  --library-path=.. \
  --no-force-link \
  --smart-io \
  -Map=.map \
  --report-mem \
  -start-group \
  --library=fx-elf \
  --library=pic30-elf \
  --library=m-elf \
  --library=c-elf \
  -end-group \

Archive member included because of file (symbol)

c:/program files (x86)/microchip/xc16/v1.20/bin/bin/../../lib\libpic30-elf.a(crt0_extendedep.o)
                              (__resetPRI)
c:/program files (x86)/microchip/xc16/v1.20/bin/bin/../../lib\libpic30-elf.a(data_init_extendedep.o)
                              c:/program files (x86)/microchip/xc16/v1.20/bin/bin/../../lib\libpic30-elf.a(crt0_extendedep.o) (__data_init_extended)
c:/program files (x86)/microchip/xc16/v1.20/bin/bin/../../lib\libm-elf.a(divsi3.epeo)
                              build/XC16-EX16_MRF24WB/production/_ext/1472/WiSteerHTTP.o (___divsi3)
c:/program files (x86)/microchip/xc16/v1.20/bin/bin/../../lib\libm-elf.a(modsi3.epeo)
                              build/XC16-EX16_MRF24WB/production/_ext/1472/WiSteerHTTP.o (___modsi3)
c:/program files (x86)/microchip/xc16/v1.20/bin/bin/../../lib\libm-elf.a(udivsi3.epeo)
                              build/XC16-EX16_MRF24WB/production/_ext/1472/MPFS2.o (___udivsi3)
c:/program files (x86)/microchip/xc16/v1.20/bin/bin/../../lib\libm-elf.a(umodsi3.epeo)
                              build/XC16-EX16_MRF24WB/production/_ext/1472/WiSteerHTTP.o (___umodsi3)
c:/program files (x86)/microchip/xc16/v1.20/bin/bin/../../lib\libm-elf.a(divmoddi3.epeo)
                              build/XC16-EX16_MRF24WB/production/_ext/1954962658/Tick.o (___udivdi3)
c:/program files (x86)/microchip/xc16/v1.20/bin/bin/../../lib\libm-elf.a(muldi3.epeo)
                              build/XC16-EX16_MRF24WB/production/_ext/1472/WiSteerTime.o (___muldi3)
c:/program files (x86)/microchip/xc16/v1.20/bin/bin/../../lib\libm-elf.a(umuldi3.epeo)
                              c:/program files (x86)/microchip/xc16/v1.20/bin/bin/../../lib\libm-elf.a(muldi3.epeo) (___umuldi3)
c:/program files (x86)/microchip/xc16/v1.20/bin/bin/../../lib\libc-elf.a(atof.epeo)
                              build/XC16-EX16_MRF24WB/production/_ext/1472/WiSteerHTTP.o (_strtod)
c:/program files (x86)/microchip/xc16/v1.20/bin/bin/../../lib\libc-elf.a(atoi.epeo)
                              build/XC16-EX16_MRF24WB/production/_ext/1472/WiSteerHTTP.o (_atoi)
c:/program files (x86)/microchip/xc16/v1.20/bin/bin/../../lib\libc-elf.a(atol.epeo)
                              build/XC16-EX16_MRF24WB/production/_ext/1472/HTTP2.o (_atol)
c:/program files (x86)/microchip/xc16/v1.20/bin/bin/../../lib\libc-elf.a(errno.epeo)
                              c:/program files (x86)/microchip/xc16/v1.20/bin/bin/../../lib\libc-elf.a(atof.epeo) (_errno)
c:/program files (x86)/microchip/xc16/v1.20/bin/bin/../../lib\libc-elf.a(ltoa.epeo)
                              build/XC16-EX16_MRF24WB/production/_ext/1472/WiSteerHTTP.o (_ultoa)
c:/program files (x86)/microchip/xc16/v1.20/bin/bin/../../lib\libc-elf.a(memcmp.epeo)
                              build/XC16-EX16_MRF24WB/production/_ext/1954962658/NBNS.o (_memcmp)
c:/program files (x86)/microchip/xc16/v1.20/bin/bin/../../lib\libc-elf.a(memcpy.epeo)
                              build/XC16-EX16_MRF24WB/production/_ext/1954962658/ARP.o (_memcpy)
c:/program files (x86)/microchip/xc16/v1.20/bin/bin/../../lib\libc-elf.a(memmove.epeo)
                              build/XC16-EX16_MRF24WB/production/_ext/1472/HTTP2.o (_memmove)
c:/program files (x86)/microchip/xc16/v1.20/bin/bin/../../lib\libc-elf.a(memset.epeo)
                              build/XC16-EX16_MRF24WB/production/_ext/1954962658/DHCP.o (_memset)
c:/program files (x86)/microchip/xc16/v1.20/bin/bin/../../lib\libc-elf.a(strchr.epeo)
                              build/XC16-EX16_MRF24WB/production/_ext/1472/WiSteerTime.o (_strchr)
c:/program files (x86)/microchip/xc16/v1.20/bin/bin/../../lib\libc-elf.a(strcmp.epeo)
                              build/XC16-EX16_MRF24WB/production/_ext/1472/HTTP2.o (_strcmp)
c:/program files (x86)/microchip/xc16/v1.20/bin/bin/../../lib\libc-elf.a(strcpy.epeo)
                              build/XC16-EX16_MRF24WB/production/_ext/1472/WiSteerHTTP.o (_strcpy)
c:/program files (x86)/microchip/xc16/v1.20/bin/bin/../../lib\libc-elf.a(strlen.epeo)
                              build/XC16-EX16_MRF24WB/production/_ext/1954962658/DHCP.o (_strlen)
c:/program files (x86)/microchip/xc16/v1.20/bin/bin/../../lib\libc-elf.a(strncmp.epeo)
                              build/XC16-EX16_MRF24WB/production/_ext/1472/WiSteerHTTP.o (_strncmp)
c:/program files (x86)/microchip/xc16/v1.20/bin/bin/../../lib\libc-elf.a(strncpy.epeo)
                              build/XC16-EX16_MRF24WB/production/_ext/1954962658/Helpers.o (_strncpy)
c:/program files (x86)/microchip/xc16/v1.20/bin/bin/../../lib\libc-elf.a(strtol.epeo)
                              build/XC16-EX16_MRF24WB/production/_ext/1472/WiSteerHTTP.o (_strtoul)
c:/program files (x86)/microchip/xc16/v1.20/bin/bin/../../lib\libc-elf.a(vsnprintf.epeo)
                              build/XC16-EX16_MRF24WB/production/_ext/1472/WiSteerHTTPtools.o (_vsnprintf)
c:/program files (x86)/microchip/xc16/v1.20/bin/bin/../../lib\libc-elf.a(snprintf_cdnopuxX.EPeo)
                              build/XC16-EX16_MRF24WB/production/_ext/243675038/WFDebugStrings.o (__snprintf_cdnopuxX)
c:/program files (x86)/microchip/xc16/v1.20/bin/bin/../../lib\libc-elf.a(vsnprintf_cdnopuxX.EPeo)
                              c:/program files (x86)/microchip/xc16/v1.20/bin/bin/../../lib\libc-elf.a(snprintf_cdnopuxX.EPeo) (__vsnprintf_cdnopuxX)
c:/program files (x86)/microchip/xc16/v1.20/bin/bin/../../lib\libc-elf.a(snprintf_cdfFnopuxX.EPeo)
                              build/XC16-EX16_MRF24WB/production/_ext/1472/WiSteerHTTP.o (__snprintf_cdfFnopuxX)
c:/program files (x86)/microchip/xc16/v1.20/bin/bin/../../lib\libc-elf.a(vsnprintf_cdfFnopuxX.EPeo)
                              c:/program files (x86)/microchip/xc16/v1.20/bin/bin/../../lib\libc-elf.a(snprintf_cdfFnopuxX.EPeo) (__vsnprintf_cdfFnopuxX)
c:/program files (x86)/microchip/xc16/v1.20/bin/bin/../../lib\libc-elf.a(snprintf_cdfFnopsuxX.EPeo)
                              (__snprintf_cdfFnopsuxX)
c:/program files (x86)/microchip/xc16/v1.20/bin/bin/../../lib\libc-elf.a(vsnprintf_cdfFnopsuxX.EPeo)
                              c:/program files (x86)/microchip/xc16/v1.20/bin/bin/../../lib\libc-elf.a(snprintf_cdfFnopsuxX.EPeo) (__vsnprintf_cdfFnopsuxX)
c:/program files (x86)/microchip/xc16/v1.20/bin/bin/../../lib\libc-elf.a(snprintf_cdnopsuxX.EPeo)
                              build/XC16-EX16_MRF24WB/production/_ext/1472/WiSteerTime.o (__snprintf_cdnopsuxX)
c:/program files (x86)/microchip/xc16/v1.20/bin/bin/../../lib\libc-elf.a(vsnprintf_cdnopsuxX.EPeo)
                              c:/program files (x86)/microchip/xc16/v1.20/bin/bin/../../lib\libc-elf.a(snprintf_cdnopsuxX.EPeo) (__vsnprintf_cdnopsuxX)
c:/program files (x86)/microchip/xc16/v1.20/bin/bin/../../lib\libc-elf.a(isalpha.epeso)
                              c:/program files (x86)/microchip/xc16/v1.20/bin/bin/../../lib\libc-elf.a(strtol.epeo) (_isalpha)
c:/program files (x86)/microchip/xc16/v1.20/bin/bin/../../lib\libc-elf.a(isspace.epeso)
                              c:/program files (x86)/microchip/xc16/v1.20/bin/bin/../../lib\libc-elf.a(atof.epeo) (_isspace)
c:/program files (x86)/microchip/xc16/v1.20/bin/bin/../../lib\libc-elf.a(isxdigit.epeso)
                              build/XC16-EX16_MRF24WB/production/_ext/243675038/WFConsoleMsgs.o (_isxdigit)
c:/program files (x86)/microchip/xc16/v1.20/bin/bin/../../lib\libc-elf.a(toupper.epeso)
                              c:/program files (x86)/microchip/xc16/v1.20/bin/bin/../../lib\libc-elf.a(strtol.epeo) (_toupper)
c:/program files (x86)/microchip/xc16/v1.20/bin/bin/../../lib\libc-elf.a(doprnt.epeo)
                              c:/program files (x86)/microchip/xc16/v1.20/bin/bin/../../lib\libc-elf.a(vsnprintf.epeo) (_vfprintf)
c:/program files (x86)/microchip/xc16/v1.20/bin/bin/../../lib\libc-elf.a(fputc.epeo)
                              c:/program files (x86)/microchip/xc16/v1.20/bin/bin/../../lib\libc-elf.a(doprnt.epeo) (_fputc)
c:/program files (x86)/microchip/xc16/v1.20/bin/bin/../../lib\libc-elf.a(powers.epeo)
                              c:/program files (x86)/microchip/xc16/v1.20/bin/bin/../../lib\libc-elf.a(doprnt.epeo) (__powers_)
c:/program files (x86)/microchip/xc16/v1.20/bin/bin/../../lib\libc-elf.a(_iob.epeo)
                              c:/program files (x86)/microchip/xc16/v1.20/bin/bin/../../lib\libc-elf.a(fputc.epeo) (__outdone)
c:/program files (x86)/microchip/xc16/v1.20/bin/bin/../../lib\libc-elf.a(doprnt_cdnopuxX.EPeo)
                              c:/program files (x86)/microchip/xc16/v1.20/bin/bin/../../lib\libc-elf.a(vsnprintf_cdnopuxX.EPeo) (__vfprintf_cdnopuxX)
c:/program files (x86)/microchip/xc16/v1.20/bin/bin/../../lib\libc-elf.a(doprnt_cdfFnopuxX.EPeo)
                              c:/program files (x86)/microchip/xc16/v1.20/bin/bin/../../lib\libc-elf.a(vsnprintf_cdfFnopuxX.EPeo) (__vfprintf_cdfFnopuxX)
c:/program files (x86)/microchip/xc16/v1.20/bin/bin/../../lib\libc-elf.a(doprnt_cdfFnopsuxX.EPeo)
                              c:/program files (x86)/microchip/xc16/v1.20/bin/bin/../../lib\libc-elf.a(vsnprintf_cdfFnopsuxX.EPeo) (__vfprintf_cdfFnopsuxX)
c:/program files (x86)/microchip/xc16/v1.20/bin/bin/../../lib\libc-elf.a(doprnt_cdnopsuxX.EPeo)
                              c:/program files (x86)/microchip/xc16/v1.20/bin/bin/../../lib\libc-elf.a(vsnprintf_cdnopsuxX.EPeo) (__vfprintf_cdnopsuxX)
c:/program files (x86)/microchip/xc16/v1.20/bin/bin/../../lib\libc-elf.a(flsbuf.epeo)
                              c:/program files (x86)/microchip/xc16/v1.20/bin/bin/../../lib\libc-elf.a(fputc.epeo) (__flsbuf)
c:/program files (x86)/microchip/xc16/v1.20/bin/bin/../../lib\libpic30-elf.a(writeep.eo)
                              c:/program files (x86)/microchip/xc16/v1.20/bin/bin/../../lib\libc-elf.a(fputc.epeo) (_write)
c:/program files (x86)/microchip/xc16/v1.20/bin/bin/../../lib\libpic30-elf.a(c30_uartep.eo)
                              c:/program files (x86)/microchip/xc16/v1.20/bin/bin/../../lib\libpic30-elf.a(writeep.eo) (___C30_UART)
c:/program files (x86)/microchip/xc16/v1.20/bin/bin/../../lib\libm-elf.a(adddf3.epeo)
                              c:/program files (x86)/microchip/xc16/v1.20/bin/bin/../../lib\libc-elf.a(doprnt.epeo) (___adddf3)
c:/program files (x86)/microchip/xc16/v1.20/bin/bin/../../lib\libm-elf.a(deqltle.epeo)
                              c:/program files (x86)/microchip/xc16/v1.20/bin/bin/../../lib\libc-elf.a(doprnt.epeo) (___ltdf2)
c:/program files (x86)/microchip/xc16/v1.20/bin/bin/../../lib\libm-elf.a(dgtge.epeo)
                              c:/program files (x86)/microchip/xc16/v1.20/bin/bin/../../lib\libc-elf.a(doprnt.epeo) (___gedf2)
c:/program files (x86)/microchip/xc16/v1.20/bin/bin/../../lib\libm-elf.a(divdf3.epeo)
                              c:/program files (x86)/microchip/xc16/v1.20/bin/bin/../../lib\libc-elf.a(doprnt.epeo) (___divdf3)
c:/program files (x86)/microchip/xc16/v1.20/bin/bin/../../lib\libm-elf.a(divsf3.epeo)
                              c:/program files (x86)/microchip/xc16/v1.20/bin/bin/../../lib\libc-elf.a(atof.epeo) (___divsf3)
c:/program files (x86)/microchip/xc16/v1.20/bin/bin/../../lib\libm-elf.a(dne.epeo)
                              c:/program files (x86)/microchip/xc16/v1.20/bin/bin/../../lib\libc-elf.a(doprnt.epeo) (___nedf2)
c:/program files (x86)/microchip/xc16/v1.20/bin/bin/../../lib\libm-elf.a(dpack.epeo)
                              c:/program files (x86)/microchip/xc16/v1.20/bin/bin/../../lib\libm-elf.a(adddf3.epeo) (__dpack)
c:/program files (x86)/microchip/xc16/v1.20/bin/bin/../../lib\libm-elf.a(dunpack2.epeo)
                              c:/program files (x86)/microchip/xc16/v1.20/bin/bin/../../lib\libm-elf.a(adddf3.epeo) (__dunpack2)
c:/program files (x86)/microchip/xc16/v1.20/bin/bin/../../lib\libm-elf.a(extendsfdf.epeo)
                              c:/program files (x86)/microchip/xc16/v1.20/bin/bin/../../lib\libc-elf.a(doprnt.epeo) (___extendsfdf2)
c:/program files (x86)/microchip/xc16/v1.20/bin/bin/../../lib\libm-elf.a(feqltle.epeo)
                              c:/program files (x86)/microchip/xc16/v1.20/bin/bin/../../lib\libc-elf.a(atof.epeo) (___eqsf2)
c:/program files (x86)/microchip/xc16/v1.20/bin/bin/../../lib\libm-elf.a(fgtge.epeo)
                              c:/program files (x86)/microchip/xc16/v1.20/bin/bin/../../lib\libc-elf.a(atof.epeo) (___gtsf2)
c:/program files (x86)/microchip/xc16/v1.20/bin/bin/../../lib\libm-elf.a(fixunsdfdi.epeo)
                              c:/program files (x86)/microchip/xc16/v1.20/bin/bin/../../lib\libc-elf.a(doprnt.epeo) (___fixunsdfdi)
c:/program files (x86)/microchip/xc16/v1.20/bin/bin/../../lib\libm-elf.a(fixunsdfsi.epeo)
                              c:/program files (x86)/microchip/xc16/v1.20/bin/bin/../../lib\libc-elf.a(doprnt.epeo) (___fixunsdfsi)
c:/program files (x86)/microchip/xc16/v1.20/bin/bin/../../lib\libm-elf.a(floatsisf.epeo)
                              c:/program files (x86)/microchip/xc16/v1.20/bin/bin/../../lib\libc-elf.a(atof.epeo) (___floatsisf)
c:/program files (x86)/microchip/xc16/v1.20/bin/bin/../../lib\libm-elf.a(floatundidf.epeo)
                              c:/program files (x86)/microchip/xc16/v1.20/bin/bin/../../lib\libc-elf.a(doprnt.epeo) (___floatundidf)
c:/program files (x86)/microchip/xc16/v1.20/bin/bin/../../lib\libm-elf.a(floatunsidf.epeo)
                              c:/program files (x86)/microchip/xc16/v1.20/bin/bin/../../lib\libc-elf.a(doprnt.epeo) (___floatunsidf)
c:/program files (x86)/microchip/xc16/v1.20/bin/bin/../../lib\libm-elf.a(fpack.epeo)
                              c:/program files (x86)/microchip/xc16/v1.20/bin/bin/../../lib\libm-elf.a(divsf3.epeo) (__fpack)
c:/program files (x86)/microchip/xc16/v1.20/bin/bin/../../lib\libm-elf.a(frexpf.epeo)
                              c:/program files (x86)/microchip/xc16/v1.20/bin/bin/../../lib\libc-elf.a(doprnt.epeo) (_frexpf)
c:/program files (x86)/microchip/xc16/v1.20/bin/bin/../../lib\libm-elf.a(funpack.epeo)
                              c:/program files (x86)/microchip/xc16/v1.20/bin/bin/../../lib\libm-elf.a(extendsfdf.epeo) (__funpack)
c:/program files (x86)/microchip/xc16/v1.20/bin/bin/../../lib\libm-elf.a(funpack2.epeo)
                              c:/program files (x86)/microchip/xc16/v1.20/bin/bin/../../lib\libm-elf.a(divsf3.epeo) (__funpack2)
c:/program files (x86)/microchip/xc16/v1.20/bin/bin/../../lib\libm-elf.a(futil.epeo)
                              c:/program files (x86)/microchip/xc16/v1.20/bin/bin/../../lib\libm-elf.a(divsf3.epeo) (__fPropagateNaN)
c:/program files (x86)/microchip/xc16/v1.20/bin/bin/../../lib\libm-elf.a(muldf3.epeo)
                              c:/program files (x86)/microchip/xc16/v1.20/bin/bin/../../lib\libc-elf.a(doprnt.epeo) (___muldf3)
c:/program files (x86)/microchip/xc16/v1.20/bin/bin/../../lib\libm-elf.a(mulsf3.epeo)
                              c:/program files (x86)/microchip/xc16/v1.20/bin/bin/../../lib\libc-elf.a(atof.epeo) (___mulsf3)
c:/program files (x86)/microchip/xc16/v1.20/bin/bin/../../lib\libm-elf.a(subdf3.epeo)
                              c:/program files (x86)/microchip/xc16/v1.20/bin/bin/../../lib\libc-elf.a(doprnt.epeo) (___subdf3)
c:/program files (x86)/microchip/xc16/v1.20/bin/bin/../../lib\libm-elf.a(truncdfsf.epeo)
                              c:/program files (x86)/microchip/xc16/v1.20/bin/bin/../../lib\libc-elf.a(doprnt.epeo) (___truncdfsf2)
c:/program files (x86)/microchip/xc16/v1.20/bin/bin/../../lib\libm-elf.a(mulsi3.epeo)
                              c:/program files (x86)/microchip/xc16/v1.20/bin/bin/../../lib\libc-elf.a(atof.epeo) (___mulsi3)
c:/program files (x86)/microchip/xc16/v1.20/bin/bin/../../lib\libm-elf.a(_frexpf.epeo)
                              c:/program files (x86)/microchip/xc16/v1.20/bin/bin/../../lib\libm-elf.a(frexpf.epeo) (__frexpf)
c:/program files (x86)/microchip/xc16/v1.20/bin/bin/../../lib\libm-elf.a(dcompare.epeo)
                              c:/program files (x86)/microchip/xc16/v1.20/bin/bin/../../lib\libm-elf.a(deqltle.epeo) (__dcompare)
c:/program files (x86)/microchip/xc16/v1.20/bin/bin/../../lib\libm-elf.a(dpropagateNaN.epeo)
                              c:/program files (x86)/microchip/xc16/v1.20/bin/bin/../../lib\libm-elf.a(dunpack2.epeo) (__dPropagateNaN)
c:/program files (x86)/microchip/xc16/v1.20/bin/bin/../../lib\libm-elf.a(dtype.epeo)
                              c:/program files (x86)/microchip/xc16/v1.20/bin/bin/../../lib\libm-elf.a(dcompare.epeo) (__dtype)
c:/program files (x86)/microchip/xc16/v1.20/bin/bin/../../lib\libm-elf.a(dunpack.epeo)
                              c:/program files (x86)/microchip/xc16/v1.20/bin/bin/../../lib\libm-elf.a(dunpack2.epeo) (__dunpack)
c:/program files (x86)/microchip/xc16/v1.20/bin/bin/../../lib\libm-elf.a(fcompare.epeo)
                              c:/program files (x86)/microchip/xc16/v1.20/bin/bin/../../lib\libm-elf.a(feqltle.epeo) (__fcompare)
c:/program files (x86)/microchip/xc16/v1.20/bin/bin/../../lib\libm-elf.a(floatdisf.epeo)
                              c:/program files (x86)/microchip/xc16/v1.20/bin/bin/../../lib\libm-elf.a(floatsisf.epeo) (___floatdisf)
c:/program files (x86)/microchip/xc16/v1.20/bin/bin/../../lib\libm-elf.a(floatundisf.epeo)
                              c:/program files (x86)/microchip/xc16/v1.20/bin/bin/../../lib\libm-elf.a(floatdisf.epeo) (___floatundisf)


Program Memory  [Origin = 0x200, Length = 0x555fe]

section                    address   length (PC units)   length (bytes) (dec)
-------                    -------   -----------------   --------------------
.text                        0x200              0x4bde          0x71cd  (29133)
.const                      0x4dde              0x2a12          0x3f1b  (16155)
MPFSData                    0x77f0             0x1c98e         0x2ae55  (175701)
.text                      0x2417e             0x1e694         0x2d9de  (186846)
.dinit                     0x42812               0x452           0x67b  (1659)
.text                      0x42c64              0x3bd4          0x59be  (22974)
MPFSHelpers                0x46838                 0xe            0x15  (21)
.text                      0x46846                 0x6             0x9  (9)

                     Total program memory used (bytes):        0x69972  (432498) 82%


Auxflash Memory  [Origin = 0x7fc000, Length = 0x3ff8]

section                    address   length (PC units)   length (bytes) (dec)
-------                    -------   -----------------   --------------------

                     Total auxflash memory used (bytes):              0  (0) <1%


Data Memory  [Origin = 0x1000, Length = 0xd000]

section                    address      alignment gaps    total length  (dec)
-------                    -------      --------------    -------------------
.bss                        0x1000                   0          0x4c78  (19576)
.data._powers_              0x5c78                   0           0x160  (352)
.bss                        0x5dd8                   0           0x31a  (794)
.data.dpowers               0x60f2                   0           0x140  (320)
.bss                        0x6232                   0           0x184  (388)
.data                       0x63b6                   0            0x6a  (106)
.bss                        0x6420                   0            0xe0  (224)
.data                       0x6500                   0            0x54  (84)
.bss                        0x6554                   0            0x26  (38)
.data._iob                  0x657a                   0            0x26  (38)
.bss                        0x65a0                   0            0x22  (34)
.data                       0x65c2                   0            0x1c  (28)
.bss                        0x65de                   0            0x56  (86)
.data                       0x6634                   0            0x10  (16)
.bss                        0x6644                   0            0x1c  (28)
.data                       0x6660                   0            0x2a  (42)
.bss                        0x668a                   0             0x8  (8)
.data                       0x6692                   0             0xc  (12)
_04F3B4805461348c           0x669e                   0             0x6  (6)
.bss                        0x66a4                   0            0x12  (18)
.data                       0x66b6                   0             0x8  (8)
.bss                        0x66be                   0             0x8  (8)
.data                       0x66c6                   0             0xe  (14)
.pbss                       0x66d4                   0             0x2  (2)
.data                       0x66d6                   0             0x6  (6)
.pbss                       0x66dc                   0             0x2  (2)
.data                       0x66de                   0             0x2  (2)
.pbss                       0x66e0                   0             0x2  (2)
.data                       0x66e2                   0             0x2  (2)
.bss                        0x66e4                   0             0x2  (2)
.data                       0x66e6                   0             0xa  (10)
.bss                        0x66f0                   0             0x2  (2)
.data.__C30_UART            0x66f2                   0             0x2  (2)
.heap                       0x66f4                   0           0x3e8  (1000)

                        Total data memory used (bytes):         0x5adc  (23260) 43%


Dynamic Memory Usage

region                     address                      maximum length  (dec)
------                     -------                      ---------------------
heap                        0x66f4                               0x3e8  (1000)
stack                       0x6adc                              0x1524  (5412)

                        Maximum dynamic memory (bytes):         0x190c  (6412)


External Symbols in Data Memory (by address):

                    0x1000                  _AppConfig
                    0x10aa                  _WiSteerCfg
                    0x1ff8                  _WiSteerLog
                    0x2ff8                  _WiSteerCfgTmp
                    0x38f4                  _ConnectionProfileID
                    0x38fa                  _HTTPControlBlocks
                    0x496a                  _httpStubs
                    0x497a                  _curHTTPID
                    0x4d7e                  _g_ScanCtx
                    0x4d84                  _g_easyConfigCtx
                    0x4e14                  _preScanResult
                    0x54e4                  _logStubs
                    0x5968                  _httpPageId
                    0x59a8                  _httpTimeScan
                    0x59d8                  _httpCatEnum
                    0x59dc                  _httpCatMainEnum
                    0x59f4                  _httpCfgCatEnum
                    0x59fc                  _httpIOpinEnum
                    0x5a00                  _httpCmdOutEnum
                    0x5a04                  _httpCfgCmdEnum
                    0x5a34                  _httpCfgIOenum
                    0x5a3c                  _httpCfgFormId
                    0x5a6c                  _httpActEnum
                    0x5a70                  _httpDevEnum
                    0x5a74                  _httpBtnEnum
                    0x5a80                  _g_tiIO
                    0x5ab0                  _g_tiIOmax
                    0x5ae0                  _g_tiIOoff
                    0x5b10                  _g_tiIOoffMax
                    0x5b40                  _g_inputState
                    0x5c30                  _g_catReqCtx
                    0x5c38                  _bufAskerLabel
                    0x5c78                  __powers_
                    0x5d28                  __npowers_
                    0x5dd8                  _UDPSocketInfo
                    0x5ef8                  _activeUDPSocket
                    0x5efa                  _UDPTxCount
                    0x5efc                  _UDPRxCount
                    0x600a                  _wsLastHostRecv
                    0x601e                  _g_discoveryMsg
                    0x60e2                  _wiSteerAuthMd5
                    0x634c                  _DhcpIpPool
                    0x63b6                  __connectionFailureStrings
                    0x63e0                  __connectionLostStrings
                    0x63ee                  __moduleName
                    0x6462                  _lastBlock
                    0x657a                  __iob
                    0x659e                  __Files
                    0x65a0                  _LCDText
                    0x65c2                  _g_actRunningRemoteOrPin
                    0x65c4                  _g_actRunningTick
                    0x65c8                  _g_actToSet
                    0x65cc                  _g_actToUnset
                    0x65d0                  _g_catReqTi
                    0x65d4                  _g_catReqTiMax
                    0x65d8                  _g_inputDefined
                    0x65da                  _g_outputAutoOff
                    0x65dc                  _g_inputToWatch
                    0x6620                  _g_rxIndexSetBeyondBuffer
                    0x6630                  _RawMoveState
                    0x6634                  _g_logStarted
                    0x6636                  _m_cLogAppend
                    0x6638                  _m_logStartId
                    0x663c                  _m_cLogChanged
                    0x6640                  _g_wslogCheckPt
                    0x6654                  _remoteNode
                    0x6660                  _g_wisteerBoostMode
                    0x6662                  _g_tiNow
                    0x6666                  _g_deviceWithOpIdx
                    0x6668                  _g_cfgShareSourceDevId
                    0x666a                  _g_cfgShareSourceDate
                    0x6672                  _g_wiSteerCom_opOrder
                    0x6674                  _g_wiSteerCom_opOrderLast
                    0x6676                  _g_wiSteerAuthMd5Ok
                    0x6678                  _g_wiSteerComReqToDo
                    0x667a                  _g_DhcpSuccessful
                    0x667c                  _g_WiFiConnectionChanged
                    0x667e                  _g_WiFiConnection
                    0x6680                  _g_dhcpInProgress
                    0x6682                  _g_prescan_adhoc_done
                    0x6684                  _g_tickConnectError
                    0x6688                  _g_bWifiConnectOk
                    0x668a                  _g_httpTooMuchData
                    0x6694                  _bDHCPServerEnabled
                    0x6698                  _g_DhcpRenew
                    0x669a                  _g_DhcpRetryTimer
                    0x669e                  _vTickReading
                    0x66a4                  _RawWindowReady
                    0x66a8                  _RawWindowState
                    0x66b0                  __outdone
                    0x66b1                  __sibuf
                    0x66b3                  __sobuf
                    0x66c6                  _dwInternalTicks
                    0x66ca                  _mpfsLastSeek
                    0x66ce                  _g_timeOffset
                    0x66d2                  _DHCPClientInitializedOnce
                    0x66e6                  _g_HostRAWDataPacketReceived
                    0x66e8                  _preScanResult_Count
                    0x66ea                  _gRFModuleVer1209orLater
                    0x66ec                  _g_WaitingForMgmtResponse
                    0x66f0                  _errno
                    0x66f2                  ___C30_UART

External Symbols in Data Memory (by name):

                    0x1000                  _AppConfig
                    0x38f4                  _ConnectionProfileID
                    0x66d2                  _DHCPClientInitializedOnce
                    0x634c                  _DhcpIpPool
                    0x38fa                  _HTTPControlBlocks
                    0x65a0                  _LCDText
                    0x6630                  _RawMoveState
                    0x66a4                  _RawWindowReady
                    0x66a8                  _RawWindowState
                    0x5efc                  _UDPRxCount
                    0x5dd8                  _UDPSocketInfo
                    0x5efa                  _UDPTxCount
                    0x10aa                  _WiSteerCfg
                    0x2ff8                  _WiSteerCfgTmp
                    0x1ff8                  _WiSteerLog
                    0x659e                  __Files
                    0x66f2                  ___C30_UART
                    0x63b6                  __connectionFailureStrings
                    0x63e0                  __connectionLostStrings
                    0x657a                  __iob
                    0x63ee                  __moduleName
                    0x5d28                  __npowers_
                    0x66b0                  __outdone
                    0x5c78                  __powers_
                    0x66b1                  __sibuf
                    0x66b3                  __sobuf
                    0x5ef8                  _activeUDPSocket
                    0x6694                  _bDHCPServerEnabled
                    0x5c38                  _bufAskerLabel
                    0x497a                  _curHTTPID
                    0x66c6                  _dwInternalTicks
                    0x66f0                  _errno
                    0x66ea                  _gRFModuleVer1209orLater
                    0x6698                  _g_DhcpRenew
                    0x669a                  _g_DhcpRetryTimer
                    0x667a                  _g_DhcpSuccessful
                    0x66e6                  _g_HostRAWDataPacketReceived
                    0x4d7e                  _g_ScanCtx
                    0x66ec                  _g_WaitingForMgmtResponse
                    0x667e                  _g_WiFiConnection
                    0x667c                  _g_WiFiConnectionChanged
                    0x65c2                  _g_actRunningRemoteOrPin
                    0x65c4                  _g_actRunningTick
                    0x65c8                  _g_actToSet
                    0x65cc                  _g_actToUnset
                    0x6688                  _g_bWifiConnectOk
                    0x5c30                  _g_catReqCtx
                    0x65d0                  _g_catReqTi
                    0x65d4                  _g_catReqTiMax
                    0x666a                  _g_cfgShareSourceDate
                    0x6668                  _g_cfgShareSourceDevId
                    0x6666                  _g_deviceWithOpIdx
                    0x6680                  _g_dhcpInProgress
                    0x601e                  _g_discoveryMsg
                    0x4d84                  _g_easyConfigCtx
                    0x668a                  _g_httpTooMuchData
                    0x65d8                  _g_inputDefined
                    0x5b40                  _g_inputState
                    0x65dc                  _g_inputToWatch
                    0x6634                  _g_logStarted
                    0x65da                  _g_outputAutoOff
                    0x6682                  _g_prescan_adhoc_done
                    0x6620                  _g_rxIndexSetBeyondBuffer
                    0x5a80                  _g_tiIO
                    0x5ab0                  _g_tiIOmax
                    0x5ae0                  _g_tiIOoff
                    0x5b10                  _g_tiIOoffMax
                    0x6662                  _g_tiNow
                    0x6684                  _g_tickConnectError
                    0x66ce                  _g_timeOffset
                    0x6676                  _g_wiSteerAuthMd5Ok
                    0x6678                  _g_wiSteerComReqToDo
                    0x6672                  _g_wiSteerCom_opOrder
                    0x6674                  _g_wiSteerCom_opOrderLast
                    0x6660                  _g_wisteerBoostMode
                    0x6640                  _g_wslogCheckPt
                    0x5a6c                  _httpActEnum
                    0x5a74                  _httpBtnEnum
                    0x59d8                  _httpCatEnum
                    0x59dc                  _httpCatMainEnum
                    0x59f4                  _httpCfgCatEnum
                    0x5a04                  _httpCfgCmdEnum
                    0x5a3c                  _httpCfgFormId
                    0x5a34                  _httpCfgIOenum
                    0x5a00                  _httpCmdOutEnum
                    0x5a70                  _httpDevEnum
                    0x59fc                  _httpIOpinEnum
                    0x5968                  _httpPageId
                    0x496a                  _httpStubs
                    0x59a8                  _httpTimeScan
                    0x6462                  _lastBlock
                    0x54e4                  _logStubs
                    0x6636                  _m_cLogAppend
                    0x663c                  _m_cLogChanged
                    0x6638                  _m_logStartId
                    0x66ca                  _mpfsLastSeek
                    0x4e14                  _preScanResult
                    0x66e8                  _preScanResult_Count
                    0x6654                  _remoteNode
                    0x669e                  _vTickReading
                    0x60e2                  _wiSteerAuthMd5
                    0x600a                  _wsLastHostRecv

External Symbols in Program Memory (by address):

                  0x000200                  __resetPRI
                  0x000226                  __psv_init
                  0x000232                  __data_init
                  0x000232                  __data_init_extended
                  0x0002d8                  __DefaultInterrupt
                  0x000302                  __OscillatorFail
                  0x00032c                  __AddressError
                  0x000356                  __StackError
                  0x000380                  __MathError
                  0x0003aa                  _main
                  0x000640                  _WF_Connect
                  0x000756                  _DisplayIPValue
                  0x0008d4                  _DefaultAppConfig
                  0x000a06                  _LoadAppConfig
                  0x000b7e                  _UpgradeAppConfig
                  0x000bf0                  _AppConfigUseWiFiMacAddress
                  0x000dda                  _SaveAppConfig
                  0x000e52                  _RestoreWifiConfig
                  0x000e86                  _LED_PUT
                  0x000f64                  _activityLedsOn
                  0x000f9a                  _activityLedsModeChange
                  0x000fbe                  _OnMdnsHostNameChanged
                  0x000fc6                  _deviceReinit
                  0x00102e                  _deviceGet
                  0x001100                  _deviceFind
                  0x00117c                  _deviceWithOpToDoGet
                  0x001264                  _deviceIsGoodCfgShareSource
                  0x001334                  _deviceGoodCfgShareSourceEnd
                  0x001362                  _deviceId
                  0x001380                  _deviceCmdAdd
                  0x001430                  _deviceCmdEnd
                  0x0014c4                  _speedBoostStart
                  0x00158e                  _speedBoostValidate
                  0x0015f0                  _speedBoostKeep
                  0x00165a                  _speedBoostKeepLow
                  0x0016c2                  _speedBoostReset
                  0x0016c8                  _isalpha
                  0x0016dc                  _isspace
                  0x0016ec                  _isxdigit
                  0x001708                  _toupper
                  0x001716                  ___divsi3
                  0x001734                  ___modsi3
                  0x001752                  ___udivsi3
                  0x001772                  ___umodsi3
                  0x0017e6                  ___udivmoddi3
                  0x0018b6                  ___udivdi3
                  0x0018c8                  ___umoddi3
                  0x0018d4                  ___divdi3
                  0x001938                  ___moddi3
                  0x001998                  ___muldi3
                  0x0019ee                  ___umuldi3
                  0x001a32                  _strtod
                  0x001c04                  _atof
                  0x001c0e                  _atoi
                  0x001c50                  _atol
                  0x001caa                  _ultoa
                  0x001cfa                  _ltoa
                  0x001d1e                  _memcmp
                  0x001d4c                  _memcpy
                  0x001d5e                  _memmove
                  0x001d84                  _memset
                  0x001d96                  _strchr
                  0x001dae                  _strcmp
                  0x001dc0                  _strcpy
                  0x001dd0                  _strlen
                  0x001de2                  _strncmp
                  0x001e08                  _strncpy
                  0x001e2e                  _strtoul
                  0x001f42                  _strtol
                  0x001fce                  _vsnprintf
                  0x001ff8                  __snprintf_cdnopuxX
                  0x001ff8                  __snprintf_cdfFnopsuxX
                  0x001ff8                  __snprintf_cdfFnopuxX
                  0x001ff8                  __snprintf_cdnopsuxX
                  0x002004                  __vsnprintf_cdfFnopuxX
                  0x002004                  __vsnprintf_cdfFnopsuxX
                  0x002004                  __vsnprintf_cdnopuxX
                  0x002004                  __vsnprintf_cdnopsuxX
                  0x00218e                  _vfprintf
                  0x00383e                  __vfprintf_cdnopsuxX
                  0x00383e                  __vfprintf_cdfFnopuxX
                  0x00383e                  __vfprintf_cdnopuxX
                  0x00383e                  __vfprintf_cdfFnopsuxX
                  0x00459e                  ___adddf3
                  0x004698                  ___ltdf2
                  0x004698                  ___eqdf2
                  0x004698                  ___ledf2
                  0x0046a2                  ___gtdf2
                  0x0046a2                  ___gedf2
                  0x0046ac                  ___divdf3
                  0x004760                  ___divsf3
                  0x0047e4                  ___nedf2
                  0x0047ee                  __dpack
                  0x004846                  __dunpack2
                  0x004868                  __dreturnNaN
                  0x00486e                  __dunpack2exit
                  0x004878                  ___extendsfdf2
                  0x0048b6                  ___eqsf2
                  0x0048b6                  ___lesf2
                  0x0048b6                  ___ltsf2
                  0x0048ba                  ___gesf2
                  0x0048ba                  ___gtsf2
                  0x0048be                  ___fixunsdfdi
                  0x004920                  ___fixunsdfsi
                  0x00496c                  ___floatsisf
                  0x004972                  ___floatundidf
                  0x0049c8                  ___floatunsidf
                  0x0049cc                  __fpack
                  0x004a18                  _frexpf
                  0x004a1e                  __funpack
                  0x004a48                  __funpack2
                  0x004a58                  __fPropagateNaN
                  0x004a6a                  __fbopExit
                  0x004a72                  __fbopReturnNaN
                  0x004a78                  ___muldf3
                  0x004b62                  ___mulsf3
                  0x004bca                  ___subdf3
                  0x004bce                  ___truncdfsf2
                  0x004c24                  ___mulp32peds3
                  0x004c24                  ___mulsi3
                  0x004c24                  ___mulp32eds3
                  0x004c30                  __frexpf
                  0x004c4a                  __dcompare
                  0x004c9c                  __dPropagateNaN
                  0x004cb8                  __dtype
                  0x004cdc                  __dunpack
                  0x004d2a                  __fcompare
                  0x004d60                  ___floatdisf
                  0x004d80                  ___floatundisf
                  0x0058ba                  _c_formInput_nochg
                  0x0058bb                  _c_formInput_post
                  0x006151                  _HTML_UP_ARROW
                  0x006154                  _HTML_DOWN_ARROW
                  0x0062e2                  _http2m_ContentTypes
                  0x006f14                  _wstime_weekDay
                  0x006f78                  _wstime_month
                  0x007642                  _helpCmd
                  0x007647                  _helpHelp
                  0x00765a                  _getwfverCmd
                  0x007663                  _getwfverHelp
                  0x00767c                  _resetCmd
                  0x007682                  _resetHelp
                  0x007691                  _clsCmd
                  0x007695                  _clsHelp
                  0x0076a3                  _seeDocHelp
                  0x0076b5                  _pingCmd
                  0x0076ba                  _pingHelp
                  0x0076cc                  _g_consoleCmd
                  0x0076ea                  _g_numCmds
                  0x0077ba                  _TCPSocketInitializer
                  0x0077ec                  _MPFS_Start
                  0x0077f4                  BEGIN_MPFS
                  0x02417e                  _HTTPNeedsAuth
                  0x02420e                  _HTTPCheckAuth
                  0x024244                  _HTTPPrint_postWifiConfig
                  0x0245da                  _HTTPPrint_postTcpIpConfig
                  0x0249ac                  _HTTPPrint_builddate
                  0x0249b8                  _HTTPPrint_tcpipVersion
                  0x0249c4                  _HTTPPrint_version
                  0x0249fe                  _HTTPPrint_led
                  0x024aa2                  _HTTPPrint_ledSelected
                  0x024b54                  _HTTPPrint_temp
                  0x024bec                  _HTTPPrint_pot
                  0x024c64                  _HTTPPrint_zcross
                  0x024c6a                  _HTTPQueryIf_zcrossOk
                  0x024c74                  _HTTPQueryIf_zcrossNotOk
                  0x024c7e                  _HTTPPrint_time
                  0x024cb0                  _HTTPPrint_timeBoot
                  0x024ce0                  _HTTPPrintIP
                  0x024d46                  _HTTPPrint_host
                  0x024d64                  _HTTPPrint_config_hostname
                  0x024d82                  _HTTPPrint_config_netbiosname
                  0x024da0                  _HTTPPrint_config_dhcpchecked
                  0x024dca                  _HTTPPrint_config_ip
                  0x024df8                  _HTTPPrint_config_gw
                  0x024e26                  _HTTPPrint_config_subnet
                  0x024e54                  _HTTPPrint_config_dns1
                  0x024e82                  _HTTPPrint_config_dns2
                  0x024eb0                  _HTTPPrint_config_mac
                  0x024f84                  _HTTPPrint_reboot
                  0x024f9c                  _HTTPPrint_rebootaddr
                  0x024fca                  _HTTPPrint_status_ok
                  0x025010                  _HTTPPrint_status_fail
                  0x025056                  _HTTPPrint_fwver
                  0x0250a8                  _HTTPPrint_ssid
                  0x0250da                  _HTTPPrint_nextSSID
                  0x0250f8                  _HTTPPrint_prevSSID
                  0x025116                  _getWlanStr
                  0x02513e                  _HTTPPrint_prevWLAN
                  0x025168                  _HTTPPrint_nextWLAN
                  0x025192                  _HTTPPrint_label
                  0x0251b0                  _HTTPQueryIf_wifiConfigured
                  0x0251be                  _HTTPQueryIf_devConfigured
                  0x02521e                  _HTTPQueryIf_wifiAndDevConfigured
                  0x025236                  _HTTPQueryIf_wifiNotConfigured
                  0x02524c                  _HTTPQueryIf_devNotConfigured
                  0x025260                  _HTTPQueryIf_logToGet
                  0x02527c                  _HTTPQueryIf_actionToGet
                  0x025298                  _HTTPQueryIf_actionToReload
                  0x0252ca                  _HTTPQueryWhile_logEnum
                  0x0253f8                  _HTTPPrint_logID
                  0x02543a                  _HTTPPrint_logTime
                  0x02547a                  _HTTPPrint_logLevel
                  0x0254b8                  _HTTPPrint_logDetails
                  0x0254de                  _HTTPPrint_actionsPost
                  0x02553e                  _HTTPPrint_actionsPostLed
                  0x025690                  _HTTPPrint_actionsPostCmd
                  0x0257d2                  _HTTPPrint_actionsPostInfo
                  0x025876                  _HTTPPrint_wifiScanPost
                  0x0259ce                  _HTTPPrint_wifiScanInProgress
                  0x025a34                  _HTTPPrint_bssCount
                  0x025a70                  _HTTPPrint_bssValid
                  0x025a9a                  _HTTPPrint_bssName
                  0x025aca                  _HTTPPrint_bssPrivacy
                  0x025b10                  _HTTPPrint_bssWlan
                  0x025b46                  _HTTPPrint_bssStrength
                  0x025b7c                  _HTTPQueryIf_pageIdIs
                  0x025ba4                  _HTTPQueryIf_pageIdIsNot
                  0x025bcc                  _HTTPPrint_pageId
                  0x025c06                  _HTTPPrint_wifiPowerMax
                  0x025c46                  _HTTPPrint_wifiFactoryPowerMax
                  0x025c82                  _HTTPPrint_postWifiPowerMax
                  0x025cf4                  _HTTPPrint_timeScanStartLow
                  0x025e4c                  _HTTPPrint_timeScanStart
                  0x025eac                  _HTTPPrint_timeDay
                  0x025eea                  _HTTPPrint_timeMonth
                  0x025f28                  _HTTPPrint_timeYear
                  0x025f64                  _HTTPPrint_timeHour
                  0x025fa2                  _HTTPPrint_timeMin
                  0x025fe0                  _HTTPPrint_timeSec
                  0x02601e                  _HTTPPrint_timeZoneId
                  0x026070                  _HTTPPrint_timeBias
                  0x0260ac                  _HTTPQueryIf_cfg_timeDlON
                  0x0260ee                  _HTTPPrint_timeDltWeekDayNo
                  0x026136                  _HTTPPrint_timeDltWeekDay
                  0x02617e                  _HTTPPrint_timeDltMonth
                  0x0261c6                  _HTTPPrint_timeDltHour
                  0x02620e                  _HTTPPrint_timeDltMin
                  0x026256                  _HTTPPrint_timeDltSec
                  0x02629e                  _HTTPPrint_timeDltBias
                  0x0262da                  _HTTPPrint_timeSdtWeekDayNo
                  0x026322                  _HTTPPrint_timeSdtWeekDay
                  0x02636a                  _HTTPPrint_timeSdtMonth
                  0x0263b2                  _HTTPPrint_timeSdtHour
                  0x0263fa                  _HTTPPrint_timeSdtMin
                  0x026442                  _HTTPPrint_timeSdtSec
                  0x02648a                  _HTTPPrint_timeSdtBias
                  0x0264c6                  _HTTPQueryWhile_catEnum
                  0x02652a                  _HTTPPrint_catEnumId
                  0x026566                  _HTTPPrint_catEnumLabel
                  0x02658e                  _HTTPPrint_cfg_label
                  0x0265b4                  _HTTPQueryIf_cfg_debugON
                  0x026638                  _HTTPQueryIf_cfg_testON
                  0x0266bc                  _MPFStestMode
                  0x026710                  _HTTPQueryIf_testON
                  0x026764                  _HTTPQueryIf_cfg_haltfON
                  0x0267e8                  _HTTPQueryIf_cfg_activityLedON
                  0x02686c                  _HTTPQueryIf_cfg_protectAllON
                  0x0268f0                  _HTTPQueryIf_cfg_homeActivityPanelON
                  0x026974                  _HTTPQueryIf_homeActivityPanelON
                  0x0269c8                  _HTTPQueryIf_cfg_boostModeON
                  0x026a4c                  _HTTPQueryIf_boostModeON
                  0x026aa0                  _HTTPQueryIf_cfg_wisteerNetBrowseON
                  0x026b24                  _HTTPQueryIf_cfg_wisteerAutoUpdateON
                  0x026b2e                  _HTTPQueryIf_cfg_mpfsUploadON
                  0x026b38                  _HTTPPrint_cfg_login
                  0x026b5e                  _HTTPPrint_cfg_pwd1
                  0x026b64                  _HTTPPrint_cfg_pwd2
                  0x026b6a                  _HTTPQueryIf_category_available
                  0x026b7c                  _HTTPQueryIf_cfg_timeServerSyncON
                  0x026c00                  _HTTPPrint_cfg_timeServer
                  0x026c26                  _HTTPPrint_cfg_catCountVal
                  0x026c62                  _HTTPPrint_cfg_catCount
                  0x026c8e                  _HTTPPrint_cfg_catCountMax
                  0x026cb4                  _HTTPPrint_cfg_catMainCatId
                  0x026d44                  _HTTPQueryWhile_cfg_catMainEnum
                  0x026dee                  _HTTPPrint_cfg_catMainEnumId
                  0x026e2c                  _HTTPPrint_cfg_catMainEnumNo
                  0x026e6c                  _HTTPPrint_cfg_catMainEnumExc
                  0x026f28                  _HTTPQueryWhile_cfg_catEnum
                  0x026f72                  _HTTPPrint_cfg_catEnumId
                  0x026fb2                  _HTTPPrint_cfg_catEnumLabel
                  0x027012                  _HTTPQueryWhile_ioPinEnum
                  0x0270b4                  _HTTPPrint_ioPinEnumId
                  0x0270f0                  _HTTPPrint_ioPinEnumLabel
                  0x02711a                  _HTTPPrint_ioPinEnumType
                  0x027182                  _HTTPQueryWhile_cmdOutEnum
                  0x0271ec                  _HTTPPrint_cmdOutEnumId
                  0x027228                  _HTTPPrint_cmdOutEnumLabel
                  0x027250                  _HTTPPrint_cfg_cmdCfgCountVal
                  0x02728c                  _HTTPPrint_cfg_cmdCfgCount
                  0x0272b8                  _HTTPPrint_cfg_cmdCfgCountMax
                  0x0272de                  _HTTPQueryWhile_cfg_cmdCfgEnum
                  0x027336                  _HTTPPrint_cfg_cmdCfgEnumId
                  0x027376                  _HTTPPrint_cfg_cmdCfgEnumLabel
                  0x027412                  _HTTPPrint_cfg_cmdCfgEnumPrior
                  0x027504                  _HTTPPrint_cfg_cmdCfgEnumImg
                  0x0275d8                  _HTTPPrint_cfg_cmdCfgEnumPin1s
                  0x0276ac                  _HTTPPrint_cfg_cmdCfgEnumPin0s
                  0x027780                  _HTTPPrint_cfg_cmdCfgEnumPinRs
                  0x027854                  _HTTPPrint_cfg_cmdCfgEnumCatId
                  0x027918                  _HTTPQueryWhile_cfg_cmdCfgEnumCatEnum
                  0x0279e6                  _HTTPPrint_cfg_cmdCfgEnumCatEnumId
                  0x027a42                  _HTTPPrint_cfg_cmdCfgEnumCatEnumNo
                  0x027a82                  _HTTPPrint_cfg_cmdCfgEnumCatEnumExc
                  0x027b46                  _HTTPPrint_cfg_cmdCfgEnumTypeVal
                  0x027c0e                  _HTTPPrint_cfg_cmdCfgEnumType
                  0x027c62                  _HTTPQueryIf_cfg_cmdCfgEnumTypeIs
                  0x027c7e                  _HTTPPrint_cfg_cmdCfgEnumPin
                  0x027d52                  _HTTPPrint_cfg_cmdCfgEnumIOtypeVal
                  0x027e3e                  _HTTPPrint_cfg_cmdCfgEnumIOtype
                  0x027e92                  _HTTPQueryIf_cfg_cmdCfgEnumIOtypeIs
                  0x027eae                  _HTTPPrint_cfg_cmdCfgEnumRact
                  0x027fa0                  _HTTPPrint_cfg_cmdCfgEnumPulse
                  0x028092                  _HTTPPrint_cfg_cmdCfgEnumTimeNext
                  0x028178                  _HTTPPrint_cfg_cmdCfgEnumTimeOff
                  0x02825e                  _HTTPPrint_cfg_cmdCfgEnumAct
                  0x028350                  _HTTPPrint_cfg_cmdCfgEnumAskTypeVal
                  0x028412                  _HTTPPrint_cfg_cmdCfgEnumAskType
                  0x028466                  _HTTPPrint_cfg_ioCountVal
                  0x0284a2                  _HTTPPrint_cfg_ioCount
                  0x0284ce                  _HTTPPrint_cfg_ioCountMax
                  0x0284f4                  _HTTPQueryWhile_cfg_ioEnum
                  0x02853e                  _HTTPPrint_cfg_ioEnumId
                  0x02857e                  _HTTPPrint_cfg_ioEnumLabel
                  0x0285e0                  _HTTPPrint_cfg_ioEnumTypeVal
                  0x028662                  _HTTPPrint_cfg_ioEnumType
                  0x028696                  _HTTPPrint_postDevIOconfig
                  0x0287fa                  _HTTPPrint_formFocus
                  0x02881e                  _HTTPPrint_postDevIOconfig_configMain
                  0x02951a                  _HTTPPrint_postDevIOconfig_configTime
                  0x029966                  _HTTPPrint_postDevIOconfig_configCmds
                  0x02a2ba                  _HTTPPrint_postDevIOconfig_configIOs
                  0x02a54a                  _HTTPPrint_postDevIOconfig_configCats
                  0x02a6a0                  _HTTPQueryWhile_actionEnum
                  0x02a740                  _HTTPPrint_actionEnumId
                  0x02a77c                  _HTTPPrint_actionEnumUnicId
                  0x02a7ee                  _HTTPPrint_actionEnumLabel
                  0x02a818                  _HTTPPrint_actionEnumImg
                  0x02a864                  _HTTPQueryIf_actionEnumON
                  0x02a898                  _HTTPQueryIf_actionEnumONavail
                  0x02a8ce                  _HTTPQueryIf_actionEnumRunning
                  0x02a904                  _HTTPQueryIf_actionEnumError
                  0x02a938                  _HTTPPrint_actionEnumStatus
                  0x02a9d8                  _HTTPPrint_actionEnumPriority
                  0x02aa46                  _HTTPPrint_actionEnumCats
                  0x02ab8c                  _HTTPPrint_actionEnumAskType
                  0x02abd6                  _HTTPQueryIf_formConfigured
                  0x02ac86                  _HTTPQueryIf_formExpanded
                  0x02acd6                  _HTTPQueryWhile_deviceEnum
                  0x02ad18                  _HTTPPrint_deviceID
                  0x02ad40                  _HTTPPrint_deviceLabel
                  0x02ad66                  _HTTPPrint_deviceMac
                  0x02add0                  _HTTPPrint_deviceIP
                  0x02ae2a                  _HTTPPrint_deviceStatus
                  0x02b156                  _HTTPPrint_deviceTime
                  0x02b1ca                  _HTTPPrint_deviceSentTime
                  0x02b23e                  _HTTPPrint_deviceFWver
                  0x02b29c                  _HTTPPrint_deviceMpfsDate
                  0x02b2e6                  _HTTPPrint_deviceBootDate
                  0x02b330                  _HTTPQueryIf_deviceLinked
                  0x02b342                  _HTTPPrint_cfg_gpsLat
                  0x02b400                  _HTTPPrint_cfg_gpsLon
                  0x02b4be                  _HTTPPrint_cfg_gpsDist
                  0x02b57c                  _HTTPPrint_gpsLatitude
                  0x02b638                  _HTTPPrint_gpsLongitude
                  0x02b6f4                  _HTTPPrint_gpsDistanceMax
                  0x02b7b0                  _HTTPQueryIf_wisteerMpfsDynamic
                  0x02b7ba                  _HTTPQueryIf_wisteerMpfsUploadON
                  0x02b7c4                  _HTTPPrint_postDevIOconfig_configTools
                  0x02b848                  _HTTPPrint_mpfsdate
                  0x02b898                  _HTTPPrint_postDevLst
                  0x02b8a2                  _HTTPPrint_actionVer
                  0x02b8e6                  _HTTPPrint_categoryMax
                  0x02b91c                  _HTTPQueryIf_actionPending
                  0x02b936                  _HTTPPrint_btnResetStatus
                  0x02b966                  _HTTPQueryWhile_btnEnum
                  0x02b9da                  _HTTPPrint_btnEnumId
                  0x02ba18                  _HTTPPrint_btnEnumLabel
                  0x02ba46                  _HTTPPrint_btnEnumStatus
                  0x02baa2                  _HTTPPrint_cfg_ioEnumDimLevel
                  0x02baf6                  _HTTPQueryIf_cfg_ioEnumTypeIs
                  0x02bb10                  _HTTPPrint_cfg_ioEnumDimLevelVal
                  0x02bb96                  _hmac_sha1_vector
                  0x02bcbe                  _hmac_sha1
                  0x02bcde                  _sha1_prf
                  0x02bd82                  _sha1_t_prf
                  0x02bf28                  _pbkdf2_sha1
                  0x02bf88                  _sha1_vector
                  0x02bfd4                  _sha1_transform
                  0x0305f4                  _WiSteerCom_AnnounceIP
                  0x03067a                  _WiSteerCom_AnnounceModeToOpCode
                  0x0306a0                  _WiSteerCom_AnnounceTask
                  0x030836                  _WiSteerCom_init
                  0x03088e                  _WiSteerCom_AnnounceSend
                  0x030a20                  _WiSteerCom_DiscoveryTask
                  0x030be2                  _WiSteerCom_DiscoveryRecv
                  0x030d4c                  _WiSteerCom_DiscoveryReply
                  0x030e6e                  _WiSteerCom_AuthMd5
                  0x030ecc                  _WiSteerCom_AuthMd5Reset
                  0x030ed6                  _WiSteerCom_AnnounceProcess
                  0x031236                  _WiSteerCom_DiscoverySendTask
                  0x031492                  _WiSteerCom_DiscoverySendTaskCat
                  0x03169c                  _WiSteerCom_DiscoverySendTaskCmd
                  0x0318a0                  _WiSteerCom_RetrieveInfoSend
                  0x03192e                  _WiSteerCom_RetrieveInfoError
                  0x031986                  _WiSteerCom_RetrieveCatProcess
                  0x031a5c                  _WiSteerCom_RetrieveCmdProcess
                  0x031b60                  _WiSteerCom_deviceSource
                  0x031bee                  _WiSteerCom_RetrieveCatInfoProcess
                  0x031d28                  _WiSteerCom_RetrieveCatErrorProcess
                  0x031e42                  _WiSteerCom_RetrieveCmdInfoProcess
                  0x031fe4                  _WiSteerCom_RetrieveCmdErrorProcess
                  0x0320fe                  _WiSteerCom_actionProcessCmdCfgOutputId
                  0x032442                  _WiSteerCom_DiscoverySendTaskCmdAction
                  0x032726                  _WiSteerCom_CmdActionProcess
                  0x032888                  _WiSteerCom_CmdActionErrorSend
                  0x0328e4                  _WiSteerCom_CmdActionInfoProcess
                  0x0329e4                  _WiSteerCom_CmdActionErrorProcess
                  0x032b1a                  _WiSteerCom_CmdActionChanged
                  0x032bac                  _WiSteerCom_DiscoverySendTaskCmdChanged
                  0x032e90                  _WiSteerCom_CmdStatusProcess
                  0x033056                  _WiSteerCom_CmdLog
                  0x03317c                  _WiSteerCom_CmdStatusInfoProcess
                  0x033274                  _cmdModeRemoteRecv
                  0x0332b0                  _WiSteerCom_CatActionAsk
                  0x0333c8                  _WiSteerCom_DiscoverySendTaskCatAction
                  0x0336be                  _WiSteerCom_CatActionProcess
                  0x0337d8                  _WiSteerCom_CatActionInfoProcess
                  0x033922                  _HTTPPrint
                  0x033e9c                  _HTTPQueryIf
                  0x034122                  _HTTPQueryWhile
                  0x0341ea                  _HTTPQueryContentType
                  0x0341f6                  _HTTPInit
                  0x034274                  _HTTPServer
                  0x035c80                  _HTTPMPFS2mSendData
                  0x03615a                  _HTTPURLDecode
                  0x03622e                  _HTTPargGet
                  0x0362ce                  _HTTPargTrimGet
                  0x0363b4                  _HTTPargSet
                  0x0365c0                  _HTTPReadPostName
                  0x0365ec                  _HTTPReadPostValue
                  0x0368ce                  _HTTPIncFile
                  0x036a3e                  _CRC32_Init
                  0x036ada                  _CRC32_Push
                  0x036b50                  _CRC32_Get
                  0x036b62                  _actionPendingClear
                  0x036b8a                  _ioPinMode
                  0x036bf6                  _ioPinInitLow
                  0x036c00                  _ioPinInit
                  0x036c2c                  _cmdCfgIsValid
                  0x036cc0                  _cmdCfgDisplayIsValid
                  0x036ce6                  _cmdCfgHiddenIsValid
                  0x036d0c                  _cmdCfgOutIsValid
                  0x036d66                  _cmdCfgCatIsValid
                  0x036db4                  _actionInit
                  0x036e00                  _actionInputInit
                  0x036f24                  _actionInputReset
                  0x036f38                  _actionInputWatchAdd
                  0x036fea                  _actionInputWatch
                  0x037078                  _actionInputChanged
                  0x03710e                  _actionInputSignal
                  0x037188                  _actionInputPulse
                  0x037248                  _actionInputPulseChoose
                  0x0373bc                  _actionInputPulseProcess
                  0x037498                  _actionInputSignalProcess
                  0x03776c                  _cmdSumCalc
                  0x0378fc                  _actionSumFromCmdId
                  0x0379d2                  _actionPostCmd
                  0x037ac4                  _actionRunningRemoteUpdate
                  0x037b54                  _actionRunningTick
                  0x037b76                  _actionStatus
                  0x037be0                  _actionProcessMask
                  0x037c88                  _actionProcess
                  0x037cbe                  _actionProcessCmdSumId
                  0x037d90                  _actTypeFromInputMode
                  0x037dde                  _actTypeFromLinkMode
                  0x037e2c                  _actionProcessCmdSum
                  0x037e66                  _actionProcessCmdCfgId
                  0x03800a                  _actionProcessCmdCfgOutputId
                  0x03864a                  _actionProcessCmdCfgOutputPin
                  0x038698                  _actionProcessCmdCfgOutputPinLow
                  0x03872c                  _actionProcessCmdCfgOutputPinStatus
                  0x03878a                  __actionProcessCmdOrCatId
                  0x03880e                  _actionProcessCmdOrCatId
                  0x0388fe                  _actionAskerGet
                  0x038976                  _actionAskerFree
                  0x038a0c                  _actionAskerError
                  0x038a54                  _actionAskerLabel
                  0x038a9e                  _actionLocalInit
                  0x038aba                  _actionProcessCatId
                  0x038dc6                  _catInCatList
                  0x038df8                  _actionCatFilter
                  0x038e3c                  _actionProcessCatCom
                  0x038ede                  _actionProcessCmdCfgInputPinStatus
                  0x038f34                  _actionAutoOff
                  0x038fc4                  _actionAutoOffReset
                  0x039032                  _actionAutoOffWatch
                  0x039136                  _actionInitToOffForIO
                  0x039190                  _actionInitToOffForIOcmd
                  0x039362                  _TCPInit
                  0x039452                  _TCPOpen
                  0x0395ae                  _TCPWasReset
                  0x0395dc                  _TCPIsConnected
                  0x039600                  _TCPDisconnect
                  0x0396a0                  _TCPClose
                  0x0396c0                  _TCPGetRemoteInfo
                  0x0396ea                  _TCPFlush
                  0x039710                  _TCPIsPutReady
                  0x03975e                  _TCPPut
                  0x039804                  _TCPPutArray
                  0x0398ea                  _TCPPutString
                  0x03990e                  _TCPGetTxFIFOFull
                  0x03993a                  _TCPDiscard
                  0x03995a                  _TCPIsGetReady
                  0x039992                  _TCPGet
                  0x039a0c                  _TCPGetArray
                  0x039ad8                  _TCPGetRxFIFOFree
                  0x039b02                  _TCPPeekArray
                  0x039bac                  _TCPPeek
                  0x039bc4                  _TCPFindArrayEx
                  0x039e34                  _TCPFindEx
                  0x039e58                  _TCPTick
                  0x03a348                  _TCPProcess
                  0x03b554                  _TCPAdjustFIFOSize
                  0x03b756                  _GetTcbInfo
                  0x03b768                  _wstimeEncode
                  0x03b96e                  _wstimeDecode
                  0x03bb62                  _wstimeMonthLength
                  0x03bbe6                  _wstimeWeekDay
                  0x03bc16                  _wstimeStToStr
                  0x03bfa8                  _wstimeToStr
                  0x03bfdc                  _wstimeStr
                  0x03c00e                  _wstickStr
                  0x03c0c8                  _wstimeLowGet
                  0x03c0e2                  _wstimeSet
                  0x03c14c                  _wstimeGet
                  0x03c160                  _ntpServerPort
                  0x03c16c                  _ntpServer
                  0x03c1ca                  _ntpTimeRecv
                  0x03c214                  _tzInfoIsUtc
                  0x03c23c                  _tzInfoHasDayLight
                  0x03c25c                  _tzInfoMakeDate
                  0x03c3c0                  _wstimeStDiff
                  0x03c47c                  _tzInfoToLocalTime
                  0x03c634                  _tzInfoToUtcTime
                  0x03c73e                  _timeBiasStr
                  0x03c7ae                  _timeBiasFromStr
                  0x03c864                  _DHCPInit
                  0x03c8c0                  _DHCPDisable
                  0x03c8e4                  _DHCPEnable
                  0x03c904                  _DHCPIsEnabled
                  0x03c918                  _DHCPIsBound
                  0x03c928                  _DHCPStateChanged
                  0x03c946                  _DHCPIsServerDetected
                  0x03c958                  _DHCPTempIPAddr
                  0x03c99a                  _DHCPTask
                  0x03d4c4                  _MPFSInit
                  0x03d4f8                  _MPFSOpen
                  0x03d64e                  _MPFSOpenID
                  0x03d6d8                  _MPFSClose
                  0x03d6fe                  _MPFSGet
                  0x03d88e                  _MPFSGetArray
                  0x03dab8                  _MPFSGetLong
                  0x03dada                  _MPFSSeek
                  0x03dcec                  _MPFSGetTimestamp
                  0x03dd32                  _MPFSGetContentTypeId
                  0x03ddb8                  _MPFSGetContentType
                  0x03de14                  _MPFSGetFlags
                  0x03de58                  _MPFSGetSize
                  0x03de9e                  _MPFSGetBytesRem
                  0x03dedc                  _MPFSGetPhysAddr
                  0x03df22                  _MPFSGetStartAddr
                  0x03df6a                  _MPFSGetEndAddr
                  0x03dfbc                  _MPFSGetFilename
                  0x03e020                  _MPFSGetPosition
                  0x03e05c                  _MPFSGetID
                  0x03e0cc                  _MPFSseekInit
                  0x03e0da                  _MPFSputHdrCorrect
                  0x03e0e0                  _MPFSLocked
                  0x03e0ea                  _DHCPServerTask
                  0x03ebf8                  _DHCPServer_Disable
                  0x03ec1a                  _DHCPServer_Enable
                  0x03ee32                  _MACProcess
                  0x03ee70                  _WFGetTCBSize
                  0x03ee7a                  _MACInit
                  0x03ee84                  _RawInit
                  0x03eed6                  _MACIsLinked
                  0x03eee4                  _MACIsTxReady
                  0x03ef3a                  _WFisTxMgmtReady
                  0x03ef74                  _WFFreeMgmtTx
                  0x03efa8                  _SendRAWManagementFrame
                  0x03efb8                  _RawGetMgmtRxBuffer
                  0x03effa                  _SetRawRxMgmtInProgress
                  0x03f012                  _isRawRxMgmtInProgress
                  0x03f01c                  _MACDiscardRx
                  0x03f026                  _MACGetFreeRxSize
                  0x03f0a0                  _MACGetHeader
                  0x03f194                  _MACPutHeader
                  0x03f1ec                  _MACFlush
                  0x03f252                  _MACSetReadPtrInRx
                  0x03f264                  _MACSetWritePtr
                  0x03f27c                  _MACSetReadPtr
                  0x03f294                  _MACCalcRxChecksum
                  0x03f2c2                  _MACMemCopyAsync
                  0x03f518                  _MACIsMemCopyDone
                  0x03f522                  _MACGet
                  0x03f54e                  _MACGetArray
                  0x03f5a8                  _MACPut
                  0x03f5d6                  _MACPutArray
                  0x03f604                  _CalcIPBufferChecksum
                  0x03f696                  _MACPowerDown
                  0x03f69c                  _MACPowerUp
                  0x03f6a2                  _LFSRSeedRand
                  0x03f6e4                  _LFSRRand
                  0x03f754                  _GenerateRandomDWORD
                  0x03f85e                  _StringToIPAddress
                  0x03f9d0                  _Base64Decode
                  0x03fb38                  _uitoa
                  0x03fbc2                  _hexatob
                  0x03fc2c                  _btohexa_high
                  0x03fc4e                  _btohexa_low
                  0x03fc6c                  _stricmppgm2ram
                  0x03fd04                  _swaps
                  0x03fd20                  _swapl
                  0x03fd80                  _CalcIPChecksum
                  0x03fe02                  _strupr
                  0x03fe40                  _FormatNetBIOSName
                  0x03fe8a                  _strnchr
                  0x03fed8                  _strncpy_m
                  0x03ff56                  _DNSBeginUsage
                  0x03ff76                  _DNSEndUsage
                  0x03ffae                  _DNSResolve
                  0x03ffee                  _DNSIsResolved
                  0x0407ec                  _wslog
                  0x0409e6                  _wsvlogf
                  0x040a08                  _wslogf
                  0x040b3a                  _wslogReset
                  0x040b5a                  _wslogWrite
                  0x040f38                  _wslogEnum
                  0x040fcc                  _wslogSeekNext
                  0x04100a                  _wslogTimeAdjust
                  0x041034                  _wslogTimeAdjustRestart
                  0x041040                  _logFatalCheckPt
                  0x04105a                  _UDPInit
                  0x04107a                  _UDPOpenEx
                  0x041194                  _UDPTask
                  0x0413d4                  _UDPIsOpened
                  0x0413f6                  _UDPClose
                  0x04144e                  _UDPSetTxBuffer
                  0x041464                  _UDPSetRxBuffer
                  0x04147a                  _UDPIsPutReady
                  0x0414b0                  _UDPPut
                  0x0414e0                  _UDPPutArray
                  0x04151c                  _UDPPutString
                  0x04153a                  _UDPFlush
                  0x0415a8                  _UDPIsGetReady
                  0x0415de                  _UDPGet
                  0x041612                  _UDPGetArray
                  0x04165e                  _UDPDiscard
                  0x041684                  _UDPDiscardRxTx
                  0x041698                  _UDPProcess
                  0x041874                  _HTTPExecuteGet
                  0x04187e                  _HTTPExecutePost
                  0x0418fc                  _HTTPPrint_tooMuchData
                  0x041922                  _HTTPPrint_out
                  0x04193c                  _HTTPPrint_outLen
                  0x041a8a                  _HTTPPrint_jsEscape
                  0x041aa4                  _HTTPPrint_jsEscapeLen
                  0x041c0a                  _HTTPPrint_htmlEscape
                  0x041c24                  _HTTPPrint_htmlEscapeLen
                  0x041dfa                  _HTTPPrint_postJSf
                  0x041e18                  _HTTPPrintTry_postJSf
                  0x041e3a                  _HTTPPrint_postJS
                  0x041e66                  _HTTPPrintTry_postJS
                  0x041eee                  _HTTPPrint_postErrorField
                  0x041f06                  _HTTPPrint_postErrorFieldArg1
                  0x041f24                  _HTTPPrint_postErrorFieldArg2
                  0x041f48                  _HashAddData
                  0x041f64                  _MD5Initialize
                  0x041fa0                  _MD5AddData
                  0x042240                  _MD5Calculate
                  0x0423c0                  _WF_CASetElements
                  0x04247e                  _WF_CASetElementsN
                  0x0424b6                  _WF_CAGetElements
                  0x042502                  _WF_CASetScanType
                  0x042512                  _WF_CAGetScanType
                  0x042524                  _WF_CASetMinChannelTime
                  0x042540                  _WF_CAGetMinChannelTime
                  0x042562                  _WF_CASetMaxChannelTime
                  0x04257e                  _WF_CAGetMaxChannelTime
                  0x0425a0                  _WF_CASetProbeDelay
                  0x0425bc                  _WF_CAGetProbeDelay
                  0x0425de                  _WF_CASetScanCount
                  0x0425ee                  _WF_CAGetScanCount
                  0x042600                  _WF_CASetRssi
                  0x042610                  _WF_CAGetRssi
                  0x042622                  _WF_CASetConnectionProfileList
                  0x042632                  _WF_CAGetConnectionProfileList
                  0x042642                  _WF_CASetListRetryCount
                  0x042652                  _WF_CAGetListRetryCount
                  0x042664                  _WF_CASetEventNotificationAction
                  0x042670                  _WF_CAGetEventNotificationAction
                  0x042680                  _WF_CASetBeaconTimeoutAction
                  0x042690                  _WF_CAGetBeaconTimeoutAction
                  0x0426a2                  _WF_CASetDeauthAction
                  0x0426b2                  _WF_CAGetDeauthAction
                  0x0426c4                  _WF_CASetChannelList
                  0x0426d6                  _WF_CAGetChannelList
                  0x042712                  _WF_CASetListenInterval
                  0x04272e                  _WF_CAGetListenInterval
                  0x042750                  _WF_CASetBeaconTimeout
                  0x042760                  _WF_CAGetBeaconTimeout
                  0x04277e                  _GetEventNotificationMask
                  0x042800                  _WF_DisableModuleConnectionManager
                  0x042c64                  _WiFiTask
                  0x042c74                  _SignalDHCPSuccessful
                  0x042c82                  _SetDhcpProgressState
                  0x042c8c                  _SignalWiFiConnectionChanged
                  0x042c9c                  _WFProcess
                  0x042d4e                  _Read8BitWFRegister
                  0x042d78                  _Write8BitWFRegister
                  0x042da0                  _Read16BitWFRegister
                  0x042dd6                  _Write16BitWFRegister
                  0x042e0a                  _WriteWFArray
                  0x042e3a                  _ReadWFArray
                  0x042f9e                  _WFEintHandler
                  0x04303e                  _ReenablePowerSaveMode
                  0x043044                  _WFHardwareInit
                  0x0430b2                  _AllocateMgmtTxBuffer
                  0x0430f8                  _DeallocateMgmtRxBuffer
                  0x043112                  _AllocateDataTxBuffer
                  0x043158                  _DeallocateDataTxBuffer
                  0x043172                  _DeallocateDataRxBuffer
                  0x043182                  _RawSendTxBuffer
                  0x04319e                  _RawMountRxBuffer
                  0x0431c0                  _RawToRawCopy
                  0x0431d8                  _PushRawWindow
                  0x0431ee                  _PopRawWindow
                  0x04320c                  _ScratchMount
                  0x043246                  _ScratchUnmount
                  0x043270                  _RawRead
                  0x043294                  _RawWrite
                  0x043326                  _RawSetIndex
                  0x04339c                  _RawGetIndex
                  0x0433c0                  _RawGetByte
                  0x043406                  _RawSetByte
                  0x0434dc                  _SendRAWDataFrame
                  0x0434fa                  _WFEasyConfigInit
                  0x043530                  _WFEasyConfigMgr
                  0x0436e2                  _WFInitScan
                  0x0436f6                  _WFStartScan
                  0x043734                  _WFRetrieveScanResult
                  0x043770                  _WFScanEventHandler
                  0x043792                  _WFGetScanResults
                  0x043806                  _WFDisplayScanMgr
                  0x0438d0                  _NBNSTask
                  0x043c7e                  _ARPSendPkt
                  0x043d52                  _ARPInit
                  0x043d84                  _ARPProcess
                  0x043e5c                  _ARPResolve
                  0x043f26                  _ARPIsResolved
                  0x043fee                  _SwapARPPacket
                  0x044026                  _dhcpConnectOk
                  0x044052                  _StackInit
                  0x0440b2                  _StackTask
                  0x04438e                  _StackApplications
                  0x0443b0                  _RenewDhcp
                  0x0443be                  _XEEInit
                  0x0443dc                  _XEEBeginRead
                  0x0443f4                  _XEERead
                  0x04443a                  _XEEEndRead
                  0x044444                  _XEEReadArray
                  0x044526                  _XEEBeginWrite
                  0x04453e                  _XEEWrite
                  0x044584                  _XEEWriteArray
                  0x0445b2                  _XEEEndWrite
                  0x0446d0                  _XEEIsBusy
                  0x044748                  _WF_CPCreate
                  0x044776                  _WF_CPDelete
                  0x04479c                  _WF_CPGetIds
                  0x0447c4                  _WF_CPSetElements
                  0x0447f8                  _WF_CPGetElements
                  0x044810                  _WF_CPSetSsidType
                  0x044826                  _WF_CPGetSsidType
                  0x04483c                  _WF_CPSetSsid
                  0x044862                  _WF_CPGetSsid
                  0x0448a2                  _WF_CPSetBssid
                  0x0448b6                  _WF_CPGetBssid
                  0x0448cc                  _WF_CPSetNetworkType
                  0x0448e2                  _WF_CPGetNetworkType
                  0x0448f8                  _WF_CPSetWepKeyType
                  0x04490e                  _WF_CPGetWepKeyType
                  0x044924                  _WF_CPSetSecurity
                  0x04498c                  _WF_CPGetSecurity
                  0x0449f8                  _WF_CPSetDefaultWepKeyIndex
                  0x044a0e                  _WF_CPGetDefaultWepKeyIndex
                  0x044a24                  _WF_CPSetAdHocBehavior
                  0x044a3a                  _WF_CPGetAdHocBehavior
                  0x044ace                  _WFEnableMRF24WB0MMode
                  0x044ae0                  _WFEnableBroadcastProbeResponse
                  0x044af2                  _WF_SetLinkDownThreshold
                  0x044b02                  _WFEnableDeferredPowerSave
                  0x044b14                  _WF_GetDeviceInfo
                  0x044b36                  _WF_SetMacAddress
                  0x044b46                  _WF_GetMacAddress
                  0x044b56                  _WF_SetMultiCastFilter
                  0x044bc4                  _WF_GetMultiCastFilter
                  0x044c2a                  _WF_SetTxDataConfirm
                  0x044c3a                  _WF_GetTxDataConfirm
                  0x044c4a                  _WF_SetRegionalDomain
                  0x044c5a                  _WF_GetRegionalDomain
                  0x044c6a                  _WF_SetRtsThreshold
                  0x044c96                  _WF_GetRtsThreshold
                  0x044cb6                  _WF_GetMacStats
                  0x044d5c                  _SendSetParamMsg
                  0x044d8c                  _SendGetParamMsg
                  0x044dc0                  _WF_ProcessEvent
                  0x044f14                  __wifiConnectOk
                  0x044f3a                  _wifiConnectOk
                  0x044f46                  _wifiDhcpOk
                  0x044f4e                  _wifiConnectError
                  0x044f80                  _wifiConnectCheck
                  0x044fe0                  _wifiConnectRetry
                  0x0450a0                  _DNSServerTask
                  0x04537e                  _SNTPClientRestart
                  0x045398                  _SNTPClient
                  0x045596                  _SNTPGetUTCSeconds
                  0x0455e8                  _IPGetHeader
                  0x045702                  _IPPutHeader
                  0x0457b4                  _IPSetRxBuffer
                  0x045802                  _WFProcessMgmtIndicateMsg
                  0x045a16                  _SendMgmtMsg
                  0x045aba                  _SignalMgmtConfirmReceivedEvent
                  0x045ac4                  _WaitForMgmtResponse
                  0x045b68                  _WaitForMgmtResponseAndReadData
                  0x045be2                  _WFSetFuncState
                  0x045c54                  _LCDInit
                  0x045ce2                  _LCDUpdate
                  0x045da6                  _LCDErase
                  0x045dc2                  _TickInit
                  0x045e6c                  _TickGet
                  0x045e9e                  _TickGetDiv256
                  0x045ed0                  _TickGetDiv64K
                  0x045f02                  _TickConvertToMilliseconds
                  0x045f30                  __T1Interrupt
                  0x045f48                  _WF_CMConnect
                  0x045f96                  _WF_CMDisconnect
                  0x045fcc                  _WF_CMGetConnectionState
                  0x04601e                  _WFisConnected
                  0x046028                  _SetLogicalConnectionState
                  0x046034                  _WF_CMCheckConnectionState
                  0x04606c                  _WF_ConvPassphrase2Key
                  0x04610c                  _WF_OutputConnectionDebugMsg
                  0x0461b2                  _WF_OutputConnectionInfo
                  0x0461ba                  _WF_AssertionFailed
                  0x0461ec                  _WF_TxPowerSetMinMax
                  0x046250                  _WF_TxPowerGetMinMax
                  0x046292                  _WF_FixTxRateWithMaxPower
                  0x0462b2                  _WF_TxPowerGetFactoryMax
                  0x0462ca                  _ConvertASCIIHexToBinary
                  0x04635a                  _HexToBin
                  0x0463b8                  _WF_Scan
                  0x04640c                  _WF_ScanGetResult
                  0x04645c                  _WF_SpiInit
                  0x04647c                  _WF_SpiEnableChipSelect
                  0x046484                  _WF_SpiDisableChipSelect
                  0x04648e                  _WFSpiTxRx
                  0x046508                  _WF_EintIsDisabled
                  0x04651e                  _WF_EintIsPending
                  0x046540                  __INT3Interrupt
                  0x046580                  _WF_EintEnable
                  0x046594                  _WF_EintDisable
                  0x04659c                  _WF_EintInit
                  0x0465ae                  _ICMPProcess
                  0x046642                  _convertAsciiToHexInPlace
                  0x0466ce                  _WF_Init
                  0x04674c                  _DelayMs
                  0x046788                  _Delay10us
                  0x0467c4                  _WriteMem
                  0x0467e6                  _WriteLatch
                  0x0467ee                  _ReadLatchLo
                  0x0467fe                  _ReadLatchHi
                  0x04680e                  _ErasePage
                  0x046838                  _ReadProgramMemory
                  0x046846                  _WiSteerStructCheck

External Symbols in Program Memory (by name):

                  0x0077f4                  BEGIN_MPFS
                  0x043d52                  _ARPInit
                  0x043f26                  _ARPIsResolved
                  0x043d84                  _ARPProcess
                  0x043e5c                  _ARPResolve
                  0x043c7e                  _ARPSendPkt
                  0x043112                  _AllocateDataTxBuffer
                  0x0430b2                  _AllocateMgmtTxBuffer
                  0x000bf0                  _AppConfigUseWiFiMacAddress
                  0x03f9d0                  _Base64Decode
                  0x036b50                  _CRC32_Get
                  0x036a3e                  _CRC32_Init
                  0x036ada                  _CRC32_Push
                  0x03f604                  _CalcIPBufferChecksum
                  0x03fd80                  _CalcIPChecksum
                  0x0462ca                  _ConvertASCIIHexToBinary
                  0x03c8c0                  _DHCPDisable
                  0x03c8e4                  _DHCPEnable
                  0x03c864                  _DHCPInit
                  0x03c918                  _DHCPIsBound
                  0x03c904                  _DHCPIsEnabled
                  0x03c946                  _DHCPIsServerDetected
                  0x03e0ea                  _DHCPServerTask
                  0x03ebf8                  _DHCPServer_Disable
                  0x03ec1a                  _DHCPServer_Enable
                  0x03c928                  _DHCPStateChanged
                  0x03c99a                  _DHCPTask
                  0x03c958                  _DHCPTempIPAddr
                  0x03ff56                  _DNSBeginUsage
                  0x03ff76                  _DNSEndUsage
                  0x03ffee                  _DNSIsResolved
                  0x03ffae                  _DNSResolve
                  0x0450a0                  _DNSServerTask
                  0x043172                  _DeallocateDataRxBuffer
                  0x043158                  _DeallocateDataTxBuffer
                  0x0430f8                  _DeallocateMgmtRxBuffer
                  0x0008d4                  _DefaultAppConfig
                  0x046788                  _Delay10us
                  0x04674c                  _DelayMs
                  0x000756                  _DisplayIPValue
                  0x04680e                  _ErasePage
                  0x03fe40                  _FormatNetBIOSName
                  0x03f754                  _GenerateRandomDWORD
                  0x04277e                  _GetEventNotificationMask
                  0x03b756                  _GetTcbInfo
                  0x006154                  _HTML_DOWN_ARROW
                  0x006151                  _HTML_UP_ARROW
                  0x02420e                  _HTTPCheckAuth
                  0x041874                  _HTTPExecuteGet
                  0x04187e                  _HTTPExecutePost
                  0x0368ce                  _HTTPIncFile
                  0x0341f6                  _HTTPInit
                  0x035c80                  _HTTPMPFS2mSendData
                  0x02417e                  _HTTPNeedsAuth
                  0x033922                  _HTTPPrint
                  0x024ce0                  _HTTPPrintIP
                  0x041e66                  _HTTPPrintTry_postJS
                  0x041e18                  _HTTPPrintTry_postJSf
                  0x02ab8c                  _HTTPPrint_actionEnumAskType
                  0x02aa46                  _HTTPPrint_actionEnumCats
                  0x02a740                  _HTTPPrint_actionEnumId
                  0x02a818                  _HTTPPrint_actionEnumImg
                  0x02a7ee                  _HTTPPrint_actionEnumLabel
                  0x02a9d8                  _HTTPPrint_actionEnumPriority
                  0x02a938                  _HTTPPrint_actionEnumStatus
                  0x02a77c                  _HTTPPrint_actionEnumUnicId
                  0x02b8a2                  _HTTPPrint_actionVer
                  0x0254de                  _HTTPPrint_actionsPost
                  0x025690                  _HTTPPrint_actionsPostCmd
                  0x0257d2                  _HTTPPrint_actionsPostInfo
                  0x02553e                  _HTTPPrint_actionsPostLed
                  0x025a34                  _HTTPPrint_bssCount
                  0x025a9a                  _HTTPPrint_bssName
                  0x025aca                  _HTTPPrint_bssPrivacy
                  0x025b46                  _HTTPPrint_bssStrength
                  0x025a70                  _HTTPPrint_bssValid
                  0x025b10                  _HTTPPrint_bssWlan
                  0x02b9da                  _HTTPPrint_btnEnumId
                  0x02ba18                  _HTTPPrint_btnEnumLabel
                  0x02ba46                  _HTTPPrint_btnEnumStatus
                  0x02b936                  _HTTPPrint_btnResetStatus
                  0x0249ac                  _HTTPPrint_builddate
                  0x02652a                  _HTTPPrint_catEnumId
                  0x026566                  _HTTPPrint_catEnumLabel
                  0x02b8e6                  _HTTPPrint_categoryMax
                  0x026c62                  _HTTPPrint_cfg_catCount
                  0x026c8e                  _HTTPPrint_cfg_catCountMax
                  0x026c26                  _HTTPPrint_cfg_catCountVal
                  0x026f72                  _HTTPPrint_cfg_catEnumId
                  0x026fb2                  _HTTPPrint_cfg_catEnumLabel
                  0x026cb4                  _HTTPPrint_cfg_catMainCatId
                  0x026e6c                  _HTTPPrint_cfg_catMainEnumExc
                  0x026dee                  _HTTPPrint_cfg_catMainEnumId
                  0x026e2c                  _HTTPPrint_cfg_catMainEnumNo
                  0x02728c                  _HTTPPrint_cfg_cmdCfgCount
                  0x0272b8                  _HTTPPrint_cfg_cmdCfgCountMax
                  0x027250                  _HTTPPrint_cfg_cmdCfgCountVal
                  0x02825e                  _HTTPPrint_cfg_cmdCfgEnumAct
                  0x028412                  _HTTPPrint_cfg_cmdCfgEnumAskType
                  0x028350                  _HTTPPrint_cfg_cmdCfgEnumAskTypeVal
                  0x027a82                  _HTTPPrint_cfg_cmdCfgEnumCatEnumExc
                  0x0279e6                  _HTTPPrint_cfg_cmdCfgEnumCatEnumId
                  0x027a42                  _HTTPPrint_cfg_cmdCfgEnumCatEnumNo
                  0x027854                  _HTTPPrint_cfg_cmdCfgEnumCatId
                  0x027e3e                  _HTTPPrint_cfg_cmdCfgEnumIOtype
                  0x027d52                  _HTTPPrint_cfg_cmdCfgEnumIOtypeVal
                  0x027336                  _HTTPPrint_cfg_cmdCfgEnumId
                  0x027504                  _HTTPPrint_cfg_cmdCfgEnumImg
                  0x027376                  _HTTPPrint_cfg_cmdCfgEnumLabel
                  0x027c7e                  _HTTPPrint_cfg_cmdCfgEnumPin
                  0x0276ac                  _HTTPPrint_cfg_cmdCfgEnumPin0s
                  0x0275d8                  _HTTPPrint_cfg_cmdCfgEnumPin1s
                  0x027780                  _HTTPPrint_cfg_cmdCfgEnumPinRs
                  0x027412                  _HTTPPrint_cfg_cmdCfgEnumPrior
                  0x027fa0                  _HTTPPrint_cfg_cmdCfgEnumPulse
                  0x027eae                  _HTTPPrint_cfg_cmdCfgEnumRact
                  0x028092                  _HTTPPrint_cfg_cmdCfgEnumTimeNext
                  0x028178                  _HTTPPrint_cfg_cmdCfgEnumTimeOff
                  0x027c0e                  _HTTPPrint_cfg_cmdCfgEnumType
                  0x027b46                  _HTTPPrint_cfg_cmdCfgEnumTypeVal
                  0x02b4be                  _HTTPPrint_cfg_gpsDist
                  0x02b342                  _HTTPPrint_cfg_gpsLat
                  0x02b400                  _HTTPPrint_cfg_gpsLon
                  0x0284a2                  _HTTPPrint_cfg_ioCount
                  0x0284ce                  _HTTPPrint_cfg_ioCountMax
                  0x028466                  _HTTPPrint_cfg_ioCountVal
                  0x02baa2                  _HTTPPrint_cfg_ioEnumDimLevel
                  0x02bb10                  _HTTPPrint_cfg_ioEnumDimLevelVal
                  0x02853e                  _HTTPPrint_cfg_ioEnumId
                  0x02857e                  _HTTPPrint_cfg_ioEnumLabel
                  0x028662                  _HTTPPrint_cfg_ioEnumType
                  0x0285e0                  _HTTPPrint_cfg_ioEnumTypeVal
                  0x02658e                  _HTTPPrint_cfg_label
                  0x026b38                  _HTTPPrint_cfg_login
                  0x026b5e                  _HTTPPrint_cfg_pwd1
                  0x026b64                  _HTTPPrint_cfg_pwd2
                  0x026c00                  _HTTPPrint_cfg_timeServer
                  0x0271ec                  _HTTPPrint_cmdOutEnumId
                  0x027228                  _HTTPPrint_cmdOutEnumLabel
                  0x024da0                  _HTTPPrint_config_dhcpchecked
                  0x024e54                  _HTTPPrint_config_dns1
                  0x024e82                  _HTTPPrint_config_dns2
                  0x024df8                  _HTTPPrint_config_gw
                  0x024d64                  _HTTPPrint_config_hostname
                  0x024dca                  _HTTPPrint_config_ip
                  0x024eb0                  _HTTPPrint_config_mac
                  0x024d82                  _HTTPPrint_config_netbiosname
                  0x024e26                  _HTTPPrint_config_subnet
                  0x02b2e6                  _HTTPPrint_deviceBootDate
                  0x02b23e                  _HTTPPrint_deviceFWver
                  0x02ad18                  _HTTPPrint_deviceID
                  0x02add0                  _HTTPPrint_deviceIP
                  0x02ad40                  _HTTPPrint_deviceLabel
                  0x02ad66                  _HTTPPrint_deviceMac
                  0x02b29c                  _HTTPPrint_deviceMpfsDate
                  0x02b1ca                  _HTTPPrint_deviceSentTime
                  0x02ae2a                  _HTTPPrint_deviceStatus
                  0x02b156                  _HTTPPrint_deviceTime
                  0x0287fa                  _HTTPPrint_formFocus
                  0x025056                  _HTTPPrint_fwver
                  0x02b6f4                  _HTTPPrint_gpsDistanceMax
                  0x02b57c                  _HTTPPrint_gpsLatitude
                  0x02b638                  _HTTPPrint_gpsLongitude
                  0x024d46                  _HTTPPrint_host
                  0x041c0a                  _HTTPPrint_htmlEscape
                  0x041c24                  _HTTPPrint_htmlEscapeLen
                  0x0270b4                  _HTTPPrint_ioPinEnumId
                  0x0270f0                  _HTTPPrint_ioPinEnumLabel
                  0x02711a                  _HTTPPrint_ioPinEnumType
                  0x041a8a                  _HTTPPrint_jsEscape
                  0x041aa4                  _HTTPPrint_jsEscapeLen
                  0x025192                  _HTTPPrint_label
                  0x0249fe                  _HTTPPrint_led
                  0x024aa2                  _HTTPPrint_ledSelected
                  0x0254b8                  _HTTPPrint_logDetails
                  0x0253f8                  _HTTPPrint_logID
                  0x02547a                  _HTTPPrint_logLevel
                  0x02543a                  _HTTPPrint_logTime
                  0x02b848                  _HTTPPrint_mpfsdate
                  0x0250da                  _HTTPPrint_nextSSID
                  0x025168                  _HTTPPrint_nextWLAN
                  0x041922                  _HTTPPrint_out
                  0x04193c                  _HTTPPrint_outLen
                  0x025bcc                  _HTTPPrint_pageId
                  0x028696                  _HTTPPrint_postDevIOconfig
                  0x02a54a                  _HTTPPrint_postDevIOconfig_configCats
                  0x029966                  _HTTPPrint_postDevIOconfig_configCmds
                  0x02a2ba                  _HTTPPrint_postDevIOconfig_configIOs
                  0x02881e                  _HTTPPrint_postDevIOconfig_configMain
                  0x02951a                  _HTTPPrint_postDevIOconfig_configTime
                  0x02b7c4                  _HTTPPrint_postDevIOconfig_configTools
                  0x02b898                  _HTTPPrint_postDevLst
                  0x041eee                  _HTTPPrint_postErrorField
                  0x041f06                  _HTTPPrint_postErrorFieldArg1
                  0x041f24                  _HTTPPrint_postErrorFieldArg2
                  0x041e3a                  _HTTPPrint_postJS
                  0x041dfa                  _HTTPPrint_postJSf
                  0x0245da                  _HTTPPrint_postTcpIpConfig
                  0x024244                  _HTTPPrint_postWifiConfig
                  0x025c82                  _HTTPPrint_postWifiPowerMax
                  0x024bec                  _HTTPPrint_pot
                  0x0250f8                  _HTTPPrint_prevSSID
                  0x02513e                  _HTTPPrint_prevWLAN
                  0x024f84                  _HTTPPrint_reboot
                  0x024f9c                  _HTTPPrint_rebootaddr
                  0x0250a8                  _HTTPPrint_ssid
                  0x025010                  _HTTPPrint_status_fail
                  0x024fca                  _HTTPPrint_status_ok
                  0x0249b8                  _HTTPPrint_tcpipVersion
                  0x024b54                  _HTTPPrint_temp
                  0x024c7e                  _HTTPPrint_time
                  0x026070                  _HTTPPrint_timeBias
                  0x024cb0                  _HTTPPrint_timeBoot
                  0x025eac                  _HTTPPrint_timeDay
                  0x02629e                  _HTTPPrint_timeDltBias
                  0x0261c6                  _HTTPPrint_timeDltHour
                  0x02620e                  _HTTPPrint_timeDltMin
                  0x02617e                  _HTTPPrint_timeDltMonth
                  0x026256                  _HTTPPrint_timeDltSec
                  0x026136                  _HTTPPrint_timeDltWeekDay
                  0x0260ee                  _HTTPPrint_timeDltWeekDayNo
                  0x025f64                  _HTTPPrint_timeHour
                  0x025fa2                  _HTTPPrint_timeMin
                  0x025eea                  _HTTPPrint_timeMonth
                  0x025e4c                  _HTTPPrint_timeScanStart
                  0x025cf4                  _HTTPPrint_timeScanStartLow
                  0x02648a                  _HTTPPrint_timeSdtBias
                  0x0263b2                  _HTTPPrint_timeSdtHour
                  0x0263fa                  _HTTPPrint_timeSdtMin
                  0x02636a                  _HTTPPrint_timeSdtMonth
                  0x026442                  _HTTPPrint_timeSdtSec
                  0x026322                  _HTTPPrint_timeSdtWeekDay
                  0x0262da                  _HTTPPrint_timeSdtWeekDayNo
                  0x025fe0                  _HTTPPrint_timeSec
                  0x025f28                  _HTTPPrint_timeYear
                  0x02601e                  _HTTPPrint_timeZoneId
                  0x0418fc                  _HTTPPrint_tooMuchData
                  0x0249c4                  _HTTPPrint_version
                  0x025c46                  _HTTPPrint_wifiFactoryPowerMax
                  0x025c06                  _HTTPPrint_wifiPowerMax
                  0x0259ce                  _HTTPPrint_wifiScanInProgress
                  0x025876                  _HTTPPrint_wifiScanPost
                  0x024c64                  _HTTPPrint_zcross
                  0x0341ea                  _HTTPQueryContentType
                  0x033e9c                  _HTTPQueryIf
                  0x02a904                  _HTTPQueryIf_actionEnumError
                  0x02a864                  _HTTPQueryIf_actionEnumON
                  0x02a898                  _HTTPQueryIf_actionEnumONavail
                  0x02a8ce                  _HTTPQueryIf_actionEnumRunning
                  0x02b91c                  _HTTPQueryIf_actionPending
                  0x02527c                  _HTTPQueryIf_actionToGet
                  0x025298                  _HTTPQueryIf_actionToReload
                  0x026a4c                  _HTTPQueryIf_boostModeON
                  0x026b6a                  _HTTPQueryIf_category_available
                  0x0267e8                  _HTTPQueryIf_cfg_activityLedON
                  0x0269c8                  _HTTPQueryIf_cfg_boostModeON
                  0x027e92                  _HTTPQueryIf_cfg_cmdCfgEnumIOtypeIs
                  0x027c62                  _HTTPQueryIf_cfg_cmdCfgEnumTypeIs
                  0x0265b4                  _HTTPQueryIf_cfg_debugON
                  0x026764                  _HTTPQueryIf_cfg_haltfON
                  0x0268f0                  _HTTPQueryIf_cfg_homeActivityPanelON
                  0x02baf6                  _HTTPQueryIf_cfg_ioEnumTypeIs
                  0x026b2e                  _HTTPQueryIf_cfg_mpfsUploadON
                  0x02686c                  _HTTPQueryIf_cfg_protectAllON
                  0x026638                  _HTTPQueryIf_cfg_testON
                  0x0260ac                  _HTTPQueryIf_cfg_timeDlON
                  0x026b7c                  _HTTPQueryIf_cfg_timeServerSyncON
                  0x026b24                  _HTTPQueryIf_cfg_wisteerAutoUpdateON
                  0x026aa0                  _HTTPQueryIf_cfg_wisteerNetBrowseON
                  0x0251be                  _HTTPQueryIf_devConfigured
                  0x02524c                  _HTTPQueryIf_devNotConfigured
                  0x02b330                  _HTTPQueryIf_deviceLinked
                  0x02abd6                  _HTTPQueryIf_formConfigured
                  0x02ac86                  _HTTPQueryIf_formExpanded
                  0x026974                  _HTTPQueryIf_homeActivityPanelON
                  0x025260                  _HTTPQueryIf_logToGet
                  0x025b7c                  _HTTPQueryIf_pageIdIs
                  0x025ba4                  _HTTPQueryIf_pageIdIsNot
                  0x026710                  _HTTPQueryIf_testON
                  0x02521e                  _HTTPQueryIf_wifiAndDevConfigured
                  0x0251b0                  _HTTPQueryIf_wifiConfigured
                  0x025236                  _HTTPQueryIf_wifiNotConfigured
                  0x02b7b0                  _HTTPQueryIf_wisteerMpfsDynamic
                  0x02b7ba                  _HTTPQueryIf_wisteerMpfsUploadON
                  0x024c74                  _HTTPQueryIf_zcrossNotOk
                  0x024c6a                  _HTTPQueryIf_zcrossOk
                  0x034122                  _HTTPQueryWhile
                  0x02a6a0                  _HTTPQueryWhile_actionEnum
                  0x02b966                  _HTTPQueryWhile_btnEnum
                  0x0264c6                  _HTTPQueryWhile_catEnum
                  0x026f28                  _HTTPQueryWhile_cfg_catEnum
                  0x026d44                  _HTTPQueryWhile_cfg_catMainEnum
                  0x0272de                  _HTTPQueryWhile_cfg_cmdCfgEnum
                  0x027918                  _HTTPQueryWhile_cfg_cmdCfgEnumCatEnum
                  0x0284f4                  _HTTPQueryWhile_cfg_ioEnum
                  0x027182                  _HTTPQueryWhile_cmdOutEnum
                  0x02acd6                  _HTTPQueryWhile_deviceEnum
                  0x027012                  _HTTPQueryWhile_ioPinEnum
                  0x0252ca                  _HTTPQueryWhile_logEnum
                  0x0365c0                  _HTTPReadPostName
                  0x0365ec                  _HTTPReadPostValue
                  0x034274                  _HTTPServer
                  0x03615a                  _HTTPURLDecode
                  0x03622e                  _HTTPargGet
                  0x0363b4                  _HTTPargSet
                  0x0362ce                  _HTTPargTrimGet
                  0x041f48                  _HashAddData
                  0x04635a                  _HexToBin
                  0x0465ae                  _ICMPProcess
                  0x0455e8                  _IPGetHeader
                  0x045702                  _IPPutHeader
                  0x0457b4                  _IPSetRxBuffer
                  0x045da6                  _LCDErase
                  0x045c54                  _LCDInit
                  0x045ce2                  _LCDUpdate
                  0x000e86                  _LED_PUT
                  0x03f6e4                  _LFSRRand
                  0x03f6a2                  _LFSRSeedRand
                  0x000a06                  _LoadAppConfig
                  0x03f294                  _MACCalcRxChecksum
                  0x03f01c                  _MACDiscardRx
                  0x03f1ec                  _MACFlush
                  0x03f522                  _MACGet
                  0x03f54e                  _MACGetArray
                  0x03f026                  _MACGetFreeRxSize
                  0x03f0a0                  _MACGetHeader
                  0x03ee7a                  _MACInit
                  0x03eed6                  _MACIsLinked
                  0x03f518                  _MACIsMemCopyDone
                  0x03eee4                  _MACIsTxReady
                  0x03f2c2                  _MACMemCopyAsync
                  0x03f696                  _MACPowerDown
                  0x03f69c                  _MACPowerUp
                  0x03ee32                  _MACProcess
                  0x03f5a8                  _MACPut
                  0x03f5d6                  _MACPutArray
                  0x03f194                  _MACPutHeader
                  0x03f27c                  _MACSetReadPtr
                  0x03f252                  _MACSetReadPtrInRx
                  0x03f264                  _MACSetWritePtr
                  0x041fa0                  _MD5AddData
                  0x042240                  _MD5Calculate
                  0x041f64                  _MD5Initialize
                  0x03d6d8                  _MPFSClose
                  0x03d6fe                  _MPFSGet
                  0x03d88e                  _MPFSGetArray
                  0x03de9e                  _MPFSGetBytesRem
                  0x03ddb8                  _MPFSGetContentType
                  0x03dd32                  _MPFSGetContentTypeId
                  0x03df6a                  _MPFSGetEndAddr
                  0x03dfbc                  _MPFSGetFilename
                  0x03de14                  _MPFSGetFlags
                  0x03e05c                  _MPFSGetID
                  0x03dab8                  _MPFSGetLong
                  0x03dedc                  _MPFSGetPhysAddr
                  0x03e020                  _MPFSGetPosition
                  0x03de58                  _MPFSGetSize
                  0x03df22                  _MPFSGetStartAddr
                  0x03dcec                  _MPFSGetTimestamp
                  0x03d4c4                  _MPFSInit
                  0x03e0e0                  _MPFSLocked
                  0x03d4f8                  _MPFSOpen
                  0x03d64e                  _MPFSOpenID
                  0x03dada                  _MPFSSeek
                  0x0077ec                  _MPFS_Start
                  0x03e0da                  _MPFSputHdrCorrect
                  0x03e0cc                  _MPFSseekInit
                  0x0266bc                  _MPFStestMode
                  0x0438d0                  _NBNSTask
                  0x000fbe                  _OnMdnsHostNameChanged
                  0x0431ee                  _PopRawWindow
                  0x0431d8                  _PushRawWindow
                  0x0433c0                  _RawGetByte
                  0x04339c                  _RawGetIndex
                  0x03efb8                  _RawGetMgmtRxBuffer
                  0x03ee84                  _RawInit
                  0x04319e                  _RawMountRxBuffer
                  0x043270                  _RawRead
                  0x043182                  _RawSendTxBuffer
                  0x043406                  _RawSetByte
                  0x043326                  _RawSetIndex
                  0x0431c0                  _RawToRawCopy
                  0x043294                  _RawWrite
                  0x042da0                  _Read16BitWFRegister
                  0x042d4e                  _Read8BitWFRegister
                  0x0467fe                  _ReadLatchHi
                  0x0467ee                  _ReadLatchLo
                  0x046838                  _ReadProgramMemory
                  0x042e3a                  _ReadWFArray
                  0x04303e                  _ReenablePowerSaveMode
                  0x0443b0                  _RenewDhcp
                  0x000e52                  _RestoreWifiConfig
                  0x045398                  _SNTPClient
                  0x04537e                  _SNTPClientRestart
                  0x045596                  _SNTPGetUTCSeconds
                  0x000dda                  _SaveAppConfig
                  0x04320c                  _ScratchMount
                  0x043246                  _ScratchUnmount
                  0x044d8c                  _SendGetParamMsg
                  0x045a16                  _SendMgmtMsg
                  0x0434dc                  _SendRAWDataFrame
                  0x03efa8                  _SendRAWManagementFrame
                  0x044d5c                  _SendSetParamMsg
                  0x042c82                  _SetDhcpProgressState
                  0x046028                  _SetLogicalConnectionState
                  0x03effa                  _SetRawRxMgmtInProgress
                  0x042c74                  _SignalDHCPSuccessful
                  0x045aba                  _SignalMgmtConfirmReceivedEvent
                  0x042c8c                  _SignalWiFiConnectionChanged
                  0x04438e                  _StackApplications
                  0x044052                  _StackInit
                  0x0440b2                  _StackTask
                  0x03f85e                  _StringToIPAddress
                  0x043fee                  _SwapARPPacket
                  0x03b554                  _TCPAdjustFIFOSize
                  0x0396a0                  _TCPClose
                  0x03993a                  _TCPDiscard
                  0x039600                  _TCPDisconnect
                  0x039bc4                  _TCPFindArrayEx
                  0x039e34                  _TCPFindEx
                  0x0396ea                  _TCPFlush
                  0x039992                  _TCPGet
                  0x039a0c                  _TCPGetArray
                  0x0396c0                  _TCPGetRemoteInfo
                  0x039ad8                  _TCPGetRxFIFOFree
                  0x03990e                  _TCPGetTxFIFOFull
                  0x039362                  _TCPInit
                  0x0395dc                  _TCPIsConnected
                  0x03995a                  _TCPIsGetReady
                  0x039710                  _TCPIsPutReady
                  0x039452                  _TCPOpen
                  0x039bac                  _TCPPeek
                  0x039b02                  _TCPPeekArray
                  0x03a348                  _TCPProcess
                  0x03975e                  _TCPPut
                  0x039804                  _TCPPutArray
                  0x0398ea                  _TCPPutString
                  0x0077ba                  _TCPSocketInitializer
                  0x039e58                  _TCPTick
                  0x0395ae                  _TCPWasReset
                  0x045f02                  _TickConvertToMilliseconds
                  0x045e6c                  _TickGet
                  0x045e9e                  _TickGetDiv256
                  0x045ed0                  _TickGetDiv64K
                  0x045dc2                  _TickInit
                  0x0413f6                  _UDPClose
                  0x04165e                  _UDPDiscard
                  0x041684                  _UDPDiscardRxTx
                  0x04153a                  _UDPFlush
                  0x0415de                  _UDPGet
                  0x041612                  _UDPGetArray
                  0x04105a                  _UDPInit
                  0x0415a8                  _UDPIsGetReady
                  0x0413d4                  _UDPIsOpened
                  0x04147a                  _UDPIsPutReady
                  0x04107a                  _UDPOpenEx
                  0x041698                  _UDPProcess
                  0x0414b0                  _UDPPut
                  0x0414e0                  _UDPPutArray
                  0x04151c                  _UDPPutString
                  0x041464                  _UDPSetRxBuffer
                  0x04144e                  _UDPSetTxBuffer
                  0x041194                  _UDPTask
                  0x000b7e                  _UpgradeAppConfig
                  0x043806                  _WFDisplayScanMgr
                  0x0434fa                  _WFEasyConfigInit
                  0x043530                  _WFEasyConfigMgr
                  0x042f9e                  _WFEintHandler
                  0x044ae0                  _WFEnableBroadcastProbeResponse
                  0x044b02                  _WFEnableDeferredPowerSave
                  0x044ace                  _WFEnableMRF24WB0MMode
                  0x03ef74                  _WFFreeMgmtTx
                  0x043792                  _WFGetScanResults
                  0x03ee70                  _WFGetTCBSize
                  0x043044                  _WFHardwareInit
                  0x0436e2                  _WFInitScan
                  0x042c9c                  _WFProcess
                  0x045802                  _WFProcessMgmtIndicateMsg
                  0x043734                  _WFRetrieveScanResult
                  0x043770                  _WFScanEventHandler
                  0x045be2                  _WFSetFuncState
                  0x04648e                  _WFSpiTxRx
                  0x0436f6                  _WFStartScan
                  0x0461ba                  _WF_AssertionFailed
                  0x042760                  _WF_CAGetBeaconTimeout
                  0x042690                  _WF_CAGetBeaconTimeoutAction
                  0x0426d6                  _WF_CAGetChannelList
                  0x042632                  _WF_CAGetConnectionProfileList
                  0x0426b2                  _WF_CAGetDeauthAction
                  0x0424b6                  _WF_CAGetElements
                  0x042670                  _WF_CAGetEventNotificationAction
                  0x042652                  _WF_CAGetListRetryCount
                  0x04272e                  _WF_CAGetListenInterval
                  0x04257e                  _WF_CAGetMaxChannelTime
                  0x042540                  _WF_CAGetMinChannelTime
                  0x0425bc                  _WF_CAGetProbeDelay
                  0x042610                  _WF_CAGetRssi
                  0x0425ee                  _WF_CAGetScanCount
                  0x042512                  _WF_CAGetScanType
                  0x042750                  _WF_CASetBeaconTimeout
                  0x042680                  _WF_CASetBeaconTimeoutAction
                  0x0426c4                  _WF_CASetChannelList
                  0x042622                  _WF_CASetConnectionProfileList
                  0x0426a2                  _WF_CASetDeauthAction
                  0x0423c0                  _WF_CASetElements
                  0x04247e                  _WF_CASetElementsN
                  0x042664                  _WF_CASetEventNotificationAction
                  0x042642                  _WF_CASetListRetryCount
                  0x042712                  _WF_CASetListenInterval
                  0x042562                  _WF_CASetMaxChannelTime
                  0x042524                  _WF_CASetMinChannelTime
                  0x0425a0                  _WF_CASetProbeDelay
                  0x042600                  _WF_CASetRssi
                  0x0425de                  _WF_CASetScanCount
                  0x042502                  _WF_CASetScanType
                  0x046034                  _WF_CMCheckConnectionState
                  0x045f48                  _WF_CMConnect
                  0x045f96                  _WF_CMDisconnect
                  0x045fcc                  _WF_CMGetConnectionState
                  0x044748                  _WF_CPCreate
                  0x044776                  _WF_CPDelete
                  0x044a3a                  _WF_CPGetAdHocBehavior
                  0x0448b6                  _WF_CPGetBssid
                  0x044a0e                  _WF_CPGetDefaultWepKeyIndex
                  0x0447f8                  _WF_CPGetElements
                  0x04479c                  _WF_CPGetIds
                  0x0448e2                  _WF_CPGetNetworkType
                  0x04498c                  _WF_CPGetSecurity
                  0x044862                  _WF_CPGetSsid
                  0x044826                  _WF_CPGetSsidType
                  0x04490e                  _WF_CPGetWepKeyType
                  0x044a24                  _WF_CPSetAdHocBehavior
                  0x0448a2                  _WF_CPSetBssid
                  0x0449f8                  _WF_CPSetDefaultWepKeyIndex
                  0x0447c4                  _WF_CPSetElements
                  0x0448cc                  _WF_CPSetNetworkType
                  0x044924                  _WF_CPSetSecurity
                  0x04483c                  _WF_CPSetSsid
                  0x044810                  _WF_CPSetSsidType
                  0x0448f8                  _WF_CPSetWepKeyType
                  0x000640                  _WF_Connect
                  0x04606c                  _WF_ConvPassphrase2Key
                  0x042800                  _WF_DisableModuleConnectionManager
                  0x046594                  _WF_EintDisable
                  0x046580                  _WF_EintEnable
                  0x04659c                  _WF_EintInit
                  0x046508                  _WF_EintIsDisabled
                  0x04651e                  _WF_EintIsPending
                  0x046292                  _WF_FixTxRateWithMaxPower
                  0x044b14                  _WF_GetDeviceInfo
                  0x044b46                  _WF_GetMacAddress
                  0x044cb6                  _WF_GetMacStats
                  0x044bc4                  _WF_GetMultiCastFilter
                  0x044c5a                  _WF_GetRegionalDomain
                  0x044c96                  _WF_GetRtsThreshold
                  0x044c3a                  _WF_GetTxDataConfirm
                  0x0466ce                  _WF_Init
                  0x04610c                  _WF_OutputConnectionDebugMsg
                  0x0461b2                  _WF_OutputConnectionInfo
                  0x044dc0                  _WF_ProcessEvent
                  0x0463b8                  _WF_Scan
                  0x04640c                  _WF_ScanGetResult
                  0x044af2                  _WF_SetLinkDownThreshold
                  0x044b36                  _WF_SetMacAddress
                  0x044b56                  _WF_SetMultiCastFilter
                  0x044c4a                  _WF_SetRegionalDomain
                  0x044c6a                  _WF_SetRtsThreshold
                  0x044c2a                  _WF_SetTxDataConfirm
                  0x046484                  _WF_SpiDisableChipSelect
                  0x04647c                  _WF_SpiEnableChipSelect
                  0x04645c                  _WF_SpiInit
                  0x0462b2                  _WF_TxPowerGetFactoryMax
                  0x046250                  _WF_TxPowerGetMinMax
                  0x0461ec                  _WF_TxPowerSetMinMax
                  0x04601e                  _WFisConnected
                  0x03ef3a                  _WFisTxMgmtReady
                  0x045ac4                  _WaitForMgmtResponse
                  0x045b68                  _WaitForMgmtResponseAndReadData
                  0x042c64                  _WiFiTask
                  0x0305f4                  _WiSteerCom_AnnounceIP
                  0x03067a                  _WiSteerCom_AnnounceModeToOpCode
                  0x030ed6                  _WiSteerCom_AnnounceProcess
                  0x03088e                  _WiSteerCom_AnnounceSend
                  0x0306a0                  _WiSteerCom_AnnounceTask
                  0x030e6e                  _WiSteerCom_AuthMd5
                  0x030ecc                  _WiSteerCom_AuthMd5Reset
                  0x0332b0                  _WiSteerCom_CatActionAsk
                  0x0337d8                  _WiSteerCom_CatActionInfoProcess
                  0x0336be                  _WiSteerCom_CatActionProcess
                  0x032b1a                  _WiSteerCom_CmdActionChanged
                  0x0329e4                  _WiSteerCom_CmdActionErrorProcess
                  0x032888                  _WiSteerCom_CmdActionErrorSend
                  0x0328e4                  _WiSteerCom_CmdActionInfoProcess
                  0x032726                  _WiSteerCom_CmdActionProcess
                  0x033056                  _WiSteerCom_CmdLog
                  0x03317c                  _WiSteerCom_CmdStatusInfoProcess
                  0x032e90                  _WiSteerCom_CmdStatusProcess
                  0x030be2                  _WiSteerCom_DiscoveryRecv
                  0x030d4c                  _WiSteerCom_DiscoveryReply
                  0x031236                  _WiSteerCom_DiscoverySendTask
                  0x031492                  _WiSteerCom_DiscoverySendTaskCat
                  0x0333c8                  _WiSteerCom_DiscoverySendTaskCatAction
                  0x03169c                  _WiSteerCom_DiscoverySendTaskCmd
                  0x032442                  _WiSteerCom_DiscoverySendTaskCmdAction
                  0x032bac                  _WiSteerCom_DiscoverySendTaskCmdChanged
                  0x030a20                  _WiSteerCom_DiscoveryTask
                  0x031d28                  _WiSteerCom_RetrieveCatErrorProcess
                  0x031bee                  _WiSteerCom_RetrieveCatInfoProcess
                  0x031986                  _WiSteerCom_RetrieveCatProcess
                  0x031fe4                  _WiSteerCom_RetrieveCmdErrorProcess
                  0x031e42                  _WiSteerCom_RetrieveCmdInfoProcess
                  0x031a5c                  _WiSteerCom_RetrieveCmdProcess
                  0x03192e                  _WiSteerCom_RetrieveInfoError
                  0x0318a0                  _WiSteerCom_RetrieveInfoSend
                  0x0320fe                  _WiSteerCom_actionProcessCmdCfgOutputId
                  0x031b60                  _WiSteerCom_deviceSource
                  0x030836                  _WiSteerCom_init
                  0x046846                  _WiSteerStructCheck
                  0x042dd6                  _Write16BitWFRegister
                  0x042d78                  _Write8BitWFRegister
                  0x0467e6                  _WriteLatch
                  0x0467c4                  _WriteMem
                  0x042e0a                  _WriteWFArray
                  0x0443dc                  _XEEBeginRead
                  0x044526                  _XEEBeginWrite
                  0x04443a                  _XEEEndRead
                  0x0445b2                  _XEEEndWrite
                  0x0443be                  _XEEInit
                  0x0446d0                  _XEEIsBusy
                  0x0443f4                  _XEERead
                  0x044444                  _XEEReadArray
                  0x04453e                  _XEEWrite
                  0x044584                  _XEEWriteArray
                  0x00032c                  __AddressError
                  0x0002d8                  __DefaultInterrupt
                  0x046540                  __INT3Interrupt
                  0x000380                  __MathError
                  0x000302                  __OscillatorFail
                  0x000356                  __StackError
                  0x045f30                  __T1Interrupt
                  0x00459e                  ___adddf3
                  0x0046ac                  ___divdf3
                  0x0018d4                  ___divdi3
                  0x004760                  ___divsf3
                  0x001716                  ___divsi3
                  0x004698                  ___eqdf2
                  0x0048b6                  ___eqsf2
                  0x004878                  ___extendsfdf2
                  0x0048be                  ___fixunsdfdi
                  0x004920                  ___fixunsdfsi
                  0x004d60                  ___floatdisf
                  0x00496c                  ___floatsisf
                  0x004972                  ___floatundidf
                  0x004d80                  ___floatundisf
                  0x0049c8                  ___floatunsidf
                  0x0046a2                  ___gedf2
                  0x0048ba                  ___gesf2
                  0x0046a2                  ___gtdf2
                  0x0048ba                  ___gtsf2
                  0x004698                  ___ledf2
                  0x0048b6                  ___lesf2
                  0x004698                  ___ltdf2
                  0x0048b6                  ___ltsf2
                  0x001938                  ___moddi3
                  0x001734                  ___modsi3
                  0x004a78                  ___muldf3
                  0x001998                  ___muldi3
                  0x004c24                  ___mulp32eds3
                  0x004c24                  ___mulp32peds3
                  0x004b62                  ___mulsf3
                  0x004c24                  ___mulsi3
                  0x0047e4                  ___nedf2
                  0x004bca                  ___subdf3
                  0x004bce                  ___truncdfsf2
                  0x0018b6                  ___udivdi3
                  0x0017e6                  ___udivmoddi3
                  0x001752                  ___udivsi3
                  0x0018c8                  ___umoddi3
                  0x001772                  ___umodsi3
                  0x0019ee                  ___umuldi3
                  0x03878a                  __actionProcessCmdOrCatId
                  0x004c9c                  __dPropagateNaN
                  0x000232                  __data_init
                  0x000232                  __data_init_extended
                  0x004c4a                  __dcompare
                  0x0047ee                  __dpack
                  0x004868                  __dreturnNaN
                  0x004cb8                  __dtype
                  0x004cdc                  __dunpack
                  0x004846                  __dunpack2
                  0x00486e                  __dunpack2exit
                  0x004a58                  __fPropagateNaN
                  0x004a6a                  __fbopExit
                  0x004a72                  __fbopReturnNaN
                  0x004d2a                  __fcompare
                  0x0049cc                  __fpack
                  0x004c30                  __frexpf
                  0x004a1e                  __funpack
                  0x004a48                  __funpack2
                  0x000226                  __psv_init
                  0x000200                  __resetPRI
                  0x001ff8                  __snprintf_cdfFnopsuxX
                  0x001ff8                  __snprintf_cdfFnopuxX
                  0x001ff8                  __snprintf_cdnopsuxX
                  0x001ff8                  __snprintf_cdnopuxX
                  0x00383e                  __vfprintf_cdfFnopsuxX
                  0x00383e                  __vfprintf_cdfFnopuxX
                  0x00383e                  __vfprintf_cdnopsuxX
                  0x00383e                  __vfprintf_cdnopuxX
                  0x002004                  __vsnprintf_cdfFnopsuxX
                  0x002004                  __vsnprintf_cdfFnopuxX
                  0x002004                  __vsnprintf_cdnopsuxX
                  0x002004                  __vsnprintf_cdnopuxX
                  0x044f14                  __wifiConnectOk
                  0x037d90                  _actTypeFromInputMode
                  0x037dde                  _actTypeFromLinkMode
                  0x038a0c                  _actionAskerError
                  0x038976                  _actionAskerFree
                  0x0388fe                  _actionAskerGet
                  0x038a54                  _actionAskerLabel
                  0x038f34                  _actionAutoOff
                  0x038fc4                  _actionAutoOffReset
                  0x039032                  _actionAutoOffWatch
                  0x038df8                  _actionCatFilter
                  0x036db4                  _actionInit
                  0x039136                  _actionInitToOffForIO
                  0x039190                  _actionInitToOffForIOcmd
                  0x037078                  _actionInputChanged
                  0x036e00                  _actionInputInit
                  0x037188                  _actionInputPulse
                  0x037248                  _actionInputPulseChoose
                  0x0373bc                  _actionInputPulseProcess
                  0x036f24                  _actionInputReset
                  0x03710e                  _actionInputSignal
                  0x037498                  _actionInputSignalProcess
                  0x036fea                  _actionInputWatch
                  0x036f38                  _actionInputWatchAdd
                  0x038a9e                  _actionLocalInit
                  0x036b62                  _actionPendingClear
                  0x0379d2                  _actionPostCmd
                  0x037c88                  _actionProcess
                  0x038e3c                  _actionProcessCatCom
                  0x038aba                  _actionProcessCatId
                  0x037e66                  _actionProcessCmdCfgId
                  0x038ede                  _actionProcessCmdCfgInputPinStatus
                  0x03800a                  _actionProcessCmdCfgOutputId
                  0x03864a                  _actionProcessCmdCfgOutputPin
                  0x038698                  _actionProcessCmdCfgOutputPinLow
                  0x03872c                  _actionProcessCmdCfgOutputPinStatus
                  0x03880e                  _actionProcessCmdOrCatId
                  0x037e2c                  _actionProcessCmdSum
                  0x037cbe                  _actionProcessCmdSumId
                  0x037be0                  _actionProcessMask
                  0x037ac4                  _actionRunningRemoteUpdate
                  0x037b54                  _actionRunningTick
                  0x037b76                  _actionStatus
                  0x0378fc                  _actionSumFromCmdId
                  0x000f9a                  _activityLedsModeChange
                  0x000f64                  _activityLedsOn
                  0x001c04                  _atof
                  0x001c0e                  _atoi
                  0x001c50                  _atol
                  0x03fc2c                  _btohexa_high
                  0x03fc4e                  _btohexa_low
                  0x0058ba                  _c_formInput_nochg
                  0x0058bb                  _c_formInput_post
                  0x038dc6                  _catInCatList
                  0x007691                  _clsCmd
                  0x007695                  _clsHelp
                  0x036d66                  _cmdCfgCatIsValid
                  0x036cc0                  _cmdCfgDisplayIsValid
                  0x036ce6                  _cmdCfgHiddenIsValid
                  0x036c2c                  _cmdCfgIsValid
                  0x036d0c                  _cmdCfgOutIsValid
                  0x033274                  _cmdModeRemoteRecv
                  0x03776c                  _cmdSumCalc
                  0x046642                  _convertAsciiToHexInPlace
                  0x001380                  _deviceCmdAdd
                  0x001430                  _deviceCmdEnd
                  0x001100                  _deviceFind
                  0x00102e                  _deviceGet
                  0x001334                  _deviceGoodCfgShareSourceEnd
                  0x001362                  _deviceId
                  0x001264                  _deviceIsGoodCfgShareSource
                  0x000fc6                  _deviceReinit
                  0x00117c                  _deviceWithOpToDoGet
                  0x044026                  _dhcpConnectOk
                  0x004a18                  _frexpf
                  0x0076cc                  _g_consoleCmd
                  0x0076ea                  _g_numCmds
                  0x025116                  _getWlanStr
                  0x00765a                  _getwfverCmd
                  0x007663                  _getwfverHelp
                  0x007642                  _helpCmd
                  0x007647                  _helpHelp
                  0x03fbc2                  _hexatob
                  0x02bcbe                  _hmac_sha1
                  0x02bb96                  _hmac_sha1_vector
                  0x0062e2                  _http2m_ContentTypes
                  0x036c00                  _ioPinInit
                  0x036bf6                  _ioPinInitLow
                  0x036b8a                  _ioPinMode
                  0x03f012                  _isRawRxMgmtInProgress
                  0x0016c8                  _isalpha
                  0x0016dc                  _isspace
                  0x0016ec                  _isxdigit
                  0x041040                  _logFatalCheckPt
                  0x001cfa                  _ltoa
                  0x0003aa                  _main
                  0x001d1e                  _memcmp
                  0x001d4c                  _memcpy
                  0x001d5e                  _memmove
                  0x001d84                  _memset
                  0x03c16c                  _ntpServer
                  0x03c160                  _ntpServerPort
                  0x03c1ca                  _ntpTimeRecv
                  0x02bf28                  _pbkdf2_sha1
                  0x0076b5                  _pingCmd
                  0x0076ba                  _pingHelp
                  0x00767c                  _resetCmd
                  0x007682                  _resetHelp
                  0x0076a3                  _seeDocHelp
                  0x02bcde                  _sha1_prf
                  0x02bd82                  _sha1_t_prf
                  0x02bfd4                  _sha1_transform
                  0x02bf88                  _sha1_vector
                  0x0015f0                  _speedBoostKeep
                  0x00165a                  _speedBoostKeepLow
                  0x0016c2                  _speedBoostReset
                  0x0014c4                  _speedBoostStart
                  0x00158e                  _speedBoostValidate
                  0x001d96                  _strchr
                  0x001dae                  _strcmp
                  0x001dc0                  _strcpy
                  0x03fc6c                  _stricmppgm2ram
                  0x001dd0                  _strlen
                  0x03fe8a                  _strnchr
                  0x001de2                  _strncmp
                  0x001e08                  _strncpy
                  0x03fed8                  _strncpy_m
                  0x001a32                  _strtod
                  0x001f42                  _strtol
                  0x001e2e                  _strtoul
                  0x03fe02                  _strupr
                  0x03fd20                  _swapl
                  0x03fd04                  _swaps
                  0x03c7ae                  _timeBiasFromStr
                  0x03c73e                  _timeBiasStr
                  0x001708                  _toupper
                  0x03c23c                  _tzInfoHasDayLight
                  0x03c214                  _tzInfoIsUtc
                  0x03c25c                  _tzInfoMakeDate
                  0x03c47c                  _tzInfoToLocalTime
                  0x03c634                  _tzInfoToUtcTime
                  0x03fb38                  _uitoa
                  0x001caa                  _ultoa
                  0x00218e                  _vfprintf
                  0x001fce                  _vsnprintf
                  0x044f80                  _wifiConnectCheck
                  0x044f4e                  _wifiConnectError
                  0x044f3a                  _wifiConnectOk
                  0x044fe0                  _wifiConnectRetry
                  0x044f46                  _wifiDhcpOk
                  0x0407ec                  _wslog
                  0x040f38                  _wslogEnum
                  0x040b3a                  _wslogReset
                  0x040fcc                  _wslogSeekNext
                  0x04100a                  _wslogTimeAdjust
                  0x041034                  _wslogTimeAdjustRestart
                  0x040b5a                  _wslogWrite
                  0x040a08                  _wslogf
                  0x03c00e                  _wstickStr
                  0x03b96e                  _wstimeDecode
                  0x03b768                  _wstimeEncode
                  0x03c14c                  _wstimeGet
                  0x03c0c8                  _wstimeLowGet
                  0x03bb62                  _wstimeMonthLength
                  0x03c0e2                  _wstimeSet
                  0x03c3c0                  _wstimeStDiff
                  0x03bc16                  _wstimeStToStr
                  0x03bfdc                  _wstimeStr
                  0x03bfa8                  _wstimeToStr
                  0x03bbe6                  _wstimeWeekDay
                  0x006f78                  _wstime_month
                  0x006f14                  _wstime_weekDay
                  0x0409e6                  _wsvlogf

Memory Configuration

Name             Origin             Length             Attributes
data             0x001000           0x00d000           a !xr
reset            0x000000           0x000004  
ivt              0x000004           0x0001fc  
program          0x000200           0x0555fe           xr
auxflash         0x7fc000           0x003ff8           xr
FGS              0xf80004           0x000002  
FOSCSEL          0xf80006           0x000002  
FOSC             0xf80008           0x000002  
FWDT             0xf8000a           0x000002  
FPOR             0xf8000c           0x000002  
FICD             0xf8000e           0x000002  
FAS              0xf80010           0x000002  
FUID0            0xf80012           0x000002  
*default*        0x000000           0xffffffff  

Linker script and memory map

LOAD build/XC16-EX16_MRF24WB/production/_ext/1954962658/ARP.o
LOAD build/XC16-EX16_MRF24WB/production/_ext/1954962658/Announce.o
LOAD build/XC16-EX16_MRF24WB/production/_ext/1954962658/AutoIP.o
LOAD build/XC16-EX16_MRF24WB/production/_ext/1954962658/BerkeleyAPI.o
LOAD build/XC16-EX16_MRF24WB/production/_ext/1954962658/DHCP.o
LOAD build/XC16-EX16_MRF24WB/production/_ext/1954962658/DHCPs.o
LOAD build/XC16-EX16_MRF24WB/production/_ext/1954962658/DNS.o
LOAD build/XC16-EX16_MRF24WB/production/_ext/1954962658/DNSs.o
LOAD build/XC16-EX16_MRF24WB/production/_ext/1954962658/Delay.o
LOAD build/XC16-EX16_MRF24WB/production/_ext/1954962658/DynDNS.o
LOAD build/XC16-EX16_MRF24WB/production/_ext/1954962658/ENC28J60.o
LOAD build/XC16-EX16_MRF24WB/production/_ext/1954962658/ENCX24J600.o
LOAD build/XC16-EX16_MRF24WB/production/_ext/1954962658/FTP.o
LOAD build/XC16-EX16_MRF24WB/production/_ext/1954962658/Hashes.o
LOAD build/XC16-EX16_MRF24WB/production/_ext/1954962658/Helpers.o
LOAD build/XC16-EX16_MRF24WB/production/_ext/1954962658/ICMP.o
LOAD build/XC16-EX16_MRF24WB/production/_ext/1954962658/IP.o
LOAD build/XC16-EX16_MRF24WB/production/_ext/1954962658/LCDBlocking.o
LOAD build/XC16-EX16_MRF24WB/production/_ext/1954962658/NBNS.o
LOAD build/XC16-EX16_MRF24WB/production/_ext/1954962658/Reboot.o
LOAD build/XC16-EX16_MRF24WB/production/_ext/1954962658/SMTP.o
LOAD build/XC16-EX16_MRF24WB/production/_ext/1954962658/SNMP.o
LOAD build/XC16-EX16_MRF24WB/production/_ext/1954962658/SNTP.o
LOAD build/XC16-EX16_MRF24WB/production/_ext/1954962658/SPIEEPROM.o
LOAD build/XC16-EX16_MRF24WB/production/_ext/1954962658/SPIFlash.o
LOAD build/XC16-EX16_MRF24WB/production/_ext/1954962658/SPIRAM.o
LOAD build/XC16-EX16_MRF24WB/production/_ext/1954962658/StackTsk.o
LOAD build/XC16-EX16_MRF24WB/production/_ext/1954962658/TCP.o
LOAD build/XC16-EX16_MRF24WB/production/_ext/1954962658/TCPPerformanceTest.o
LOAD build/XC16-EX16_MRF24WB/production/_ext/1954962658/TFTPc.o
LOAD build/XC16-EX16_MRF24WB/production/_ext/1954962658/Telnet.o
LOAD build/XC16-EX16_MRF24WB/production/_ext/1954962658/Tick.o
LOAD build/XC16-EX16_MRF24WB/production/_ext/1954962658/UART.o
LOAD build/XC16-EX16_MRF24WB/production/_ext/1954962658/UART2TCPBridge.o
LOAD build/XC16-EX16_MRF24WB/production/_ext/1954962658/UDP.o
LOAD build/XC16-EX16_MRF24WB/production/_ext/1954962658/UDPPerformanceTest.o
LOAD build/XC16-EX16_MRF24WB/production/_ext/1954962658/ZeroconfHelper.o
LOAD build/XC16-EX16_MRF24WB/production/_ext/1954962658/ZeroconfLinkLocal.o
LOAD build/XC16-EX16_MRF24WB/production/_ext/1954962658/ZeroconfMulticastDNS.o
LOAD build/XC16-EX16_MRF24WB/production/_ext/243675038/WFConnectionAlgorithm.o
LOAD build/XC16-EX16_MRF24WB/production/_ext/243675038/WFConnectionManager.o
LOAD build/XC16-EX16_MRF24WB/production/_ext/243675038/WFConnectionProfile.o
LOAD build/XC16-EX16_MRF24WB/production/_ext/243675038/WFConsole.o
LOAD build/XC16-EX16_MRF24WB/production/_ext/243675038/WFConsoleIfconfig.o
LOAD build/XC16-EX16_MRF24WB/production/_ext/243675038/WFConsoleIwconfig.o
LOAD build/XC16-EX16_MRF24WB/production/_ext/243675038/WFConsoleIwpriv.o
LOAD build/XC16-EX16_MRF24WB/production/_ext/243675038/WFConsoleMsgHandler.o
LOAD build/XC16-EX16_MRF24WB/production/_ext/243675038/WFConsoleMsgs.o
LOAD build/XC16-EX16_MRF24WB/production/_ext/243675038/WFDataTxRx.o
LOAD build/XC16-EX16_MRF24WB/production/_ext/243675038/WFDriverCom.o
LOAD build/XC16-EX16_MRF24WB/production/_ext/243675038/WFDriverRaw.o
LOAD build/XC16-EX16_MRF24WB/production/_ext/243675038/WFEasyConfig.o
LOAD build/XC16-EX16_MRF24WB/production/_ext/243675038/WFEventHandler.o
LOAD build/XC16-EX16_MRF24WB/production/_ext/243675038/WFInit.o
LOAD build/XC16-EX16_MRF24WB/production/_ext/243675038/WFMac.o
LOAD build/XC16-EX16_MRF24WB/production/_ext/243675038/WFMgmtMsg.o
LOAD build/XC16-EX16_MRF24WB/production/_ext/243675038/WFParamMsg.o
LOAD build/XC16-EX16_MRF24WB/production/_ext/243675038/WFPowerSave.o
LOAD build/XC16-EX16_MRF24WB/production/_ext/243675038/WFScan.o
LOAD build/XC16-EX16_MRF24WB/production/_ext/243675038/WFTxPower.o
LOAD build/XC16-EX16_MRF24WB/production/_ext/243675038/WF_Eint.o
LOAD build/XC16-EX16_MRF24WB/production/_ext/243675038/WF_Spi.o
LOAD build/XC16-EX16_MRF24WB/production/_ext/243675038/WFDebugStrings.o
LOAD build/XC16-EX16_MRF24WB/production/_ext/243675038/WF_pbkdf2.o
LOAD build/XC16-EX16_MRF24WB/production/_ext/1472/UARTConfig.o
LOAD build/XC16-EX16_MRF24WB/production/_ext/1472/WF_Config.o
LOAD build/XC16-EX16_MRF24WB/production/_ext/1472/HTTP2.o
LOAD build/XC16-EX16_MRF24WB/production/_ext/1472/MPFS2.o
LOAD build/XC16-EX16_MRF24WB/production/_ext/1472/WiSteerHTTP.o
LOAD build/XC16-EX16_MRF24WB/production/_ext/1472/WiSteerMain.o
LOAD build/XC16-EX16_MRF24WB/production/_ext/1472/WiSteerHTTPtools.o
LOAD build/XC16-EX16_MRF24WB/production/_ext/1472/WiSteerUpdate.o
LOAD build/XC16-EX16_MRF24WB/production/WiSteerUpdateHlp.o
LOAD build/XC16-EX16_MRF24WB/production/_ext/1472/WiSteerLog.o
LOAD build/XC16-EX16_MRF24WB/production/_ext/1472/WiSteerTime.o
LOAD build/XC16-EX16_MRF24WB/production/_ext/1472/WiSteerCom.o
LOAD build/XC16-EX16_MRF24WB/production/_ext/1472/WiSteerAction.o
LOAD build/XC16-EX16_MRF24WB/production/_ext/1472/WiSteerMpfsSource.o
LOAD build/XC16-EX16_MRF24WB/production/_ext/1472/WiSteerStructSizeCheck.o
LOAD build/XC16-EX16_MRF24WB/production/_ext/1472/pic32helpers.o
                    0x0001                  __MPLAB_BUILD = 0x1
LOAD c:/program files (x86)/microchip/xc16/v1.20/bin/bin/../../lib/PIC24E\libp24EP512GU810-elf.a
                    0xf80004                  __FGS = 0xf80004
                    0xf80006                  __FOSCSEL = 0xf80006
                    0xf80008                  __FOSC = 0xf80008
                    0xf8000a                  __FWDT = 0xf8000a
                    0xf8000c                  __FPOR = 0xf8000c
                    0xf8000e                  __FICD = 0xf8000e
                    0xf80010                  __FAS = 0xf80010
                    0xf80012                  __FUID0 = 0xf80012
                    0x0004                  __IVT_BASE = 0x4
                    0x1000                  __DATA_BASE = 0x1000
                    0xd000                  __DATA_LENGTH = 0xd000
                    0xd000                  __DMA_BASE = 0xd000
                    0xdfff                  __DMA_END = 0xdfff
                    0x7fc000                  __CODE_BASE = 0x7fc000
                    0x3ffa                  __CODE_LENGTH = 0x3ffa

.reset            0x000000          0x4
                  0x000000          0x2 SHORT 0x200 ABSOLUTE (__reset)
                  0x000001          0x2 SHORT 0x4
                  0x000002          0x2 SHORT 0x0 ((ABSOLUTE (__reset) >> 0x10) & 0x7f)
                  0x000003          0x2 SHORT 0x0

.text             0x000200       0x4bde
 *(.init)
 .init            0x000200         0x32 c:/program files (x86)/microchip/xc16/v1.20/bin/bin/../../lib\libpic30-elf.a(crt0_extendedep.o)
                  0x000200                  __resetPRI
                  0x000200                  __reset
                  0x000226                  __psv_init
 .init            0x000232         0x9a c:/program files (x86)/microchip/xc16/v1.20/bin/bin/../../lib\libpic30-elf.a(data_init_extendedep.o)
                  0x000232                  __data_init
                  0x000232                  __data_init_extended
 *(.user_init)
 *(.handle)
 .handle          0x0002cc          0xc jump_table
 *(.isr*)
 .isr.text        0x0002d8       0x13f0 build/XC16-EX16_MRF24WB/production/_ext/1472/WiSteerMain.o
                  0x0002d8                  __DefaultInterrupt
                  0x000302                  __OscillatorFail
                  0x00032c                  __AddressError
                  0x000356                  __StackError
                  0x000380                  __MathError
                  0x0003aa                  _main
                  0x000640                  _WF_Connect
                  0x000756                  _DisplayIPValue
                  0x0008d4                  _DefaultAppConfig
                  0x000a06                  _LoadAppConfig
                  0x000b7e                  _UpgradeAppConfig
                  0x000bf0                  _AppConfigUseWiFiMacAddress
                  0x000dda                  _SaveAppConfig
                  0x000e52                  _RestoreWifiConfig
                  0x000e86                  _LED_PUT
                  0x000f64                  _activityLedsOn
                  0x000f9a                  _activityLedsModeChange
                  0x000fbe                  _OnMdnsHostNameChanged
                  0x000fc6                  _deviceReinit
                  0x00102e                  _deviceGet
                  0x001100                  _deviceFind
                  0x00117c                  _deviceWithOpToDoGet
                  0x001264                  _deviceIsGoodCfgShareSource
                  0x001334                  _deviceGoodCfgShareSourceEnd
                  0x001362                  _deviceId
                  0x001380                  _deviceCmdAdd
                  0x001430                  _deviceCmdEnd
                  0x0014c4                  _speedBoostStart
                  0x00158e                  _speedBoostValidate
                  0x0015f0                  _speedBoostKeep
                  0x00165a                  _speedBoostKeepLow
                  0x0016c2                  _speedBoostReset
 *(.libc)
 .libc            0x0016c8         0x14 c:/program files (x86)/microchip/xc16/v1.20/bin/bin/../../lib\libc-elf.a(isalpha.epeso)
                  0x0016c8                  _isalpha
 .libc            0x0016dc         0x10 c:/program files (x86)/microchip/xc16/v1.20/bin/bin/../../lib\libc-elf.a(isspace.epeso)
                  0x0016dc                  _isspace
 .libc            0x0016ec         0x1c c:/program files (x86)/microchip/xc16/v1.20/bin/bin/../../lib\libc-elf.a(isxdigit.epeso)
                  0x0016ec                  _isxdigit
 .libc            0x001708          0xe c:/program files (x86)/microchip/xc16/v1.20/bin/bin/../../lib\libc-elf.a(toupper.epeso)
                  0x001708                  _toupper
 *(.libm)
 *(.libdsp)
 *(.lib*)
 .libm.divsi3     0x001716         0x1e c:/program files (x86)/microchip/xc16/v1.20/bin/bin/../../lib\libm-elf.a(divsi3.epeo)
                  0x001716                  ___divsi3
 .libm.modsi3     0x001734         0x1e c:/program files (x86)/microchip/xc16/v1.20/bin/bin/../../lib\libm-elf.a(modsi3.epeo)
                  0x001734                  ___modsi3
 .libm.udivsi3    0x001752         0x20 c:/program files (x86)/microchip/xc16/v1.20/bin/bin/../../lib\libm-elf.a(udivsi3.epeo)
                  0x001752                  ___udivsi3
 .libm.umodsi3    0x001772          0x6 c:/program files (x86)/microchip/xc16/v1.20/bin/bin/../../lib\libm-elf.a(umodsi3.epeo)
                  0x001772                  ___umodsi3
 .libm.__PplusBdi.__PplusBdi
                  0x001778         0x2c c:/program files (x86)/microchip/xc16/v1.20/bin/bin/../../lib\libm-elf.a(divmoddi3.epeo)
 .libm.__PminusBdi.__PminusBdi
                  0x0017a4         0x42 c:/program files (x86)/microchip/xc16/v1.20/bin/bin/../../lib\libm-elf.a(divmoddi3.epeo)
 .libm.__udivmoddi3.__udivmoddi3
                  0x0017e6         0xd0 c:/program files (x86)/microchip/xc16/v1.20/bin/bin/../../lib\libm-elf.a(divmoddi3.epeo)
                  0x0017e6                  ___udivmoddi3
 .libm.__udivdi3.__udivdi3
                  0x0018b6         0x12 c:/program files (x86)/microchip/xc16/v1.20/bin/bin/../../lib\libm-elf.a(divmoddi3.epeo)
                  0x0018b6                  ___udivdi3
 .libm.__umoddi3.__umoddi3
                  0x0018c8          0xc c:/program files (x86)/microchip/xc16/v1.20/bin/bin/../../lib\libm-elf.a(divmoddi3.epeo)
                  0x0018c8                  ___umoddi3
 .libm.__divdi3.__divdi3
                  0x0018d4         0x64 c:/program files (x86)/microchip/xc16/v1.20/bin/bin/../../lib\libm-elf.a(divmoddi3.epeo)
                  0x0018d4                  ___divdi3
 .libm.__moddi3.__moddi3
                  0x001938         0x60 c:/program files (x86)/microchip/xc16/v1.20/bin/bin/../../lib\libm-elf.a(divmoddi3.epeo)
                  0x001938                  ___moddi3
 .libm.__muldi3.__muldi3
                  0x001998         0x56 c:/program files (x86)/microchip/xc16/v1.20/bin/bin/../../lib\libm-elf.a(muldi3.epeo)
                  0x001998                  ___muldi3
 .libm.umuldi3    0x0019ee         0x44 c:/program files (x86)/microchip/xc16/v1.20/bin/bin/../../lib\libm-elf.a(umuldi3.epeo)
                  0x0019ee                  ___umuldi3
 .libc.strtod.strtod
                  0x001a32        0x1d2 c:/program files (x86)/microchip/xc16/v1.20/bin/bin/../../lib\libc-elf.a(atof.epeo)
                  0x001a32                  _strtod
 .libc.atof.atof
                  0x001c04          0xa c:/program files (x86)/microchip/xc16/v1.20/bin/bin/../../lib\libc-elf.a(atof.epeo)
                  0x001c04                  _atof
 .libc.atoi.atoi
                  0x001c0e         0x42 c:/program files (x86)/microchip/xc16/v1.20/bin/bin/../../lib\libc-elf.a(atoi.epeo)
                  0x001c0e                  _atoi
 .libc.atol.atol
                  0x001c50         0x5a c:/program files (x86)/microchip/xc16/v1.20/bin/bin/../../lib\libc-elf.a(atol.epeo)
                  0x001c50                  _atol
 .libc.ultoa.ultoa
                  0x001caa         0x50 c:/program files (x86)/microchip/xc16/v1.20/bin/bin/../../lib\libc-elf.a(ltoa.epeo)
                  0x001caa                  _ultoa
 .libc.ltoa.ltoa
                  0x001cfa         0x24 c:/program files (x86)/microchip/xc16/v1.20/bin/bin/../../lib\libc-elf.a(ltoa.epeo)
                  0x001cfa                  _ltoa
 .libc.memcmp.memcmp
                  0x001d1e         0x2e c:/program files (x86)/microchip/xc16/v1.20/bin/bin/../../lib\libc-elf.a(memcmp.epeo)
                  0x001d1e                  _memcmp
 .libc.memcpy.memcpy
                  0x001d4c         0x12 c:/program files (x86)/microchip/xc16/v1.20/bin/bin/../../lib\libc-elf.a(memcpy.epeo)
                  0x001d4c                  _memcpy
 .libc.memmove.memmove
                  0x001d5e         0x26 c:/program files (x86)/microchip/xc16/v1.20/bin/bin/../../lib\libc-elf.a(memmove.epeo)
                  0x001d5e                  _memmove
 .libc.memset.memset
                  0x001d84         0x12 c:/program files (x86)/microchip/xc16/v1.20/bin/bin/../../lib\libc-elf.a(memset.epeo)
                  0x001d84                  _memset
 .libc.strchr.strchr
                  0x001d96         0x18 c:/program files (x86)/microchip/xc16/v1.20/bin/bin/../../lib\libc-elf.a(strchr.epeo)
                  0x001d96                  _strchr
 .libc.strcmp.strcmp
                  0x001dae         0x12 c:/program files (x86)/microchip/xc16/v1.20/bin/bin/../../lib\libc-elf.a(strcmp.epeo)
                  0x001dae                  _strcmp
 .libc.strcpy.strcpy
                  0x001dc0         0x10 c:/program files (x86)/microchip/xc16/v1.20/bin/bin/../../lib\libc-elf.a(strcpy.epeo)
                  0x001dc0                  _strcpy
 .libc.strlen.strlen
                  0x001dd0         0x12 c:/program files (x86)/microchip/xc16/v1.20/bin/bin/../../lib\libc-elf.a(strlen.epeo)
                  0x001dd0                  _strlen
 .libc.strncmp.strncmp
                  0x001de2         0x26 c:/program files (x86)/microchip/xc16/v1.20/bin/bin/../../lib\libc-elf.a(strncmp.epeo)
                  0x001de2                  _strncmp
 .libc.strncpy.strncpy
                  0x001e08         0x26 c:/program files (x86)/microchip/xc16/v1.20/bin/bin/../../lib\libc-elf.a(strncpy.epeo)
                  0x001e08                  _strncpy
 .libc.strtoul.strtoul
                  0x001e2e        0x114 c:/program files (x86)/microchip/xc16/v1.20/bin/bin/../../lib\libc-elf.a(strtol.epeo)
                  0x001e2e                  _strtoul
 .libc.strtol.strtol
                  0x001f42         0x8c c:/program files (x86)/microchip/xc16/v1.20/bin/bin/../../lib\libc-elf.a(strtol.epeo)
                  0x001f42                  _strtol
 .libc.vsnprintf.vsnprintf
                  0x001fce         0x2a c:/program files (x86)/microchip/xc16/v1.20/bin/bin/../../lib\libc-elf.a(vsnprintf.epeo)
                  0x001fce                  _vsnprintf
 .libc._snprintf_cdfFnopsuxX._snprintf_cdfFnopsuxX
                  0x001ff8          0xc c:/program files (x86)/microchip/xc16/v1.20/bin/bin/../../lib\libc-elf.a(snprintf_cdfFnopsuxX.EPeo)
                  0x001ff8                  __snprintf_cdnopsuxX
                  0x001ff8                  __snprintf_cdnopuxX
                  0x001ff8                  __snprintf_cdfFnopsuxX
                  0x001ff8                  __snprintf_cdfFnopuxX
 .libc._vsnprintf_cdfFnopsuxX._vsnprintf_cdfFnopsuxX
                  0x002004         0x2a c:/program files (x86)/microchip/xc16/v1.20/bin/bin/../../lib\libc-elf.a(vsnprintf_cdfFnopsuxX.EPeo)
                  0x002004                  __vsnprintf_cdnopuxX
                  0x002004                  __vsnprintf_cdnopsuxX
                  0x002004                  __vsnprintf_cdfFnopsuxX
                  0x002004                  __vsnprintf_cdfFnopuxX
 .libc.fround.fround
                  0x00202e         0x98 c:/program files (x86)/microchip/xc16/v1.20/bin/bin/../../lib\libc-elf.a(doprnt.epeo)
 .libc.scale.scale
                  0x0020c6         0xc8 c:/program files (x86)/microchip/xc16/v1.20/bin/bin/../../lib\libc-elf.a(doprnt.epeo)
 .libc.vfprintf.vfprintf
                  0x00218e       0x14c4 c:/program files (x86)/microchip/xc16/v1.20/bin/bin/../../lib\libc-elf.a(doprnt.epeo)
                  0x00218e                  _vfprintf
 .libc.fputc.fputc
                  0x003652         0x8c c:/program files (x86)/microchip/xc16/v1.20/bin/bin/../../lib\libc-elf.a(fputc.epeo)
                  0x003652                  _fputc
 .libc.fround.fround
                  0x0036de         0x98 c:/program files (x86)/microchip/xc16/v1.20/bin/bin/../../lib\libc-elf.a(doprnt_cdfFnopsuxX.EPeo)
 .libc.scale.scale
                  0x003776         0xc8 c:/program files (x86)/microchip/xc16/v1.20/bin/bin/../../lib\libc-elf.a(doprnt_cdfFnopsuxX.EPeo)
 .libc._vfprintf_cdfFnopsuxX._vfprintf_cdfFnopsuxX
                  0x00383e        0xc78 c:/program files (x86)/microchip/xc16/v1.20/bin/bin/../../lib\libc-elf.a(doprnt_cdfFnopsuxX.EPeo)
                  0x00383e                  __vfprintf_cdnopuxX
                  0x00383e                  __vfprintf_cdnopsuxX
                  0x00383e                  __vfprintf_cdfFnopuxX
                  0x00383e                  __vfprintf_cdfFnopsuxX
 .libc._flsbuf._flsbuf
                  0x0044b6         0x80 c:/program files (x86)/microchip/xc16/v1.20/bin/bin/../../lib\libc-elf.a(flsbuf.epeo)
                  0x0044b6                  __flsbuf
 .libc.dowrite.dowrite
                  0x004536          0x8 c:/program files (x86)/microchip/xc16/v1.20/bin/bin/../../lib\libpic30-elf.a(writeep.eo)
 .libc.write      0x00453e         0x60 c:/program files (x86)/microchip/xc16/v1.20/bin/bin/../../lib\libpic30-elf.a(writeep.eo)
                  0x00453e                  _write
 .libm.adddf3     0x00459e         0xfa c:/program files (x86)/microchip/xc16/v1.20/bin/bin/../../lib\libm-elf.a(adddf3.epeo)
                  0x00459e                  ___adddf3
 .libm.eqdf2      0x004698          0xa c:/program files (x86)/microchip/xc16/v1.20/bin/bin/../../lib\libm-elf.a(deqltle.epeo)
                  0x004698                  ___eqdf2
                  0x004698                  ___ltdf2
                  0x004698                  ___ledf2
 .libm.gtdf2      0x0046a2          0xa c:/program files (x86)/microchip/xc16/v1.20/bin/bin/../../lib\libm-elf.a(dgtge.epeo)
                  0x0046a2                  ___gtdf2
                  0x0046a2                  ___gedf2
 .libm.divdf3     0x0046ac         0xb4 c:/program files (x86)/microchip/xc16/v1.20/bin/bin/../../lib\libm-elf.a(divdf3.epeo)
                  0x0046ac                  ___divdf3
 .libm.divfs3     0x004760         0x84 c:/program files (x86)/microchip/xc16/v1.20/bin/bin/../../lib\libm-elf.a(divsf3.epeo)
                  0x004760                  ___divsf3
 .libm.nedf2      0x0047e4          0xa c:/program files (x86)/microchip/xc16/v1.20/bin/bin/../../lib\libm-elf.a(dne.epeo)
                  0x0047e4                  ___nedf2
 .libm.dpack      0x0047ee         0x58 c:/program files (x86)/microchip/xc16/v1.20/bin/bin/../../lib\libm-elf.a(dpack.epeo)
                  0x0047ee                  __dpack
 .libm.dunpack2
                  0x004846         0x32 c:/program files (x86)/microchip/xc16/v1.20/bin/bin/../../lib\libm-elf.a(dunpack2.epeo)
                  0x004846                  __dunpack2
                  0x004868                  __dreturnNaN
                  0x00486e                  __dunpack2exit
 .libm.extendsfdf2
                  0x004878         0x3e c:/program files (x86)/microchip/xc16/v1.20/bin/bin/../../lib\libm-elf.a(extendsfdf.epeo)
                  0x004878                  ___extendsfdf2
 .libm.eqsf2      0x0048b6          0x4 c:/program files (x86)/microchip/xc16/v1.20/bin/bin/../../lib\libm-elf.a(feqltle.epeo)
                  0x0048b6                  ___eqsf2
                  0x0048b6                  ___ltsf2
                  0x0048b6                  ___lesf2
 .libm.gtsf2      0x0048ba          0x4 c:/program files (x86)/microchip/xc16/v1.20/bin/bin/../../lib\libm-elf.a(fgtge.epeo)
                  0x0048ba                  ___gesf2
                  0x0048ba                  ___gtsf2
 .libm.fixunsdfdi
                  0x0048be         0x62 c:/program files (x86)/microchip/xc16/v1.20/bin/bin/../../lib\libm-elf.a(fixunsdfdi.epeo)
                  0x0048be                  ___fixunsdfdi
 .libm.fixunsdfsi
                  0x004920         0x4c c:/program files (x86)/microchip/xc16/v1.20/bin/bin/../../lib\libm-elf.a(fixunsdfsi.epeo)
                  0x004920                  ___fixunsdfsi
 .libm.floatsisf
                  0x00496c          0x6 c:/program files (x86)/microchip/xc16/v1.20/bin/bin/../../lib\libm-elf.a(floatsisf.epeo)
                  0x00496c                  ___floatsisf
 .libm.floatundidf
                  0x004972         0x56 c:/program files (x86)/microchip/xc16/v1.20/bin/bin/../../lib\libm-elf.a(floatundidf.epeo)
                  0x004972                  ___floatundidf
 .libm.floatunsidf
                  0x0049c8          0x4 c:/program files (x86)/microchip/xc16/v1.20/bin/bin/../../lib\libm-elf.a(floatunsidf.epeo)
                  0x0049c8                  ___floatunsidf
 .libm.fpack      0x0049cc         0x4c c:/program files (x86)/microchip/xc16/v1.20/bin/bin/../../lib\libm-elf.a(fpack.epeo)
                  0x0049cc                  __fpack
 .libm.frexpf     0x004a18          0x6 c:/program files (x86)/microchip/xc16/v1.20/bin/bin/../../lib\libm-elf.a(frexpf.epeo)
                  0x004a18                  _frexpf
 .libm.funpack    0x004a1e         0x2a c:/program files (x86)/microchip/xc16/v1.20/bin/bin/../../lib\libm-elf.a(funpack.epeo)
                  0x004a1e                  __funpack
 .libm.funpack2
                  0x004a48         0x10 c:/program files (x86)/microchip/xc16/v1.20/bin/bin/../../lib\libm-elf.a(funpack2.epeo)
                  0x004a48                  __funpack2
 .libm.fPropagateNaN
                  0x004a58         0x12 c:/program files (x86)/microchip/xc16/v1.20/bin/bin/../../lib\libm-elf.a(futil.epeo)
                  0x004a58                  __fPropagateNaN
 .libm.fbobExit
                  0x004a6a          0x8 c:/program files (x86)/microchip/xc16/v1.20/bin/bin/../../lib\libm-elf.a(futil.epeo)
                  0x004a6a                  __fbopExit
 .libm.fbopReturnNaN
                  0x004a72          0x6 c:/program files (x86)/microchip/xc16/v1.20/bin/bin/../../lib\libm-elf.a(futil.epeo)
                  0x004a72                  __fbopReturnNaN
 .libm.muldf3     0x004a78         0xea c:/program files (x86)/microchip/xc16/v1.20/bin/bin/../../lib\libm-elf.a(muldf3.epeo)
                  0x004a78                  ___muldf3
 .libm.mulsf3     0x004b62         0x68 c:/program files (x86)/microchip/xc16/v1.20/bin/bin/../../lib\libm-elf.a(mulsf3.epeo)
                  0x004b62                  ___mulsf3
 .libm.subdf3     0x004bca          0x4 c:/program files (x86)/microchip/xc16/v1.20/bin/bin/../../lib\libm-elf.a(subdf3.epeo)
                  0x004bca                  ___subdf3
 .libm.truncdfsf2
                  0x004bce         0x56 c:/program files (x86)/microchip/xc16/v1.20/bin/bin/../../lib\libm-elf.a(truncdfsf.epeo)
                  0x004bce                  ___truncdfsf2
 .libm.mulsi3     0x004c24          0xc c:/program files (x86)/microchip/xc16/v1.20/bin/bin/../../lib\libm-elf.a(mulsi3.epeo)
                  0x004c24                  ___mulp32peds3
                  0x004c24                  ___mulsi3
                  0x004c24                  ___mulp32eds3
 .libm.frexpf     0x004c30         0x1a c:/program files (x86)/microchip/xc16/v1.20/bin/bin/../../lib\libm-elf.a(_frexpf.epeo)
                  0x004c30                  __frexpf
 .libm.dcompare
                  0x004c4a         0x52 c:/program files (x86)/microchip/xc16/v1.20/bin/bin/../../lib\libm-elf.a(dcompare.epeo)
                  0x004c4a                  __dcompare
 .libm.dPropagateNaN
                  0x004c9c         0x1c c:/program files (x86)/microchip/xc16/v1.20/bin/bin/../../lib\libm-elf.a(dpropagateNaN.epeo)
                  0x004c9c                  __dPropagateNaN
 .libm.dtype      0x004cb8         0x24 c:/program files (x86)/microchip/xc16/v1.20/bin/bin/../../lib\libm-elf.a(dtype.epeo)
                  0x004cb8                  __dtype
 .libm.dunpack    0x004cdc         0x4e c:/program files (x86)/microchip/xc16/v1.20/bin/bin/../../lib\libm-elf.a(dunpack.epeo)
                  0x004cdc                  __dunpack
 .libm.fcompare
                  0x004d2a         0x36 c:/program files (x86)/microchip/xc16/v1.20/bin/bin/../../lib\libm-elf.a(fcompare.epeo)
                  0x004d2a                  __fcompare
 .libm.floatdisf
                  0x004d60         0x20 c:/program files (x86)/microchip/xc16/v1.20/bin/bin/../../lib\libm-elf.a(floatdisf.epeo)
                  0x004d60                  ___floatdisf
 .libm.floatundisf
                  0x004d80         0x5e c:/program files (x86)/microchip/xc16/v1.20/bin/bin/../../lib\libm-elf.a(floatundisf.epeo)
                  0x004d80                  ___floatundisf

usercode
 *(usercode)

__FGS
 *(__FGS.sec*)

__FOSCSEL         0xf80006          0x2
 *(__FOSCSEL.sec*)
 __FOSCSEL.sec    0xf80006          0x2 build/XC16-EX16_MRF24WB/production/_ext/1472/WiSteerMain.o

__FOSC            0xf80008          0x2
 *(__FOSC.sec*)
 __FOSC.sec       0xf80008          0x2 build/XC16-EX16_MRF24WB/production/_ext/1472/WiSteerMain.o

__FWDT            0xf8000a          0x2
 *(__FWDT.sec*)
 __FWDT.sec       0xf8000a          0x2 build/XC16-EX16_MRF24WB/production/_ext/1472/WiSteerMain.o

__FPOR
 *(__FPOR.sec*)

__FICD
 *(__FICD.sec*)

__FAS
 *(__FAS.sec*)

__FUID0
 *(__FUID0.sec*)

.comment
 *(.comment)

.debug_info       0x000000      0x3813a
 *(.debug_info)
 .debug_info      0x000000        0xc85 build/XC16-EX16_MRF24WB/production/_ext/1954962658/ARP.o
 .debug_info      0x000c85        0x158 build/XC16-EX16_MRF24WB/production/_ext/1954962658/Announce.o
 .debug_info      0x000ddd        0x156 build/XC16-EX16_MRF24WB/production/_ext/1954962658/AutoIP.o
 .debug_info      0x000f33        0x15b build/XC16-EX16_MRF24WB/production/_ext/1954962658/BerkeleyAPI.o
 .debug_info      0x00108e       0x12b7 build/XC16-EX16_MRF24WB/production/_ext/1954962658/DHCP.o
 .debug_info      0x002345       0x13bc build/XC16-EX16_MRF24WB/production/_ext/1954962658/DHCPs.o
 .debug_info      0x003701        0xea7 build/XC16-EX16_MRF24WB/production/_ext/1954962658/DNS.o
 .debug_info      0x0045a8        0xc06 build/XC16-EX16_MRF24WB/production/_ext/1954962658/DNSs.o
 .debug_info      0x0051ae        0x1ea build/XC16-EX16_MRF24WB/production/_ext/1954962658/Delay.o
 .debug_info      0x005398        0x156 build/XC16-EX16_MRF24WB/production/_ext/1954962658/DynDNS.o
 .debug_info      0x0054ee        0x10d build/XC16-EX16_MRF24WB/production/_ext/1954962658/ENC28J60.o
 .debug_info      0x0055fb        0x10f build/XC16-EX16_MRF24WB/production/_ext/1954962658/ENCX24J600.o
 .debug_info      0x00570a        0x153 build/XC16-EX16_MRF24WB/production/_ext/1954962658/FTP.o
 .debug_info      0x00585d        0x524 build/XC16-EX16_MRF24WB/production/_ext/1954962658/Hashes.o
 .debug_info      0x005d81       0x107e build/XC16-EX16_MRF24WB/production/_ext/1954962658/Helpers.o
 .debug_info      0x006dff        0x74a build/XC16-EX16_MRF24WB/production/_ext/1954962658/ICMP.o
 .debug_info      0x007549        0xca6 build/XC16-EX16_MRF24WB/production/_ext/1954962658/IP.o
 .debug_info      0x0081ef        0x8f0 build/XC16-EX16_MRF24WB/production/_ext/1954962658/LCDBlocking.o
 .debug_info      0x008adf        0xd8c build/XC16-EX16_MRF24WB/production/_ext/1954962658/NBNS.o
 .debug_info      0x00986b        0x156 build/XC16-EX16_MRF24WB/production/_ext/1954962658/Reboot.o
 .debug_info      0x0099c1        0x154 build/XC16-EX16_MRF24WB/production/_ext/1954962658/SMTP.o
 .debug_info      0x009b15        0x154 build/XC16-EX16_MRF24WB/production/_ext/1954962658/SNMP.o
 .debug_info      0x009c69        0x515 build/XC16-EX16_MRF24WB/production/_ext/1954962658/SNTP.o
 .debug_info      0x00a17e       0x11a7 build/XC16-EX16_MRF24WB/production/_ext/1954962658/SPIEEPROM.o
 .debug_info      0x00b325        0x10d build/XC16-EX16_MRF24WB/production/_ext/1954962658/SPIFlash.o
 .debug_info      0x00b432        0x10b build/XC16-EX16_MRF24WB/production/_ext/1954962658/SPIRAM.o
 .debug_info      0x00b53d        0xc30 build/XC16-EX16_MRF24WB/production/_ext/1954962658/StackTsk.o
 .debug_info      0x00c16d       0x2329 build/XC16-EX16_MRF24WB/production/_ext/1954962658/TCP.o
 .debug_info      0x00e496        0x162 build/XC16-EX16_MRF24WB/production/_ext/1954962658/TCPPerformanceTest.o
 .debug_info      0x00e5f8        0x155 build/XC16-EX16_MRF24WB/production/_ext/1954962658/TFTPc.o
 .debug_info      0x00e74d        0x156 build/XC16-EX16_MRF24WB/production/_ext/1954962658/Telnet.o
 .debug_info      0x00e8a3        0xb31 build/XC16-EX16_MRF24WB/production/_ext/1954962658/Tick.o
 .debug_info      0x00f3d4        0x154 build/XC16-EX16_MRF24WB/production/_ext/1954962658/UART.o
 .debug_info      0x00f528        0x15e build/XC16-EX16_MRF24WB/production/_ext/1954962658/UART2TCPBridge.o
 .debug_info      0x00f686       0x12da build/XC16-EX16_MRF24WB/production/_ext/1954962658/UDP.o
 .debug_info      0x010960        0x162 build/XC16-EX16_MRF24WB/production/_ext/1954962658/UDPPerformanceTest.o
 .debug_info      0x010ac2        0x15e build/XC16-EX16_MRF24WB/production/_ext/1954962658/ZeroconfHelper.o
 .debug_info      0x010c20        0x161 build/XC16-EX16_MRF24WB/production/_ext/1954962658/ZeroconfLinkLocal.o
 .debug_info      0x010d81        0x164 build/XC16-EX16_MRF24WB/production/_ext/1954962658/ZeroconfMulticastDNS.o
 .debug_info      0x010ee5       0x15a1 build/XC16-EX16_MRF24WB/production/_ext/243675038/WFConnectionAlgorithm.o
 .debug_info      0x012486        0x83d build/XC16-EX16_MRF24WB/production/_ext/243675038/WFConnectionManager.o
 .debug_info      0x012cc3       0x1312 build/XC16-EX16_MRF24WB/production/_ext/243675038/WFConnectionProfile.o
 .debug_info      0x013fd5        0x15e build/XC16-EX16_MRF24WB/production/_ext/243675038/WFConsole.o
 .debug_info      0x014133        0x166 build/XC16-EX16_MRF24WB/production/_ext/243675038/WFConsoleIfconfig.o
 .debug_info      0x014299        0x166 build/XC16-EX16_MRF24WB/production/_ext/243675038/WFConsoleIwconfig.o
 .debug_info      0x0143ff        0x164 build/XC16-EX16_MRF24WB/production/_ext/243675038/WFConsoleIwpriv.o
 .debug_info      0x014563        0x28e build/XC16-EX16_MRF24WB/production/_ext/243675038/WFConsoleMsgHandler.o
 .debug_info      0x0147f1        0x5ab build/XC16-EX16_MRF24WB/production/_ext/243675038/WFConsoleMsgs.o
 .debug_info      0x014d9c        0x15f build/XC16-EX16_MRF24WB/production/_ext/243675038/WFDataTxRx.o
 .debug_info      0x014efb        0xe9b build/XC16-EX16_MRF24WB/production/_ext/243675038/WFDriverCom.o
 .debug_info      0x015d96        0xc24 build/XC16-EX16_MRF24WB/production/_ext/243675038/WFDriverRaw.o
 .debug_info      0x0169ba       0x1062 build/XC16-EX16_MRF24WB/production/_ext/243675038/WFEasyConfig.o
 .debug_info      0x017a1c        0x5a0 build/XC16-EX16_MRF24WB/production/_ext/243675038/WFEventHandler.o
 .debug_info      0x017fbc        0xcef build/XC16-EX16_MRF24WB/production/_ext/243675038/WFInit.o
 .debug_info      0x018cab       0x14f7 build/XC16-EX16_MRF24WB/production/_ext/243675038/WFMac.o
 .debug_info      0x01a1a2        0xb29 build/XC16-EX16_MRF24WB/production/_ext/243675038/WFMgmtMsg.o
 .debug_info      0x01accb       0x137f build/XC16-EX16_MRF24WB/production/_ext/243675038/WFParamMsg.o
 .debug_info      0x01c04a        0x160 build/XC16-EX16_MRF24WB/production/_ext/243675038/WFPowerSave.o
 .debug_info      0x01c1aa        0x7ca build/XC16-EX16_MRF24WB/production/_ext/243675038/WFScan.o
 .debug_info      0x01c974        0x97d build/XC16-EX16_MRF24WB/production/_ext/243675038/WFTxPower.o
 .debug_info      0x01d2f1        0x845 build/XC16-EX16_MRF24WB/production/_ext/243675038/WF_Eint.o
 .debug_info      0x01db36        0x8bd build/XC16-EX16_MRF24WB/production/_ext/243675038/WF_Spi.o
 .debug_info      0x01e3f3        0xcce build/XC16-EX16_MRF24WB/production/_ext/243675038/WFDebugStrings.o
 .debug_info      0x01f0c1        0xb3b build/XC16-EX16_MRF24WB/production/_ext/243675038/WF_pbkdf2.o
 .debug_info      0x01fbfc        0x13e build/XC16-EX16_MRF24WB/production/_ext/1472/UARTConfig.o
 .debug_info      0x01fd3a       0x1298 build/XC16-EX16_MRF24WB/production/_ext/1472/WF_Config.o
 .debug_info      0x020fd2       0x1337 build/XC16-EX16_MRF24WB/production/_ext/1472/HTTP2.o
 .debug_info      0x022309       0x10f8 build/XC16-EX16_MRF24WB/production/_ext/1472/MPFS2.o
 .debug_info      0x023401       0x6d5a build/XC16-EX16_MRF24WB/production/_ext/1472/WiSteerHTTP.o
 .debug_info      0x02a15b       0x3916 build/XC16-EX16_MRF24WB/production/_ext/1472/WiSteerMain.o
 .debug_info      0x02da71        0xc5e build/XC16-EX16_MRF24WB/production/_ext/1472/WiSteerHTTPtools.o
 .debug_info      0x02e6cf        0x14a build/XC16-EX16_MRF24WB/production/_ext/1472/WiSteerUpdate.o
 .debug_info      0x02e819         0x86 build/XC16-EX16_MRF24WB/production/WiSteerUpdateHlp.o
 .debug_info      0x02e89f       0x19c6 build/XC16-EX16_MRF24WB/production/_ext/1472/WiSteerLog.o
 .debug_info      0x030265       0x1a30 build/XC16-EX16_MRF24WB/production/_ext/1472/WiSteerTime.o
 .debug_info      0x031c95       0x3379 build/XC16-EX16_MRF24WB/production/_ext/1472/WiSteerCom.o
 .debug_info      0x03500e       0x2f36 build/XC16-EX16_MRF24WB/production/_ext/1472/WiSteerAction.o
 .debug_info      0x037f44         0x82 build/XC16-EX16_MRF24WB/production/_ext/1472/WiSteerMpfsSource.o
 .debug_info      0x037fc6        0x174 build/XC16-EX16_MRF24WB/production/_ext/1472/WiSteerStructSizeCheck.o
 *(.gnu.linkonce.wi.*)

.debug_abbrev     0x000000       0x5503
 *(.debug_abbrev)
 .debug_abbrev    0x000000        0x1cb build/XC16-EX16_MRF24WB/production/_ext/1954962658/ARP.o
 .debug_abbrev    0x0001cb         0x1f build/XC16-EX16_MRF24WB/production/_ext/1954962658/Announce.o
 .debug_abbrev    0x0001ea         0x1f build/XC16-EX16_MRF24WB/production/_ext/1954962658/AutoIP.o
 .debug_abbrev    0x000209         0x1f build/XC16-EX16_MRF24WB/production/_ext/1954962658/BerkeleyAPI.o
 .debug_abbrev    0x000228        0x22f build/XC16-EX16_MRF24WB/production/_ext/1954962658/DHCP.o
 .debug_abbrev    0x000457        0x1fe build/XC16-EX16_MRF24WB/production/_ext/1954962658/DHCPs.o
 .debug_abbrev    0x000655        0x1db build/XC16-EX16_MRF24WB/production/_ext/1954962658/DNS.o
 .debug_abbrev    0x000830        0x1b3 build/XC16-EX16_MRF24WB/production/_ext/1954962658/DNSs.o
 .debug_abbrev    0x0009e3         0x68 build/XC16-EX16_MRF24WB/production/_ext/1954962658/Delay.o
 .debug_abbrev    0x000a4b         0x1f build/XC16-EX16_MRF24WB/production/_ext/1954962658/DynDNS.o
 .debug_abbrev    0x000a6a         0x1f build/XC16-EX16_MRF24WB/production/_ext/1954962658/ENC28J60.o
 .debug_abbrev    0x000a89         0x1f build/XC16-EX16_MRF24WB/production/_ext/1954962658/ENCX24J600.o
 .debug_abbrev    0x000aa8         0x1f build/XC16-EX16_MRF24WB/production/_ext/1954962658/FTP.o
 .debug_abbrev    0x000ac7        0x14c build/XC16-EX16_MRF24WB/production/_ext/1954962658/Hashes.o
 .debug_abbrev    0x000c13        0x1bb build/XC16-EX16_MRF24WB/production/_ext/1954962658/Helpers.o
 .debug_abbrev    0x000dce         0xf0 build/XC16-EX16_MRF24WB/production/_ext/1954962658/ICMP.o
 .debug_abbrev    0x000ebe        0x1c0 build/XC16-EX16_MRF24WB/production/_ext/1954962658/IP.o
 .debug_abbrev    0x00107e        0x132 build/XC16-EX16_MRF24WB/production/_ext/1954962658/LCDBlocking.o
 .debug_abbrev    0x0011b0        0x1aa build/XC16-EX16_MRF24WB/production/_ext/1954962658/NBNS.o
 .debug_abbrev    0x00135a         0x1f build/XC16-EX16_MRF24WB/production/_ext/1954962658/Reboot.o
 .debug_abbrev    0x001379         0x1f build/XC16-EX16_MRF24WB/production/_ext/1954962658/SMTP.o
 .debug_abbrev    0x001398         0x1f build/XC16-EX16_MRF24WB/production/_ext/1954962658/SNMP.o
 .debug_abbrev    0x0013b7        0x102 build/XC16-EX16_MRF24WB/production/_ext/1954962658/SNTP.o
 .debug_abbrev    0x0014b9        0x214 build/XC16-EX16_MRF24WB/production/_ext/1954962658/SPIEEPROM.o
 .debug_abbrev    0x0016cd         0x1f build/XC16-EX16_MRF24WB/production/_ext/1954962658/SPIFlash.o
 .debug_abbrev    0x0016ec         0x1f build/XC16-EX16_MRF24WB/production/_ext/1954962658/SPIRAM.o
 .debug_abbrev    0x00170b        0x1ac build/XC16-EX16_MRF24WB/production/_ext/1954962658/StackTsk.o
 .debug_abbrev    0x0018b7        0x246 build/XC16-EX16_MRF24WB/production/_ext/1954962658/TCP.o
 .debug_abbrev    0x001afd         0x1f build/XC16-EX16_MRF24WB/production/_ext/1954962658/TCPPerformanceTest.o
 .debug_abbrev    0x001b1c         0x1f build/XC16-EX16_MRF24WB/production/_ext/1954962658/TFTPc.o
 .debug_abbrev    0x001b3b         0x1f build/XC16-EX16_MRF24WB/production/_ext/1954962658/Telnet.o
 .debug_abbrev    0x001b5a        0x1cc build/XC16-EX16_MRF24WB/production/_ext/1954962658/Tick.o
 .debug_abbrev    0x001d26         0x1f build/XC16-EX16_MRF24WB/production/_ext/1954962658/UART.o
 .debug_abbrev    0x001d45         0x1f build/XC16-EX16_MRF24WB/production/_ext/1954962658/UART2TCPBridge.o
 .debug_abbrev    0x001d64        0x23e build/XC16-EX16_MRF24WB/production/_ext/1954962658/UDP.o
 .debug_abbrev    0x001fa2         0x1f build/XC16-EX16_MRF24WB/production/_ext/1954962658/UDPPerformanceTest.o
 .debug_abbrev    0x001fc1         0x1f build/XC16-EX16_MRF24WB/production/_ext/1954962658/ZeroconfHelper.o
 .debug_abbrev    0x001fe0         0x1f build/XC16-EX16_MRF24WB/production/_ext/1954962658/ZeroconfLinkLocal.o
 .debug_abbrev    0x001fff         0x1f build/XC16-EX16_MRF24WB/production/_ext/1954962658/ZeroconfMulticastDNS.o
 .debug_abbrev    0x00201e        0x1a1 build/XC16-EX16_MRF24WB/production/_ext/243675038/WFConnectionAlgorithm.o
 .debug_abbrev    0x0021bf        0x14a build/XC16-EX16_MRF24WB/production/_ext/243675038/WFConnectionManager.o
 .debug_abbrev    0x002309        0x19d build/XC16-EX16_MRF24WB/production/_ext/243675038/WFConnectionProfile.o
 .debug_abbrev    0x0024a6         0x1f build/XC16-EX16_MRF24WB/production/_ext/243675038/WFConsole.o
 .debug_abbrev    0x0024c5         0x1f build/XC16-EX16_MRF24WB/production/_ext/243675038/WFConsoleIfconfig.o
 .debug_abbrev    0x0024e4         0x1f build/XC16-EX16_MRF24WB/production/_ext/243675038/WFConsoleIwconfig.o
 .debug_abbrev    0x002503         0x1f build/XC16-EX16_MRF24WB/production/_ext/243675038/WFConsoleIwpriv.o
 .debug_abbrev    0x002522         0x94 build/XC16-EX16_MRF24WB/production/_ext/243675038/WFConsoleMsgHandler.o
 .debug_abbrev    0x0025b6         0xff build/XC16-EX16_MRF24WB/production/_ext/243675038/WFConsoleMsgs.o
 .debug_abbrev    0x0026b5         0x1f build/XC16-EX16_MRF24WB/production/_ext/243675038/WFDataTxRx.o
 .debug_abbrev    0x0026d4        0x1ec build/XC16-EX16_MRF24WB/production/_ext/243675038/WFDriverCom.o
 .debug_abbrev    0x0028c0        0x1c8 build/XC16-EX16_MRF24WB/production/_ext/243675038/WFDriverRaw.o
 .debug_abbrev    0x002a88        0x200 build/XC16-EX16_MRF24WB/production/_ext/243675038/WFEasyConfig.o
 .debug_abbrev    0x002c88        0x125 build/XC16-EX16_MRF24WB/production/_ext/243675038/WFEventHandler.o
 .debug_abbrev    0x002dad        0x16c build/XC16-EX16_MRF24WB/production/_ext/243675038/WFInit.o
 .debug_abbrev    0x002f19        0x1f9 build/XC16-EX16_MRF24WB/production/_ext/243675038/WFMac.o
 .debug_abbrev    0x003112        0x16a build/XC16-EX16_MRF24WB/production/_ext/243675038/WFMgmtMsg.o
 .debug_abbrev    0x00327c        0x141 build/XC16-EX16_MRF24WB/production/_ext/243675038/WFParamMsg.o
 .debug_abbrev    0x0033bd         0x1f build/XC16-EX16_MRF24WB/production/_ext/243675038/WFPowerSave.o
 .debug_abbrev    0x0033dc         0xfa build/XC16-EX16_MRF24WB/production/_ext/243675038/WFScan.o
 .debug_abbrev    0x0034d6        0x109 build/XC16-EX16_MRF24WB/production/_ext/243675038/WFTxPower.o
 .debug_abbrev    0x0035df         0xce build/XC16-EX16_MRF24WB/production/_ext/243675038/WF_Eint.o
 .debug_abbrev    0x0036ad        0x145 build/XC16-EX16_MRF24WB/production/_ext/243675038/WF_Spi.o
 .debug_abbrev    0x0037f2        0x1a1 build/XC16-EX16_MRF24WB/production/_ext/243675038/WFDebugStrings.o
 .debug_abbrev    0x003993        0x176 build/XC16-EX16_MRF24WB/production/_ext/243675038/WF_pbkdf2.o
 .debug_abbrev    0x003b09         0x1f build/XC16-EX16_MRF24WB/production/_ext/1472/UARTConfig.o
 .debug_abbrev    0x003b28        0x20f build/XC16-EX16_MRF24WB/production/_ext/1472/WF_Config.o
 .debug_abbrev    0x003d37        0x248 build/XC16-EX16_MRF24WB/production/_ext/1472/HTTP2.o
 .debug_abbrev    0x003f7f        0x205 build/XC16-EX16_MRF24WB/production/_ext/1472/MPFS2.o
 .debug_abbrev    0x004184        0x2fb build/XC16-EX16_MRF24WB/production/_ext/1472/WiSteerHTTP.o
 .debug_abbrev    0x00447f        0x330 build/XC16-EX16_MRF24WB/production/_ext/1472/WiSteerMain.o
 .debug_abbrev    0x0047af        0x18c build/XC16-EX16_MRF24WB/production/_ext/1472/WiSteerHTTPtools.o
 .debug_abbrev    0x00493b         0x1f build/XC16-EX16_MRF24WB/production/_ext/1472/WiSteerUpdate.o
 .debug_abbrev    0x00495a         0x14 build/XC16-EX16_MRF24WB/production/WiSteerUpdateHlp.o
 .debug_abbrev    0x00496e        0x30b build/XC16-EX16_MRF24WB/production/_ext/1472/WiSteerLog.o
 .debug_abbrev    0x004c79        0x255 build/XC16-EX16_MRF24WB/production/_ext/1472/WiSteerTime.o
 .debug_abbrev    0x004ece        0x30b build/XC16-EX16_MRF24WB/production/_ext/1472/WiSteerCom.o
 .debug_abbrev    0x0051d9        0x2e7 build/XC16-EX16_MRF24WB/production/_ext/1472/WiSteerAction.o
 .debug_abbrev    0x0054c0         0x10 build/XC16-EX16_MRF24WB/production/_ext/1472/WiSteerMpfsSource.o
 .debug_abbrev    0x0054d0         0x32 build/XC16-EX16_MRF24WB/production/_ext/1472/WiSteerStructSizeCheck.o
 .debug_abbrev    0x005502          0x1 build/XC16-EX16_MRF24WB/production/_ext/1472/pic32helpers.o

.debug_line       0x000000      0x1e10c
 *(.debug_line)
 .debug_line      0x000000        0x405 build/XC16-EX16_MRF24WB/production/_ext/1954962658/ARP.o
 .debug_line      0x000405         0x24 build/XC16-EX16_MRF24WB/production/_ext/1954962658/Announce.o
 .debug_line      0x000429         0x24 build/XC16-EX16_MRF24WB/production/_ext/1954962658/AutoIP.o
 .debug_line      0x00044d         0x24 build/XC16-EX16_MRF24WB/production/_ext/1954962658/BerkeleyAPI.o
 .debug_line      0x000471        0xc1d build/XC16-EX16_MRF24WB/production/_ext/1954962658/DHCP.o
 .debug_line      0x00108e        0xbef build/XC16-EX16_MRF24WB/production/_ext/1954962658/DHCPs.o
 .debug_line      0x001c7d        0x817 build/XC16-EX16_MRF24WB/production/_ext/1954962658/DNS.o
 .debug_line      0x002494        0x400 build/XC16-EX16_MRF24WB/production/_ext/1954962658/DNSs.o
 .debug_line      0x002894         0xf2 build/XC16-EX16_MRF24WB/production/_ext/1954962658/Delay.o
 .debug_line      0x002986         0x24 build/XC16-EX16_MRF24WB/production/_ext/1954962658/DynDNS.o
 .debug_line      0x0029aa         0x24 build/XC16-EX16_MRF24WB/production/_ext/1954962658/ENC28J60.o
 .debug_line      0x0029ce         0x24 build/XC16-EX16_MRF24WB/production/_ext/1954962658/ENCX24J600.o
 .debug_line      0x0029f2         0x24 build/XC16-EX16_MRF24WB/production/_ext/1954962658/FTP.o
 .debug_line      0x002a16        0x38a build/XC16-EX16_MRF24WB/production/_ext/1954962658/Hashes.o
 .debug_line      0x002da0        0xac8 build/XC16-EX16_MRF24WB/production/_ext/1954962658/Helpers.o
 .debug_line      0x003868        0x162 build/XC16-EX16_MRF24WB/production/_ext/1954962658/ICMP.o
 .debug_line      0x0039ca        0x2b9 build/XC16-EX16_MRF24WB/production/_ext/1954962658/IP.o
 .debug_line      0x003c83        0x3c0 build/XC16-EX16_MRF24WB/production/_ext/1954962658/LCDBlocking.o
 .debug_line      0x004043        0x409 build/XC16-EX16_MRF24WB/production/_ext/1954962658/NBNS.o
 .debug_line      0x00444c         0x24 build/XC16-EX16_MRF24WB/production/_ext/1954962658/Reboot.o
 .debug_line      0x004470         0x24 build/XC16-EX16_MRF24WB/production/_ext/1954962658/SMTP.o
 .debug_line      0x004494         0x24 build/XC16-EX16_MRF24WB/production/_ext/1954962658/SNMP.o
 .debug_line      0x0044b8        0x32d build/XC16-EX16_MRF24WB/production/_ext/1954962658/SNTP.o
 .debug_line      0x0047e5        0x623 build/XC16-EX16_MRF24WB/production/_ext/1954962658/SPIEEPROM.o
 .debug_line      0x004e08         0x24 build/XC16-EX16_MRF24WB/production/_ext/1954962658/SPIFlash.o
 .debug_line      0x004e2c         0x24 build/XC16-EX16_MRF24WB/production/_ext/1954962658/SPIRAM.o
 .debug_line      0x004e50        0x3ed build/XC16-EX16_MRF24WB/production/_ext/1954962658/StackTsk.o
 .debug_line      0x00523d       0x2758 build/XC16-EX16_MRF24WB/production/_ext/1954962658/TCP.o
 .debug_line      0x007995         0x24 build/XC16-EX16_MRF24WB/production/_ext/1954962658/TCPPerformanceTest.o
 .debug_line      0x0079b9         0x24 build/XC16-EX16_MRF24WB/production/_ext/1954962658/TFTPc.o
 .debug_line      0x0079dd         0x24 build/XC16-EX16_MRF24WB/production/_ext/1954962658/Telnet.o
 .debug_line      0x007a01        0x320 build/XC16-EX16_MRF24WB/production/_ext/1954962658/Tick.o
 .debug_line      0x007d21         0x24 build/XC16-EX16_MRF24WB/production/_ext/1954962658/UART.o
 .debug_line      0x007d45         0x24 build/XC16-EX16_MRF24WB/production/_ext/1954962658/UART2TCPBridge.o
 .debug_line      0x007d69        0x947 build/XC16-EX16_MRF24WB/production/_ext/1954962658/UDP.o
 .debug_line      0x0086b0         0x24 build/XC16-EX16_MRF24WB/production/_ext/1954962658/UDPPerformanceTest.o
 .debug_line      0x0086d4         0x24 build/XC16-EX16_MRF24WB/production/_ext/1954962658/ZeroconfHelper.o
 .debug_line      0x0086f8         0x24 build/XC16-EX16_MRF24WB/production/_ext/1954962658/ZeroconfLinkLocal.o
 .debug_line      0x00871c         0x24 build/XC16-EX16_MRF24WB/production/_ext/1954962658/ZeroconfMulticastDNS.o
 .debug_line      0x008740        0x7a2 build/XC16-EX16_MRF24WB/production/_ext/243675038/WFConnectionAlgorithm.o
 .debug_line      0x008ee2        0x2e2 build/XC16-EX16_MRF24WB/production/_ext/243675038/WFConnectionManager.o
 .debug_line      0x0091c4        0x5e4 build/XC16-EX16_MRF24WB/production/_ext/243675038/WFConnectionProfile.o
 .debug_line      0x0097a8         0x24 build/XC16-EX16_MRF24WB/production/_ext/243675038/WFConsole.o
 .debug_line      0x0097cc         0x24 build/XC16-EX16_MRF24WB/production/_ext/243675038/WFConsoleIfconfig.o
 .debug_line      0x0097f0         0x24 build/XC16-EX16_MRF24WB/production/_ext/243675038/WFConsoleIwconfig.o
 .debug_line      0x009814         0x24 build/XC16-EX16_MRF24WB/production/_ext/243675038/WFConsoleIwpriv.o
 .debug_line      0x009838        0x125 build/XC16-EX16_MRF24WB/production/_ext/243675038/WFConsoleMsgHandler.o
 .debug_line      0x00995d        0x185 build/XC16-EX16_MRF24WB/production/_ext/243675038/WFConsoleMsgs.o
 .debug_line      0x009ae2         0x24 build/XC16-EX16_MRF24WB/production/_ext/243675038/WFDataTxRx.o
 .debug_line      0x009b06        0x783 build/XC16-EX16_MRF24WB/production/_ext/243675038/WFDriverCom.o
 .debug_line      0x00a289        0x6a8 build/XC16-EX16_MRF24WB/production/_ext/243675038/WFDriverRaw.o
 .debug_line      0x00a931        0x58e build/XC16-EX16_MRF24WB/production/_ext/243675038/WFEasyConfig.o
 .debug_line      0x00aebf        0x3a7 build/XC16-EX16_MRF24WB/production/_ext/243675038/WFEventHandler.o
 .debug_line      0x00b266        0x188 build/XC16-EX16_MRF24WB/production/_ext/243675038/WFInit.o
 .debug_line      0x00b3ee        0xf1a build/XC16-EX16_MRF24WB/production/_ext/243675038/WFMac.o
 .debug_line      0x00c308        0x331 build/XC16-EX16_MRF24WB/production/_ext/243675038/WFMgmtMsg.o
 .debug_line      0x00c639        0x4e7 build/XC16-EX16_MRF24WB/production/_ext/243675038/WFParamMsg.o
 .debug_line      0x00cb20         0x24 build/XC16-EX16_MRF24WB/production/_ext/243675038/WFPowerSave.o
 .debug_line      0x00cb44        0x1eb build/XC16-EX16_MRF24WB/production/_ext/243675038/WFScan.o
 .debug_line      0x00cd2f        0x1f9 build/XC16-EX16_MRF24WB/production/_ext/243675038/WFTxPower.o
 .debug_line      0x00cf28        0x205 build/XC16-EX16_MRF24WB/production/_ext/243675038/WF_Eint.o
 .debug_line      0x00d12d        0x225 build/XC16-EX16_MRF24WB/production/_ext/243675038/WF_Spi.o
 .debug_line      0x00d352        0x285 build/XC16-EX16_MRF24WB/production/_ext/243675038/WFDebugStrings.o
 .debug_line      0x00d5d7        0x7ff build/XC16-EX16_MRF24WB/production/_ext/243675038/WF_pbkdf2.o
 .debug_line      0x00ddd6         0x24 build/XC16-EX16_MRF24WB/production/_ext/1472/UARTConfig.o
 .debug_line      0x00ddfa        0x4df build/XC16-EX16_MRF24WB/production/_ext/1472/WF_Config.o
 .debug_line      0x00e2d9       0x22d8 build/XC16-EX16_MRF24WB/production/_ext/1472/HTTP2.o
 .debug_line      0x0105b1        0xac0 build/XC16-EX16_MRF24WB/production/_ext/1472/MPFS2.o
 .debug_line      0x011071       0x5858 build/XC16-EX16_MRF24WB/production/_ext/1472/WiSteerHTTP.o
 .debug_line      0x0168c9       0x157a build/XC16-EX16_MRF24WB/production/_ext/1472/WiSteerMain.o
 .debug_line      0x017e43        0x647 build/XC16-EX16_MRF24WB/production/_ext/1472/WiSteerHTTPtools.o
 .debug_line      0x01848a         0x24 build/XC16-EX16_MRF24WB/production/_ext/1472/WiSteerUpdate.o
 .debug_line      0x0184ae         0x78 build/XC16-EX16_MRF24WB/production/WiSteerUpdateHlp.o
 .debug_line      0x018526        0x957 build/XC16-EX16_MRF24WB/production/_ext/1472/WiSteerLog.o
 .debug_line      0x018e7d        0xb78 build/XC16-EX16_MRF24WB/production/_ext/1472/WiSteerTime.o
 .debug_line      0x0199f5       0x2395 build/XC16-EX16_MRF24WB/production/_ext/1472/WiSteerCom.o
 .debug_line      0x01bd8a       0x22a5 build/XC16-EX16_MRF24WB/production/_ext/1472/WiSteerAction.o
 .debug_line      0x01e02f         0x5c build/XC16-EX16_MRF24WB/production/_ext/1472/WiSteerMpfsSource.o
 .debug_line      0x01e08b         0x5d build/XC16-EX16_MRF24WB/production/_ext/1472/WiSteerStructSizeCheck.o
 .debug_line      0x01e0e8         0x24 build/XC16-EX16_MRF24WB/production/_ext/1472/pic32helpers.o

.debug_frame      0x000000       0x4f98
 *(.debug_frame)
 .debug_frame     0x000000         0x84 build/XC16-EX16_MRF24WB/production/_ext/1954962658/ARP.o
 .debug_frame     0x000084         0xc4 build/XC16-EX16_MRF24WB/production/_ext/1954962658/DHCP.o
 .debug_frame     0x000148         0xf4 build/XC16-EX16_MRF24WB/production/_ext/1954962658/DHCPs.o
 .debug_frame     0x00023c         0x74 build/XC16-EX16_MRF24WB/production/_ext/1954962658/DNS.o
 .debug_frame     0x0002b0         0x64 build/XC16-EX16_MRF24WB/production/_ext/1954962658/DNSs.o
 .debug_frame     0x000314         0x34 build/XC16-EX16_MRF24WB/production/_ext/1954962658/Delay.o
 .debug_frame     0x000348         0x64 build/XC16-EX16_MRF24WB/production/_ext/1954962658/Hashes.o
 .debug_frame     0x0003ac        0x124 build/XC16-EX16_MRF24WB/production/_ext/1954962658/Helpers.o
 .debug_frame     0x0004d0         0x24 build/XC16-EX16_MRF24WB/production/_ext/1954962658/ICMP.o
 .debug_frame     0x0004f4         0x54 build/XC16-EX16_MRF24WB/production/_ext/1954962658/IP.o
 .debug_frame     0x000548         0x54 build/XC16-EX16_MRF24WB/production/_ext/1954962658/LCDBlocking.o
 .debug_frame     0x00059c         0x44 build/XC16-EX16_MRF24WB/production/_ext/1954962658/NBNS.o
 .debug_frame     0x0005e0         0x44 build/XC16-EX16_MRF24WB/production/_ext/1954962658/SNTP.o
 .debug_frame     0x000624         0xc4 build/XC16-EX16_MRF24WB/production/_ext/1954962658/SPIEEPROM.o
 .debug_frame     0x0006e8         0x64 build/XC16-EX16_MRF24WB/production/_ext/1954962658/StackTsk.o
 .debug_frame     0x00074c        0x244 build/XC16-EX16_MRF24WB/production/_ext/1954962658/TCP.o
 .debug_frame     0x000990         0x84 build/XC16-EX16_MRF24WB/production/_ext/1954962658/Tick.o
 .debug_frame     0x000a14        0x144 build/XC16-EX16_MRF24WB/production/_ext/1954962658/UDP.o
 .debug_frame     0x000b58        0x254 build/XC16-EX16_MRF24WB/production/_ext/243675038/WFConnectionAlgorithm.o
 .debug_frame     0x000dac         0x94 build/XC16-EX16_MRF24WB/production/_ext/243675038/WFConnectionManager.o
 .debug_frame     0x000e40        0x184 build/XC16-EX16_MRF24WB/production/_ext/243675038/WFConnectionProfile.o
 .debug_frame     0x000fc4         0x24 build/XC16-EX16_MRF24WB/production/_ext/243675038/WFConsoleMsgHandler.o
 .debug_frame     0x000fe8         0x34 build/XC16-EX16_MRF24WB/production/_ext/243675038/WFConsoleMsgs.o
 .debug_frame     0x00101c        0x154 build/XC16-EX16_MRF24WB/production/_ext/243675038/WFDriverCom.o
 .debug_frame     0x001170        0x164 build/XC16-EX16_MRF24WB/production/_ext/243675038/WFDriverRaw.o
 .debug_frame     0x0012d4         0xdc build/XC16-EX16_MRF24WB/production/_ext/243675038/WFEasyConfig.o
 .debug_frame     0x0013b0         0x44 build/XC16-EX16_MRF24WB/production/_ext/243675038/WFEventHandler.o
 .debug_frame     0x0013f4         0x34 build/XC16-EX16_MRF24WB/production/_ext/243675038/WFInit.o
 .debug_frame     0x001428        0x224 build/XC16-EX16_MRF24WB/production/_ext/243675038/WFMac.o
 .debug_frame     0x00164c         0x64 build/XC16-EX16_MRF24WB/production/_ext/243675038/WFMgmtMsg.o
 .debug_frame     0x0016b0        0x134 build/XC16-EX16_MRF24WB/production/_ext/243675038/WFParamMsg.o
 .debug_frame     0x0017e4         0x44 build/XC16-EX16_MRF24WB/production/_ext/243675038/WFScan.o
 .debug_frame     0x001828         0x54 build/XC16-EX16_MRF24WB/production/_ext/243675038/WFTxPower.o
 .debug_frame     0x00187c         0x74 build/XC16-EX16_MRF24WB/production/_ext/243675038/WF_Eint.o
 .debug_frame     0x0018f0         0x64 build/XC16-EX16_MRF24WB/production/_ext/243675038/WF_Spi.o
 .debug_frame     0x001954        0x130 build/XC16-EX16_MRF24WB/production/_ext/243675038/WFDebugStrings.o
 .debug_frame     0x001a84         0xd4 build/XC16-EX16_MRF24WB/production/_ext/243675038/WF_pbkdf2.o
 .debug_frame     0x001b58         0xfc build/XC16-EX16_MRF24WB/production/_ext/1472/WF_Config.o
 .debug_frame     0x001c54        0x1a4 build/XC16-EX16_MRF24WB/production/_ext/1472/HTTP2.o
 .debug_frame     0x001df8        0x1c0 build/XC16-EX16_MRF24WB/production/_ext/1472/MPFS2.o
 .debug_frame     0x001fb8       0x196c build/XC16-EX16_MRF24WB/production/_ext/1472/WiSteerHTTP.o
 .debug_frame     0x003924        0x2c0 build/XC16-EX16_MRF24WB/production/_ext/1472/WiSteerMain.o
 .debug_frame     0x003be4        0x1b0 build/XC16-EX16_MRF24WB/production/_ext/1472/WiSteerHTTPtools.o
 .debug_frame     0x003d94        0x138 build/XC16-EX16_MRF24WB/production/_ext/1472/WiSteerLog.o
 .debug_frame     0x003ecc        0x3ec build/XC16-EX16_MRF24WB/production/_ext/1472/WiSteerTime.o
 .debug_frame     0x0042b8        0x82c build/XC16-EX16_MRF24WB/production/_ext/1472/WiSteerCom.o
 .debug_frame     0x004ae4        0x490 build/XC16-EX16_MRF24WB/production/_ext/1472/WiSteerAction.o
 .debug_frame     0x004f74         0x24 build/XC16-EX16_MRF24WB/production/_ext/1472/WiSteerStructSizeCheck.o

.debug_str        0x000000       0x1550
 *(.debug_str)
 .debug_str       0x000000         0x18 build/XC16-EX16_MRF24WB/production/_ext/1954962658/ARP.o
 .debug_str       0x000018         0x48 build/XC16-EX16_MRF24WB/production/_ext/1954962658/DHCP.o
 .debug_str       0x000060         0x52 build/XC16-EX16_MRF24WB/production/_ext/1954962658/DHCPs.o
 .debug_str       0x0000b2          0xa build/XC16-EX16_MRF24WB/production/_ext/1954962658/DNS.o
 .debug_str       0x0000bc          0xa build/XC16-EX16_MRF24WB/production/_ext/1954962658/DNSs.o
 .debug_str       0x0000c6         0x11 build/XC16-EX16_MRF24WB/production/_ext/1954962658/Hashes.o
 .debug_str       0x0000d7          0x9 build/XC16-EX16_MRF24WB/production/_ext/1954962658/Helpers.o
 .debug_str       0x0000e0         0x13 build/XC16-EX16_MRF24WB/production/_ext/1954962658/IP.o
 .debug_str       0x0000f3         0x26 build/XC16-EX16_MRF24WB/production/_ext/1954962658/LCDBlocking.o
 .debug_str       0x000119         0x23 build/XC16-EX16_MRF24WB/production/_ext/1954962658/NBNS.o
 .debug_str       0x00013c         0x64 build/XC16-EX16_MRF24WB/production/_ext/1954962658/SPIEEPROM.o
 .debug_str       0x0001a0         0x41 build/XC16-EX16_MRF24WB/production/_ext/1954962658/StackTsk.o
 .debug_str       0x0001e1         0xcb build/XC16-EX16_MRF24WB/production/_ext/1954962658/TCP.o
 .debug_str       0x0002ac         0x42 build/XC16-EX16_MRF24WB/production/_ext/1954962658/Tick.o
 .debug_str       0x0002ee         0x72 build/XC16-EX16_MRF24WB/production/_ext/1954962658/UDP.o
 .debug_str       0x000360         0xe4 build/XC16-EX16_MRF24WB/production/_ext/243675038/WFConnectionAlgorithm.o
 .debug_str       0x000444         0x15 build/XC16-EX16_MRF24WB/production/_ext/243675038/WFConnectionManager.o
 .debug_str       0x000459         0xbe build/XC16-EX16_MRF24WB/production/_ext/243675038/WFConnectionProfile.o
 .debug_str       0x000517         0x4b build/XC16-EX16_MRF24WB/production/_ext/243675038/WFConsoleMsgs.o
 .debug_str       0x000562         0x97 build/XC16-EX16_MRF24WB/production/_ext/243675038/WFDriverCom.o
 .debug_str       0x0005f9         0xb9 build/XC16-EX16_MRF24WB/production/_ext/243675038/WFDriverRaw.o
 .debug_str       0x0006b2         0x55 build/XC16-EX16_MRF24WB/production/_ext/243675038/WFEasyConfig.o
 .debug_str       0x000707          0xb build/XC16-EX16_MRF24WB/production/_ext/243675038/WFEventHandler.o
 .debug_str       0x000712         0x22 build/XC16-EX16_MRF24WB/production/_ext/243675038/WFInit.o
 .debug_str       0x000734         0x5d build/XC16-EX16_MRF24WB/production/_ext/243675038/WFMac.o
 .debug_str       0x000791         0x63 build/XC16-EX16_MRF24WB/production/_ext/243675038/WFMgmtMsg.o
 .debug_str       0x0007f4         0x49 build/XC16-EX16_MRF24WB/production/_ext/243675038/WFParamMsg.o
 .debug_str       0x00083d          0x8 build/XC16-EX16_MRF24WB/production/_ext/243675038/WFTxPower.o
 .debug_str       0x000845         0x32 build/XC16-EX16_MRF24WB/production/_ext/243675038/WF_Eint.o
 .debug_str       0x000877         0x44 build/XC16-EX16_MRF24WB/production/_ext/243675038/WF_Spi.o
 .debug_str       0x0008bb         0x56 build/XC16-EX16_MRF24WB/production/_ext/243675038/WFDebugStrings.o
 .debug_str       0x000911         0x52 build/XC16-EX16_MRF24WB/production/_ext/243675038/WF_pbkdf2.o
 .debug_str       0x000963         0x6b build/XC16-EX16_MRF24WB/production/_ext/1472/WF_Config.o
 .debug_str       0x0009ce         0x59 build/XC16-EX16_MRF24WB/production/_ext/1472/HTTP2.o
 .debug_str       0x000a27         0x41 build/XC16-EX16_MRF24WB/production/_ext/1472/MPFS2.o
 .debug_str       0x000a68        0x2fa build/XC16-EX16_MRF24WB/production/_ext/1472/WiSteerHTTP.o
 .debug_str       0x000d62        0x208 build/XC16-EX16_MRF24WB/production/_ext/1472/WiSteerMain.o
 .debug_str       0x000f6a         0x6b build/XC16-EX16_MRF24WB/production/_ext/1472/WiSteerHTTPtools.o
 .debug_str       0x000fd5         0xa0 build/XC16-EX16_MRF24WB/production/_ext/1472/WiSteerLog.o
 .debug_str       0x001075         0xc5 build/XC16-EX16_MRF24WB/production/_ext/1472/WiSteerTime.o
 .debug_str       0x00113a        0x20d build/XC16-EX16_MRF24WB/production/_ext/1472/WiSteerCom.o
 .debug_str       0x001347        0x209 build/XC16-EX16_MRF24WB/production/_ext/1472/WiSteerAction.o

.debug_loc
 *(.debug_loc)

.debug_macinfo
 *(.debug_macinfo)

.debug_pubnames
                  0x000000       0x50aa
 *(.debug_pubnames)
 .debug_pubnames
                  0x000000         0x6f build/XC16-EX16_MRF24WB/production/_ext/1954962658/ARP.o
 .debug_pubnames
                  0x00006f         0xcc build/XC16-EX16_MRF24WB/production/_ext/1954962658/DHCP.o
 .debug_pubnames
                  0x00013b         0x78 build/XC16-EX16_MRF24WB/production/_ext/1954962658/DHCPs.o
 .debug_pubnames
                  0x0001b3         0x55 build/XC16-EX16_MRF24WB/production/_ext/1954962658/DNS.o
 .debug_pubnames
                  0x000208         0x24 build/XC16-EX16_MRF24WB/production/_ext/1954962658/DNSs.o
 .debug_pubnames
                  0x00022c         0x2c build/XC16-EX16_MRF24WB/production/_ext/1954962658/Delay.o
 .debug_pubnames
                  0x000258         0x62 build/XC16-EX16_MRF24WB/production/_ext/1954962658/Hashes.o
 .debug_pubnames
                  0x0002ba        0x11b build/XC16-EX16_MRF24WB/production/_ext/1954962658/Helpers.o
 .debug_pubnames
                  0x0003d5         0x22 build/XC16-EX16_MRF24WB/production/_ext/1954962658/ICMP.o
 .debug_pubnames
                  0x0003f7         0x44 build/XC16-EX16_MRF24WB/production/_ext/1954962658/IP.o
 .debug_pubnames
                  0x00043b         0x45 build/XC16-EX16_MRF24WB/production/_ext/1954962658/LCDBlocking.o
 .debug_pubnames
                  0x000480         0x1f build/XC16-EX16_MRF24WB/production/_ext/1954962658/NBNS.o
 .debug_pubnames
                  0x00049f         0x4d build/XC16-EX16_MRF24WB/production/_ext/1954962658/SNTP.o
 .debug_pubnames
                  0x0004ec         0xaa build/XC16-EX16_MRF24WB/production/_ext/1954962658/SPIEEPROM.o
 .debug_pubnames
                  0x000596         0x98 build/XC16-EX16_MRF24WB/production/_ext/1954962658/StackTsk.o
 .debug_pubnames
                  0x00062e        0x1c9 build/XC16-EX16_MRF24WB/production/_ext/1954962658/TCP.o
 .debug_pubnames
                  0x0007f7         0xa3 build/XC16-EX16_MRF24WB/production/_ext/1954962658/Tick.o
 .debug_pubnames
                  0x00089a        0x168 build/XC16-EX16_MRF24WB/production/_ext/1954962658/UDP.o
 .debug_pubnames
                  0x000a02        0x375 build/XC16-EX16_MRF24WB/production/_ext/243675038/WFConnectionAlgorithm.o
 .debug_pubnames
                  0x000d77         0xbb build/XC16-EX16_MRF24WB/production/_ext/243675038/WFConnectionManager.o
 .debug_pubnames
                  0x000e32        0x1d6 build/XC16-EX16_MRF24WB/production/_ext/243675038/WFConnectionProfile.o
 .debug_pubnames
                  0x001008         0x2f build/XC16-EX16_MRF24WB/production/_ext/243675038/WFConsoleMsgHandler.o
 .debug_pubnames
                  0x001037         0xee build/XC16-EX16_MRF24WB/production/_ext/243675038/WFConsoleMsgs.o
 .debug_pubnames
                  0x001125        0x1ab build/XC16-EX16_MRF24WB/production/_ext/243675038/WFDriverCom.o
 .debug_pubnames
                  0x0012d0        0x1c8 build/XC16-EX16_MRF24WB/production/_ext/243675038/WFDriverRaw.o
 .debug_pubnames
                  0x001498        0x100 build/XC16-EX16_MRF24WB/production/_ext/243675038/WFEasyConfig.o
 .debug_pubnames
                  0x001598         0x2f build/XC16-EX16_MRF24WB/production/_ext/243675038/WFEventHandler.o
 .debug_pubnames
                  0x0015c7         0x3a build/XC16-EX16_MRF24WB/production/_ext/243675038/WFInit.o
 .debug_pubnames
                  0x001601        0x252 build/XC16-EX16_MRF24WB/production/_ext/243675038/WFMac.o
 .debug_pubnames
                  0x001853         0xb0 build/XC16-EX16_MRF24WB/production/_ext/243675038/WFMgmtMsg.o
 .debug_pubnames
                  0x001903        0x1c7 build/XC16-EX16_MRF24WB/production/_ext/243675038/WFParamMsg.o
 .debug_pubnames
                  0x001aca         0x33 build/XC16-EX16_MRF24WB/production/_ext/243675038/WFScan.o
 .debug_pubnames
                  0x001afd         0x7b build/XC16-EX16_MRF24WB/production/_ext/243675038/WFTxPower.o
 .debug_pubnames
                  0x001b78         0x85 build/XC16-EX16_MRF24WB/production/_ext/243675038/WF_Eint.o
 .debug_pubnames
                  0x001bfd         0x66 build/XC16-EX16_MRF24WB/production/_ext/243675038/WF_Spi.o
 .debug_pubnames
                  0x001c63         0xae build/XC16-EX16_MRF24WB/production/_ext/243675038/WFDebugStrings.o
 .debug_pubnames
                  0x001d11         0x84 build/XC16-EX16_MRF24WB/production/_ext/243675038/WF_pbkdf2.o
 .debug_pubnames
                  0x001d95         0xde build/XC16-EX16_MRF24WB/production/_ext/1472/WF_Config.o
 .debug_pubnames
                  0x001e73        0x183 build/XC16-EX16_MRF24WB/production/_ext/1472/HTTP2.o
 .debug_pubnames
                  0x001ff6        0x1b6 build/XC16-EX16_MRF24WB/production/_ext/1472/MPFS2.o
 .debug_pubnames
                  0x0021ac       0x1b29 build/XC16-EX16_MRF24WB/production/_ext/1472/WiSteerHTTP.o
 .debug_pubnames
                  0x003cd5        0x36e build/XC16-EX16_MRF24WB/production/_ext/1472/WiSteerMain.o
 .debug_pubnames
                  0x004043        0x1b1 build/XC16-EX16_MRF24WB/production/_ext/1472/WiSteerHTTPtools.o
 .debug_pubnames
                  0x0041f4        0x10c build/XC16-EX16_MRF24WB/production/_ext/1472/WiSteerLog.o
 .debug_pubnames
                  0x004300        0x1c4 build/XC16-EX16_MRF24WB/production/_ext/1472/WiSteerTime.o
 .debug_pubnames
                  0x0044c4        0x5ad build/XC16-EX16_MRF24WB/production/_ext/1472/WiSteerCom.o
 .debug_pubnames
                  0x004a71        0x610 build/XC16-EX16_MRF24WB/production/_ext/1472/WiSteerAction.o
 .debug_pubnames
                  0x005081         0x29 build/XC16-EX16_MRF24WB/production/_ext/1472/WiSteerStructSizeCheck.o

.debug_ranges
 *(.debug_ranges)

.debug_aranges    0x000000        0x4b8
 *(.debug_aranges)
 .debug_aranges
                  0x000000         0x18 build/XC16-EX16_MRF24WB/production/_ext/1954962658/ARP.o
 .debug_aranges
                  0x000018         0x18 build/XC16-EX16_MRF24WB/production/_ext/1954962658/DHCP.o
 .debug_aranges
                  0x000030         0x18 build/XC16-EX16_MRF24WB/production/_ext/1954962658/DHCPs.o
 .debug_aranges
                  0x000048         0x18 build/XC16-EX16_MRF24WB/production/_ext/1954962658/DNS.o
 .debug_aranges
                  0x000060         0x18 build/XC16-EX16_MRF24WB/production/_ext/1954962658/DNSs.o
 .debug_aranges
                  0x000078         0x18 build/XC16-EX16_MRF24WB/production/_ext/1954962658/Delay.o
 .debug_aranges
                  0x000090         0x18 build/XC16-EX16_MRF24WB/production/_ext/1954962658/Hashes.o
 .debug_aranges
                  0x0000a8         0x18 build/XC16-EX16_MRF24WB/production/_ext/1954962658/Helpers.o
 .debug_aranges
                  0x0000c0         0x18 build/XC16-EX16_MRF24WB/production/_ext/1954962658/ICMP.o
 .debug_aranges
                  0x0000d8         0x18 build/XC16-EX16_MRF24WB/production/_ext/1954962658/IP.o
 .debug_aranges
                  0x0000f0         0x18 build/XC16-EX16_MRF24WB/production/_ext/1954962658/LCDBlocking.o
 .debug_aranges
                  0x000108         0x18 build/XC16-EX16_MRF24WB/production/_ext/1954962658/NBNS.o
 .debug_aranges
                  0x000120         0x18 build/XC16-EX16_MRF24WB/production/_ext/1954962658/SNTP.o
 .debug_aranges
                  0x000138         0x18 build/XC16-EX16_MRF24WB/production/_ext/1954962658/SPIEEPROM.o
 .debug_aranges
                  0x000150         0x18 build/XC16-EX16_MRF24WB/production/_ext/1954962658/StackTsk.o
 .debug_aranges
                  0x000168         0x18 build/XC16-EX16_MRF24WB/production/_ext/1954962658/TCP.o
 .debug_aranges
                  0x000180         0x18 build/XC16-EX16_MRF24WB/production/_ext/1954962658/Tick.o
 .debug_aranges
                  0x000198         0x18 build/XC16-EX16_MRF24WB/production/_ext/1954962658/UDP.o
 .debug_aranges
                  0x0001b0         0x18 build/XC16-EX16_MRF24WB/production/_ext/243675038/WFConnectionAlgorithm.o
 .debug_aranges
                  0x0001c8         0x18 build/XC16-EX16_MRF24WB/production/_ext/243675038/WFConnectionManager.o
 .debug_aranges
                  0x0001e0         0x18 build/XC16-EX16_MRF24WB/production/_ext/243675038/WFConnectionProfile.o
 .debug_aranges
                  0x0001f8         0x18 build/XC16-EX16_MRF24WB/production/_ext/243675038/WFConsoleMsgHandler.o
 .debug_aranges
                  0x000210         0x18 build/XC16-EX16_MRF24WB/production/_ext/243675038/WFConsoleMsgs.o
 .debug_aranges
                  0x000228         0x18 build/XC16-EX16_MRF24WB/production/_ext/243675038/WFDriverCom.o
 .debug_aranges
                  0x000240         0x18 build/XC16-EX16_MRF24WB/production/_ext/243675038/WFDriverRaw.o
 .debug_aranges
                  0x000258         0x18 build/XC16-EX16_MRF24WB/production/_ext/243675038/WFEasyConfig.o
 .debug_aranges
                  0x000270         0x18 build/XC16-EX16_MRF24WB/production/_ext/243675038/WFEventHandler.o
 .debug_aranges
                  0x000288         0x18 build/XC16-EX16_MRF24WB/production/_ext/243675038/WFInit.o
 .debug_aranges
                  0x0002a0         0x18 build/XC16-EX16_MRF24WB/production/_ext/243675038/WFMac.o
 .debug_aranges
                  0x0002b8         0x18 build/XC16-EX16_MRF24WB/production/_ext/243675038/WFMgmtMsg.o
 .debug_aranges
                  0x0002d0         0x18 build/XC16-EX16_MRF24WB/production/_ext/243675038/WFParamMsg.o
 .debug_aranges
                  0x0002e8         0x18 build/XC16-EX16_MRF24WB/production/_ext/243675038/WFScan.o
 .debug_aranges
                  0x000300         0x18 build/XC16-EX16_MRF24WB/production/_ext/243675038/WFTxPower.o
 .debug_aranges
                  0x000318         0x18 build/XC16-EX16_MRF24WB/production/_ext/243675038/WF_Eint.o
 .debug_aranges
                  0x000330         0x18 build/XC16-EX16_MRF24WB/production/_ext/243675038/WF_Spi.o
 .debug_aranges
                  0x000348         0x18 build/XC16-EX16_MRF24WB/production/_ext/243675038/WFDebugStrings.o
 .debug_aranges
                  0x000360         0x18 build/XC16-EX16_MRF24WB/production/_ext/243675038/WF_pbkdf2.o
 .debug_aranges
                  0x000378         0x18 build/XC16-EX16_MRF24WB/production/_ext/1472/WF_Config.o
 .debug_aranges
                  0x000390         0x18 build/XC16-EX16_MRF24WB/production/_ext/1472/HTTP2.o
 .debug_aranges
                  0x0003a8         0x18 build/XC16-EX16_MRF24WB/production/_ext/1472/MPFS2.o
 .debug_aranges
                  0x0003c0         0x18 build/XC16-EX16_MRF24WB/production/_ext/1472/WiSteerHTTP.o
 .debug_aranges
                  0x0003d8         0x18 build/XC16-EX16_MRF24WB/production/_ext/1472/WiSteerMain.o
 .debug_aranges
                  0x0003f0         0x18 build/XC16-EX16_MRF24WB/production/_ext/1472/WiSteerHTTPtools.o
 .debug_aranges
                  0x000408         0x18 build/XC16-EX16_MRF24WB/production/WiSteerUpdateHlp.o
 .debug_aranges
                  0x000420         0x18 build/XC16-EX16_MRF24WB/production/_ext/1472/WiSteerLog.o
 .debug_aranges
                  0x000438         0x18 build/XC16-EX16_MRF24WB/production/_ext/1472/WiSteerTime.o
 .debug_aranges
                  0x000450         0x18 build/XC16-EX16_MRF24WB/production/_ext/1472/WiSteerCom.o
 .debug_aranges
                  0x000468         0x18 build/XC16-EX16_MRF24WB/production/_ext/1472/WiSteerAction.o
 .debug_aranges
                  0x000480         0x20 build/XC16-EX16_MRF24WB/production/_ext/1472/WiSteerMpfsSource.o
 .debug_aranges
                  0x0004a0         0x18 build/XC16-EX16_MRF24WB/production/_ext/1472/WiSteerStructSizeCheck.o

.ivt              0x000004        0x130
                  0x000004          0x4 LONG 0x302 DEFINED (__OscillatorFail)?ABSOLUTE (__OscillatorFail):ABSOLUTE (__DefaultInterrupt)
                  0x000006          0x4 LONG 0x32c DEFINED (__AddressError)?ABSOLUTE (__AddressError):ABSOLUTE (__DefaultInterrupt)
                  0x000008          0x4 LONG 0x2d8 DEFINED (__HardTrapError)?ABSOLUTE (__HardTrapError):ABSOLUTE (__DefaultInterrupt)
                  0x00000a          0x4 LONG 0x356 DEFINED (__StackError)?ABSOLUTE (__StackError):ABSOLUTE (__DefaultInterrupt)
                  0x00000c          0x4 LONG 0x380 DEFINED (__MathError)?ABSOLUTE (__MathError):ABSOLUTE (__DefaultInterrupt)
                  0x00000e          0x4 LONG 0x2d8 DEFINED (__DMACError)?ABSOLUTE (__DMACError):ABSOLUTE (__DefaultInterrupt)
                  0x000010          0x4 LONG 0x2d8 DEFINED (__SoftTrapError)?ABSOLUTE (__SoftTrapError):ABSOLUTE (__DefaultInterrupt)
                  0x000012          0x4 LONG 0x2d8 DEFINED (__ReservedTrap7)?ABSOLUTE (__ReservedTrap7):ABSOLUTE (__DefaultInterrupt)
                  0x000014          0x4 LONG 0x2d8 DEFINED (__INT0Interrupt)?ABSOLUTE (__INT0Interrupt):ABSOLUTE (__DefaultInterrupt)
                  0x000016          0x4 LONG 0x2d8 DEFINED (__IC1Interrupt)?ABSOLUTE (__IC1Interrupt):ABSOLUTE (__DefaultInterrupt)
                  0x000018          0x4 LONG 0x2d8 DEFINED (__OC1Interrupt)?ABSOLUTE (__OC1Interrupt):ABSOLUTE (__DefaultInterrupt)
                  0x00001a          0x4 LONG 0x45f30 DEFINED (__T1Interrupt)?ABSOLUTE (__T1Interrupt):ABSOLUTE (__DefaultInterrupt)
                  0x00001c          0x4 LONG 0x2d8 DEFINED (__DMA0Interrupt)?ABSOLUTE (__DMA0Interrupt):ABSOLUTE (__DefaultInterrupt)
                  0x00001e          0x4 LONG 0x2d8 DEFINED (__IC2Interrupt)?ABSOLUTE (__IC2Interrupt):ABSOLUTE (__DefaultInterrupt)
                  0x000020          0x4 LONG 0x2d8 DEFINED (__OC2Interrupt)?ABSOLUTE (__OC2Interrupt):ABSOLUTE (__DefaultInterrupt)
                  0x000022          0x4 LONG 0x2d8 DEFINED (__T2Interrupt)?ABSOLUTE (__T2Interrupt):ABSOLUTE (__DefaultInterrupt)
                  0x000024          0x4 LONG 0x2d8 DEFINED (__T3Interrupt)?ABSOLUTE (__T3Interrupt):ABSOLUTE (__DefaultInterrupt)
                  0x000026          0x4 LONG 0x2d8 DEFINED (__SPI1ErrInterrupt)?ABSOLUTE (__SPI1ErrInterrupt):ABSOLUTE (__DefaultInterrupt)
                  0x000028          0x4 LONG 0x2d8 DEFINED (__SPI1Interrupt)?ABSOLUTE (__SPI1Interrupt):ABSOLUTE (__DefaultInterrupt)
                  0x00002a          0x4 LONG 0x2d8 DEFINED (__U1RXInterrupt)?ABSOLUTE (__U1RXInterrupt):ABSOLUTE (__DefaultInterrupt)
                  0x00002c          0x4 LONG 0x2d8 DEFINED (__U1TXInterrupt)?ABSOLUTE (__U1TXInterrupt):ABSOLUTE (__DefaultInterrupt)
                  0x00002e          0x4 LONG 0x2d8 DEFINED (__AD1Interrupt)?ABSOLUTE (__AD1Interrupt):ABSOLUTE (__DefaultInterrupt)
                  0x000030          0x4 LONG 0x2d8 DEFINED (__DMA1Interrupt)?ABSOLUTE (__DMA1Interrupt):ABSOLUTE (__DefaultInterrupt)
                  0x000032          0x4 LONG 0x2d8 DEFINED (__NVMInterrupt)?ABSOLUTE (__NVMInterrupt):ABSOLUTE (__DefaultInterrupt)
                  0x000034          0x4 LONG 0x2d8 DEFINED (__SI2C1Interrupt)?ABSOLUTE (__SI2C1Interrupt):ABSOLUTE (__DefaultInterrupt)
                  0x000036          0x4 LONG 0x2d8 DEFINED (__MI2C1Interrupt)?ABSOLUTE (__MI2C1Interrupt):ABSOLUTE (__DefaultInterrupt)
                  0x000038          0x4 LONG 0x2d8 DEFINED (__CM1Interrupt)?ABSOLUTE (__CM1Interrupt):ABSOLUTE (__DefaultInterrupt)
                  0x00003a          0x4 LONG 0x2d8 DEFINED (__CNInterrupt)?ABSOLUTE (__CNInterrupt):ABSOLUTE (__DefaultInterrupt)
                  0x00003c          0x4 LONG 0x2d8 DEFINED (__INT1Interrupt)?ABSOLUTE (__INT1Interrupt):ABSOLUTE (__DefaultInterrupt)
                  0x00003e          0x4 LONG 0x2d8 DEFINED (__AD2Interrupt)?ABSOLUTE (__AD2Interrupt):ABSOLUTE (__DefaultInterrupt)
                  0x000040          0x4 LONG 0x2d8 DEFINED (__IC7Interrupt)?ABSOLUTE (__IC7Interrupt):ABSOLUTE (__DefaultInterrupt)
                  0x000042          0x4 LONG 0x2d8 DEFINED (__IC8Interrupt)?ABSOLUTE (__IC8Interrupt):ABSOLUTE (__DefaultInterrupt)
                  0x000044          0x4 LONG 0x2d8 DEFINED (__DMA2Interrupt)?ABSOLUTE (__DMA2Interrupt):ABSOLUTE (__DefaultInterrupt)
                  0x000046          0x4 LONG 0x2d8 DEFINED (__OC3Interrupt)?ABSOLUTE (__OC3Interrupt):ABSOLUTE (__DefaultInterrupt)
                  0x000048          0x4 LONG 0x2d8 DEFINED (__OC4Interrupt)?ABSOLUTE (__OC4Interrupt):ABSOLUTE (__DefaultInterrupt)
                  0x00004a          0x4 LONG 0x2d8 DEFINED (__T4Interrupt)?ABSOLUTE (__T4Interrupt):ABSOLUTE (__DefaultInterrupt)
                  0x00004c          0x4 LONG 0x2d8 DEFINED (__T5Interrupt)?ABSOLUTE (__T5Interrupt):ABSOLUTE (__DefaultInterrupt)
                  0x00004e          0x4 LONG 0x2d8 DEFINED (__INT2Interrupt)?ABSOLUTE (__INT2Interrupt):ABSOLUTE (__DefaultInterrupt)
                  0x000050          0x4 LONG 0x2d8 DEFINED (__U2RXInterrupt)?ABSOLUTE (__U2RXInterrupt):ABSOLUTE (__DefaultInterrupt)
                  0x000052          0x4 LONG 0x2d8 DEFINED (__U2TXInterrupt)?ABSOLUTE (__U2TXInterrupt):ABSOLUTE (__DefaultInterrupt)
                  0x000054          0x4 LONG 0x2d8 DEFINED (__SPI2ErrInterrupt)?ABSOLUTE (__SPI2ErrInterrupt):ABSOLUTE (__DefaultInterrupt)
                  0x000056          0x4 LONG 0x2d8 DEFINED (__SPI2Interrupt)?ABSOLUTE (__SPI2Interrupt):ABSOLUTE (__DefaultInterrupt)
                  0x000058          0x4 LONG 0x2d8 DEFINED (__C1RxRdyInterrupt)?ABSOLUTE (__C1RxRdyInterrupt):ABSOLUTE (__DefaultInterrupt)
                  0x00005a          0x4 LONG 0x2d8 DEFINED (__C1Interrupt)?ABSOLUTE (__C1Interrupt):ABSOLUTE (__DefaultInterrupt)
                  0x00005c          0x4 LONG 0x2d8 DEFINED (__DMA3Interrupt)?ABSOLUTE (__DMA3Interrupt):ABSOLUTE (__DefaultInterrupt)
                  0x00005e          0x4 LONG 0x2d8 DEFINED (__IC3Interrupt)?ABSOLUTE (__IC3Interrupt):ABSOLUTE (__DefaultInterrupt)
                  0x000060          0x4 LONG 0x2d8 DEFINED (__IC4Interrupt)?ABSOLUTE (__IC4Interrupt):ABSOLUTE (__DefaultInterrupt)
                  0x000062          0x4 LONG 0x2d8 DEFINED (__IC5Interrupt)?ABSOLUTE (__IC5Interrupt):ABSOLUTE (__DefaultInterrupt)
                  0x000064          0x4 LONG 0x2d8 DEFINED (__IC6Interrupt)?ABSOLUTE (__IC6Interrupt):ABSOLUTE (__DefaultInterrupt)
                  0x000066          0x4 LONG 0x2d8 DEFINED (__OC5Interrupt)?ABSOLUTE (__OC5Interrupt):ABSOLUTE (__DefaultInterrupt)
                  0x000068          0x4 LONG 0x2d8 DEFINED (__OC6Interrupt)?ABSOLUTE (__OC6Interrupt):ABSOLUTE (__DefaultInterrupt)
                  0x00006a          0x4 LONG 0x2d8 DEFINED (__OC7Interrupt)?ABSOLUTE (__OC7Interrupt):ABSOLUTE (__DefaultInterrupt)
                  0x00006c          0x4 LONG 0x2d8 DEFINED (__OC8Interrupt)?ABSOLUTE (__OC8Interrupt):ABSOLUTE (__DefaultInterrupt)
                  0x00006e          0x4 LONG 0x2d8 DEFINED (__PMPInterrupt)?ABSOLUTE (__PMPInterrupt):ABSOLUTE (__DefaultInterrupt)
                  0x000070          0x4 LONG 0x2d8 DEFINED (__DMA4Interrupt)?ABSOLUTE (__DMA4Interrupt):ABSOLUTE (__DefaultInterrupt)
                  0x000072          0x4 LONG 0x2d8 DEFINED (__T6Interrupt)?ABSOLUTE (__T6Interrupt):ABSOLUTE (__DefaultInterrupt)
                  0x000074          0x4 LONG 0x2d8 DEFINED (__T7Interrupt)?ABSOLUTE (__T7Interrupt):ABSOLUTE (__DefaultInterrupt)
                  0x000076          0x4 LONG 0x2d8 DEFINED (__SI2C2Interrupt)?ABSOLUTE (__SI2C2Interrupt):ABSOLUTE (__DefaultInterrupt)
                  0x000078          0x4 LONG 0x2d8 DEFINED (__MI2C2Interrupt)?ABSOLUTE (__MI2C2Interrupt):ABSOLUTE (__DefaultInterrupt)
                  0x00007a          0x4 LONG 0x2d8 DEFINED (__T8Interrupt)?ABSOLUTE (__T8Interrupt):ABSOLUTE (__DefaultInterrupt)
                  0x00007c          0x4 LONG 0x2d8 DEFINED (__T9Interrupt)?ABSOLUTE (__T9Interrupt):ABSOLUTE (__DefaultInterrupt)
                  0x00007e          0x4 LONG 0x46540 DEFINED (__INT3Interrupt)?ABSOLUTE (__INT3Interrupt):ABSOLUTE (__DefaultInterrupt)
                  0x000080          0x4 LONG 0x2d8 DEFINED (__INT4Interrupt)?ABSOLUTE (__INT4Interrupt):ABSOLUTE (__DefaultInterrupt)
                  0x000082          0x4 LONG 0x2d8 DEFINED (__C2RxRdyInterrupt)?ABSOLUTE (__C2RxRdyInterrupt):ABSOLUTE (__DefaultInterrupt)
                  0x000084          0x4 LONG 0x2d8 DEFINED (__C2Interrupt)?ABSOLUTE (__C2Interrupt):ABSOLUTE (__DefaultInterrupt)
                  0x000086          0x4 LONG 0x2d8 DEFINED (__Interrupt57)?ABSOLUTE (__Interrupt57):ABSOLUTE (__DefaultInterrupt)
                  0x000088          0x4 LONG 0x2d8 DEFINED (__Interrupt58)?ABSOLUTE (__Interrupt58):ABSOLUTE (__DefaultInterrupt)
                  0x00008a          0x4 LONG 0x2d8 DEFINED (__DCIEInterrupt)?ABSOLUTE (__DCIEInterrupt):ABSOLUTE (__DefaultInterrupt)
                  0x00008c          0x4 LONG 0x2d8 DEFINED (__DCIInterrupt)?ABSOLUTE (__DCIInterrupt):ABSOLUTE (__DefaultInterrupt)
                  0x00008e          0x4 LONG 0x2d8 DEFINED (__DMA5Interrupt)?ABSOLUTE (__DMA5Interrupt):ABSOLUTE (__DefaultInterrupt)
                  0x000090          0x4 LONG 0x2d8 DEFINED (__RTCCInterrupt)?ABSOLUTE (__RTCCInterrupt):ABSOLUTE (__DefaultInterrupt)
                  0x000092          0x4 LONG 0x2d8 DEFINED (__Interrupt63)?ABSOLUTE (__Interrupt63):ABSOLUTE (__DefaultInterrupt)
                  0x000094          0x4 LONG 0x2d8 DEFINED (__Interrupt64)?ABSOLUTE (__Interrupt64):ABSOLUTE (__DefaultInterrupt)
                  0x000096          0x4 LONG 0x2d8 DEFINED (__U1ErrInterrupt)?ABSOLUTE (__U1ErrInterrupt):ABSOLUTE (__DefaultInterrupt)
                  0x000098          0x4 LONG 0x2d8 DEFINED (__U2ErrInterrupt)?ABSOLUTE (__U2ErrInterrupt):ABSOLUTE (__DefaultInterrupt)
                  0x00009a          0x4 LONG 0x2d8 DEFINED (__CRCInterrupt)?ABSOLUTE (__CRCInterrupt):ABSOLUTE (__DefaultInterrupt)
                  0x00009c          0x4 LONG 0x2d8 DEFINED (__DMA6Interrupt)?ABSOLUTE (__DMA6Interrupt):ABSOLUTE (__DefaultInterrupt)
                  0x00009e          0x4 LONG 0x2d8 DEFINED (__DMA7Interrupt)?ABSOLUTE (__DMA7Interrupt):ABSOLUTE (__DefaultInterrupt)
                  0x0000a0          0x4 LONG 0x2d8 DEFINED (__C1TxReqInterrupt)?ABSOLUTE (__C1TxReqInterrupt):ABSOLUTE (__DefaultInterrupt)
                  0x0000a2          0x4 LONG 0x2d8 DEFINED (__C2TxReqInterrupt)?ABSOLUTE (__C2TxReqInterrupt):ABSOLUTE (__DefaultInterrupt)
                  0x0000a4          0x4 LONG 0x2d8 DEFINED (__Interrupt72)?ABSOLUTE (__Interrupt72):ABSOLUTE (__DefaultInterrupt)
                  0x0000a6          0x4 LONG 0x2d8 DEFINED (__Interrupt73)?ABSOLUTE (__Interrupt73):ABSOLUTE (__DefaultInterrupt)
                  0x0000a8          0x4 LONG 0x2d8 DEFINED (__Interrupt74)?ABSOLUTE (__Interrupt74):ABSOLUTE (__DefaultInterrupt)
                  0x0000aa          0x4 LONG 0x2d8 DEFINED (__Interrupt75)?ABSOLUTE (__Interrupt75):ABSOLUTE (__DefaultInterrupt)
                  0x0000ac          0x4 LONG 0x2d8 DEFINED (__Interrupt76)?ABSOLUTE (__Interrupt76):ABSOLUTE (__DefaultInterrupt)
                  0x0000ae          0x4 LONG 0x2d8 DEFINED (__Interrupt77)?ABSOLUTE (__Interrupt77):ABSOLUTE (__DefaultInterrupt)
                  0x0000b0          0x4 LONG 0x2d8 DEFINED (__Interrupt78)?ABSOLUTE (__Interrupt78):ABSOLUTE (__DefaultInterrupt)
                  0x0000b2          0x4 LONG 0x2d8 DEFINED (__Interrupt79)?ABSOLUTE (__Interrupt79):ABSOLUTE (__DefaultInterrupt)
                  0x0000b4          0x4 LONG 0x2d8 DEFINED (__Interrupt80)?ABSOLUTE (__Interrupt80):ABSOLUTE (__DefaultInterrupt)
                  0x0000b6          0x4 LONG 0x2d8 DEFINED (__U3ErrInterrupt)?ABSOLUTE (__U3ErrInterrupt):ABSOLUTE (__DefaultInterrupt)
                  0x0000b8          0x4 LONG 0x2d8 DEFINED (__U3RXInterrupt)?ABSOLUTE (__U3RXInterrupt):ABSOLUTE (__DefaultInterrupt)
                  0x0000ba          0x4 LONG 0x2d8 DEFINED (__U3TXInterrupt)?ABSOLUTE (__U3TXInterrupt):ABSOLUTE (__DefaultInterrupt)
                  0x0000bc          0x4 LONG 0x2d8 DEFINED (__Interrupt84)?ABSOLUTE (__Interrupt84):ABSOLUTE (__DefaultInterrupt)
                  0x0000be          0x4 LONG 0x2d8 DEFINED (__Interrupt85)?ABSOLUTE (__Interrupt85):ABSOLUTE (__DefaultInterrupt)
                  0x0000c0          0x4 LONG 0x2d8 DEFINED (__USB1Interrupt)?ABSOLUTE (__USB1Interrupt):ABSOLUTE (__DefaultInterrupt)
                  0x0000c2          0x4 LONG 0x2d8 DEFINED (__U4ErrInterrupt)?ABSOLUTE (__U4ErrInterrupt):ABSOLUTE (__DefaultInterrupt)
                  0x0000c4          0x4 LONG 0x2d8 DEFINED (__U4RXInterrupt)?ABSOLUTE (__U4RXInterrupt):ABSOLUTE (__DefaultInterrupt)
                  0x0000c6          0x4 LONG 0x2d8 DEFINED (__U4TXInterrupt)?ABSOLUTE (__U4TXInterrupt):ABSOLUTE (__DefaultInterrupt)
                  0x0000c8          0x4 LONG 0x2d8 DEFINED (__SPI3ErrInterrupt)?ABSOLUTE (__SPI3ErrInterrupt):ABSOLUTE (__DefaultInterrupt)
                  0x0000ca          0x4 LONG 0x2d8 DEFINED (__SPI3Interrupt)?ABSOLUTE (__SPI3Interrupt):ABSOLUTE (__DefaultInterrupt)
                  0x0000cc          0x4 LONG 0x2d8 DEFINED (__OC9Interrupt)?ABSOLUTE (__OC9Interrupt):ABSOLUTE (__DefaultInterrupt)
                  0x0000ce          0x4 LONG 0x2d8 DEFINED (__IC9Interrupt)?ABSOLUTE (__IC9Interrupt):ABSOLUTE (__DefaultInterrupt)
                  0x0000d0          0x4 LONG 0x2d8 DEFINED (__Interrupt94)?ABSOLUTE (__Interrupt94):ABSOLUTE (__DefaultInterrupt)
                  0x0000d2          0x4 LONG 0x2d8 DEFINED (__Interrupt95)?ABSOLUTE (__Interrupt95):ABSOLUTE (__DefaultInterrupt)
                  0x0000d4          0x4 LONG 0x2d8 DEFINED (__Interrupt96)?ABSOLUTE (__Interrupt96):ABSOLUTE (__DefaultInterrupt)
                  0x0000d6          0x4 LONG 0x2d8 DEFINED (__Interrupt97)?ABSOLUTE (__Interrupt97):ABSOLUTE (__DefaultInterrupt)
                  0x0000d8          0x4 LONG 0x2d8 DEFINED (__Interrupt98)?ABSOLUTE (__Interrupt98):ABSOLUTE (__DefaultInterrupt)
                  0x0000da          0x4 LONG 0x2d8 DEFINED (__Interrupt99)?ABSOLUTE (__Interrupt99):ABSOLUTE (__DefaultInterrupt)
                  0x0000dc          0x4 LONG 0x2d8 DEFINED (__Interrupt100)?ABSOLUTE (__Interrupt100):ABSOLUTE (__DefaultInterrupt)
                  0x0000de          0x4 LONG 0x2d8 DEFINED (__Interrupt101)?ABSOLUTE (__Interrupt101):ABSOLUTE (__DefaultInterrupt)
                  0x0000e0          0x4 LONG 0x2d8 DEFINED (__Interrupt102)?ABSOLUTE (__Interrupt102):ABSOLUTE (__DefaultInterrupt)
                  0x0000e2          0x4 LONG 0x2d8 DEFINED (__Interrupt103)?ABSOLUTE (__Interrupt103):ABSOLUTE (__DefaultInterrupt)
                  0x0000e4          0x4 LONG 0x2d8 DEFINED (__Interrupt104)?ABSOLUTE (__Interrupt104):ABSOLUTE (__DefaultInterrupt)
                  0x0000e6          0x4 LONG 0x2d8 DEFINED (__Interrupt105)?ABSOLUTE (__Interrupt105):ABSOLUTE (__DefaultInterrupt)
                  0x0000e8          0x4 LONG 0x2d8 DEFINED (__Interrupt106)?ABSOLUTE (__Interrupt106):ABSOLUTE (__DefaultInterrupt)
                  0x0000ea          0x4 LONG 0x2d8 DEFINED (__Interrupt107)?ABSOLUTE (__Interrupt107):ABSOLUTE (__DefaultInterrupt)
                  0x0000ec          0x4 LONG 0x2d8 DEFINED (__Interrupt108)?ABSOLUTE (__Interrupt108):ABSOLUTE (__DefaultInterrupt)
                  0x0000ee          0x4 LONG 0x2d8 DEFINED (__Interrupt109)?ABSOLUTE (__Interrupt109):ABSOLUTE (__DefaultInterrupt)
                  0x0000f0          0x4 LONG 0x2d8 DEFINED (__Interrupt110)?ABSOLUTE (__Interrupt110):ABSOLUTE (__DefaultInterrupt)
                  0x0000f2          0x4 LONG 0x2d8 DEFINED (__Interrupt111)?ABSOLUTE (__Interrupt111):ABSOLUTE (__DefaultInterrupt)
                  0x0000f4          0x4 LONG 0x2d8 DEFINED (__Interrupt112)?ABSOLUTE (__Interrupt112):ABSOLUTE (__DefaultInterrupt)
                  0x0000f6          0x4 LONG 0x2d8 DEFINED (__Interrupt113)?ABSOLUTE (__Interrupt113):ABSOLUTE (__DefaultInterrupt)
                  0x0000f8          0x4 LONG 0x2d8 DEFINED (__Interrupt114)?ABSOLUTE (__Interrupt114):ABSOLUTE (__DefaultInterrupt)
                  0x0000fa          0x4 LONG 0x2d8 DEFINED (__Interrupt115)?ABSOLUTE (__Interrupt115):ABSOLUTE (__DefaultInterrupt)
                  0x0000fc          0x4 LONG 0x2d8 DEFINED (__Interrupt116)?ABSOLUTE (__Interrupt116):ABSOLUTE (__DefaultInterrupt)
                  0x0000fe          0x4 LONG 0x2d8 DEFINED (__Interrupt117)?ABSOLUTE (__Interrupt117):ABSOLUTE (__DefaultInterrupt)
                  0x000100          0x4 LONG 0x2d8 DEFINED (__DMA8Interrupt)?ABSOLUTE (__DMA8Interrupt):ABSOLUTE (__DefaultInterrupt)
                  0x000102          0x4 LONG 0x2d8 DEFINED (__DMA9Interrupt)?ABSOLUTE (__DMA9Interrupt):ABSOLUTE (__DefaultInterrupt)
                  0x000104          0x4 LONG 0x2d8 DEFINED (__DMA10Interrupt)?ABSOLUTE (__DMA10Interrupt):ABSOLUTE (__DefaultInterrupt)
                  0x000106          0x4 LONG 0x2d8 DEFINED (__DMA11Interrupt)?ABSOLUTE (__DMA11Interrupt):ABSOLUTE (__DefaultInterrupt)
                  0x000108          0x4 LONG 0x2d8 DEFINED (__SPI4ErrInterrupt)?ABSOLUTE (__SPI4ErrInterrupt):ABSOLUTE (__DefaultInterrupt)
                  0x00010a          0x4 LONG 0x2d8 DEFINED (__SPI4Interrupt)?ABSOLUTE (__SPI4Interrupt):ABSOLUTE (__DefaultInterrupt)
                  0x00010c          0x4 LONG 0x2d8 DEFINED (__OC10Interrupt)?ABSOLUTE (__OC10Interrupt):ABSOLUTE (__DefaultInterrupt)
                  0x00010e          0x4 LONG 0x2d8 DEFINED (__IC10Interrupt)?ABSOLUTE (__IC10Interrupt):ABSOLUTE (__DefaultInterrupt)
                  0x000110          0x4 LONG 0x2d8 DEFINED (__OC11Interrupt)?ABSOLUTE (__OC11Interrupt):ABSOLUTE (__DefaultInterrupt)
                  0x000112          0x4 LONG 0x2d8 DEFINED (__IC11Interrupt)?ABSOLUTE (__IC11Interrupt):ABSOLUTE (__DefaultInterrupt)
                  0x000114          0x4 LONG 0x2d8 DEFINED (__OC12Interrupt)?ABSOLUTE (__OC12Interrupt):ABSOLUTE (__DefaultInterrupt)
                  0x000116          0x4 LONG 0x2d8 DEFINED (__IC12Interrupt)?ABSOLUTE (__IC12Interrupt):ABSOLUTE (__DefaultInterrupt)
                  0x000118          0x4 LONG 0x2d8 DEFINED (__DMA12Interrupt)?ABSOLUTE (__DMA12Interrupt):ABSOLUTE (__DefaultInterrupt)
                  0x00011a          0x4 LONG 0x2d8 DEFINED (__DMA13Interrupt)?ABSOLUTE (__DMA13Interrupt):ABSOLUTE (__DefaultInterrupt)
                  0x00011c          0x4 LONG 0x2d8 DEFINED (__DMA14Interrupt)?ABSOLUTE (__DMA14Interrupt):ABSOLUTE (__DefaultInterrupt)
                  0x00011e          0x4 LONG 0x2d8 DEFINED (__Interrupt133)?ABSOLUTE (__Interrupt133):ABSOLUTE (__DefaultInterrupt)
                  0x000120          0x4 LONG 0x2d8 DEFINED (__OC13Interrupt)?ABSOLUTE (__OC13Interrupt):ABSOLUTE (__DefaultInterrupt)
                  0x000122          0x4 LONG 0x2d8 DEFINED (__IC13Interrupt)?ABSOLUTE (__IC13Interrupt):ABSOLUTE (__DefaultInterrupt)
                  0x000124          0x4 LONG 0x2d8 DEFINED (__OC14Interrupt)?ABSOLUTE (__OC14Interrupt):ABSOLUTE (__DefaultInterrupt)
                  0x000126          0x4 LONG 0x2d8 DEFINED (__IC14Interrupt)?ABSOLUTE (__IC14Interrupt):ABSOLUTE (__DefaultInterrupt)
                  0x000128          0x4 LONG 0x2d8 DEFINED (__OC15Interrupt)?ABSOLUTE (__OC15Interrupt):ABSOLUTE (__DefaultInterrupt)
                  0x00012a          0x4 LONG 0x2d8 DEFINED (__IC15Interrupt)?ABSOLUTE (__IC15Interrupt):ABSOLUTE (__DefaultInterrupt)
                  0x00012c          0x4 LONG 0x2d8 DEFINED (__OC16Interrupt)?ABSOLUTE (__OC16Interrupt):ABSOLUTE (__DefaultInterrupt)
                  0x00012e          0x4 LONG 0x2d8 DEFINED (__IC16Interrupt)?ABSOLUTE (__IC16Interrupt):ABSOLUTE (__DefaultInterrupt)
                  0x000130          0x4 LONG 0x2d8 DEFINED (__ICDInterrupt)?ABSOLUTE (__ICDInterrupt):ABSOLUTE (__DefaultInterrupt)
                  0x000132          0x4 LONG 0x2d8 DEFINED (__JTAGInterrupt)?ABSOLUTE (__JTAGInterrupt):ABSOLUTE (__DefaultInterrupt)
                    0x0000                  WREG0 = 0x0
                    0x0000                  _WREG0 = 0x0
                    0x0002                  WREG1 = 0x2
                    0x0002                  _WREG1 = 0x2
                    0x0004                  WREG2 = 0x4
                    0x0004                  _WREG2 = 0x4
                    0x0006                  WREG3 = 0x6
                    0x0006                  _WREG3 = 0x6
                    0x0008                  WREG4 = 0x8
                    0x0008                  _WREG4 = 0x8
                    0x000a                  WREG5 = 0xa
                    0x000a                  _WREG5 = 0xa
                    0x000c                  WREG6 = 0xc
                    0x000c                  _WREG6 = 0xc
                    0x000e                  WREG7 = 0xe
                    0x000e                  _WREG7 = 0xe
                    0x0010                  WREG8 = 0x10
                    0x0010                  _WREG8 = 0x10
                    0x0012                  WREG9 = 0x12
                    0x0012                  _WREG9 = 0x12
                    0x0014                  WREG10 = 0x14
                    0x0014                  _WREG10 = 0x14
                    0x0016                  WREG11 = 0x16
                    0x0016                  _WREG11 = 0x16
                    0x0018                  WREG12 = 0x18
                    0x0018                  _WREG12 = 0x18
                    0x001a                  WREG13 = 0x1a
                    0x001a                  _WREG13 = 0x1a
                    0x001c                  WREG14 = 0x1c
                    0x001c                  _WREG14 = 0x1c
                    0x001e                  WREG15 = 0x1e
                    0x001e                  _WREG15 = 0x1e
                    0x0020                  SPLIM = 0x20
                    0x0020                  _SPLIM = 0x20
                    0x002e                  PCL = 0x2e
                    0x002e                  _PCL = 0x2e
                    0x0030                  PCH = 0x30
                    0x0030                  _PCH = 0x30
                    0x0032                  DSRPAG = 0x32
                    0x0032                  _DSRPAG = 0x32
                    0x0032                  _DSRPAGbits = 0x32
                    0x0034                  DSWPAG = 0x34
                    0x0034                  _DSWPAG = 0x34
                    0x0034                  _DSWPAGbits = 0x34
                    0x0036                  RCOUNT = 0x36
                    0x0036                  _RCOUNT = 0x36
                    0x0042                  SR = 0x42
                    0x0042                  _SR = 0x42
                    0x0042                  _SRbits = 0x42
                    0x0044                  CORCON = 0x44
                    0x0044                  _CORCON = 0x44
                    0x0044                  _CORCONbits = 0x44
                    0x0052                  DISICNT = 0x52
                    0x0052                  _DISICNT = 0x52
                    0x0054                  TBLPAG = 0x54
                    0x0054                  _TBLPAG = 0x54
                    0x0054                  _TBLPAGbits = 0x54
                    0x0058                  MSTRPR = 0x58
                    0x0058                  _MSTRPR = 0x58
                    0x0100                  TMR1 = 0x100
                    0x0100                  _TMR1 = 0x100
                    0x0102                  PR1 = 0x102
                    0x0102                  _PR1 = 0x102
                    0x0104                  T1CON = 0x104
                    0x0104                  _T1CON = 0x104
                    0x0104                  _T1CONbits = 0x104
                    0x0106                  TMR2 = 0x106
                    0x0106                  _TMR2 = 0x106
                    0x0108                  TMR3HLD = 0x108
                    0x0108                  _TMR3HLD = 0x108
                    0x010a                  TMR3 = 0x10a
                    0x010a                  _TMR3 = 0x10a
                    0x010c                  PR2 = 0x10c
                    0x010c                  _PR2 = 0x10c
                    0x010e                  PR3 = 0x10e
                    0x010e                  _PR3 = 0x10e
                    0x0110                  T2CON = 0x110
                    0x0110                  _T2CON = 0x110
                    0x0110                  _T2CONbits = 0x110
                    0x0112                  T3CON = 0x112
                    0x0112                  _T3CON = 0x112
                    0x0112                  _T3CONbits = 0x112
                    0x0114                  TMR4 = 0x114
                    0x0114                  _TMR4 = 0x114
                    0x0116                  TMR5HLD = 0x116
                    0x0116                  _TMR5HLD = 0x116
                    0x0118                  TMR5 = 0x118
                    0x0118                  _TMR5 = 0x118
                    0x011a                  PR4 = 0x11a
                    0x011a                  _PR4 = 0x11a
                    0x011c                  PR5 = 0x11c
                    0x011c                  _PR5 = 0x11c
                    0x011e                  T4CON = 0x11e
                    0x011e                  _T4CON = 0x11e
                    0x011e                  _T4CONbits = 0x11e
                    0x0120                  T5CON = 0x120
                    0x0120                  _T5CON = 0x120
                    0x0120                  _T5CONbits = 0x120
                    0x0122                  TMR6 = 0x122
                    0x0122                  _TMR6 = 0x122
                    0x0124                  TMR7HLD = 0x124
                    0x0124                  _TMR7HLD = 0x124
                    0x0126                  TMR7 = 0x126
                    0x0126                  _TMR7 = 0x126
                    0x0128                  PR6 = 0x128
                    0x0128                  _PR6 = 0x128
                    0x012a                  PR7 = 0x12a
                    0x012a                  _PR7 = 0x12a
                    0x012c                  T6CON = 0x12c
                    0x012c                  _T6CON = 0x12c
                    0x012c                  _T6CONbits = 0x12c
                    0x012e                  T7CON = 0x12e
                    0x012e                  _T7CON = 0x12e
                    0x012e                  _T7CONbits = 0x12e
                    0x0130                  TMR8 = 0x130
                    0x0130                  _TMR8 = 0x130
                    0x0132                  TMR9HLD = 0x132
                    0x0132                  _TMR9HLD = 0x132
                    0x0134                  TMR9 = 0x134
                    0x0134                  _TMR9 = 0x134
                    0x0136                  PR8 = 0x136
                    0x0136                  _PR8 = 0x136
                    0x0138                  PR9 = 0x138
                    0x0138                  _PR9 = 0x138
                    0x013a                  T8CON = 0x13a
                    0x013a                  _T8CON = 0x13a
                    0x013a                  _T8CONbits = 0x13a
                    0x013c                  T9CON = 0x13c
                    0x013c                  _T9CON = 0x13c
                    0x013c                  _T9CONbits = 0x13c
                    0x0140                  IC1CON1 = 0x140
                    0x0140                  _IC1CON1 = 0x140
                    0x0140                  _IC1CON1bits = 0x140
                    0x0142                  IC1CON2 = 0x142
                    0x0142                  _IC1CON2 = 0x142
                    0x0142                  _IC1CON2bits = 0x142
                    0x0144                  IC1BUF = 0x144
                    0x0144                  _IC1BUF = 0x144
                    0x0146                  IC1TMR = 0x146
                    0x0146                  _IC1TMR = 0x146
                    0x0148                  IC2CON1 = 0x148
                    0x0148                  _IC2CON1 = 0x148
                    0x0148                  _IC2CON1bits = 0x148
                    0x014a                  IC2CON2 = 0x14a
                    0x014a                  _IC2CON2 = 0x14a
                    0x014a                  _IC2CON2bits = 0x14a
                    0x014c                  IC2BUF = 0x14c
                    0x014c                  _IC2BUF = 0x14c
                    0x014e                  IC2TMR = 0x14e
                    0x014e                  _IC2TMR = 0x14e
                    0x0150                  IC3CON1 = 0x150
                    0x0150                  _IC3CON1 = 0x150
                    0x0150                  _IC3CON1bits = 0x150
                    0x0152                  IC3CON2 = 0x152
                    0x0152                  _IC3CON2 = 0x152
                    0x0152                  _IC3CON2bits = 0x152
                    0x0154                  IC3BUF = 0x154
                    0x0154                  _IC3BUF = 0x154
                    0x0156                  IC3TMR = 0x156
                    0x0156                  _IC3TMR = 0x156
                    0x0158                  IC4CON1 = 0x158
                    0x0158                  _IC4CON1 = 0x158
                    0x0158                  _IC4CON1bits = 0x158
                    0x015a                  IC4CON2 = 0x15a
                    0x015a                  _IC4CON2 = 0x15a
                    0x015a                  _IC4CON2bits = 0x15a
                    0x015c                  IC4BUF = 0x15c
                    0x015c                  _IC4BUF = 0x15c
                    0x015e                  IC4TMR = 0x15e
                    0x015e                  _IC4TMR = 0x15e
                    0x0160                  IC5CON1 = 0x160
                    0x0160                  _IC5CON1 = 0x160
                    0x0160                  _IC5CON1bits = 0x160
                    0x0162                  IC5CON2 = 0x162
                    0x0162                  _IC5CON2 = 0x162
                    0x0162                  _IC5CON2bits = 0x162
                    0x0164                  IC5BUF = 0x164
                    0x0164                  _IC5BUF = 0x164
                    0x0166                  IC5TMR = 0x166
                    0x0166                  _IC5TMR = 0x166
                    0x0168                  IC6CON1 = 0x168
                    0x0168                  _IC6CON1 = 0x168
                    0x0168                  _IC6CON1bits = 0x168
                    0x016a                  IC6CON2 = 0x16a
                    0x016a                  _IC6CON2 = 0x16a
                    0x016a                  _IC6CON2bits = 0x16a
                    0x016c                  IC6BUF = 0x16c
                    0x016c                  _IC6BUF = 0x16c
                    0x016e                  IC6TMR = 0x16e
                    0x016e                  _IC6TMR = 0x16e
                    0x0170                  IC7CON1 = 0x170
                    0x0170                  _IC7CON1 = 0x170
                    0x0170                  _IC7CON1bits = 0x170
                    0x0172                  IC7CON2 = 0x172
                    0x0172                  _IC7CON2 = 0x172
                    0x0172                  _IC7CON2bits = 0x172
                    0x0174                  IC7BUF = 0x174
                    0x0174                  _IC7BUF = 0x174
                    0x0176                  IC7TMR = 0x176
                    0x0176                  _IC7TMR = 0x176
                    0x0178                  IC8CON1 = 0x178
                    0x0178                  _IC8CON1 = 0x178
                    0x0178                  _IC8CON1bits = 0x178
                    0x017a                  IC8CON2 = 0x17a
                    0x017a                  _IC8CON2 = 0x17a
                    0x017a                  _IC8CON2bits = 0x17a
                    0x017c                  IC8BUF = 0x17c
                    0x017c                  _IC8BUF = 0x17c
                    0x017e                  IC8TMR = 0x17e
                    0x017e                  _IC8TMR = 0x17e
                    0x0180                  IC9CON1 = 0x180
                    0x0180                  _IC9CON1 = 0x180
                    0x0180                  _IC9CON1bits = 0x180
                    0x0182                  IC9CON2 = 0x182
                    0x0182                  _IC9CON2 = 0x182
                    0x0182                  _IC9CON2bits = 0x182
                    0x0184                  IC9BUF = 0x184
                    0x0184                  _IC9BUF = 0x184
                    0x0186                  IC9TMR = 0x186
                    0x0186                  _IC9TMR = 0x186
                    0x0188                  IC10CON1 = 0x188
                    0x0188                  _IC10CON1 = 0x188
                    0x0188                  _IC10CON1bits = 0x188
                    0x018a                  IC10CON2 = 0x18a
                    0x018a                  _IC10CON2 = 0x18a
                    0x018a                  _IC10CON2bits = 0x18a
                    0x018c                  IC10BUF = 0x18c
                    0x018c                  _IC10BUF = 0x18c
                    0x018e                  IC10TMR = 0x18e
                    0x018e                  _IC10TMR = 0x18e
                    0x0190                  IC11CON1 = 0x190
                    0x0190                  _IC11CON1 = 0x190
                    0x0190                  _IC11CON1bits = 0x190
                    0x0192                  IC11CON2 = 0x192
                    0x0192                  _IC11CON2 = 0x192
                    0x0192                  _IC11CON2bits = 0x192
                    0x0194                  IC11BUF = 0x194
                    0x0194                  _IC11BUF = 0x194
                    0x0196                  IC11TMR = 0x196
                    0x0196                  _IC11TMR = 0x196
                    0x0198                  IC12CON1 = 0x198
                    0x0198                  _IC12CON1 = 0x198
                    0x0198                  _IC12CON1bits = 0x198
                    0x019a                  IC12CON2 = 0x19a
                    0x019a                  _IC12CON2 = 0x19a
                    0x019a                  _IC12CON2bits = 0x19a
                    0x019c                  IC12BUF = 0x19c
                    0x019c                  _IC12BUF = 0x19c
                    0x019e                  IC12TMR = 0x19e
                    0x019e                  _IC12TMR = 0x19e
                    0x01a0                  IC13CON1 = 0x1a0
                    0x01a0                  _IC13CON1 = 0x1a0
                    0x01a0                  _IC13CON1bits = 0x1a0
                    0x01a2                  IC13CON2 = 0x1a2
                    0x01a2                  _IC13CON2 = 0x1a2
                    0x01a2                  _IC13CON2bits = 0x1a2
                    0x01a4                  IC13BUF = 0x1a4
                    0x01a4                  _IC13BUF = 0x1a4
                    0x01a6                  IC13TMR = 0x1a6
                    0x01a6                  _IC13TMR = 0x1a6
                    0x01a8                  IC14CON1 = 0x1a8
                    0x01a8                  _IC14CON1 = 0x1a8
                    0x01a8                  _IC14CON1bits = 0x1a8
                    0x01aa                  IC14CON2 = 0x1aa
                    0x01aa                  _IC14CON2 = 0x1aa
                    0x01aa                  _IC14CON2bits = 0x1aa
                    0x01ac                  IC14BUF = 0x1ac
                    0x01ac                  _IC14BUF = 0x1ac
                    0x01ae                  IC14TMR = 0x1ae
                    0x01ae                  _IC14TMR = 0x1ae
                    0x01b0                  IC15CON1 = 0x1b0
                    0x01b0                  _IC15CON1 = 0x1b0
                    0x01b0                  _IC15CON1bits = 0x1b0
                    0x01b2                  IC15CON2 = 0x1b2
                    0x01b2                  _IC15CON2 = 0x1b2
                    0x01b2                  _IC15CON2bits = 0x1b2
                    0x01b4                  IC15BUF = 0x1b4
                    0x01b4                  _IC15BUF = 0x1b4
                    0x01b6                  IC15TMR = 0x1b6
                    0x01b6                  _IC15TMR = 0x1b6
                    0x01b8                  IC16CON1 = 0x1b8
                    0x01b8                  _IC16CON1 = 0x1b8
                    0x01b8                  _IC16CON1bits = 0x1b8
                    0x01ba                  IC16CON2 = 0x1ba
                    0x01ba                  _IC16CON2 = 0x1ba
                    0x01ba                  _IC16CON2bits = 0x1ba
                    0x01bc                  IC16BUF = 0x1bc
                    0x01bc                  _IC16BUF = 0x1bc
                    0x01be                  IC16TMR = 0x1be
                    0x01be                  _IC16TMR = 0x1be
                    0x0200                  I2C1RCV = 0x200
                    0x0200                  _I2C1RCV = 0x200
                    0x0202                  I2C1TRN = 0x202
                    0x0202                  _I2C1TRN = 0x202
                    0x0204                  I2C1BRG = 0x204
                    0x0204                  _I2C1BRG = 0x204
                    0x0206                  I2C1CON = 0x206
                    0x0206                  _I2C1CON = 0x206
                    0x0206                  _I2C1CONbits = 0x206
                    0x0208                  I2C1STAT = 0x208
                    0x0208                  _I2C1STAT = 0x208
                    0x0208                  _I2C1STATbits = 0x208
                    0x020a                  I2C1ADD = 0x20a
                    0x020a                  _I2C1ADD = 0x20a
                    0x020c                  I2C1MSK = 0x20c
                    0x020c                  _I2C1MSK = 0x20c
                    0x0210                  I2C2RCV = 0x210
                    0x0210                  _I2C2RCV = 0x210
                    0x0212                  I2C2TRN = 0x212
                    0x0212                  _I2C2TRN = 0x212
                    0x0214                  I2C2BRG = 0x214
                    0x0214                  _I2C2BRG = 0x214
                    0x0216                  I2C2CON = 0x216
                    0x0216                  _I2C2CON = 0x216
                    0x0216                  _I2C2CONbits = 0x216
                    0x0218                  I2C2STAT = 0x218
                    0x0218                  _I2C2STAT = 0x218
                    0x0218                  _I2C2STATbits = 0x218
                    0x021a                  I2C2ADD = 0x21a
                    0x021a                  _I2C2ADD = 0x21a
                    0x021c                  I2C2MSK = 0x21c
                    0x021c                  _I2C2MSK = 0x21c
                    0x0220                  U1MODE = 0x220
                    0x0220                  _U1MODE = 0x220
                    0x0220                  _U1MODEbits = 0x220
                    0x0222                  U1STA = 0x222
                    0x0222                  _U1STA = 0x222
                    0x0222                  _U1STAbits = 0x222
                    0x0224                  U1TXREG = 0x224
                    0x0224                  _U1TXREG = 0x224
                    0x0226                  U1RXREG = 0x226
                    0x0226                  _U1RXREG = 0x226
                    0x0228                  U1BRG = 0x228
                    0x0228                  _U1BRG = 0x228
                    0x0230                  U2MODE = 0x230
                    0x0230                  _U2MODE = 0x230
                    0x0230                  _U2MODEbits = 0x230
                    0x0232                  U2STA = 0x232
                    0x0232                  _U2STA = 0x232
                    0x0232                  _U2STAbits = 0x232
                    0x0234                  U2TXREG = 0x234
                    0x0234                  _U2TXREG = 0x234
                    0x0236                  U2RXREG = 0x236
                    0x0236                  _U2RXREG = 0x236
                    0x0238                  U2BRG = 0x238
                    0x0238                  _U2BRG = 0x238
                    0x0240                  SPI1STAT = 0x240
                    0x0240                  _SPI1STAT = 0x240
                    0x0240                  _SPI1STATbits = 0x240
                    0x0242                  SPI1CON1 = 0x242
                    0x0242                  _SPI1CON1 = 0x242
                    0x0242                  _SPI1CON1bits = 0x242
                    0x0244                  SPI1CON2 = 0x244
                    0x0244                  _SPI1CON2 = 0x244
                    0x0244                  _SPI1CON2bits = 0x244
                    0x0248                  SPI1BUF = 0x248
                    0x0248                  _SPI1BUF = 0x248
                    0x0250                  U3MODE = 0x250
                    0x0250                  _U3MODE = 0x250
                    0x0250                  _U3MODEbits = 0x250
                    0x0252                  U3STA = 0x252
                    0x0252                  _U3STA = 0x252
                    0x0252                  _U3STAbits = 0x252
                    0x0254                  U3TXREG = 0x254
                    0x0254                  _U3TXREG = 0x254
                    0x0256                  U3RXREG = 0x256
                    0x0256                  _U3RXREG = 0x256
                    0x0258                  U3BRG = 0x258
                    0x0258                  _U3BRG = 0x258
                    0x0260                  SPI2STAT = 0x260
                    0x0260                  _SPI2STAT = 0x260
                    0x0260                  _SPI2STATbits = 0x260
                    0x0262                  SPI2CON1 = 0x262
                    0x0262                  _SPI2CON1 = 0x262
                    0x0262                  _SPI2CON1bits = 0x262
                    0x0264                  SPI2CON2 = 0x264
                    0x0264                  _SPI2CON2 = 0x264
                    0x0264                  _SPI2CON2bits = 0x264
                    0x0268                  SPI2BUF = 0x268
                    0x0268                  _SPI2BUF = 0x268
                    0x0280                  DCICON1 = 0x280
                    0x0280                  _DCICON1 = 0x280
                    0x0280                  _DCICON1bits = 0x280
                    0x0282                  DCICON2 = 0x282
                    0x0282                  _DCICON2 = 0x282
                    0x0282                  _DCICON2bits = 0x282
                    0x0284                  DCICON3 = 0x284
                    0x0284                  _DCICON3 = 0x284
                    0x0284                  _DCICON3bits = 0x284
                    0x0286                  DCISTAT = 0x286
                    0x0286                  _DCISTAT = 0x286
                    0x0286                  _DCISTATbits = 0x286
                    0x0288                  TSCON = 0x288
                    0x0288                  _TSCON = 0x288
                    0x0288                  _TSCONbits = 0x288
                    0x028c                  RSCON = 0x28c
                    0x028c                  _RSCON = 0x28c
                    0x028c                  _RSCONbits = 0x28c
                    0x0290                  RXBUF0 = 0x290
                    0x0290                  _RXBUF0 = 0x290
                    0x0292                  RXBUF1 = 0x292
                    0x0292                  _RXBUF1 = 0x292
                    0x0294                  RXBUF2 = 0x294
                    0x0294                  _RXBUF2 = 0x294
                    0x0296                  RXBUF3 = 0x296
                    0x0296                  _RXBUF3 = 0x296
                    0x0298                  TXBUF0 = 0x298
                    0x0298                  _TXBUF0 = 0x298
                    0x029a                  TXBUF1 = 0x29a
                    0x029a                  _TXBUF1 = 0x29a
                    0x029c                  TXBUF2 = 0x29c
                    0x029c                  _TXBUF2 = 0x29c
                    0x029e                  TXBUF3 = 0x29e
                    0x029e                  _TXBUF3 = 0x29e
                    0x02a0                  SPI3STAT = 0x2a0
                    0x02a0                  _SPI3STAT = 0x2a0
                    0x02a0                  _SPI3STATbits = 0x2a0
                    0x02a2                  SPI3CON1 = 0x2a2
                    0x02a2                  _SPI3CON1 = 0x2a2
                    0x02a2                  _SPI3CON1bits = 0x2a2
                    0x02a4                  SPI3CON2 = 0x2a4
                    0x02a4                  _SPI3CON2 = 0x2a4
                    0x02a4                  _SPI3CON2bits = 0x2a4
                    0x02a8                  SPI3BUF = 0x2a8
                    0x02a8                  _SPI3BUF = 0x2a8
                    0x02b0                  U4MODE = 0x2b0
                    0x02b0                  _U4MODE = 0x2b0
                    0x02b0                  _U4MODEbits = 0x2b0
                    0x02b2                  U4STA = 0x2b2
                    0x02b2                  _U4STA = 0x2b2
                    0x02b2                  _U4STAbits = 0x2b2
                    0x02b4                  U4TXREG = 0x2b4
                    0x02b4                  _U4TXREG = 0x2b4
                    0x02b6                  U4RXREG = 0x2b6
                    0x02b6                  _U4RXREG = 0x2b6
                    0x02b8                  U4BRG = 0x2b8
                    0x02b8                  _U4BRG = 0x2b8
                    0x02c0                  SPI4STAT = 0x2c0
                    0x02c0                  _SPI4STAT = 0x2c0
                    0x02c0                  _SPI4STATbits = 0x2c0
                    0x02c2                  SPI4CON1 = 0x2c2
                    0x02c2                  _SPI4CON1 = 0x2c2
                    0x02c2                  _SPI4CON1bits = 0x2c2
                    0x02c4                  SPI4CON2 = 0x2c4
                    0x02c4                  _SPI4CON2 = 0x2c4
                    0x02c4                  _SPI4CON2bits = 0x2c4
                    0x02c8                  SPI4BUF = 0x2c8
                    0x02c8                  _SPI4BUF = 0x2c8
                    0x0300                  ADC1BUF0 = 0x300
                    0x0300                  _ADC1BUF0 = 0x300
                    0x0302                  ADC1BUF1 = 0x302
                    0x0302                  _ADC1BUF1 = 0x302
                    0x0304                  ADC1BUF2 = 0x304
                    0x0304                  _ADC1BUF2 = 0x304
                    0x0306                  ADC1BUF3 = 0x306
                    0x0306                  _ADC1BUF3 = 0x306
                    0x0308                  ADC1BUF4 = 0x308
                    0x0308                  _ADC1BUF4 = 0x308
                    0x030a                  ADC1BUF5 = 0x30a
                    0x030a                  _ADC1BUF5 = 0x30a
                    0x030c                  ADC1BUF6 = 0x30c
                    0x030c                  _ADC1BUF6 = 0x30c
                    0x030e                  ADC1BUF7 = 0x30e
                    0x030e                  _ADC1BUF7 = 0x30e
                    0x0310                  ADC1BUF8 = 0x310
                    0x0310                  _ADC1BUF8 = 0x310
                    0x0312                  ADC1BUF9 = 0x312
                    0x0312                  _ADC1BUF9 = 0x312
                    0x0314                  ADC1BUFA = 0x314
                    0x0314                  _ADC1BUFA = 0x314
                    0x0316                  ADC1BUFB = 0x316
                    0x0316                  _ADC1BUFB = 0x316
                    0x0318                  ADC1BUFC = 0x318
                    0x0318                  _ADC1BUFC = 0x318
                    0x031a                  ADC1BUFD = 0x31a
                    0x031a                  _ADC1BUFD = 0x31a
                    0x031c                  ADC1BUFE = 0x31c
                    0x031c                  _ADC1BUFE = 0x31c
                    0x031e                  ADC1BUFF = 0x31e
                    0x031e                  _ADC1BUFF = 0x31e
                    0x0320                  AD1CON1 = 0x320
                    0x0320                  _AD1CON1 = 0x320
                    0x0320                  _AD1CON1bits = 0x320
                    0x0322                  AD1CON2 = 0x322
                    0x0322                  _AD1CON2 = 0x322
                    0x0322                  _AD1CON2bits = 0x322
                    0x0324                  AD1CON3 = 0x324
                    0x0324                  _AD1CON3 = 0x324
                    0x0324                  _AD1CON3bits = 0x324
                    0x0326                  AD1CHS123 = 0x326
                    0x0326                  _AD1CHS123 = 0x326
                    0x0326                  _AD1CHS123bits = 0x326
                    0x0328                  AD1CHS0 = 0x328
                    0x0328                  _AD1CHS0 = 0x328
                    0x0328                  _AD1CHS0bits = 0x328
                    0x032e                  AD1CSSH = 0x32e
                    0x032e                  _AD1CSSH = 0x32e
                    0x032e                  _AD1CSSHbits = 0x32e
                    0x0330                  AD1CSSL = 0x330
                    0x0330                  _AD1CSSL = 0x330
                    0x0330                  _AD1CSSLbits = 0x330
                    0x0332                  AD1CON4 = 0x332
                    0x0332                  _AD1CON4 = 0x332
                    0x0332                  _AD1CON4bits = 0x332
                    0x0340                  ADC2BUF0 = 0x340
                    0x0340                  _ADC2BUF0 = 0x340
                    0x0342                  ADC2BUF1 = 0x342
                    0x0342                  _ADC2BUF1 = 0x342
                    0x0344                  ADC2BUF2 = 0x344
                    0x0344                  _ADC2BUF2 = 0x344
                    0x0346                  ADC2BUF3 = 0x346
                    0x0346                  _ADC2BUF3 = 0x346
                    0x0348                  ADC2BUF4 = 0x348
                    0x0348                  _ADC2BUF4 = 0x348
                    0x034a                  ADC2BUF5 = 0x34a
                    0x034a                  _ADC2BUF5 = 0x34a
                    0x034c                  ADC2BUF6 = 0x34c
                    0x034c                  _ADC2BUF6 = 0x34c
                    0x034e                  ADC2BUF7 = 0x34e
                    0x034e                  _ADC2BUF7 = 0x34e
                    0x0350                  ADC2BUF8 = 0x350
                    0x0350                  _ADC2BUF8 = 0x350
                    0x0352                  ADC2BUF9 = 0x352
                    0x0352                  _ADC2BUF9 = 0x352
                    0x0354                  ADC2BUFA = 0x354
                    0x0354                  _ADC2BUFA = 0x354
                    0x0356                  ADC2BUFB = 0x356
                    0x0356                  _ADC2BUFB = 0x356
                    0x0358                  ADC2BUFC = 0x358
                    0x0358                  _ADC2BUFC = 0x358
                    0x035a                  ADC2BUFD = 0x35a
                    0x035a                  _ADC2BUFD = 0x35a
                    0x035c                  ADC2BUFE = 0x35c
                    0x035c                  _ADC2BUFE = 0x35c
                    0x035e                  ADC2BUFF = 0x35e
                    0x035e                  _ADC2BUFF = 0x35e
                    0x0360                  AD2CON1 = 0x360
                    0x0360                  _AD2CON1 = 0x360
                    0x0360                  _AD2CON1bits = 0x360
                    0x0362                  AD2CON2 = 0x362
                    0x0362                  _AD2CON2 = 0x362
                    0x0362                  _AD2CON2bits = 0x362
                    0x0364                  AD2CON3 = 0x364
                    0x0364                  _AD2CON3 = 0x364
                    0x0364                  _AD2CON3bits = 0x364
                    0x0366                  AD2CHS123 = 0x366
                    0x0366                  _AD2CHS123 = 0x366
                    0x0366                  _AD2CHS123bits = 0x366
                    0x0368                  AD2CHS0 = 0x368
                    0x0368                  _AD2CHS0 = 0x368
                    0x0368                  _AD2CHS0bits = 0x368
                    0x0370                  AD2CSSL = 0x370
                    0x0370                  _AD2CSSL = 0x370
                    0x0370                  _AD2CSSLbits = 0x370
                    0x0372                  AD2CON4 = 0x372
                    0x0372                  _AD2CON4 = 0x372
                    0x0372                  _AD2CON4bits = 0x372
                    0x0400                  C1CTRL1 = 0x400
                    0x0400                  _C1CTRL1 = 0x400
                    0x0400                  _C1CTRL1bits = 0x400
                    0x0402                  C1CTRL2 = 0x402
                    0x0402                  _C1CTRL2 = 0x402
                    0x0402                  _C1CTRL2bits = 0x402
                    0x0404                  C1VEC = 0x404
                    0x0404                  _C1VEC = 0x404
                    0x0404                  _C1VECbits = 0x404
                    0x0406                  C1FCTRL = 0x406
                    0x0406                  _C1FCTRL = 0x406
                    0x0406                  _C1FCTRLbits = 0x406
                    0x0408                  C1FIFO = 0x408
                    0x0408                  _C1FIFO = 0x408
                    0x0408                  _C1FIFObits = 0x408
                    0x040a                  C1INTF = 0x40a
                    0x040a                  _C1INTF = 0x40a
                    0x040a                  _C1INTFbits = 0x40a
                    0x040c                  C1INTE = 0x40c
                    0x040c                  _C1INTE = 0x40c
                    0x040c                  _C1INTEbits = 0x40c
                    0x040e                  C1EC = 0x40e
                    0x040e                  _C1EC = 0x40e
                    0x040e                  _C1ECbits = 0x40e
                    0x040e                  C1RERRCNT = 0x40e
                    0x040e                  _C1RERRCNT = 0x40e
                    0x040f                  C1TERRCNT = 0x40f
                    0x040f                  _C1TERRCNT = 0x40f
                    0x0410                  C1CFG1 = 0x410
                    0x0410                  _C1CFG1 = 0x410
                    0x0410                  _C1CFG1bits = 0x410
                    0x0412                  C1CFG2 = 0x412
                    0x0412                  _C1CFG2 = 0x412
                    0x0412                  _C1CFG2bits = 0x412
                    0x0414                  C1FEN1 = 0x414
                    0x0414                  _C1FEN1 = 0x414
                    0x0414                  _C1FEN1bits = 0x414
                    0x0418                  C1FMSKSEL1 = 0x418
                    0x0418                  _C1FMSKSEL1 = 0x418
                    0x0418                  _C1FMSKSEL1bits = 0x418
                    0x041a                  C1FMSKSEL2 = 0x41a
                    0x041a                  _C1FMSKSEL2 = 0x41a
                    0x041a                  _C1FMSKSEL2bits = 0x41a
                    0x0420                  C1BUFPNT1 = 0x420
                    0x0420                  _C1BUFPNT1 = 0x420
                    0x0420                  _C1BUFPNT1bits = 0x420
                    0x0420                  C1RXFUL1 = 0x420
                    0x0420                  _C1RXFUL1 = 0x420
                    0x0420                  _C1RXFUL1bits = 0x420
                    0x0422                  C1BUFPNT2 = 0x422
                    0x0422                  _C1BUFPNT2 = 0x422
                    0x0422                  _C1BUFPNT2bits = 0x422
                    0x0422                  C1RXFUL2 = 0x422
                    0x0422                  _C1RXFUL2 = 0x422
                    0x0422                  _C1RXFUL2bits = 0x422
                    0x0424                  C1BUFPNT3 = 0x424
                    0x0424                  _C1BUFPNT3 = 0x424
                    0x0424                  _C1BUFPNT3bits = 0x424
                    0x0426                  C1BUFPNT4 = 0x426
                    0x0426                  _C1BUFPNT4 = 0x426
                    0x0426                  _C1BUFPNT4bits = 0x426
                    0x0428                  C1RXOVF1 = 0x428
                    0x0428                  _C1RXOVF1 = 0x428
                    0x0428                  _C1RXOVF1bits = 0x428
                    0x042a                  C1RXOVF2 = 0x42a
                    0x042a                  _C1RXOVF2 = 0x42a
                    0x042a                  _C1RXOVF2bits = 0x42a
                    0x0430                  C1RXM0SID = 0x430
                    0x0430                  _C1RXM0SID = 0x430
                    0x0430                  _C1RXM0SIDbits = 0x430
                    0x0430                  C1TR01CON = 0x430
                    0x0430                  _C1TR01CON = 0x430
                    0x0430                  _C1TR01CONbits = 0x430
                    0x0432                  C1RXM0EID = 0x432
                    0x0432                  _C1RXM0EID = 0x432
                    0x0432                  _C1RXM0EIDbits = 0x432
                    0x0432                  C1TR23CON = 0x432
                    0x0432                  _C1TR23CON = 0x432
                    0x0432                  _C1TR23CONbits = 0x432
                    0x0434                  C1RXM1SID = 0x434
                    0x0434                  _C1RXM1SID = 0x434
                    0x0434                  _C1RXM1SIDbits = 0x434
                    0x0434                  C1TR45CON = 0x434
                    0x0434                  _C1TR45CON = 0x434
                    0x0434                  _C1TR45CONbits = 0x434
                    0x0436                  C1RXM1EID = 0x436
                    0x0436                  _C1RXM1EID = 0x436
                    0x0436                  _C1RXM1EIDbits = 0x436
                    0x0436                  C1TR67CON = 0x436
                    0x0436                  _C1TR67CON = 0x436
                    0x0436                  _C1TR67CONbits = 0x436
                    0x0438                  C1RXM2SID = 0x438
                    0x0438                  _C1RXM2SID = 0x438
                    0x0438                  _C1RXM2SIDbits = 0x438
                    0x043a                  C1RXM2EID = 0x43a
                    0x043a                  _C1RXM2EID = 0x43a
                    0x043a                  _C1RXM2EIDbits = 0x43a
                    0x0440                  C1RXD = 0x440
                    0x0440                  _C1RXD = 0x440
                    0x0440                  C1RXF0SID = 0x440
                    0x0440                  _C1RXF0SID = 0x440
                    0x0440                  _C1RXF0SIDbits = 0x440
                    0x0442                  C1RXF0EID = 0x442
                    0x0442                  _C1RXF0EID = 0x442
                    0x0442                  _C1RXF0EIDbits = 0x442
                    0x0442                  C1TXD = 0x442
                    0x0442                  _C1TXD = 0x442
                    0x0442                  _C1TXDbits = 0x442
                    0x0444                  C1RXF1SID = 0x444
                    0x0444                  _C1RXF1SID = 0x444
                    0x0444                  _C1RXF1SIDbits = 0x444
                    0x0446                  C1RXF1EID = 0x446
                    0x0446                  _C1RXF1EID = 0x446
                    0x0446                  _C1RXF1EIDbits = 0x446
                    0x0448                  C1RXF2SID = 0x448
                    0x0448                  _C1RXF2SID = 0x448
                    0x0448                  _C1RXF2SIDbits = 0x448
                    0x044a                  C1RXF2EID = 0x44a
                    0x044a                  _C1RXF2EID = 0x44a
                    0x044a                  _C1RXF2EIDbits = 0x44a
                    0x044c                  C1RXF3SID = 0x44c
                    0x044c                  _C1RXF3SID = 0x44c
                    0x044c                  _C1RXF3SIDbits = 0x44c
                    0x044e                  C1RXF3EID = 0x44e
                    0x044e                  _C1RXF3EID = 0x44e
                    0x044e                  _C1RXF3EIDbits = 0x44e
                    0x0450                  C1RXF4SID = 0x450
                    0x0450                  _C1RXF4SID = 0x450
                    0x0450                  _C1RXF4SIDbits = 0x450
                    0x0452                  C1RXF4EID = 0x452
                    0x0452                  _C1RXF4EID = 0x452
                    0x0452                  _C1RXF4EIDbits = 0x452
                    0x0454                  C1RXF5SID = 0x454
                    0x0454                  _C1RXF5SID = 0x454
                    0x0454                  _C1RXF5SIDbits = 0x454
                    0x0456                  C1RXF5EID = 0x456
                    0x0456                  _C1RXF5EID = 0x456
                    0x0456                  _C1RXF5EIDbits = 0x456
                    0x0458                  C1RXF6SID = 0x458
                    0x0458                  _C1RXF6SID = 0x458
                    0x0458                  _C1RXF6SIDbits = 0x458
                    0x045a                  C1RXF6EID = 0x45a
                    0x045a                  _C1RXF6EID = 0x45a
                    0x045a                  _C1RXF6EIDbits = 0x45a
                    0x045c                  C1RXF7SID = 0x45c
                    0x045c                  _C1RXF7SID = 0x45c
                    0x045c                  _C1RXF7SIDbits = 0x45c
                    0x045e                  C1RXF7EID = 0x45e
                    0x045e                  _C1RXF7EID = 0x45e
                    0x045e                  _C1RXF7EIDbits = 0x45e
                    0x0460                  C1RXF8SID = 0x460
                    0x0460                  _C1RXF8SID = 0x460
                    0x0460                  _C1RXF8SIDbits = 0x460
                    0x0462                  C1RXF8EID = 0x462
                    0x0462                  _C1RXF8EID = 0x462
                    0x0462                  _C1RXF8EIDbits = 0x462
                    0x0464                  C1RXF9SID = 0x464
                    0x0464                  _C1RXF9SID = 0x464
                    0x0464                  _C1RXF9SIDbits = 0x464
                    0x0466                  C1RXF9EID = 0x466
                    0x0466                  _C1RXF9EID = 0x466
                    0x0466                  _C1RXF9EIDbits = 0x466
                    0x0468                  C1RXF10SID = 0x468
                    0x0468                  _C1RXF10SID = 0x468
                    0x0468                  _C1RXF10SIDbits = 0x468
                    0x046a                  C1RXF10EID = 0x46a
                    0x046a                  _C1RXF10EID = 0x46a
                    0x046a                  _C1RXF10EIDbits = 0x46a
                    0x046c                  C1RXF11SID = 0x46c
                    0x046c                  _C1RXF11SID = 0x46c
                    0x046c                  _C1RXF11SIDbits = 0x46c
                    0x046e                  C1RXF11EID = 0x46e
                    0x046e                  _C1RXF11EID = 0x46e
                    0x046e                  _C1RXF11EIDbits = 0x46e
                    0x0470                  C1RXF12SID = 0x470
                    0x0470                  _C1RXF12SID = 0x470
                    0x0470                  _C1RXF12SIDbits = 0x470
                    0x0472                  C1RXF12EID = 0x472
                    0x0472                  _C1RXF12EID = 0x472
                    0x0472                  _C1RXF12EIDbits = 0x472
                    0x0474                  C1RXF13SID = 0x474
                    0x0474                  _C1RXF13SID = 0x474
                    0x0474                  _C1RXF13SIDbits = 0x474
                    0x0476                  C1RXF13EID = 0x476
                    0x0476                  _C1RXF13EID = 0x476
                    0x0476                  _C1RXF13EIDbits = 0x476
                    0x0478                  C1RXF14SID = 0x478
                    0x0478                  _C1RXF14SID = 0x478
                    0x0478                  _C1RXF14SIDbits = 0x478
                    0x047a                  C1RXF14EID = 0x47a
                    0x047a                  _C1RXF14EID = 0x47a
                    0x047a                  _C1RXF14EIDbits = 0x47a
                    0x047c                  C1RXF15SID = 0x47c
                    0x047c                  _C1RXF15SID = 0x47c
                    0x047c                  _C1RXF15SIDbits = 0x47c
                    0x047e                  C1RXF15EID = 0x47e
                    0x047e                  _C1RXF15EID = 0x47e
                    0x047e                  _C1RXF15EIDbits = 0x47e
                    0x0488                  U1OTGIR = 0x488
                    0x0488                  _U1OTGIR = 0x488
                    0x0488                  _U1OTGIRbits = 0x488
                    0x048a                  U1OTGIE = 0x48a
                    0x048a                  _U1OTGIE = 0x48a
                    0x048a                  _U1OTGIEbits = 0x48a
                    0x048c                  U1OTGSTAT = 0x48c
                    0x048c                  _U1OTGSTAT = 0x48c
                    0x048c                  _U1OTGSTATbits = 0x48c
                    0x048e                  U1OTGCON = 0x48e
                    0x048e                  _U1OTGCON = 0x48e
                    0x048e                  _U1OTGCONbits = 0x48e
                    0x0490                  U1PWRC = 0x490
                    0x0490                  _U1PWRC = 0x490
                    0x0490                  _U1PWRCbits = 0x490
                    0x04c0                  U1IR = 0x4c0
                    0x04c0                  _U1IR = 0x4c0
                    0x04c0                  _U1IRbits = 0x4c0
                    0x04c2                  U1IE = 0x4c2
                    0x04c2                  _U1IE = 0x4c2
                    0x04c2                  _U1IEbits = 0x4c2
                    0x04c4                  U1EIR = 0x4c4
                    0x04c4                  _U1EIR = 0x4c4
                    0x04c4                  _U1EIRbits = 0x4c4
                    0x04c6                  U1EIE = 0x4c6
                    0x04c6                  _U1EIE = 0x4c6
                    0x04c6                  _U1EIEbits = 0x4c6
                    0x04c8                  U1STAT = 0x4c8
                    0x04c8                  _U1STAT = 0x4c8
                    0x04c8                  _U1STATbits = 0x4c8
                    0x04ca                  U1CON = 0x4ca
                    0x04ca                  _U1CON = 0x4ca
                    0x04ca                  _U1CONbits = 0x4ca
                    0x04cc                  U1ADDR = 0x4cc
                    0x04cc                  _U1ADDR = 0x4cc
                    0x04cc                  _U1ADDRbits = 0x4cc
                    0x04ce                  U1BDTP1 = 0x4ce
                    0x04ce                  _U1BDTP1 = 0x4ce
                    0x04ce                  _U1BDTP1bits = 0x4ce
                    0x04d0                  U1FRML = 0x4d0
                    0x04d0                  _U1FRML = 0x4d0
                    0x04d0                  _U1FRMLbits = 0x4d0
                    0x04d2                  U1FRMH = 0x4d2
                    0x04d2                  _U1FRMH = 0x4d2
                    0x04d2                  _U1FRMHbits = 0x4d2
                    0x04d4                  U1TOK = 0x4d4
                    0x04d4                  _U1TOK = 0x4d4
                    0x04d4                  _U1TOKbits = 0x4d4
                    0x04d6                  U1SOF = 0x4d6
                    0x04d6                  _U1SOF = 0x4d6
                    0x04d6                  _U1SOFbits = 0x4d6
                    0x04d8                  U1BDTP2 = 0x4d8
                    0x04d8                  _U1BDTP2 = 0x4d8
                    0x04d8                  _U1BDTP2bits = 0x4d8
                    0x04da                  U1BDTP3 = 0x4da
                    0x04da                  _U1BDTP3 = 0x4da
                    0x04da                  _U1BDTP3bits = 0x4da
                    0x04dc                  U1CNFG1 = 0x4dc
                    0x04dc                  _U1CNFG1 = 0x4dc
                    0x04dc                  _U1CNFG1bits = 0x4dc
                    0x04de                  U1CNFG2 = 0x4de
                    0x04de                  _U1CNFG2 = 0x4de
                    0x04de                  _U1CNFG2bits = 0x4de
                    0x04e0                  U1EP0 = 0x4e0
                    0x04e0                  _U1EP0 = 0x4e0
                    0x04e0                  _U1EP0bits = 0x4e0
                    0x04e2                  U1EP1 = 0x4e2
                    0x04e2                  _U1EP1 = 0x4e2
                    0x04e2                  _U1EP1bits = 0x4e2
                    0x04e4                  U1EP2 = 0x4e4
                    0x04e4                  _U1EP2 = 0x4e4
                    0x04e4                  _U1EP2bits = 0x4e4
                    0x04e6                  U1EP3 = 0x4e6
                    0x04e6                  _U1EP3 = 0x4e6
                    0x04e6                  _U1EP3bits = 0x4e6
                    0x04e8                  U1EP4 = 0x4e8
                    0x04e8                  _U1EP4 = 0x4e8
                    0x04e8                  _U1EP4bits = 0x4e8
                    0x04ea                  U1EP5 = 0x4ea
                    0x04ea                  _U1EP5 = 0x4ea
                    0x04ea                  _U1EP5bits = 0x4ea
                    0x04ec                  U1EP6 = 0x4ec
                    0x04ec                  _U1EP6 = 0x4ec
                    0x04ec                  _U1EP6bits = 0x4ec
                    0x04ee                  U1EP7 = 0x4ee
                    0x04ee                  _U1EP7 = 0x4ee
                    0x04ee                  _U1EP7bits = 0x4ee
                    0x04f0                  U1EP8 = 0x4f0
                    0x04f0                  _U1EP8 = 0x4f0
                    0x04f0                  _U1EP8bits = 0x4f0
                    0x04f2                  U1EP9 = 0x4f2
                    0x04f2                  _U1EP9 = 0x4f2
                    0x04f2                  _U1EP9bits = 0x4f2
                    0x04f4                  U1EP10 = 0x4f4
                    0x04f4                  _U1EP10 = 0x4f4
                    0x04f4                  _U1EP10bits = 0x4f4
                    0x04f6                  U1EP11 = 0x4f6
                    0x04f6                  _U1EP11 = 0x4f6
                    0x04f6                  _U1EP11bits = 0x4f6
                    0x04f8                  U1EP12 = 0x4f8
                    0x04f8                  _U1EP12 = 0x4f8
                    0x04f8                  _U1EP12bits = 0x4f8
                    0x04fa                  U1EP13 = 0x4fa
                    0x04fa                  _U1EP13 = 0x4fa
                    0x04fa                  _U1EP13bits = 0x4fa
                    0x04fc                  U1EP14 = 0x4fc
                    0x04fc                  _U1EP14 = 0x4fc
                    0x04fc                  _U1EP14bits = 0x4fc
                    0x04fe                  U1EP15 = 0x4fe
                    0x04fe                  _U1EP15 = 0x4fe
                    0x04fe                  _U1EP15bits = 0x4fe
                    0x0500                  C2CTRL1 = 0x500
                    0x0500                  _C2CTRL1 = 0x500
                    0x0500                  _C2CTRL1bits = 0x500
                    0x0502                  C2CTRL2 = 0x502
                    0x0502                  _C2CTRL2 = 0x502
                    0x0502                  _C2CTRL2bits = 0x502
                    0x0504                  C2VEC = 0x504
                    0x0504                  _C2VEC = 0x504
                    0x0504                  _C2VECbits = 0x504
                    0x0506                  C2FCTRL = 0x506
                    0x0506                  _C2FCTRL = 0x506
                    0x0506                  _C2FCTRLbits = 0x506
                    0x0508                  C2FIFO = 0x508
                    0x0508                  _C2FIFO = 0x508
                    0x0508                  _C2FIFObits = 0x508
                    0x050a                  C2INTF = 0x50a
                    0x050a                  _C2INTF = 0x50a
                    0x050a                  _C2INTFbits = 0x50a
                    0x050c                  C2INTE = 0x50c
                    0x050c                  _C2INTE = 0x50c
                    0x050c                  _C2INTEbits = 0x50c
                    0x050e                  C2EC = 0x50e
                    0x050e                  _C2EC = 0x50e
                    0x050e                  _C2ECbits = 0x50e
                    0x050e                  C2RERRCNT = 0x50e
                    0x050e                  _C2RERRCNT = 0x50e
                    0x050f                  C2TERRCNT = 0x50f
                    0x050f                  _C2TERRCNT = 0x50f
                    0x0510                  C2CFG1 = 0x510
                    0x0510                  _C2CFG1 = 0x510
                    0x0510                  _C2CFG1bits = 0x510
                    0x0512                  C2CFG2 = 0x512
                    0x0512                  _C2CFG2 = 0x512
                    0x0512                  _C2CFG2bits = 0x512
                    0x0514                  C2FEN1 = 0x514
                    0x0514                  _C2FEN1 = 0x514
                    0x0514                  _C2FEN1bits = 0x514
                    0x0518                  C2FMSKSEL1 = 0x518
                    0x0518                  _C2FMSKSEL1 = 0x518
                    0x0518                  _C2FMSKSEL1bits = 0x518
                    0x051a                  C2FMSKSEL2 = 0x51a
                    0x051a                  _C2FMSKSEL2 = 0x51a
                    0x051a                  _C2FMSKSEL2bits = 0x51a
                    0x0520                  C2BUFPNT1 = 0x520
                    0x0520                  _C2BUFPNT1 = 0x520
                    0x0520                  _C2BUFPNT1bits = 0x520
                    0x0520                  C2RXFUL1 = 0x520
                    0x0520                  _C2RXFUL1 = 0x520
                    0x0520                  _C2RXFUL1bits = 0x520
                    0x0522                  C2BUFPNT2 = 0x522
                    0x0522                  _C2BUFPNT2 = 0x522
                    0x0522                  _C2BUFPNT2bits = 0x522
                    0x0522                  C2RXFUL2 = 0x522
                    0x0522                  _C2RXFUL2 = 0x522
                    0x0522                  _C2RXFUL2bits = 0x522
                    0x0524                  C2BUFPNT3 = 0x524
                    0x0524                  _C2BUFPNT3 = 0x524
                    0x0524                  _C2BUFPNT3bits = 0x524
                    0x0526                  C2BUFPNT4 = 0x526
                    0x0526                  _C2BUFPNT4 = 0x526
                    0x0526                  _C2BUFPNT4bits = 0x526
                    0x0528                  C2RXOVF1 = 0x528
                    0x0528                  _C2RXOVF1 = 0x528
                    0x0528                  _C2RXOVF1bits = 0x528
                    0x052a                  C2RXOVF2 = 0x52a
                    0x052a                  _C2RXOVF2 = 0x52a
                    0x052a                  _C2RXOVF2bits = 0x52a
                    0x0530                  C2RXM0SID = 0x530
                    0x0530                  _C2RXM0SID = 0x530
                    0x0530                  _C2RXM0SIDbits = 0x530
                    0x0530                  C2TR01CON = 0x530
                    0x0530                  _C2TR01CON = 0x530
                    0x0530                  _C2TR01CONbits = 0x530
                    0x0532                  C2RXM0EID = 0x532
                    0x0532                  _C2RXM0EID = 0x532
                    0x0532                  _C2RXM0EIDbits = 0x532
                    0x0532                  C2TR23CON = 0x532
                    0x0532                  _C2TR23CON = 0x532
                    0x0532                  _C2TR23CONbits = 0x532
                    0x0534                  C2RXM1SID = 0x534
                    0x0534                  _C2RXM1SID = 0x534
                    0x0534                  _C2RXM1SIDbits = 0x534
                    0x0534                  C2TR45CON = 0x534
                    0x0534                  _C2TR45CON = 0x534
                    0x0534                  _C2TR45CONbits = 0x534
                    0x0536                  C2RXM1EID = 0x536
                    0x0536                  _C2RXM1EID = 0x536
                    0x0536                  _C2RXM1EIDbits = 0x536
                    0x0536                  C2TR67CON = 0x536
                    0x0536                  _C2TR67CON = 0x536
                    0x0536                  _C2TR67CONbits = 0x536
                    0x0538                  C2RXM2SID = 0x538
                    0x0538                  _C2RXM2SID = 0x538
                    0x0538                  _C2RXM2SIDbits = 0x538
                    0x053a                  C2RXM2EID = 0x53a
                    0x053a                  _C2RXM2EID = 0x53a
                    0x053a                  _C2RXM2EIDbits = 0x53a
                    0x0540                  C2RXD = 0x540
                    0x0540                  _C2RXD = 0x540
                    0x0540                  C2RXF0SID = 0x540
                    0x0540                  _C2RXF0SID = 0x540
                    0x0540                  _C2RXF0SIDbits = 0x540
                    0x0542                  C2RXF0EID = 0x542
                    0x0542                  _C2RXF0EID = 0x542
                    0x0542                  _C2RXF0EIDbits = 0x542
                    0x0542                  C2TXD = 0x542
                    0x0542                  _C2TXD = 0x542
                    0x0542                  _C2TXDbits = 0x542
                    0x0544                  C2RXF1SID = 0x544
                    0x0544                  _C2RXF1SID = 0x544
                    0x0544                  _C2RXF1SIDbits = 0x544
                    0x0546                  C2RXF1EID = 0x546
                    0x0546                  _C2RXF1EID = 0x546
                    0x0546                  _C2RXF1EIDbits = 0x546
                    0x0548                  C2RXF2SID = 0x548
                    0x0548                  _C2RXF2SID = 0x548
                    0x0548                  _C2RXF2SIDbits = 0x548
                    0x054a                  C2RXF2EID = 0x54a
                    0x054a                  _C2RXF2EID = 0x54a
                    0x054a                  _C2RXF2EIDbits = 0x54a
                    0x054c                  C2RXF3SID = 0x54c
                    0x054c                  _C2RXF3SID = 0x54c
                    0x054c                  _C2RXF3SIDbits = 0x54c
                    0x054e                  C2RXF3EID = 0x54e
                    0x054e                  _C2RXF3EID = 0x54e
                    0x054e                  _C2RXF3EIDbits = 0x54e
                    0x0550                  C2RXF4SID = 0x550
                    0x0550                  _C2RXF4SID = 0x550
                    0x0550                  _C2RXF4SIDbits = 0x550
                    0x0552                  C2RXF4EID = 0x552
                    0x0552                  _C2RXF4EID = 0x552
                    0x0552                  _C2RXF4EIDbits = 0x552
                    0x0554                  C2RXF5SID = 0x554
                    0x0554                  _C2RXF5SID = 0x554
                    0x0554                  _C2RXF5SIDbits = 0x554
                    0x0556                  C2RXF5EID = 0x556
                    0x0556                  _C2RXF5EID = 0x556
                    0x0556                  _C2RXF5EIDbits = 0x556
                    0x0558                  C2RXF6SID = 0x558
                    0x0558                  _C2RXF6SID = 0x558
                    0x0558                  _C2RXF6SIDbits = 0x558
                    0x055a                  C2RXF6EID = 0x55a
                    0x055a                  _C2RXF6EID = 0x55a
                    0x055a                  _C2RXF6EIDbits = 0x55a
                    0x055c                  C2RXF7SID = 0x55c
                    0x055c                  _C2RXF7SID = 0x55c
                    0x055c                  _C2RXF7SIDbits = 0x55c
                    0x055e                  C2RXF7EID = 0x55e
                    0x055e                  _C2RXF7EID = 0x55e
                    0x055e                  _C2RXF7EIDbits = 0x55e
                    0x0560                  C2RXF8SID = 0x560
                    0x0560                  _C2RXF8SID = 0x560
                    0x0560                  _C2RXF8SIDbits = 0x560
                    0x0562                  C2RXF8EID = 0x562
                    0x0562                  _C2RXF8EID = 0x562
                    0x0562                  _C2RXF8EIDbits = 0x562
                    0x0564                  C2RXF9SID = 0x564
                    0x0564                  _C2RXF9SID = 0x564
                    0x0564                  _C2RXF9SIDbits = 0x564
                    0x0566                  C2RXF9EID = 0x566
                    0x0566                  _C2RXF9EID = 0x566
                    0x0566                  _C2RXF9EIDbits = 0x566
                    0x0568                  C2RXF10SID = 0x568
                    0x0568                  _C2RXF10SID = 0x568
                    0x0568                  _C2RXF10SIDbits = 0x568
                    0x056a                  C2RXF10EID = 0x56a
                    0x056a                  _C2RXF10EID = 0x56a
                    0x056a                  _C2RXF10EIDbits = 0x56a
                    0x056c                  C2RXF11SID = 0x56c
                    0x056c                  _C2RXF11SID = 0x56c
                    0x056c                  _C2RXF11SIDbits = 0x56c
                    0x056e                  C2RXF11EID = 0x56e
                    0x056e                  _C2RXF11EID = 0x56e
                    0x056e                  _C2RXF11EIDbits = 0x56e
                    0x0570                  C2RXF12SID = 0x570
                    0x0570                  _C2RXF12SID = 0x570
                    0x0570                  _C2RXF12SIDbits = 0x570
                    0x0572                  C2RXF12EID = 0x572
                    0x0572                  _C2RXF12EID = 0x572
                    0x0572                  _C2RXF12EIDbits = 0x572
                    0x0574                  C2RXF13SID = 0x574
                    0x0574                  _C2RXF13SID = 0x574
                    0x0574                  _C2RXF13SIDbits = 0x574
                    0x0576                  C2RXF13EID = 0x576
                    0x0576                  _C2RXF13EID = 0x576
                    0x0576                  _C2RXF13EIDbits = 0x576
                    0x0578                  C2RXF14SID = 0x578
                    0x0578                  _C2RXF14SID = 0x578
                    0x0578                  _C2RXF14SIDbits = 0x578
                    0x057a                  C2RXF14EID = 0x57a
                    0x057a                  _C2RXF14EID = 0x57a
                    0x057a                  _C2RXF14EIDbits = 0x57a
                    0x057c                  C2RXF15SID = 0x57c
                    0x057c                  _C2RXF15SID = 0x57c
                    0x057c                  _C2RXF15SIDbits = 0x57c
                    0x057e                  C2RXF15EID = 0x57e
                    0x057e                  _C2RXF15EID = 0x57e
                    0x057e                  _C2RXF15EIDbits = 0x57e
                    0x0580                  U1PWMRRS = 0x580
                    0x0580                  _U1PWMRRS = 0x580
                    0x0580                  _U1PWMRRSbits = 0x580
                    0x0582                  U1PWMCON = 0x582
                    0x0582                  _U1PWMCON = 0x582
                    0x0582                  _U1PWMCONbits = 0x582
                    0x0600                  PMCON = 0x600
                    0x0600                  _PMCON = 0x600
                    0x0600                  _PMCONbits = 0x600
                    0x0602                  PMMODE = 0x602
                    0x0602                  _PMMODE = 0x602
                    0x0602                  _PMMODEbits = 0x602
                    0x0604                  PMADDR = 0x604
                    0x0604                  _PMADDR = 0x604
                    0x0604                  _PMADDRbits = 0x604
                    0x0604                  PMDOUT1 = 0x604
                    0x0604                  _PMDOUT1 = 0x604
                    0x0604                  _PMDOUT1bits = 0x604
                    0x0606                  PMDOUT2 = 0x606
                    0x0606                  _PMDOUT2 = 0x606
                    0x0608                  PMDIN1 = 0x608
                    0x0608                  _PMDIN1 = 0x608
                    0x060a                  PMDIN2 = 0x60a
                    0x060a                  _PMDIN2 = 0x60a
                    0x060c                  PMAEN = 0x60c
                    0x060c                  _PMAEN = 0x60c
                    0x060c                  _PMAENbits = 0x60c
                    0x060e                  PMSTAT = 0x60e
                    0x060e                  _PMSTAT = 0x60e
                    0x060e                  _PMSTATbits = 0x60e
                    0x0620                  ALRMVAL = 0x620
                    0x0620                  _ALRMVAL = 0x620
                    0x0622                  ALCFGRPT = 0x622
                    0x0622                  _ALCFGRPT = 0x622
                    0x0622                  _ALCFGRPTbits = 0x622
                    0x0624                  RTCVAL = 0x624
                    0x0624                  _RTCVAL = 0x624
                    0x0626                  RCFGCAL = 0x626
                    0x0626                  _RCFGCAL = 0x626
                    0x0626                  _RCFGCALbits = 0x626
                    0x0640                  CRCCON1 = 0x640
                    0x0640                  _CRCCON1 = 0x640
                    0x0640                  _CRCCON1bits = 0x640
                    0x0642                  CRCCON2 = 0x642
                    0x0642                  _CRCCON2 = 0x642
                    0x0642                  _CRCCON2bits = 0x642
                    0x0644                  CRCXORL = 0x644
                    0x0644                  _CRCXORL = 0x644
                    0x0644                  _CRCXORLbits = 0x644
                    0x0646                  CRCXORH = 0x646
                    0x0646                  _CRCXORH = 0x646
                    0x0646                  _CRCXORHbits = 0x646
                    0x0648                  CRCDAT = 0x648
                    0x0648                  _CRCDAT = 0x648
                    0x0648                  CRCDATL = 0x648
                    0x0648                  _CRCDATL = 0x648
                    0x064a                  CRCDATH = 0x64a
                    0x064a                  _CRCDATH = 0x64a
                    0x064c                  CRCWDAT = 0x64c
                    0x064c                  _CRCWDAT = 0x64c
                    0x064c                  CRCWDATL = 0x64c
                    0x064c                  _CRCWDATL = 0x64c
                    0x064e                  CRCWDATH = 0x64e
                    0x064e                  _CRCWDATH = 0x64e
                    0x0680                  RPOR0 = 0x680
                    0x0680                  _RPOR0 = 0x680
                    0x0680                  _RPOR0bits = 0x680
                    0x0682                  RPOR1 = 0x682
                    0x0682                  _RPOR1 = 0x682
                    0x0682                  _RPOR1bits = 0x682
                    0x0684                  RPOR2 = 0x684
                    0x0684                  _RPOR2 = 0x684
                    0x0684                  _RPOR2bits = 0x684
                    0x0686                  RPOR3 = 0x686
                    0x0686                  _RPOR3 = 0x686
                    0x0686                  _RPOR3bits = 0x686
                    0x0688                  RPOR4 = 0x688
                    0x0688                  _RPOR4 = 0x688
                    0x0688                  _RPOR4bits = 0x688
                    0x068a                  RPOR5 = 0x68a
                    0x068a                  _RPOR5 = 0x68a
                    0x068a                  _RPOR5bits = 0x68a
                    0x068c                  RPOR6 = 0x68c
                    0x068c                  _RPOR6 = 0x68c
                    0x068c                  _RPOR6bits = 0x68c
                    0x068e                  RPOR7 = 0x68e
                    0x068e                  _RPOR7 = 0x68e
                    0x068e                  _RPOR7bits = 0x68e
                    0x0690                  RPOR8 = 0x690
                    0x0690                  _RPOR8 = 0x690
                    0x0690                  _RPOR8bits = 0x690
                    0x0692                  RPOR9 = 0x692
                    0x0692                  _RPOR9 = 0x692
                    0x0692                  _RPOR9bits = 0x692
                    0x0696                  RPOR11 = 0x696
                    0x0696                  _RPOR11 = 0x696
                    0x0696                  _RPOR11bits = 0x696
                    0x0698                  RPOR12 = 0x698
                    0x0698                  _RPOR12 = 0x698
                    0x0698                  _RPOR12bits = 0x698
                    0x069a                  RPOR13 = 0x69a
                    0x069a                  _RPOR13 = 0x69a
                    0x069a                  _RPOR13bits = 0x69a
                    0x069c                  RPOR14 = 0x69c
                    0x069c                  _RPOR14 = 0x69c
                    0x069c                  _RPOR14bits = 0x69c
                    0x069e                  RPOR15 = 0x69e
                    0x069e                  _RPOR15 = 0x69e
                    0x069e                  _RPOR15bits = 0x69e
                    0x06a0                  RPINR0 = 0x6a0
                    0x06a0                  _RPINR0 = 0x6a0
                    0x06a0                  _RPINR0bits = 0x6a0
                    0x06a2                  RPINR1 = 0x6a2
                    0x06a2                  _RPINR1 = 0x6a2
                    0x06a2                  _RPINR1bits = 0x6a2
                    0x06a4                  RPINR2 = 0x6a4
                    0x06a4                  _RPINR2 = 0x6a4
                    0x06a4                  _RPINR2bits = 0x6a4
                    0x06a6                  RPINR3 = 0x6a6
                    0x06a6                  _RPINR3 = 0x6a6
                    0x06a6                  _RPINR3bits = 0x6a6
                    0x06a8                  RPINR4 = 0x6a8
                    0x06a8                  _RPINR4 = 0x6a8
                    0x06a8                  _RPINR4bits = 0x6a8
                    0x06aa                  RPINR5 = 0x6aa
                    0x06aa                  _RPINR5 = 0x6aa
                    0x06aa                  _RPINR5bits = 0x6aa
                    0x06ac                  RPINR6 = 0x6ac
                    0x06ac                  _RPINR6 = 0x6ac
                    0x06ac                  _RPINR6bits = 0x6ac
                    0x06ae                  RPINR7 = 0x6ae
                    0x06ae                  _RPINR7 = 0x6ae
                    0x06ae                  _RPINR7bits = 0x6ae
                    0x06b0                  RPINR8 = 0x6b0
                    0x06b0                  _RPINR8 = 0x6b0
                    0x06b0                  _RPINR8bits = 0x6b0
                    0x06b2                  RPINR9 = 0x6b2
                    0x06b2                  _RPINR9 = 0x6b2
                    0x06b2                  _RPINR9bits = 0x6b2
                    0x06b4                  RPINR10 = 0x6b4
                    0x06b4                  _RPINR10 = 0x6b4
                    0x06b4                  _RPINR10bits = 0x6b4
                    0x06b6                  RPINR11 = 0x6b6
                    0x06b6                  _RPINR11 = 0x6b6
                    0x06b6                  _RPINR11bits = 0x6b6
                    0x06b8                  RPINR12 = 0x6b8
                    0x06b8                  _RPINR12 = 0x6b8
                    0x06b8                  _RPINR12bits = 0x6b8
                    0x06ba                  RPINR13 = 0x6ba
                    0x06ba                  _RPINR13 = 0x6ba
                    0x06ba                  _RPINR13bits = 0x6ba
                    0x06bc                  RPINR14 = 0x6bc
                    0x06bc                  _RPINR14 = 0x6bc
                    0x06bc                  _RPINR14bits = 0x6bc
                    0x06be                  RPINR15 = 0x6be
                    0x06be                  _RPINR15 = 0x6be
                    0x06be                  _RPINR15bits = 0x6be
                    0x06c0                  RPINR16 = 0x6c0
                    0x06c0                  _RPINR16 = 0x6c0
                    0x06c0                  _RPINR16bits = 0x6c0
                    0x06c2                  RPINR17 = 0x6c2
                    0x06c2                  _RPINR17 = 0x6c2
                    0x06c2                  _RPINR17bits = 0x6c2
                    0x06c4                  RPINR18 = 0x6c4
                    0x06c4                  _RPINR18 = 0x6c4
                    0x06c4                  _RPINR18bits = 0x6c4
                    0x06c6                  RPINR19 = 0x6c6
                    0x06c6                  _RPINR19 = 0x6c6
                    0x06c6                  _RPINR19bits = 0x6c6
                    0x06c8                  RPINR20 = 0x6c8
                    0x06c8                  _RPINR20 = 0x6c8
                    0x06c8                  _RPINR20bits = 0x6c8
                    0x06ca                  RPINR21 = 0x6ca
                    0x06ca                  _RPINR21 = 0x6ca
                    0x06ca                  _RPINR21bits = 0x6ca
                    0x06ce                  RPINR23 = 0x6ce
                    0x06ce                  _RPINR23 = 0x6ce
                    0x06ce                  _RPINR23bits = 0x6ce
                    0x06d0                  RPINR24 = 0x6d0
                    0x06d0                  _RPINR24 = 0x6d0
                    0x06d0                  _RPINR24bits = 0x6d0
                    0x06d2                  RPINR25 = 0x6d2
                    0x06d2                  _RPINR25 = 0x6d2
                    0x06d2                  _RPINR25bits = 0x6d2
                    0x06d4                  RPINR26 = 0x6d4
                    0x06d4                  _RPINR26 = 0x6d4
                    0x06d4                  _RPINR26bits = 0x6d4
                    0x06d6                  RPINR27 = 0x6d6
                    0x06d6                  _RPINR27 = 0x6d6
                    0x06d6                  _RPINR27bits = 0x6d6
                    0x06d8                  RPINR28 = 0x6d8
                    0x06d8                  _RPINR28 = 0x6d8
                    0x06d8                  _RPINR28bits = 0x6d8
                    0x06da                  RPINR29 = 0x6da
                    0x06da                  _RPINR29 = 0x6da
                    0x06da                  _RPINR29bits = 0x6da
                    0x06dc                  RPINR30 = 0x6dc
                    0x06dc                  _RPINR30 = 0x6dc
                    0x06dc                  _RPINR30bits = 0x6dc
                    0x06de                  RPINR31 = 0x6de
                    0x06de                  _RPINR31 = 0x6de
                    0x06de                  _RPINR31bits = 0x6de
                    0x06e0                  RPINR32 = 0x6e0
                    0x06e0                  _RPINR32 = 0x6e0
                    0x06e0                  _RPINR32bits = 0x6e0
                    0x06e2                  RPINR33 = 0x6e2
                    0x06e2                  _RPINR33 = 0x6e2
                    0x06e2                  _RPINR33bits = 0x6e2
                    0x06e4                  RPINR34 = 0x6e4
                    0x06e4                  _RPINR34 = 0x6e4
                    0x06e4                  _RPINR34bits = 0x6e4
                    0x06e6                  RPINR35 = 0x6e6
                    0x06e6                  _RPINR35 = 0x6e6
                    0x06e6                  _RPINR35bits = 0x6e6
                    0x06e8                  RPINR36 = 0x6e8
                    0x06e8                  _RPINR36 = 0x6e8
                    0x06e8                  _RPINR36bits = 0x6e8
                    0x06ea                  RPINR37 = 0x6ea
                    0x06ea                  _RPINR37 = 0x6ea
                    0x06ea                  _RPINR37bits = 0x6ea
                    0x06ec                  RPINR38 = 0x6ec
                    0x06ec                  _RPINR38 = 0x6ec
                    0x06ec                  _RPINR38bits = 0x6ec
                    0x06f0                  RPINR40 = 0x6f0
                    0x06f0                  _RPINR40 = 0x6f0
                    0x06f0                  _RPINR40bits = 0x6f0
                    0x06f2                  RPINR41 = 0x6f2
                    0x06f2                  _RPINR41 = 0x6f2
                    0x06f2                  _RPINR41bits = 0x6f2
                    0x06f4                  RPINR42 = 0x6f4
                    0x06f4                  _RPINR42 = 0x6f4
                    0x06f4                  _RPINR42bits = 0x6f4
                    0x06f6                  RPINR43 = 0x6f6
                    0x06f6                  _RPINR43 = 0x6f6
                    0x06f6                  _RPINR43bits = 0x6f6
                    0x06fa                  RPINR45 = 0x6fa
                    0x06fa                  _RPINR45 = 0x6fa
                    0x06fa                  _RPINR45bits = 0x6fa
                    0x0728                  NVMCON = 0x728
                    0x0728                  _NVMCON = 0x728
                    0x0728                  _NVMCONbits = 0x728
                    0x072a                  NVMADR = 0x72a
                    0x072a                  _NVMADR = 0x72a
                    0x072c                  NVMADRU = 0x72c
                    0x072c                  _NVMADRU = 0x72c
                    0x072c                  _NVMADRUbits = 0x72c
                    0x072e                  NVMKEY = 0x72e
                    0x072e                  _NVMKEY = 0x72e
                    0x0740                  RCON = 0x740
                    0x0740                  _RCON = 0x740
                    0x0740                  _RCONbits = 0x740
                    0x0742                  OSCCON = 0x742
                    0x0742                  _OSCCON = 0x742
                    0x0742                  _OSCCONbits = 0x742
                    0x0742                  OSCCONL = 0x742
                    0x0742                  _OSCCONL = 0x742
                    0x0743                  OSCCONH = 0x743
                    0x0743                  _OSCCONH = 0x743
                    0x0744                  CLKDIV = 0x744
                    0x0744                  _CLKDIV = 0x744
                    0x0744                  _CLKDIVbits = 0x744
                    0x0746                  PLLFBD = 0x746
                    0x0746                  _PLLFBD = 0x746
                    0x0746                  _PLLFBDbits = 0x746
                    0x0748                  OSCTUN = 0x748
                    0x0748                  _OSCTUN = 0x748
                    0x0748                  _OSCTUNbits = 0x748
                    0x074e                  REFOCON = 0x74e
                    0x074e                  _REFOCON = 0x74e
                    0x074e                  _REFOCONbits = 0x74e
                    0x0758                  ACLKCON3 = 0x758
                    0x0758                  _ACLKCON3 = 0x758
                    0x0758                  _ACLKCON3bits = 0x758
                    0x075a                  ACLKDIV3 = 0x75a
                    0x075a                  _ACLKDIV3 = 0x75a
                    0x075a                  _ACLKDIV3bits = 0x75a
                    0x0760                  PMD1 = 0x760
                    0x0760                  _PMD1 = 0x760
                    0x0760                  _PMD1bits = 0x760
                    0x0762                  PMD2 = 0x762
                    0x0762                  _PMD2 = 0x762
                    0x0762                  _PMD2bits = 0x762
                    0x0764                  PMD3 = 0x764
                    0x0764                  _PMD3 = 0x764
                    0x0764                  _PMD3bits = 0x764
                    0x0766                  PMD4 = 0x766
                    0x0766                  _PMD4 = 0x766
                    0x0766                  _PMD4bits = 0x766
                    0x0768                  PMD5 = 0x768
                    0x0768                  _PMD5 = 0x768
                    0x0768                  _PMD5bits = 0x768
                    0x076a                  PMD6 = 0x76a
                    0x076a                  _PMD6 = 0x76a
                    0x076a                  _PMD6bits = 0x76a
                    0x076c                  PMD7 = 0x76c
                    0x076c                  _PMD7 = 0x76c
                    0x076c                  _PMD7bits = 0x76c
                    0x0800                  IFS0 = 0x800
                    0x0800                  _IFS0 = 0x800
                    0x0800                  _IFS0bits = 0x800
                    0x0802                  IFS1 = 0x802
                    0x0802                  _IFS1 = 0x802
                    0x0802                  _IFS1bits = 0x802
                    0x0804                  IFS2 = 0x804
                    0x0804                  _IFS2 = 0x804
                    0x0804                  _IFS2bits = 0x804
                    0x0806                  IFS3 = 0x806
                    0x0806                  _IFS3 = 0x806
                    0x0806                  _IFS3bits = 0x806
                    0x0808                  IFS4 = 0x808
                    0x0808                  _IFS4 = 0x808
                    0x0808                  _IFS4bits = 0x808
                    0x080a                  IFS5 = 0x80a
                    0x080a                  _IFS5 = 0x80a
                    0x080a                  _IFS5bits = 0x80a
                    0x080e                  IFS7 = 0x80e
                    0x080e                  _IFS7 = 0x80e
                    0x080e                  _IFS7bits = 0x80e
                    0x0810                  IFS8 = 0x810
                    0x0810                  _IFS8 = 0x810
                    0x0810                  _IFS8bits = 0x810
                    0x0820                  IEC0 = 0x820
                    0x0820                  _IEC0 = 0x820
                    0x0820                  _IEC0bits = 0x820
                    0x0822                  IEC1 = 0x822
                    0x0822                  _IEC1 = 0x822
                    0x0822                  _IEC1bits = 0x822
                    0x0824                  IEC2 = 0x824
                    0x0824                  _IEC2 = 0x824
                    0x0824                  _IEC2bits = 0x824
                    0x0826                  IEC3 = 0x826
                    0x0826                  _IEC3 = 0x826
                    0x0826                  _IEC3bits = 0x826
                    0x0828                  IEC4 = 0x828
                    0x0828                  _IEC4 = 0x828
                    0x0828                  _IEC4bits = 0x828
                    0x082a                  IEC5 = 0x82a
                    0x082a                  _IEC5 = 0x82a
                    0x082a                  _IEC5bits = 0x82a
                    0x082e                  IEC7 = 0x82e
                    0x082e                  _IEC7 = 0x82e
                    0x082e                  _IEC7bits = 0x82e
                    0x0830                  IEC8 = 0x830
                    0x0830                  _IEC8 = 0x830
                    0x0830                  _IEC8bits = 0x830
                    0x0840                  IPC0 = 0x840
                    0x0840                  _IPC0 = 0x840
                    0x0840                  _IPC0bits = 0x840
                    0x0842                  IPC1 = 0x842
                    0x0842                  _IPC1 = 0x842
                    0x0842                  _IPC1bits = 0x842
                    0x0844                  IPC2 = 0x844
                    0x0844                  _IPC2 = 0x844
                    0x0844                  _IPC2bits = 0x844
                    0x0846                  IPC3 = 0x846
                    0x0846                  _IPC3 = 0x846
                    0x0846                  _IPC3bits = 0x846
                    0x0848                  IPC4 = 0x848
                    0x0848                  _IPC4 = 0x848
                    0x0848                  _IPC4bits = 0x848
                    0x084a                  IPC5 = 0x84a
                    0x084a                  _IPC5 = 0x84a
                    0x084a                  _IPC5bits = 0x84a
                    0x084c                  IPC6 = 0x84c
                    0x084c                  _IPC6 = 0x84c
                    0x084c                  _IPC6bits = 0x84c
                    0x084e                  IPC7 = 0x84e
                    0x084e                  _IPC7 = 0x84e
                    0x084e                  _IPC7bits = 0x84e
                    0x0850                  IPC8 = 0x850
                    0x0850                  _IPC8 = 0x850
                    0x0850                  _IPC8bits = 0x850
                    0x0852                  IPC9 = 0x852
                    0x0852                  _IPC9 = 0x852
                    0x0852                  _IPC9bits = 0x852
                    0x0854                  IPC10 = 0x854
                    0x0854                  _IPC10 = 0x854
                    0x0854                  _IPC10bits = 0x854
                    0x0856                  IPC11 = 0x856
                    0x0856                  _IPC11 = 0x856
                    0x0856                  _IPC11bits = 0x856
                    0x0858                  IPC12 = 0x858
                    0x0858                  _IPC12 = 0x858
                    0x0858                  _IPC12bits = 0x858
                    0x085a                  IPC13 = 0x85a
                    0x085a                  _IPC13 = 0x85a
                    0x085a                  _IPC13bits = 0x85a
                    0x085c                  IPC14 = 0x85c
                    0x085c                  _IPC14 = 0x85c
                    0x085c                  _IPC14bits = 0x85c
                    0x085e                  IPC15 = 0x85e
                    0x085e                  _IPC15 = 0x85e
                    0x085e                  _IPC15bits = 0x85e
                    0x0860                  IPC16 = 0x860
                    0x0860                  _IPC16 = 0x860
                    0x0860                  _IPC16bits = 0x860
                    0x0862                  IPC17 = 0x862
                    0x0862                  _IPC17 = 0x862
                    0x0862                  _IPC17bits = 0x862
                    0x0868                  IPC20 = 0x868
                    0x0868                  _IPC20 = 0x868
                    0x0868                  _IPC20bits = 0x868
                    0x086a                  IPC21 = 0x86a
                    0x086a                  _IPC21 = 0x86a
                    0x086a                  _IPC21bits = 0x86a
                    0x086c                  IPC22 = 0x86c
                    0x086c                  _IPC22 = 0x86c
                    0x086c                  _IPC22bits = 0x86c
                    0x086e                  IPC23 = 0x86e
                    0x086e                  _IPC23 = 0x86e
                    0x086e                  _IPC23bits = 0x86e
                    0x087a                  IPC29 = 0x87a
                    0x087a                  _IPC29 = 0x87a
                    0x087a                  _IPC29bits = 0x87a
                    0x087c                  IPC30 = 0x87c
                    0x087c                  _IPC30 = 0x87c
                    0x087c                  _IPC30bits = 0x87c
                    0x087e                  IPC31 = 0x87e
                    0x087e                  _IPC31 = 0x87e
                    0x087e                  _IPC31bits = 0x87e
                    0x0880                  IPC32 = 0x880
                    0x0880                  _IPC32 = 0x880
                    0x0880                  _IPC32bits = 0x880
                    0x0882                  IPC33 = 0x882
                    0x0882                  _IPC33 = 0x882
                    0x0882                  _IPC33bits = 0x882
                    0x0884                  IPC34 = 0x884
                    0x0884                  _IPC34 = 0x884
                    0x0884                  _IPC34bits = 0x884
                    0x0886                  IPC35 = 0x886
                    0x0886                  _IPC35 = 0x886
                    0x0886                  _IPC35bits = 0x886
                    0x08c0                  INTCON1 = 0x8c0
                    0x08c0                  _INTCON1 = 0x8c0
                    0x08c0                  _INTCON1bits = 0x8c0
                    0x08c2                  INTCON2 = 0x8c2
                    0x08c2                  _INTCON2 = 0x8c2
                    0x08c2                  _INTCON2bits = 0x8c2
                    0x08c4                  INTCON3 = 0x8c4
                    0x08c4                  _INTCON3 = 0x8c4
                    0x08c4                  _INTCON3bits = 0x8c4
                    0x08c6                  INTCON4 = 0x8c6
                    0x08c6                  _INTCON4 = 0x8c6
                    0x08c6                  _INTCON4bits = 0x8c6
                    0x08c8                  INTTREG = 0x8c8
                    0x08c8                  _INTTREG = 0x8c8
                    0x08c8                  _INTTREGbits = 0x8c8
                    0x0900                  OC1CON1 = 0x900
                    0x0900                  _OC1CON1 = 0x900
                    0x0900                  _OC1CON1bits = 0x900
                    0x0902                  OC1CON2 = 0x902
                    0x0902                  _OC1CON2 = 0x902
                    0x0902                  _OC1CON2bits = 0x902
                    0x0904                  OC1RS = 0x904
                    0x0904                  _OC1RS = 0x904
                    0x0906                  OC1R = 0x906
                    0x0906                  _OC1R = 0x906
                    0x0908                  OC1TMR = 0x908
                    0x0908                  _OC1TMR = 0x908
                    0x090a                  OC2CON1 = 0x90a
                    0x090a                  _OC2CON1 = 0x90a
                    0x090a                  _OC2CON1bits = 0x90a
                    0x090c                  OC2CON2 = 0x90c
                    0x090c                  _OC2CON2 = 0x90c
                    0x090c                  _OC2CON2bits = 0x90c
                    0x090e                  OC2RS = 0x90e
                    0x090e                  _OC2RS = 0x90e
                    0x0910                  OC2R = 0x910
                    0x0910                  _OC2R = 0x910
                    0x0912                  OC2TMR = 0x912
                    0x0912                  _OC2TMR = 0x912
                    0x0914                  OC3CON1 = 0x914
                    0x0914                  _OC3CON1 = 0x914
                    0x0914                  _OC3CON1bits = 0x914
                    0x0916                  OC3CON2 = 0x916
                    0x0916                  _OC3CON2 = 0x916
                    0x0916                  _OC3CON2bits = 0x916
                    0x0918                  OC3RS = 0x918
                    0x0918                  _OC3RS = 0x918
                    0x091a                  OC3R = 0x91a
                    0x091a                  _OC3R = 0x91a
                    0x091c                  OC3TMR = 0x91c
                    0x091c                  _OC3TMR = 0x91c
                    0x091e                  OC4CON1 = 0x91e
                    0x091e                  _OC4CON1 = 0x91e
                    0x091e                  _OC4CON1bits = 0x91e
                    0x0920                  OC4CON2 = 0x920
                    0x0920                  _OC4CON2 = 0x920
                    0x0920                  _OC4CON2bits = 0x920
                    0x0922                  OC4RS = 0x922
                    0x0922                  _OC4RS = 0x922
                    0x0924                  OC4R = 0x924
                    0x0924                  _OC4R = 0x924
                    0x0926                  OC4TMR = 0x926
                    0x0926                  _OC4TMR = 0x926
                    0x0928                  OC5CON1 = 0x928
                    0x0928                  _OC5CON1 = 0x928
                    0x0928                  _OC5CON1bits = 0x928
                    0x092a                  OC5CON2 = 0x92a
                    0x092a                  _OC5CON2 = 0x92a
                    0x092a                  _OC5CON2bits = 0x92a
                    0x092c                  OC5RS = 0x92c
                    0x092c                  _OC5RS = 0x92c
                    0x092e                  OC5R = 0x92e
                    0x092e                  _OC5R = 0x92e
                    0x0930                  OC5TMR = 0x930
                    0x0930                  _OC5TMR = 0x930
                    0x0932                  OC6CON1 = 0x932
                    0x0932                  _OC6CON1 = 0x932
                    0x0932                  _OC6CON1bits = 0x932
                    0x0934                  OC6CON2 = 0x934
                    0x0934                  _OC6CON2 = 0x934
                    0x0934                  _OC6CON2bits = 0x934
                    0x0936                  OC6RS = 0x936
                    0x0936                  _OC6RS = 0x936
                    0x0938                  OC6R = 0x938
                    0x0938                  _OC6R = 0x938
                    0x093a                  OC6TMR = 0x93a
                    0x093a                  _OC6TMR = 0x93a
                    0x093c                  OC7CON1 = 0x93c
                    0x093c                  _OC7CON1 = 0x93c
                    0x093c                  _OC7CON1bits = 0x93c
                    0x093e                  OC7CON2 = 0x93e
                    0x093e                  _OC7CON2 = 0x93e
                    0x093e                  _OC7CON2bits = 0x93e
                    0x0940                  OC7RS = 0x940
                    0x0940                  _OC7RS = 0x940
                    0x0942                  OC7R = 0x942
                    0x0942                  _OC7R = 0x942
                    0x0944                  OC7TMR = 0x944
                    0x0944                  _OC7TMR = 0x944
                    0x0946                  OC8CON1 = 0x946
                    0x0946                  _OC8CON1 = 0x946
                    0x0946                  _OC8CON1bits = 0x946
                    0x0948                  OC8CON2 = 0x948
                    0x0948                  _OC8CON2 = 0x948
                    0x0948                  _OC8CON2bits = 0x948
                    0x094a                  OC8RS = 0x94a
                    0x094a                  _OC8RS = 0x94a
                    0x094c                  OC8R = 0x94c
                    0x094c                  _OC8R = 0x94c
                    0x094e                  OC8TMR = 0x94e
                    0x094e                  _OC8TMR = 0x94e
                    0x0950                  OC9CON1 = 0x950
                    0x0950                  _OC9CON1 = 0x950
                    0x0950                  _OC9CON1bits = 0x950
                    0x0952                  OC9CON2 = 0x952
                    0x0952                  _OC9CON2 = 0x952
                    0x0952                  _OC9CON2bits = 0x952
                    0x0954                  OC9RS = 0x954
                    0x0954                  _OC9RS = 0x954
                    0x0956                  OC9R = 0x956
                    0x0956                  _OC9R = 0x956
                    0x0958                  OC9TMR = 0x958
                    0x0958                  _OC9TMR = 0x958
                    0x095a                  OC10CON1 = 0x95a
                    0x095a                  _OC10CON1 = 0x95a
                    0x095a                  _OC10CON1bits = 0x95a
                    0x095c                  OC10CON2 = 0x95c
                    0x095c                  _OC10CON2 = 0x95c
                    0x095c                  _OC10CON2bits = 0x95c
                    0x095e                  OC10RS = 0x95e
                    0x095e                  _OC10RS = 0x95e
                    0x0960                  OC10R = 0x960
                    0x0960                  _OC10R = 0x960
                    0x0962                  OC10TMR = 0x962
                    0x0962                  _OC10TMR = 0x962
                    0x0964                  OC11CON1 = 0x964
                    0x0964                  _OC11CON1 = 0x964
                    0x0964                  _OC11CON1bits = 0x964
                    0x0966                  OC11CON2 = 0x966
                    0x0966                  _OC11CON2 = 0x966
                    0x0966                  _OC11CON2bits = 0x966
                    0x0968                  OC11RS = 0x968
                    0x0968                  _OC11RS = 0x968
                    0x096a                  OC11R = 0x96a
                    0x096a                  _OC11R = 0x96a
                    0x096c                  OC11TMR = 0x96c
                    0x096c                  _OC11TMR = 0x96c
                    0x096e                  OC12CON1 = 0x96e
                    0x096e                  _OC12CON1 = 0x96e
                    0x096e                  _OC12CON1bits = 0x96e
                    0x0970                  OC12CON2 = 0x970
                    0x0970                  _OC12CON2 = 0x970
                    0x0970                  _OC12CON2bits = 0x970
                    0x0972                  OC12RS = 0x972
                    0x0972                  _OC12RS = 0x972
                    0x0974                  OC12R = 0x974
                    0x0974                  _OC12R = 0x974
                    0x0976                  OC12TMR = 0x976
                    0x0976                  _OC12TMR = 0x976
                    0x0978                  OC13CON1 = 0x978
                    0x0978                  _OC13CON1 = 0x978
                    0x0978                  _OC13CON1bits = 0x978
                    0x097a                  OC13CON2 = 0x97a
                    0x097a                  _OC13CON2 = 0x97a
                    0x097a                  _OC13CON2bits = 0x97a
                    0x097c                  OC13RS = 0x97c
                    0x097c                  _OC13RS = 0x97c
                    0x097e                  OC13R = 0x97e
                    0x097e                  _OC13R = 0x97e
                    0x0980                  OC13TMR = 0x980
                    0x0980                  _OC13TMR = 0x980
                    0x0982                  OC14CON1 = 0x982
                    0x0982                  _OC14CON1 = 0x982
                    0x0982                  _OC14CON1bits = 0x982
                    0x0984                  OC14CON2 = 0x984
                    0x0984                  _OC14CON2 = 0x984
                    0x0984                  _OC14CON2bits = 0x984
                    0x0986                  OC14RS = 0x986
                    0x0986                  _OC14RS = 0x986
                    0x0988                  OC14R = 0x988
                    0x0988                  _OC14R = 0x988
                    0x098a                  OC14TMR = 0x98a
                    0x098a                  _OC14TMR = 0x98a
                    0x098c                  OC15CON1 = 0x98c
                    0x098c                  _OC15CON1 = 0x98c
                    0x098c                  _OC15CON1bits = 0x98c
                    0x098e                  OC15CON2 = 0x98e
                    0x098e                  _OC15CON2 = 0x98e
                    0x098e                  _OC15CON2bits = 0x98e
                    0x0990                  OC15RS = 0x990
                    0x0990                  _OC15RS = 0x990
                    0x0992                  OC15R = 0x992
                    0x0992                  _OC15R = 0x992
                    0x0994                  OC15TMR = 0x994
                    0x0994                  _OC15TMR = 0x994
                    0x0996                  OC16CON1 = 0x996
                    0x0996                  _OC16CON1 = 0x996
                    0x0996                  _OC16CON1bits = 0x996
                    0x0998                  OC16CON2 = 0x998
                    0x0998                  _OC16CON2 = 0x998
                    0x0998                  _OC16CON2bits = 0x998
                    0x099a                  OC16RS = 0x99a
                    0x099a                  _OC16RS = 0x99a
                    0x099c                  OC16R = 0x99c
                    0x099c                  _OC16R = 0x99c
                    0x099e                  OC16TMR = 0x99e
                    0x099e                  _OC16TMR = 0x99e
                    0x0a80                  CMSTAT = 0xa80
                    0x0a80                  _CMSTAT = 0xa80
                    0x0a80                  _CMSTATbits = 0xa80
                    0x0a82                  CVRCON = 0xa82
                    0x0a82                  _CVRCON = 0xa82
                    0x0a82                  _CVRCONbits = 0xa82
                    0x0a84                  CM1CON = 0xa84
                    0x0a84                  _CM1CON = 0xa84
                    0x0a84                  _CM1CONbits = 0xa84
                    0x0a86                  CM1MSKSRC = 0xa86
                    0x0a86                  _CM1MSKSRC = 0xa86
                    0x0a86                  _CM1MSKSRCbits = 0xa86
                    0x0a88                  CM1MSKCON = 0xa88
                    0x0a88                  _CM1MSKCON = 0xa88
                    0x0a88                  _CM1MSKCONbits = 0xa88
                    0x0a8a                  CM1FLTR = 0xa8a
                    0x0a8a                  _CM1FLTR = 0xa8a
                    0x0a8a                  _CM1FLTRbits = 0xa8a
                    0x0a8c                  CM2CON = 0xa8c
                    0x0a8c                  _CM2CON = 0xa8c
                    0x0a8c                  _CM2CONbits = 0xa8c
                    0x0a8e                  CM2MSKSRC = 0xa8e
                    0x0a8e                  _CM2MSKSRC = 0xa8e
                    0x0a8e                  _CM2MSKSRCbits = 0xa8e
                    0x0a90                  CM2MSKCON = 0xa90
                    0x0a90                  _CM2MSKCON = 0xa90
                    0x0a90                  _CM2MSKCONbits = 0xa90
                    0x0a92                  CM2FLTR = 0xa92
                    0x0a92                  _CM2FLTR = 0xa92
                    0x0a92                  _CM2FLTRbits = 0xa92
                    0x0a94                  CM3CON = 0xa94
                    0x0a94                  _CM3CON = 0xa94
                    0x0a94                  _CM3CONbits = 0xa94
                    0x0a96                  CM3MSKSRC = 0xa96
                    0x0a96                  _CM3MSKSRC = 0xa96
                    0x0a96                  _CM3MSKSRCbits = 0xa96
                    0x0a98                  CM3MSKCON = 0xa98
                    0x0a98                  _CM3MSKCON = 0xa98
                    0x0a98                  _CM3MSKCONbits = 0xa98
                    0x0a9a                  CM3FLTR = 0xa9a
                    0x0a9a                  _CM3FLTR = 0xa9a
                    0x0a9a                  _CM3FLTRbits = 0xa9a
                    0x0b00                  DMA0CON = 0xb00
                    0x0b00                  _DMA0CON = 0xb00
                    0x0b00                  _DMA0CONbits = 0xb00
                    0x0b02                  DMA0REQ = 0xb02
                    0x0b02                  _DMA0REQ = 0xb02
                    0x0b02                  _DMA0REQbits = 0xb02
                    0x0b04                  DMA0STAL = 0xb04
                    0x0b04                  _DMA0STAL = 0xb04
                    0x0b06                  DMA0STAH = 0xb06
                    0x0b06                  _DMA0STAH = 0xb06
                    0x0b06                  _DMA0STAHbits = 0xb06
                    0x0b08                  DMA0STBL = 0xb08
                    0x0b08                  _DMA0STBL = 0xb08
                    0x0b0a                  DMA0STBH = 0xb0a
                    0x0b0a                  _DMA0STBH = 0xb0a
                    0x0b0a                  _DMA0STBHbits = 0xb0a
                    0x0b0c                  DMA0PAD = 0xb0c
                    0x0b0c                  _DMA0PAD = 0xb0c
                    0x0b0e                  DMA0CNT = 0xb0e
                    0x0b0e                  _DMA0CNT = 0xb0e
                    0x0b0e                  _DMA0CNTbits = 0xb0e
                    0x0b10                  DMA1CON = 0xb10
                    0x0b10                  _DMA1CON = 0xb10
                    0x0b10                  _DMA1CONbits = 0xb10
                    0x0b12                  DMA1REQ = 0xb12
                    0x0b12                  _DMA1REQ = 0xb12
                    0x0b12                  _DMA1REQbits = 0xb12
                    0x0b14                  DMA1STAL = 0xb14
                    0x0b14                  _DMA1STAL = 0xb14
                    0x0b16                  DMA1STAH = 0xb16
                    0x0b16                  _DMA1STAH = 0xb16
                    0x0b16                  _DMA1STAHbits = 0xb16
                    0x0b18                  DMA1STBL = 0xb18
                    0x0b18                  _DMA1STBL = 0xb18
                    0x0b1a                  DMA1STBH = 0xb1a
                    0x0b1a                  _DMA1STBH = 0xb1a
                    0x0b1a                  _DMA1STBHbits = 0xb1a
                    0x0b1c                  DMA1PAD = 0xb1c
                    0x0b1c                  _DMA1PAD = 0xb1c
                    0x0b1e                  DMA1CNT = 0xb1e
                    0x0b1e                  _DMA1CNT = 0xb1e
                    0x0b1e                  _DMA1CNTbits = 0xb1e
                    0x0b20                  DMA2CON = 0xb20
                    0x0b20                  _DMA2CON = 0xb20
                    0x0b20                  _DMA2CONbits = 0xb20
                    0x0b22                  DMA2REQ = 0xb22
                    0x0b22                  _DMA2REQ = 0xb22
                    0x0b22                  _DMA2REQbits = 0xb22
                    0x0b24                  DMA2STAL = 0xb24
                    0x0b24                  _DMA2STAL = 0xb24
                    0x0b26                  DMA2STAH = 0xb26
                    0x0b26                  _DMA2STAH = 0xb26
                    0x0b26                  _DMA2STAHbits = 0xb26
                    0x0b28                  DMA2STBL = 0xb28
                    0x0b28                  _DMA2STBL = 0xb28
                    0x0b2a                  DMA2STBH = 0xb2a
                    0x0b2a                  _DMA2STBH = 0xb2a
                    0x0b2a                  _DMA2STBHbits = 0xb2a
                    0x0b2c                  DMA2PAD = 0xb2c
                    0x0b2c                  _DMA2PAD = 0xb2c
                    0x0b2e                  DMA2CNT = 0xb2e
                    0x0b2e                  _DMA2CNT = 0xb2e
                    0x0b2e                  _DMA2CNTbits = 0xb2e
                    0x0b30                  DMA3CON = 0xb30
                    0x0b30                  _DMA3CON = 0xb30
                    0x0b30                  _DMA3CONbits = 0xb30
                    0x0b32                  DMA3REQ = 0xb32
                    0x0b32                  _DMA3REQ = 0xb32
                    0x0b32                  _DMA3REQbits = 0xb32
                    0x0b34                  DMA3STAL = 0xb34
                    0x0b34                  _DMA3STAL = 0xb34
                    0x0b36                  DMA3STAH = 0xb36
                    0x0b36                  _DMA3STAH = 0xb36
                    0x0b36                  _DMA3STAHbits = 0xb36
                    0x0b38                  DMA3STBL = 0xb38
                    0x0b38                  _DMA3STBL = 0xb38
                    0x0b3a                  DMA3STBH = 0xb3a
                    0x0b3a                  _DMA3STBH = 0xb3a
                    0x0b3a                  _DMA3STBHbits = 0xb3a
                    0x0b3c                  DMA3PAD = 0xb3c
                    0x0b3c                  _DMA3PAD = 0xb3c
                    0x0b3e                  DMA3CNT = 0xb3e
                    0x0b3e                  _DMA3CNT = 0xb3e
                    0x0b3e                  _DMA3CNTbits = 0xb3e
                    0x0b40                  DMA4CON = 0xb40
                    0x0b40                  _DMA4CON = 0xb40
                    0x0b40                  _DMA4CONbits = 0xb40
                    0x0b42                  DMA4REQ = 0xb42
                    0x0b42                  _DMA4REQ = 0xb42
                    0x0b42                  _DMA4REQbits = 0xb42
                    0x0b44                  DMA4STAL = 0xb44
                    0x0b44                  _DMA4STAL = 0xb44
                    0x0b46                  DMA4STAH = 0xb46
                    0x0b46                  _DMA4STAH = 0xb46
                    0x0b46                  _DMA4STAHbits = 0xb46
                    0x0b48                  DMA4STBL = 0xb48
                    0x0b48                  _DMA4STBL = 0xb48
                    0x0b4a                  DMA4STBH = 0xb4a
                    0x0b4a                  _DMA4STBH = 0xb4a
                    0x0b4a                  _DMA4STBHbits = 0xb4a
                    0x0b4c                  DMA4PAD = 0xb4c
                    0x0b4c                  _DMA4PAD = 0xb4c
                    0x0b4e                  DMA4CNT = 0xb4e
                    0x0b4e                  _DMA4CNT = 0xb4e
                    0x0b4e                  _DMA4CNTbits = 0xb4e
                    0x0b50                  DMA5CON = 0xb50
                    0x0b50                  _DMA5CON = 0xb50
                    0x0b50                  _DMA5CONbits = 0xb50
                    0x0b52                  DMA5REQ = 0xb52
                    0x0b52                  _DMA5REQ = 0xb52
                    0x0b52                  _DMA5REQbits = 0xb52
                    0x0b54                  DMA5STAL = 0xb54
                    0x0b54                  _DMA5STAL = 0xb54
                    0x0b56                  DMA5STAH = 0xb56
                    0x0b56                  _DMA5STAH = 0xb56
                    0x0b56                  _DMA5STAHbits = 0xb56
                    0x0b58                  DMA5STBL = 0xb58
                    0x0b58                  _DMA5STBL = 0xb58
                    0x0b5a                  DMA5STBH = 0xb5a
                    0x0b5a                  _DMA5STBH = 0xb5a
                    0x0b5a                  _DMA5STBHbits = 0xb5a
                    0x0b5c                  DMA5PAD = 0xb5c
                    0x0b5c                  _DMA5PAD = 0xb5c
                    0x0b5e                  DMA5CNT = 0xb5e
                    0x0b5e                  _DMA5CNT = 0xb5e
                    0x0b5e                  _DMA5CNTbits = 0xb5e
                    0x0b60                  DMA6CON = 0xb60
                    0x0b60                  _DMA6CON = 0xb60
                    0x0b60                  _DMA6CONbits = 0xb60
                    0x0b62                  DMA6REQ = 0xb62
                    0x0b62                  _DMA6REQ = 0xb62
                    0x0b62                  _DMA6REQbits = 0xb62
                    0x0b64                  DMA6STAL = 0xb64
                    0x0b64                  _DMA6STAL = 0xb64
                    0x0b66                  DMA6STAH = 0xb66
                    0x0b66                  _DMA6STAH = 0xb66
                    0x0b66                  _DMA6STAHbits = 0xb66
                    0x0b68                  DMA6STBL = 0xb68
                    0x0b68                  _DMA6STBL = 0xb68
                    0x0b6a                  DMA6STBH = 0xb6a
                    0x0b6a                  _DMA6STBH = 0xb6a
                    0x0b6a                  _DMA6STBHbits = 0xb6a
                    0x0b6c                  DMA6PAD = 0xb6c
                    0x0b6c                  _DMA6PAD = 0xb6c
                    0x0b6e                  DMA6CNT = 0xb6e
                    0x0b6e                  _DMA6CNT = 0xb6e
                    0x0b6e                  _DMA6CNTbits = 0xb6e
                    0x0b70                  DMA7CON = 0xb70
                    0x0b70                  _DMA7CON = 0xb70
                    0x0b70                  _DMA7CONbits = 0xb70
                    0x0b72                  DMA7REQ = 0xb72
                    0x0b72                  _DMA7REQ = 0xb72
                    0x0b72                  _DMA7REQbits = 0xb72
                    0x0b74                  DMA7STAL = 0xb74
                    0x0b74                  _DMA7STAL = 0xb74
                    0x0b76                  DMA7STAH = 0xb76
                    0x0b76                  _DMA7STAH = 0xb76
                    0x0b76                  _DMA7STAHbits = 0xb76
                    0x0b78                  DMA7STBL = 0xb78
                    0x0b78                  _DMA7STBL = 0xb78
                    0x0b7a                  DMA7STBH = 0xb7a
                    0x0b7a                  _DMA7STBH = 0xb7a
                    0x0b7a                  _DMA7STBHbits = 0xb7a
                    0x0b7c                  DMA7PAD = 0xb7c
                    0x0b7c                  _DMA7PAD = 0xb7c
                    0x0b7e                  DMA7CNT = 0xb7e
                    0x0b7e                  _DMA7CNT = 0xb7e
                    0x0b7e                  _DMA7CNTbits = 0xb7e
                    0x0b80                  DMA8CON = 0xb80
                    0x0b80                  _DMA8CON = 0xb80
                    0x0b80                  _DMA8CONbits = 0xb80
                    0x0b82                  DMA8REQ = 0xb82
                    0x0b82                  _DMA8REQ = 0xb82
                    0x0b82                  _DMA8REQbits = 0xb82
                    0x0b84                  DMA8STAL = 0xb84
                    0x0b84                  _DMA8STAL = 0xb84
                    0x0b86                  DMA8STAH = 0xb86
                    0x0b86                  _DMA8STAH = 0xb86
                    0x0b86                  _DMA8STAHbits = 0xb86
                    0x0b88                  DMA8STBL = 0xb88
                    0x0b88                  _DMA8STBL = 0xb88
                    0x0b8a                  DMA8STBH = 0xb8a
                    0x0b8a                  _DMA8STBH = 0xb8a
                    0x0b8a                  _DMA8STBHbits = 0xb8a
                    0x0b8c                  DMA8PAD = 0xb8c
                    0x0b8c                  _DMA8PAD = 0xb8c
                    0x0b8e                  DMA8CNT = 0xb8e
                    0x0b8e                  _DMA8CNT = 0xb8e
                    0x0b8e                  _DMA8CNTbits = 0xb8e
                    0x0b90                  DMA9CON = 0xb90
                    0x0b90                  _DMA9CON = 0xb90
                    0x0b90                  _DMA9CONbits = 0xb90
                    0x0b92                  DMA9REQ = 0xb92
                    0x0b92                  _DMA9REQ = 0xb92
                    0x0b92                  _DMA9REQbits = 0xb92
                    0x0b94                  DMA9STAL = 0xb94
                    0x0b94                  _DMA9STAL = 0xb94
                    0x0b96                  DMA9STAH = 0xb96
                    0x0b96                  _DMA9STAH = 0xb96
                    0x0b96                  _DMA9STAHbits = 0xb96
                    0x0b98                  DMA9STBL = 0xb98
                    0x0b98                  _DMA9STBL = 0xb98
                    0x0b9a                  DMA9STBH = 0xb9a
                    0x0b9a                  _DMA9STBH = 0xb9a
                    0x0b9a                  _DMA9STBHbits = 0xb9a
                    0x0b9c                  DMA9PAD = 0xb9c
                    0x0b9c                  _DMA9PAD = 0xb9c
                    0x0b9e                  DMA9CNT = 0xb9e
                    0x0b9e                  _DMA9CNT = 0xb9e
                    0x0b9e                  _DMA9CNTbits = 0xb9e
                    0x0ba0                  DMA10CON = 0xba0
                    0x0ba0                  _DMA10CON = 0xba0
                    0x0ba0                  _DMA10CONbits = 0xba0
                    0x0ba2                  DMA10REQ = 0xba2
                    0x0ba2                  _DMA10REQ = 0xba2
                    0x0ba2                  _DMA10REQbits = 0xba2
                    0x0ba4                  DMA10STAL = 0xba4
                    0x0ba4                  _DMA10STAL = 0xba4
                    0x0ba6                  DMA10STAH = 0xba6
                    0x0ba6                  _DMA10STAH = 0xba6
                    0x0ba6                  _DMA10STAHbits = 0xba6
                    0x0ba8                  DMA10STBL = 0xba8
                    0x0ba8                  _DMA10STBL = 0xba8
                    0x0baa                  DMA10STBH = 0xbaa
                    0x0baa                  _DMA10STBH = 0xbaa
                    0x0baa                  _DMA10STBHbits = 0xbaa
                    0x0bac                  DMA10PAD = 0xbac
                    0x0bac                  _DMA10PAD = 0xbac
                    0x0bae                  DMA10CNT = 0xbae
                    0x0bae                  _DMA10CNT = 0xbae
                    0x0bae                  _DMA10CNTbits = 0xbae
                    0x0bb0                  DMA11CON = 0xbb0
                    0x0bb0                  _DMA11CON = 0xbb0
                    0x0bb0                  _DMA11CONbits = 0xbb0
                    0x0bb2                  DMA11REQ = 0xbb2
                    0x0bb2                  _DMA11REQ = 0xbb2
                    0x0bb2                  _DMA11REQbits = 0xbb2
                    0x0bb4                  DMA11STAL = 0xbb4
                    0x0bb4                  _DMA11STAL = 0xbb4
                    0x0bb6                  DMA11STAH = 0xbb6
                    0x0bb6                  _DMA11STAH = 0xbb6
                    0x0bb6                  _DMA11STAHbits = 0xbb6
                    0x0bb8                  DMA11STBL = 0xbb8
                    0x0bb8                  _DMA11STBL = 0xbb8
                    0x0bba                  DMA11STBH = 0xbba
                    0x0bba                  _DMA11STBH = 0xbba
                    0x0bba                  _DMA11STBHbits = 0xbba
                    0x0bbc                  DMA11PAD = 0xbbc
                    0x0bbc                  _DMA11PAD = 0xbbc
                    0x0bbe                  DMA11CNT = 0xbbe
                    0x0bbe                  _DMA11CNT = 0xbbe
                    0x0bbe                  _DMA11CNTbits = 0xbbe
                    0x0bc0                  DMA12CON = 0xbc0
                    0x0bc0                  _DMA12CON = 0xbc0
                    0x0bc0                  _DMA12CONbits = 0xbc0
                    0x0bc2                  DMA12REQ = 0xbc2
                    0x0bc2                  _DMA12REQ = 0xbc2
                    0x0bc2                  _DMA12REQbits = 0xbc2
                    0x0bc4                  DMA12STAL = 0xbc4
                    0x0bc4                  _DMA12STAL = 0xbc4
                    0x0bc6                  DMA12STAH = 0xbc6
                    0x0bc6                  _DMA12STAH = 0xbc6
                    0x0bc6                  _DMA12STAHbits = 0xbc6
                    0x0bc8                  DMA12STBL = 0xbc8
                    0x0bc8                  _DMA12STBL = 0xbc8
                    0x0bca                  DMA12STBH = 0xbca
                    0x0bca                  _DMA12STBH = 0xbca
                    0x0bca                  _DMA12STBHbits = 0xbca
                    0x0bcc                  DMA12PAD = 0xbcc
                    0x0bcc                  _DMA12PAD = 0xbcc
                    0x0bce                  DMA12CNT = 0xbce
                    0x0bce                  _DMA12CNT = 0xbce
                    0x0bce                  _DMA12CNTbits = 0xbce
                    0x0bd0                  DMA13CON = 0xbd0
                    0x0bd0                  _DMA13CON = 0xbd0
                    0x0bd0                  _DMA13CONbits = 0xbd0
                    0x0bd2                  DMA13REQ = 0xbd2
                    0x0bd2                  _DMA13REQ = 0xbd2
                    0x0bd2                  _DMA13REQbits = 0xbd2
                    0x0bd4                  DMA13STAL = 0xbd4
                    0x0bd4                  _DMA13STAL = 0xbd4
                    0x0bd6                  DMA13STAH = 0xbd6
                    0x0bd6                  _DMA13STAH = 0xbd6
                    0x0bd6                  _DMA13STAHbits = 0xbd6
                    0x0bd8                  DMA13STBL = 0xbd8
                    0x0bd8                  _DMA13STBL = 0xbd8
                    0x0bda                  DMA13STBH = 0xbda
                    0x0bda                  _DMA13STBH = 0xbda
                    0x0bda                  _DMA13STBHbits = 0xbda
                    0x0bdc                  DMA13PAD = 0xbdc
                    0x0bdc                  _DMA13PAD = 0xbdc
                    0x0bde                  DMA13CNT = 0xbde
                    0x0bde                  _DMA13CNT = 0xbde
                    0x0bde                  _DMA13CNTbits = 0xbde
                    0x0be0                  DMA14CON = 0xbe0
                    0x0be0                  _DMA14CON = 0xbe0
                    0x0be0                  _DMA14CONbits = 0xbe0
                    0x0be2                  DMA14REQ = 0xbe2
                    0x0be2                  _DMA14REQ = 0xbe2
                    0x0be2                  _DMA14REQbits = 0xbe2
                    0x0be4                  DMA14STAL = 0xbe4
                    0x0be4                  _DMA14STAL = 0xbe4
                    0x0be6                  DMA14STAH = 0xbe6
                    0x0be6                  _DMA14STAH = 0xbe6
                    0x0be6                  _DMA14STAHbits = 0xbe6
                    0x0be8                  DMA14STBL = 0xbe8
                    0x0be8                  _DMA14STBL = 0xbe8
                    0x0bea                  DMA14STBH = 0xbea
                    0x0bea                  _DMA14STBH = 0xbea
                    0x0bea                  _DMA14STBHbits = 0xbea
                    0x0bec                  DMA14PAD = 0xbec
                    0x0bec                  _DMA14PAD = 0xbec
                    0x0bee                  DMA14CNT = 0xbee
                    0x0bee                  _DMA14CNT = 0xbee
                    0x0bee                  _DMA14CNTbits = 0xbee
                    0x0bf0                  DMAPWC = 0xbf0
                    0x0bf0                  _DMAPWC = 0xbf0
                    0x0bf0                  _DMAPWCbits = 0xbf0
                    0x0bf2                  DMARQC = 0xbf2
                    0x0bf2                  _DMARQC = 0xbf2
                    0x0bf2                  _DMARQCbits = 0xbf2
                    0x0bf4                  DMAPPS = 0xbf4
                    0x0bf4                  _DMAPPS = 0xbf4
                    0x0bf4                  _DMAPPSbits = 0xbf4
                    0x0bf6                  DMALCA = 0xbf6
                    0x0bf6                  _DMALCA = 0xbf6
                    0x0bf6                  _DMALCAbits = 0xbf6
                    0x0bf8                  DSADRL = 0xbf8
                    0x0bf8                  _DSADRL = 0xbf8
                    0x0bfa                  DSADRH = 0xbfa
                    0x0bfa                  _DSADRH = 0xbfa
                    0x0bfa                  _DSADRHbits = 0xbfa
                    0x0e00                  TRISA = 0xe00
                    0x0e00                  _TRISA = 0xe00
                    0x0e00                  _TRISAbits = 0xe00
                    0x0e02                  PORTA = 0xe02
                    0x0e02                  _PORTA = 0xe02
                    0x0e02                  _PORTAbits = 0xe02
                    0x0e04                  LATA = 0xe04
                    0x0e04                  _LATA = 0xe04
                    0x0e04                  _LATAbits = 0xe04
                    0x0e06                  ODCA = 0xe06
                    0x0e06                  _ODCA = 0xe06
                    0x0e06                  _ODCAbits = 0xe06
                    0x0e08                  CNENA = 0xe08
                    0x0e08                  _CNENA = 0xe08
                    0x0e08                  _CNENAbits = 0xe08
                    0x0e0a                  CNPUA = 0xe0a
                    0x0e0a                  _CNPUA = 0xe0a
                    0x0e0a                  _CNPUAbits = 0xe0a
                    0x0e0c                  CNPDA = 0xe0c
                    0x0e0c                  _CNPDA = 0xe0c
                    0x0e0c                  _CNPDAbits = 0xe0c
                    0x0e0e                  ANSELA = 0xe0e
                    0x0e0e                  _ANSELA = 0xe0e
                    0x0e0e                  _ANSELAbits = 0xe0e
                    0x0e10                  TRISB = 0xe10
                    0x0e10                  _TRISB = 0xe10
                    0x0e10                  _TRISBbits = 0xe10
                    0x0e12                  PORTB = 0xe12
                    0x0e12                  _PORTB = 0xe12
                    0x0e12                  _PORTBbits = 0xe12
                    0x0e14                  LATB = 0xe14
                    0x0e14                  _LATB = 0xe14
                    0x0e14                  _LATBbits = 0xe14
                    0x0e18                  CNENB = 0xe18
                    0x0e18                  _CNENB = 0xe18
                    0x0e18                  _CNENBbits = 0xe18
                    0x0e1a                  CNPUB = 0xe1a
                    0x0e1a                  _CNPUB = 0xe1a
                    0x0e1a                  _CNPUBbits = 0xe1a
                    0x0e1c                  CNPDB = 0xe1c
                    0x0e1c                  _CNPDB = 0xe1c
                    0x0e1c                  _CNPDBbits = 0xe1c
                    0x0e1e                  ANSELB = 0xe1e
                    0x0e1e                  _ANSELB = 0xe1e
                    0x0e1e                  _ANSELBbits = 0xe1e
                    0x0e20                  TRISC = 0xe20
                    0x0e20                  _TRISC = 0xe20
                    0x0e20                  _TRISCbits = 0xe20
                    0x0e22                  PORTC = 0xe22
                    0x0e22                  _PORTC = 0xe22
                    0x0e22                  _PORTCbits = 0xe22
                    0x0e24                  LATC = 0xe24
                    0x0e24                  _LATC = 0xe24
                    0x0e24                  _LATCbits = 0xe24
                    0x0e28                  CNENC = 0xe28
                    0x0e28                  _CNENC = 0xe28
                    0x0e28                  _CNENCbits = 0xe28
                    0x0e2a                  CNPUC = 0xe2a
                    0x0e2a                  _CNPUC = 0xe2a
                    0x0e2a                  _CNPUCbits = 0xe2a
                    0x0e2c                  CNPDC = 0xe2c
                    0x0e2c                  _CNPDC = 0xe2c
                    0x0e2c                  _CNPDCbits = 0xe2c
                    0x0e2e                  ANSELC = 0xe2e
                    0x0e2e                  _ANSELC = 0xe2e
                    0x0e2e                  _ANSELCbits = 0xe2e
                    0x0e30                  TRISD = 0xe30
                    0x0e30                  _TRISD = 0xe30
                    0x0e30                  _TRISDbits = 0xe30
                    0x0e32                  PORTD = 0xe32
                    0x0e32                  _PORTD = 0xe32
                    0x0e32                  _PORTDbits = 0xe32
                    0x0e34                  LATD = 0xe34
                    0x0e34                  _LATD = 0xe34
                    0x0e34                  _LATDbits = 0xe34
                    0x0e36                  ODCD = 0xe36
                    0x0e36                  _ODCD = 0xe36
                    0x0e36                  _ODCDbits = 0xe36
                    0x0e38                  CNEND = 0xe38
                    0x0e38                  _CNEND = 0xe38
                    0x0e38                  _CNENDbits = 0xe38
                    0x0e3a                  CNPUD = 0xe3a
                    0x0e3a                  _CNPUD = 0xe3a
                    0x0e3a                  _CNPUDbits = 0xe3a
                    0x0e3c                  CNPDD = 0xe3c
                    0x0e3c                  _CNPDD = 0xe3c
                    0x0e3c                  _CNPDDbits = 0xe3c
                    0x0e3e                  ANSELD = 0xe3e
                    0x0e3e                  _ANSELD = 0xe3e
                    0x0e3e                  _ANSELDbits = 0xe3e
                    0x0e40                  TRISE = 0xe40
                    0x0e40                  _TRISE = 0xe40
                    0x0e40                  _TRISEbits = 0xe40
                    0x0e42                  PORTE = 0xe42
                    0x0e42                  _PORTE = 0xe42
                    0x0e42                  _PORTEbits = 0xe42
                    0x0e44                  LATE = 0xe44
                    0x0e44                  _LATE = 0xe44
                    0x0e44                  _LATEbits = 0xe44
                    0x0e48                  CNENE = 0xe48
                    0x0e48                  _CNENE = 0xe48
                    0x0e48                  _CNENEbits = 0xe48
                    0x0e4a                  CNPUE = 0xe4a
                    0x0e4a                  _CNPUE = 0xe4a
                    0x0e4a                  _CNPUEbits = 0xe4a
                    0x0e4c                  CNPDE = 0xe4c
                    0x0e4c                  _CNPDE = 0xe4c
                    0x0e4c                  _CNPDEbits = 0xe4c
                    0x0e4e                  ANSELE = 0xe4e
                    0x0e4e                  _ANSELE = 0xe4e
                    0x0e4e                  _ANSELEbits = 0xe4e
                    0x0e50                  TRISF = 0xe50
                    0x0e50                  _TRISF = 0xe50
                    0x0e50                  _TRISFbits = 0xe50
                    0x0e52                  PORTF = 0xe52
                    0x0e52                  _PORTF = 0xe52
                    0x0e52                  _PORTFbits = 0xe52
                    0x0e54                  LATF = 0xe54
                    0x0e54                  _LATF = 0xe54
                    0x0e54                  _LATFbits = 0xe54
                    0x0e56                  ODCF = 0xe56
                    0x0e56                  _ODCF = 0xe56
                    0x0e56                  _ODCFbits = 0xe56
                    0x0e58                  CNENF = 0xe58
                    0x0e58                  _CNENF = 0xe58
                    0x0e58                  _CNENFbits = 0xe58
                    0x0e5a                  CNPUF = 0xe5a
                    0x0e5a                  _CNPUF = 0xe5a
                    0x0e5a                  _CNPUFbits = 0xe5a
                    0x0e5c                  CNPDF = 0xe5c
                    0x0e5c                  _CNPDF = 0xe5c
                    0x0e5c                  _CNPDFbits = 0xe5c
                    0x0e60                  TRISG = 0xe60
                    0x0e60                  _TRISG = 0xe60
                    0x0e60                  _TRISGbits = 0xe60
                    0x0e62                  PORTG = 0xe62
                    0x0e62                  _PORTG = 0xe62
                    0x0e62                  _PORTGbits = 0xe62
                    0x0e64                  LATG = 0xe64
                    0x0e64                  _LATG = 0xe64
                    0x0e64                  _LATGbits = 0xe64
                    0x0e66                  ODCG = 0xe66
                    0x0e66                  _ODCG = 0xe66
                    0x0e66                  _ODCGbits = 0xe66
                    0x0e68                  CNENG = 0xe68
                    0x0e68                  _CNENG = 0xe68
                    0x0e68                  _CNENGbits = 0xe68
                    0x0e6a                  CNPUG = 0xe6a
                    0x0e6a                  _CNPUG = 0xe6a
                    0x0e6a                  _CNPUGbits = 0xe6a
                    0x0e6c                  CNPDG = 0xe6c
                    0x0e6c                  _CNPDG = 0xe6c
                    0x0e6c                  _CNPDGbits = 0xe6c
                    0x0e6e                  ANSELG = 0xe6e
                    0x0e6e                  _ANSELG = 0xe6e
                    0x0e6e                  _ANSELGbits = 0xe6e
                    0x0efe                  PADCFG1 = 0xefe
                    0x0efe                  _PADCFG1 = 0xefe
                    0x0efe                  _PADCFG1bits = 0xefe
                    0x0440                  CAN1 = 0x440
                    0x0440                  _CAN1 = 0x440
                    0x0540                  CAN2 = 0x540
                    0x0540                  _CAN2 = 0x540
                    0x0144                  IC1 = 0x144
                    0x0144                  _IC1 = 0x144
                    0x014c                  IC2 = 0x14c
                    0x014c                  _IC2 = 0x14c
                    0x0154                  IC3 = 0x154
                    0x0154                  _IC3 = 0x154
                    0x015c                  IC4 = 0x15c
                    0x015c                  _IC4 = 0x15c
                    0x0164                  IC5 = 0x164
                    0x0164                  _IC5 = 0x164
                    0x016c                  IC6 = 0x16c
                    0x016c                  _IC6 = 0x16c
                    0x0174                  IC7 = 0x174
                    0x0174                  _IC7 = 0x174
                    0x017c                  IC8 = 0x17c
                    0x017c                  _IC8 = 0x17c
                    0x0904                  OC1 = 0x904
                    0x0904                  _OC1 = 0x904
                    0x090e                  OC2 = 0x90e
                    0x090e                  _OC2 = 0x90e
                    0x0918                  OC3 = 0x918
                    0x0918                  _OC3 = 0x918
                    0x0922                  OC4 = 0x922
                    0x0922                  _OC4 = 0x922
                    0x092c                  OC5 = 0x92c
                    0x092c                  _OC5 = 0x92c
                    0x0936                  OC6 = 0x936
                    0x0936                  _OC6 = 0x936
                    0x0940                  OC7 = 0x940
                    0x0940                  _OC7 = 0x940
                    0x094a                  OC8 = 0x94a
                    0x094a                  _OC8 = 0x94a
                    0x0240                  SPI1 = 0x240
                    0x0240                  _SPI1 = 0x240
                    0x0260                  SPI2 = 0x260
                    0x0260                  _SPI2 = 0x260
                    0x0220                  UART1 = 0x220
                    0x0220                  _UART1 = 0x220
                    0x0230                  UART2 = 0x230
                    0x0230                  _UART2 = 0x230
START GROUP
LOAD c:/program files (x86)/microchip/xc16/v1.20/bin/bin/../../lib\libfx-elf.a
LOAD c:/program files (x86)/microchip/xc16/v1.20/bin/bin/../../lib\libpic30-elf.a
LOAD c:/program files (x86)/microchip/xc16/v1.20/bin/bin/../../lib\libm-elf.a
LOAD c:/program files (x86)/microchip/xc16/v1.20/bin/bin/../../lib\libc-elf.a
END GROUP
OUTPUT(dist/XC16-EX16_MRF24WB/production/MPLAB.X.production.elf elf32-pic30)
LOAD jump_table
LOAD heap
LOAD data_init

.debug_pubtypes
                  0x0004b8       0x2cb3
 .debug_pubtypes
                  0x0004b8         0xa9 build/XC16-EX16_MRF24WB/production/_ext/1954962658/ARP.o
 .debug_pubtypes
                  0x000561         0x12 build/XC16-EX16_MRF24WB/production/_ext/1954962658/Announce.o
 .debug_pubtypes
                  0x000573         0x12 build/XC16-EX16_MRF24WB/production/_ext/1954962658/AutoIP.o
 .debug_pubtypes
                  0x000585         0x12 build/XC16-EX16_MRF24WB/production/_ext/1954962658/BerkeleyAPI.o
 .debug_pubtypes
                  0x000597        0x10f build/XC16-EX16_MRF24WB/production/_ext/1954962658/DHCP.o
 .debug_pubtypes
                  0x0006a6        0x122 build/XC16-EX16_MRF24WB/production/_ext/1954962658/DHCPs.o
 .debug_pubtypes
                  0x0007c8         0xd8 build/XC16-EX16_MRF24WB/production/_ext/1954962658/DNS.o
 .debug_pubtypes
                  0x0008a0         0x9b build/XC16-EX16_MRF24WB/production/_ext/1954962658/DNSs.o
 .debug_pubtypes
                  0x00093b         0x25 build/XC16-EX16_MRF24WB/production/_ext/1954962658/Delay.o
 .debug_pubtypes
                  0x000960         0x12 build/XC16-EX16_MRF24WB/production/_ext/1954962658/DynDNS.o
 .debug_pubtypes
                  0x000972         0x12 build/XC16-EX16_MRF24WB/production/_ext/1954962658/ENC28J60.o
 .debug_pubtypes
                  0x000984         0x12 build/XC16-EX16_MRF24WB/production/_ext/1954962658/ENCX24J600.o
 .debug_pubtypes
                  0x000996         0x12 build/XC16-EX16_MRF24WB/production/_ext/1954962658/FTP.o
 .debug_pubtypes
                  0x0009a8         0x49 build/XC16-EX16_MRF24WB/production/_ext/1954962658/Hashes.o
 .debug_pubtypes
                  0x0009f1         0x90 build/XC16-EX16_MRF24WB/production/_ext/1954962658/Helpers.o
 .debug_pubtypes
                  0x000a81         0x64 build/XC16-EX16_MRF24WB/production/_ext/1954962658/ICMP.o
 .debug_pubtypes
                  0x000ae5         0xb7 build/XC16-EX16_MRF24WB/production/_ext/1954962658/IP.o
 .debug_pubtypes
                  0x000b9c         0x93 build/XC16-EX16_MRF24WB/production/_ext/1954962658/LCDBlocking.o
 .debug_pubtypes
                  0x000c2f         0xe6 build/XC16-EX16_MRF24WB/production/_ext/1954962658/NBNS.o
 .debug_pubtypes
                  0x000d15         0x12 build/XC16-EX16_MRF24WB/production/_ext/1954962658/Reboot.o
 .debug_pubtypes
                  0x000d27         0x12 build/XC16-EX16_MRF24WB/production/_ext/1954962658/SMTP.o
 .debug_pubtypes
                  0x000d39         0x12 build/XC16-EX16_MRF24WB/production/_ext/1954962658/SNMP.o
 .debug_pubtypes
                  0x000d4b         0x69 build/XC16-EX16_MRF24WB/production/_ext/1954962658/SNTP.o
 .debug_pubtypes
                  0x000db4         0xf8 build/XC16-EX16_MRF24WB/production/_ext/1954962658/SPIEEPROM.o
 .debug_pubtypes
                  0x000eac         0x12 build/XC16-EX16_MRF24WB/production/_ext/1954962658/SPIFlash.o
 .debug_pubtypes
                  0x000ebe         0x12 build/XC16-EX16_MRF24WB/production/_ext/1954962658/SPIRAM.o
 .debug_pubtypes
                  0x000ed0         0xbe build/XC16-EX16_MRF24WB/production/_ext/1954962658/StackTsk.o
 .debug_pubtypes
                  0x000f8e        0x14f build/XC16-EX16_MRF24WB/production/_ext/1954962658/TCP.o
 .debug_pubtypes
                  0x0010dd         0x12 build/XC16-EX16_MRF24WB/production/_ext/1954962658/TCPPerformanceTest.o
 .debug_pubtypes
                  0x0010ef         0x12 build/XC16-EX16_MRF24WB/production/_ext/1954962658/TFTPc.o
 .debug_pubtypes
                  0x001101         0x12 build/XC16-EX16_MRF24WB/production/_ext/1954962658/Telnet.o
 .debug_pubtypes
                  0x001113         0xb1 build/XC16-EX16_MRF24WB/production/_ext/1954962658/Tick.o
 .debug_pubtypes
                  0x0011c4         0x12 build/XC16-EX16_MRF24WB/production/_ext/1954962658/UART.o
 .debug_pubtypes
                  0x0011d6         0x12 build/XC16-EX16_MRF24WB/production/_ext/1954962658/UART2TCPBridge.o
 .debug_pubtypes
                  0x0011e8        0x116 build/XC16-EX16_MRF24WB/production/_ext/1954962658/UDP.o
 .debug_pubtypes
                  0x0012fe         0x12 build/XC16-EX16_MRF24WB/production/_ext/1954962658/UDPPerformanceTest.o
 .debug_pubtypes
                  0x001310         0x12 build/XC16-EX16_MRF24WB/production/_ext/1954962658/ZeroconfHelper.o
 .debug_pubtypes
                  0x001322         0x12 build/XC16-EX16_MRF24WB/production/_ext/1954962658/ZeroconfLinkLocal.o
 .debug_pubtypes
                  0x001334         0x12 build/XC16-EX16_MRF24WB/production/_ext/1954962658/ZeroconfMulticastDNS.o
 .debug_pubtypes
                  0x001346         0xb6 build/XC16-EX16_MRF24WB/production/_ext/243675038/WFConnectionAlgorithm.o
 .debug_pubtypes
                  0x0013fc         0x3a build/XC16-EX16_MRF24WB/production/_ext/243675038/WFConnectionManager.o
 .debug_pubtypes
                  0x001436         0xb4 build/XC16-EX16_MRF24WB/production/_ext/243675038/WFConnectionProfile.o
 .debug_pubtypes
                  0x0014ea         0x12 build/XC16-EX16_MRF24WB/production/_ext/243675038/WFConsole.o
 .debug_pubtypes
                  0x0014fc         0x12 build/XC16-EX16_MRF24WB/production/_ext/243675038/WFConsoleIfconfig.o
 .debug_pubtypes
                  0x00150e         0x12 build/XC16-EX16_MRF24WB/production/_ext/243675038/WFConsoleIwconfig.o
 .debug_pubtypes
                  0x001520         0x12 build/XC16-EX16_MRF24WB/production/_ext/243675038/WFConsoleIwpriv.o
 .debug_pubtypes
                  0x001532         0x43 build/XC16-EX16_MRF24WB/production/_ext/243675038/WFConsoleMsgHandler.o
 .debug_pubtypes
                  0x001575         0x68 build/XC16-EX16_MRF24WB/production/_ext/243675038/WFConsoleMsgs.o
 .debug_pubtypes
                  0x0015dd         0x12 build/XC16-EX16_MRF24WB/production/_ext/243675038/WFDataTxRx.o
 .debug_pubtypes
                  0x0015ef         0xb2 build/XC16-EX16_MRF24WB/production/_ext/243675038/WFDriverCom.o
 .debug_pubtypes
                  0x0016a1         0x57 build/XC16-EX16_MRF24WB/production/_ext/243675038/WFDriverRaw.o
 .debug_pubtypes
                  0x0016f8         0xff build/XC16-EX16_MRF24WB/production/_ext/243675038/WFEasyConfig.o
 .debug_pubtypes
                  0x0017f7         0x69 build/XC16-EX16_MRF24WB/production/_ext/243675038/WFEventHandler.o
 .debug_pubtypes
                  0x001860         0xc0 build/XC16-EX16_MRF24WB/production/_ext/243675038/WFInit.o
 .debug_pubtypes
                  0x001920         0xab build/XC16-EX16_MRF24WB/production/_ext/243675038/WFMac.o
 .debug_pubtypes
                  0x0019cb         0x6b build/XC16-EX16_MRF24WB/production/_ext/243675038/WFMgmtMsg.o
 .debug_pubtypes
                  0x001a36         0x94 build/XC16-EX16_MRF24WB/production/_ext/243675038/WFParamMsg.o
 .debug_pubtypes
                  0x001aca         0x12 build/XC16-EX16_MRF24WB/production/_ext/243675038/WFPowerSave.o
 .debug_pubtypes
                  0x001adc         0x4c build/XC16-EX16_MRF24WB/production/_ext/243675038/WFScan.o
 .debug_pubtypes
                  0x001b28         0x42 build/XC16-EX16_MRF24WB/production/_ext/243675038/WFTxPower.o
 .debug_pubtypes
                  0x001b6a         0xc0 build/XC16-EX16_MRF24WB/production/_ext/243675038/WF_Eint.o
 .debug_pubtypes
                  0x001c2a         0xa5 build/XC16-EX16_MRF24WB/production/_ext/243675038/WF_Spi.o
 .debug_pubtypes
                  0x001ccf         0xa3 build/XC16-EX16_MRF24WB/production/_ext/243675038/WFDebugStrings.o
 .debug_pubtypes
                  0x001d72         0x68 build/XC16-EX16_MRF24WB/production/_ext/243675038/WF_pbkdf2.o
 .debug_pubtypes
                  0x001dda         0x12 build/XC16-EX16_MRF24WB/production/_ext/1472/UARTConfig.o
 .debug_pubtypes
                  0x001dec        0x159 build/XC16-EX16_MRF24WB/production/_ext/1472/WF_Config.o
 .debug_pubtypes
                  0x001f45         0xe8 build/XC16-EX16_MRF24WB/production/_ext/1472/HTTP2.o
 .debug_pubtypes
                  0x00202d         0xd2 build/XC16-EX16_MRF24WB/production/_ext/1472/MPFS2.o
 .debug_pubtypes
                  0x0020ff        0x3a4 build/XC16-EX16_MRF24WB/production/_ext/1472/WiSteerHTTP.o
 .debug_pubtypes
                  0x0024a3        0x3d5 build/XC16-EX16_MRF24WB/production/_ext/1472/WiSteerMain.o
 .debug_pubtypes
                  0x002878         0xe8 build/XC16-EX16_MRF24WB/production/_ext/1472/WiSteerHTTPtools.o
 .debug_pubtypes
                  0x002960         0x12 build/XC16-EX16_MRF24WB/production/_ext/1472/WiSteerUpdate.o
 .debug_pubtypes
                  0x002972        0x16a build/XC16-EX16_MRF24WB/production/_ext/1472/WiSteerLog.o
 .debug_pubtypes
                  0x002adc        0x162 build/XC16-EX16_MRF24WB/production/_ext/1472/WiSteerTime.o
 .debug_pubtypes
                  0x002c3e        0x357 build/XC16-EX16_MRF24WB/production/_ext/1472/WiSteerCom.o
 .debug_pubtypes
                  0x002f95        0x1c4 build/XC16-EX16_MRF24WB/production/_ext/1472/WiSteerAction.o
 .debug_pubtypes
                  0x003159         0x12 build/XC16-EX16_MRF24WB/production/_ext/1472/WiSteerStructSizeCheck.o

__c30_signature
                  0x00316c        0x378
 __c30_signature
                  0x00316c          0x6 build/XC16-EX16_MRF24WB/production/_ext/1954962658/ARP.o
 __c30_signature
                  0x003172          0x6 build/XC16-EX16_MRF24WB/production/_ext/1954962658/Announce.o
 __c30_signature
                  0x003178          0x6 build/XC16-EX16_MRF24WB/production/_ext/1954962658/AutoIP.o
 __c30_signature
                  0x00317e          0x6 build/XC16-EX16_MRF24WB/production/_ext/1954962658/BerkeleyAPI.o
 __c30_signature
                  0x003184          0x6 build/XC16-EX16_MRF24WB/production/_ext/1954962658/DHCP.o
 __c30_signature
                  0x00318a          0x6 build/XC16-EX16_MRF24WB/production/_ext/1954962658/DHCPs.o
 __c30_signature
                  0x003190          0x6 build/XC16-EX16_MRF24WB/production/_ext/1954962658/DNS.o
 __c30_signature
                  0x003196          0x6 build/XC16-EX16_MRF24WB/production/_ext/1954962658/DNSs.o
 __c30_signature
                  0x00319c          0x6 build/XC16-EX16_MRF24WB/production/_ext/1954962658/Delay.o
 __c30_signature
                  0x0031a2          0x6 build/XC16-EX16_MRF24WB/production/_ext/1954962658/DynDNS.o
 __c30_signature
                  0x0031a8          0x6 build/XC16-EX16_MRF24WB/production/_ext/1954962658/ENC28J60.o
 __c30_signature
                  0x0031ae          0x6 build/XC16-EX16_MRF24WB/production/_ext/1954962658/ENCX24J600.o
 __c30_signature
                  0x0031b4          0x6 build/XC16-EX16_MRF24WB/production/_ext/1954962658/FTP.o
 __c30_signature
                  0x0031ba          0x6 build/XC16-EX16_MRF24WB/production/_ext/1954962658/Hashes.o
 __c30_signature
                  0x0031c0          0x6 build/XC16-EX16_MRF24WB/production/_ext/1954962658/Helpers.o
 __c30_signature
                  0x0031c6          0x6 build/XC16-EX16_MRF24WB/production/_ext/1954962658/ICMP.o
 __c30_signature
                  0x0031cc          0x6 build/XC16-EX16_MRF24WB/production/_ext/1954962658/IP.o
 __c30_signature
                  0x0031d2          0x6 build/XC16-EX16_MRF24WB/production/_ext/1954962658/LCDBlocking.o
 __c30_signature
                  0x0031d8          0x6 build/XC16-EX16_MRF24WB/production/_ext/1954962658/NBNS.o
 __c30_signature
                  0x0031de          0x6 build/XC16-EX16_MRF24WB/production/_ext/1954962658/Reboot.o
 __c30_signature
                  0x0031e4          0x6 build/XC16-EX16_MRF24WB/production/_ext/1954962658/SMTP.o
 __c30_signature
                  0x0031ea          0x6 build/XC16-EX16_MRF24WB/production/_ext/1954962658/SNMP.o
 __c30_signature
                  0x0031f0          0x6 build/XC16-EX16_MRF24WB/production/_ext/1954962658/SNTP.o
 __c30_signature
                  0x0031f6          0x6 build/XC16-EX16_MRF24WB/production/_ext/1954962658/SPIEEPROM.o
 __c30_signature
                  0x0031fc          0x6 build/XC16-EX16_MRF24WB/production/_ext/1954962658/SPIFlash.o
 __c30_signature
                  0x003202          0x6 build/XC16-EX16_MRF24WB/production/_ext/1954962658/SPIRAM.o
 __c30_signature
                  0x003208          0x6 build/XC16-EX16_MRF24WB/production/_ext/1954962658/StackTsk.o
 __c30_signature
                  0x00320e          0x6 build/XC16-EX16_MRF24WB/production/_ext/1954962658/TCP.o
 __c30_signature
                  0x003214          0x6 build/XC16-EX16_MRF24WB/production/_ext/1954962658/TCPPerformanceTest.o
 __c30_signature
                  0x00321a          0x6 build/XC16-EX16_MRF24WB/production/_ext/1954962658/TFTPc.o
 __c30_signature
                  0x003220          0x6 build/XC16-EX16_MRF24WB/production/_ext/1954962658/Telnet.o
 __c30_signature
                  0x003226          0x6 build/XC16-EX16_MRF24WB/production/_ext/1954962658/Tick.o
 __c30_signature
                  0x00322c          0x6 build/XC16-EX16_MRF24WB/production/_ext/1954962658/UART.o
 __c30_signature
                  0x003232          0x6 build/XC16-EX16_MRF24WB/production/_ext/1954962658/UART2TCPBridge.o
 __c30_signature
                  0x003238          0x6 build/XC16-EX16_MRF24WB/production/_ext/1954962658/UDP.o
 __c30_signature
                  0x00323e          0x6 build/XC16-EX16_MRF24WB/production/_ext/1954962658/UDPPerformanceTest.o
 __c30_signature
                  0x003244          0x6 build/XC16-EX16_MRF24WB/production/_ext/1954962658/ZeroconfHelper.o
 __c30_signature
                  0x00324a          0x6 build/XC16-EX16_MRF24WB/production/_ext/1954962658/ZeroconfLinkLocal.o
 __c30_signature
                  0x003250          0x6 build/XC16-EX16_MRF24WB/production/_ext/1954962658/ZeroconfMulticastDNS.o
 __c30_signature
                  0x003256          0x6 build/XC16-EX16_MRF24WB/production/_ext/243675038/WFConnectionAlgorithm.o
 __c30_signature
                  0x00325c          0x6 build/XC16-EX16_MRF24WB/production/_ext/243675038/WFConnectionManager.o
 __c30_signature
                  0x003262          0x6 build/XC16-EX16_MRF24WB/production/_ext/243675038/WFConnectionProfile.o
 __c30_signature
                  0x003268          0x6 build/XC16-EX16_MRF24WB/production/_ext/243675038/WFConsole.o
 __c30_signature
                  0x00326e          0x6 build/XC16-EX16_MRF24WB/production/_ext/243675038/WFConsoleIfconfig.o
 __c30_signature
                  0x003274          0x6 build/XC16-EX16_MRF24WB/production/_ext/243675038/WFConsoleIwconfig.o
 __c30_signature
                  0x00327a          0x6 build/XC16-EX16_MRF24WB/production/_ext/243675038/WFConsoleIwpriv.o
 __c30_signature
                  0x003280          0x6 build/XC16-EX16_MRF24WB/production/_ext/243675038/WFConsoleMsgHandler.o
 __c30_signature
                  0x003286          0x6 build/XC16-EX16_MRF24WB/production/_ext/243675038/WFConsoleMsgs.o
 __c30_signature
                  0x00328c          0x6 build/XC16-EX16_MRF24WB/production/_ext/243675038/WFDataTxRx.o
 __c30_signature
                  0x003292          0x6 build/XC16-EX16_MRF24WB/production/_ext/243675038/WFDriverCom.o
 __c30_signature
                  0x003298          0x6 build/XC16-EX16_MRF24WB/production/_ext/243675038/WFDriverRaw.o
 __c30_signature
                  0x00329e          0x6 build/XC16-EX16_MRF24WB/production/_ext/243675038/WFEasyConfig.o
 __c30_signature
                  0x0032a4          0x6 build/XC16-EX16_MRF24WB/production/_ext/243675038/WFEventHandler.o
 __c30_signature
                  0x0032aa          0x6 build/XC16-EX16_MRF24WB/production/_ext/243675038/WFInit.o
 __c30_signature
                  0x0032b0          0x6 build/XC16-EX16_MRF24WB/production/_ext/243675038/WFMac.o
 __c30_signature
                  0x0032b6          0x6 build/XC16-EX16_MRF24WB/production/_ext/243675038/WFMgmtMsg.o
 __c30_signature
                  0x0032bc          0x6 build/XC16-EX16_MRF24WB/production/_ext/243675038/WFParamMsg.o
 __c30_signature
                  0x0032c2          0x6 build/XC16-EX16_MRF24WB/production/_ext/243675038/WFPowerSave.o
 __c30_signature
                  0x0032c8          0x6 build/XC16-EX16_MRF24WB/production/_ext/243675038/WFScan.o
 __c30_signature
                  0x0032ce          0x6 build/XC16-EX16_MRF24WB/production/_ext/243675038/WFTxPower.o
 __c30_signature
                  0x0032d4          0x6 build/XC16-EX16_MRF24WB/production/_ext/243675038/WF_Eint.o
 __c30_signature
                  0x0032da          0x6 build/XC16-EX16_MRF24WB/production/_ext/243675038/WF_Spi.o
 __c30_signature
                  0x0032e0          0x6 build/XC16-EX16_MRF24WB/production/_ext/243675038/WFDebugStrings.o
 __c30_signature
                  0x0032e6          0x6 build/XC16-EX16_MRF24WB/production/_ext/243675038/WF_pbkdf2.o
 __c30_signature
                  0x0032ec          0x6 build/XC16-EX16_MRF24WB/production/_ext/1472/UARTConfig.o
 __c30_signature
                  0x0032f2          0x6 build/XC16-EX16_MRF24WB/production/_ext/1472/WF_Config.o
 __c30_signature
                  0x0032f8          0x6 build/XC16-EX16_MRF24WB/production/_ext/1472/HTTP2.o
 __c30_signature
                  0x0032fe          0x6 build/XC16-EX16_MRF24WB/production/_ext/1472/MPFS2.o
 __c30_signature
                  0x003304          0x6 build/XC16-EX16_MRF24WB/production/_ext/1472/WiSteerHTTP.o
 __c30_signature
                  0x00330a          0x6 build/XC16-EX16_MRF24WB/production/_ext/1472/WiSteerMain.o
 __c30_signature
                  0x003310          0x6 build/XC16-EX16_MRF24WB/production/_ext/1472/WiSteerHTTPtools.o
 __c30_signature
                  0x003316          0x6 build/XC16-EX16_MRF24WB/production/_ext/1472/WiSteerUpdate.o
 __c30_signature
                  0x00331c          0x6 build/XC16-EX16_MRF24WB/production/_ext/1472/WiSteerLog.o
 __c30_signature
                  0x003322          0x6 build/XC16-EX16_MRF24WB/production/_ext/1472/WiSteerTime.o
 __c30_signature
                  0x003328          0x6 build/XC16-EX16_MRF24WB/production/_ext/1472/WiSteerCom.o
 __c30_signature
                  0x00332e          0x6 build/XC16-EX16_MRF24WB/production/_ext/1472/WiSteerAction.o
 __c30_signature
                  0x003334          0x6 build/XC16-EX16_MRF24WB/production/_ext/1472/WiSteerStructSizeCheck.o
 __c30_signature
                  0x00333a          0x6 build/XC16-EX16_MRF24WB/production/_ext/1472/pic32helpers.o
 __c30_signature
                  0x003340          0x6 c:/program files (x86)/microchip/xc16/v1.20/bin/bin/../../lib\libpic30-elf.a(crt0_extendedep.o)
 __c30_signature
                  0x003346          0x6 c:/program files (x86)/microchip/xc16/v1.20/bin/bin/../../lib\libpic30-elf.a(data_init_extendedep.o)
 __c30_signature
                  0x00334c          0x6 c:/program files (x86)/microchip/xc16/v1.20/bin/bin/../../lib\libm-elf.a(divsi3.epeo)
 __c30_signature
                  0x003352          0x6 c:/program files (x86)/microchip/xc16/v1.20/bin/bin/../../lib\libm-elf.a(modsi3.epeo)
 __c30_signature
                  0x003358          0x6 c:/program files (x86)/microchip/xc16/v1.20/bin/bin/../../lib\libm-elf.a(udivsi3.epeo)
 __c30_signature
                  0x00335e          0x6 c:/program files (x86)/microchip/xc16/v1.20/bin/bin/../../lib\libm-elf.a(umodsi3.epeo)
 __c30_signature
                  0x003364          0x6 c:/program files (x86)/microchip/xc16/v1.20/bin/bin/../../lib\libm-elf.a(divmoddi3.epeo)
 __c30_signature
                  0x00336a          0x6 c:/program files (x86)/microchip/xc16/v1.20/bin/bin/../../lib\libm-elf.a(muldi3.epeo)
 __c30_signature
                  0x003370          0x6 c:/program files (x86)/microchip/xc16/v1.20/bin/bin/../../lib\libm-elf.a(umuldi3.epeo)
 __c30_signature
                  0x003376          0x6 c:/program files (x86)/microchip/xc16/v1.20/bin/bin/../../lib\libc-elf.a(atof.epeo)
 __c30_signature
                  0x00337c          0x6 c:/program files (x86)/microchip/xc16/v1.20/bin/bin/../../lib\libc-elf.a(atoi.epeo)
 __c30_signature
                  0x003382          0x6 c:/program files (x86)/microchip/xc16/v1.20/bin/bin/../../lib\libc-elf.a(atol.epeo)
 __c30_signature
                  0x003388          0x6 c:/program files (x86)/microchip/xc16/v1.20/bin/bin/../../lib\libc-elf.a(errno.epeo)
 __c30_signature
                  0x00338e          0x6 c:/program files (x86)/microchip/xc16/v1.20/bin/bin/../../lib\libc-elf.a(ltoa.epeo)
 __c30_signature
                  0x003394          0x6 c:/program files (x86)/microchip/xc16/v1.20/bin/bin/../../lib\libc-elf.a(memcmp.epeo)
 __c30_signature
                  0x00339a          0x6 c:/program files (x86)/microchip/xc16/v1.20/bin/bin/../../lib\libc-elf.a(memcpy.epeo)
 __c30_signature
                  0x0033a0          0x6 c:/program files (x86)/microchip/xc16/v1.20/bin/bin/../../lib\libc-elf.a(memmove.epeo)
 __c30_signature
                  0x0033a6          0x6 c:/program files (x86)/microchip/xc16/v1.20/bin/bin/../../lib\libc-elf.a(memset.epeo)
 __c30_signature
                  0x0033ac          0x6 c:/program files (x86)/microchip/xc16/v1.20/bin/bin/../../lib\libc-elf.a(strchr.epeo)
 __c30_signature
                  0x0033b2          0x6 c:/program files (x86)/microchip/xc16/v1.20/bin/bin/../../lib\libc-elf.a(strcmp.epeo)
 __c30_signature
                  0x0033b8          0x6 c:/program files (x86)/microchip/xc16/v1.20/bin/bin/../../lib\libc-elf.a(strcpy.epeo)
 __c30_signature
                  0x0033be          0x6 c:/program files (x86)/microchip/xc16/v1.20/bin/bin/../../lib\libc-elf.a(strlen.epeo)
 __c30_signature
                  0x0033c4          0x6 c:/program files (x86)/microchip/xc16/v1.20/bin/bin/../../lib\libc-elf.a(strncmp.epeo)
 __c30_signature
                  0x0033ca          0x6 c:/program files (x86)/microchip/xc16/v1.20/bin/bin/../../lib\libc-elf.a(strncpy.epeo)
 __c30_signature
                  0x0033d0          0x6 c:/program files (x86)/microchip/xc16/v1.20/bin/bin/../../lib\libc-elf.a(strtol.epeo)
 __c30_signature
                  0x0033d6          0x6 c:/program files (x86)/microchip/xc16/v1.20/bin/bin/../../lib\libc-elf.a(vsnprintf.epeo)
 __c30_signature
                  0x0033dc          0x6 c:/program files (x86)/microchip/xc16/v1.20/bin/bin/../../lib\libc-elf.a(snprintf_cdfFnopsuxX.EPeo)
 __c30_signature
                  0x0033e2          0x6 c:/program files (x86)/microchip/xc16/v1.20/bin/bin/../../lib\libc-elf.a(vsnprintf_cdfFnopsuxX.EPeo)
 __c30_signature
                  0x0033e8          0x6 c:/program files (x86)/microchip/xc16/v1.20/bin/bin/../../lib\libc-elf.a(doprnt.epeo)
 __c30_signature
                  0x0033ee          0x6 c:/program files (x86)/microchip/xc16/v1.20/bin/bin/../../lib\libc-elf.a(fputc.epeo)
 __c30_signature
                  0x0033f4          0x6 c:/program files (x86)/microchip/xc16/v1.20/bin/bin/../../lib\libc-elf.a(powers.epeo)
 __c30_signature
                  0x0033fa          0x6 c:/program files (x86)/microchip/xc16/v1.20/bin/bin/../../lib\libc-elf.a(_iob.epeo)
 __c30_signature
                  0x003400          0x6 c:/program files (x86)/microchip/xc16/v1.20/bin/bin/../../lib\libc-elf.a(doprnt_cdfFnopsuxX.EPeo)
 __c30_signature
                  0x003406          0x6 c:/program files (x86)/microchip/xc16/v1.20/bin/bin/../../lib\libc-elf.a(flsbuf.epeo)
 __c30_signature
                  0x00340c          0x6 c:/program files (x86)/microchip/xc16/v1.20/bin/bin/../../lib\libpic30-elf.a(writeep.eo)
 __c30_signature
                  0x003412          0x6 c:/program files (x86)/microchip/xc16/v1.20/bin/bin/../../lib\libpic30-elf.a(c30_uartep.eo)
 __c30_signature
                  0x003418          0x6 c:/program files (x86)/microchip/xc16/v1.20/bin/bin/../../lib\libm-elf.a(adddf3.epeo)
 __c30_signature
                  0x00341e          0x6 c:/program files (x86)/microchip/xc16/v1.20/bin/bin/../../lib\libm-elf.a(deqltle.epeo)
 __c30_signature
                  0x003424          0x6 c:/program files (x86)/microchip/xc16/v1.20/bin/bin/../../lib\libm-elf.a(dgtge.epeo)
 __c30_signature
                  0x00342a          0x6 c:/program files (x86)/microchip/xc16/v1.20/bin/bin/../../lib\libm-elf.a(divdf3.epeo)
 __c30_signature
                  0x003430          0x6 c:/program files (x86)/microchip/xc16/v1.20/bin/bin/../../lib\libm-elf.a(divsf3.epeo)
 __c30_signature
                  0x003436          0x6 c:/program files (x86)/microchip/xc16/v1.20/bin/bin/../../lib\libm-elf.a(dne.epeo)
 __c30_signature
                  0x00343c          0x6 c:/program files (x86)/microchip/xc16/v1.20/bin/bin/../../lib\libm-elf.a(dpack.epeo)
 __c30_signature
                  0x003442          0x6 c:/program files (x86)/microchip/xc16/v1.20/bin/bin/../../lib\libm-elf.a(dunpack2.epeo)
 __c30_signature
                  0x003448          0x6 c:/program files (x86)/microchip/xc16/v1.20/bin/bin/../../lib\libm-elf.a(extendsfdf.epeo)
 __c30_signature
                  0x00344e          0x6 c:/program files (x86)/microchip/xc16/v1.20/bin/bin/../../lib\libm-elf.a(feqltle.epeo)
 __c30_signature
                  0x003454          0x6 c:/program files (x86)/microchip/xc16/v1.20/bin/bin/../../lib\libm-elf.a(fgtge.epeo)
 __c30_signature
                  0x00345a          0x6 c:/program files (x86)/microchip/xc16/v1.20/bin/bin/../../lib\libm-elf.a(fixunsdfdi.epeo)
 __c30_signature
                  0x003460          0x6 c:/program files (x86)/microchip/xc16/v1.20/bin/bin/../../lib\libm-elf.a(fixunsdfsi.epeo)
 __c30_signature
                  0x003466          0x6 c:/program files (x86)/microchip/xc16/v1.20/bin/bin/../../lib\libm-elf.a(floatsisf.epeo)
 __c30_signature
                  0x00346c          0x6 c:/program files (x86)/microchip/xc16/v1.20/bin/bin/../../lib\libm-elf.a(floatundidf.epeo)
 __c30_signature
                  0x003472          0x6 c:/program files (x86)/microchip/xc16/v1.20/bin/bin/../../lib\libm-elf.a(floatunsidf.epeo)
 __c30_signature
                  0x003478          0x6 c:/program files (x86)/microchip/xc16/v1.20/bin/bin/../../lib\libm-elf.a(fpack.epeo)
 __c30_signature
                  0x00347e          0x6 c:/program files (x86)/microchip/xc16/v1.20/bin/bin/../../lib\libm-elf.a(frexpf.epeo)
 __c30_signature
                  0x003484          0x6 c:/program files (x86)/microchip/xc16/v1.20/bin/bin/../../lib\libm-elf.a(funpack.epeo)
 __c30_signature
                  0x00348a          0x6 c:/program files (x86)/microchip/xc16/v1.20/bin/bin/../../lib\libm-elf.a(funpack2.epeo)
 __c30_signature
                  0x003490          0x6 c:/program files (x86)/microchip/xc16/v1.20/bin/bin/../../lib\libm-elf.a(futil.epeo)
 __c30_signature
                  0x003496          0x6 c:/program files (x86)/microchip/xc16/v1.20/bin/bin/../../lib\libm-elf.a(muldf3.epeo)
 __c30_signature
                  0x00349c          0x6 c:/program files (x86)/microchip/xc16/v1.20/bin/bin/../../lib\libm-elf.a(mulsf3.epeo)
 __c30_signature
                  0x0034a2          0x6 c:/program files (x86)/microchip/xc16/v1.20/bin/bin/../../lib\libm-elf.a(subdf3.epeo)
 __c30_signature
                  0x0034a8          0x6 c:/program files (x86)/microchip/xc16/v1.20/bin/bin/../../lib\libm-elf.a(truncdfsf.epeo)
 __c30_signature
                  0x0034ae          0x6 c:/program files (x86)/microchip/xc16/v1.20/bin/bin/../../lib\libm-elf.a(mulsi3.epeo)
 __c30_signature
                  0x0034b4          0x6 c:/program files (x86)/microchip/xc16/v1.20/bin/bin/../../lib\libm-elf.a(_frexpf.epeo)
 __c30_signature
                  0x0034ba          0x6 c:/program files (x86)/microchip/xc16/v1.20/bin/bin/../../lib\libm-elf.a(dcompare.epeo)
 __c30_signature
                  0x0034c0          0x6 c:/program files (x86)/microchip/xc16/v1.20/bin/bin/../../lib\libm-elf.a(dpropagateNaN.epeo)
 __c30_signature
                  0x0034c6          0x6 c:/program files (x86)/microchip/xc16/v1.20/bin/bin/../../lib\libm-elf.a(dtype.epeo)
 __c30_signature
                  0x0034cc          0x6 c:/program files (x86)/microchip/xc16/v1.20/bin/bin/../../lib\libm-elf.a(dunpack.epeo)
 __c30_signature
                  0x0034d2          0x6 c:/program files (x86)/microchip/xc16/v1.20/bin/bin/../../lib\libm-elf.a(fcompare.epeo)
 __c30_signature
                  0x0034d8          0x6 c:/program files (x86)/microchip/xc16/v1.20/bin/bin/../../lib\libm-elf.a(floatdisf.epeo)
 __c30_signature
                  0x0034de          0x6 c:/program files (x86)/microchip/xc16/v1.20/bin/bin/../../lib\libm-elf.a(floatundisf.epeo)

.bss                0x1000       0x4c78
 .bss               0x1000       0x28fa build/XC16-EX16_MRF24WB/production/_ext/1472/WiSteerMain.o
                    0x1000                  _AppConfig
                    0x10aa                  _WiSteerCfg
                    0x1ff8                  _WiSteerLog
                    0x2ff8                  _WiSteerCfgTmp
                    0x38f4                  _ConnectionProfileID
 .bss               0x38fa       0x1484 build/XC16-EX16_MRF24WB/production/_ext/1472/HTTP2.o
                    0x38fa                  _HTTPControlBlocks
                    0x496a                  _httpStubs
                    0x497a                  _curHTTPID
 .bss               0x4d7e        0x762 build/XC16-EX16_MRF24WB/production/_ext/243675038/WFEasyConfig.o
                    0x4d7e                  _g_ScanCtx
                    0x4d84                  _g_easyConfigCtx
                    0x4e14                  _preScanResult
 .bss               0x54e0        0x5a0 build/XC16-EX16_MRF24WB/production/_ext/1472/WiSteerHTTP.o
                    0x54e4                  _logStubs
                    0x5968                  _httpPageId
                    0x59a8                  _httpTimeScan
                    0x59d8                  _httpCatEnum
                    0x59dc                  _httpCatMainEnum
                    0x59f4                  _httpCfgCatEnum
                    0x59fc                  _httpIOpinEnum
                    0x5a00                  _httpCmdOutEnum
                    0x5a04                  _httpCfgCmdEnum
                    0x5a34                  _httpCfgIOenum
                    0x5a3c                  _httpCfgFormId
                    0x5a6c                  _httpActEnum
                    0x5a70                  _httpDevEnum
                    0x5a74                  _httpBtnEnum
 .bss               0x5a80        0x1f8 build/XC16-EX16_MRF24WB/production/_ext/1472/WiSteerAction.o
                    0x5a80                  _g_tiIO
                    0x5ab0                  _g_tiIOmax
                    0x5ae0                  _g_tiIOoff
                    0x5b10                  _g_tiIOoffMax
                    0x5b40                  _g_inputState
                    0x5c30                  _g_catReqCtx
                    0x5c38                  _bufAskerLabel

.data._powers_      0x5c78        0x160
 .data._powers_
                    0x5c78        0x160 c:/program files (x86)/microchip/xc16/v1.20/bin/bin/../../lib\libc-elf.a(powers.epeo)
                    0x5c78                  __powers_
                    0x5d28                  __npowers_

.bss                0x5dd8        0x31a
 .bss               0x5dd8        0x12c build/XC16-EX16_MRF24WB/production/_ext/1954962658/UDP.o
                    0x5dd8                  _UDPSocketInfo
                    0x5ef8                  _activeUDPSocket
                    0x5efa                  _UDPTxCount
                    0x5efc                  _UDPRxCount
 .bss               0x5f04        0x106 build/XC16-EX16_MRF24WB/production/_ext/1954962658/TCP.o
 .bss               0x600a         0xe8 build/XC16-EX16_MRF24WB/production/_ext/1472/WiSteerCom.o
                    0x600a                  _wsLastHostRecv
                    0x601e                  _g_discoveryMsg
                    0x60e2                  _wiSteerAuthMd5

.data.dpowers       0x60f2        0x140
 .data.dpowers      0x60f2         0xa0 c:/program files (x86)/microchip/xc16/v1.20/bin/bin/../../lib\libc-elf.a(doprnt.epeo)
 .data.dpowers      0x6192         0xa0 c:/program files (x86)/microchip/xc16/v1.20/bin/bin/../../lib\libc-elf.a(doprnt_cdfFnopsuxX.EPeo)

.bss                0x6232        0x184
 .bss               0x6232         0x90 build/XC16-EX16_MRF24WB/production/_ext/1472/WiSteerTime.o
 .bss               0x62c2         0x8a build/XC16-EX16_MRF24WB/production/_ext/1472/MPFS2.o
 .bss               0x634c         0x6a build/XC16-EX16_MRF24WB/production/_ext/1954962658/DHCPs.o
                    0x634c                  _DhcpIpPool

.data               0x63b6         0x6a
 .data              0x63b6         0x6a build/XC16-EX16_MRF24WB/production/_ext/243675038/WFDebugStrings.o
                    0x63b6                  __connectionFailureStrings
                    0x63e0                  __connectionLostStrings
                    0x63ee                  __moduleName

.bss                0x6420         0xe0
 .bss               0x6420         0x42 build/XC16-EX16_MRF24WB/production/_ext/1954962658/DNSs.o
 .bss               0x6462         0x40 build/XC16-EX16_MRF24WB/production/_ext/1954962658/Hashes.o
                    0x6462                  _lastBlock
 .bss               0x64a2         0x32 build/XC16-EX16_MRF24WB/production/_ext/243675038/WFDebugStrings.o
 .bss               0x64d4         0x2c build/XC16-EX16_MRF24WB/production/_ext/1954962658/DHCP.o

.data               0x6500         0x54
 .data              0x6500         0x2a c:/program files (x86)/microchip/xc16/v1.20/bin/bin/../../lib\libc-elf.a(doprnt.epeo)
 .data              0x652a         0x2a c:/program files (x86)/microchip/xc16/v1.20/bin/bin/../../lib\libc-elf.a(doprnt_cdfFnopsuxX.EPeo)

.bss                0x6554         0x26
 .bss               0x6554         0x26 build/XC16-EX16_MRF24WB/production/_ext/1954962658/SPIEEPROM.o

.data._iob          0x657a         0x26
 .data._iob         0x657a         0x26 c:/program files (x86)/microchip/xc16/v1.20/bin/bin/../../lib\libc-elf.a(_iob.epeo)
                    0x657a                  __iob
                    0x659e                  __Files

.bss                0x65a0         0x22
 .bss               0x65a0         0x22 build/XC16-EX16_MRF24WB/production/_ext/1954962658/LCDBlocking.o
                    0x65a0                  _LCDText

.data               0x65c2         0x1c
 .data              0x65c2         0x1c build/XC16-EX16_MRF24WB/production/_ext/1472/WiSteerAction.o
                    0x65c2                  _g_actRunningRemoteOrPin
                    0x65c4                  _g_actRunningTick
                    0x65c8                  _g_actToSet
                    0x65cc                  _g_actToUnset
                    0x65d0                  _g_catReqTi
                    0x65d4                  _g_catReqTiMax
                    0x65d8                  _g_inputDefined
                    0x65da                  _g_outputAutoOff
                    0x65dc                  _g_inputToWatch

.bss                0x65de         0x56
 .bss               0x65de         0x18 build/XC16-EX16_MRF24WB/production/_ext/1954962658/DNS.o
 .bss               0x65f6         0x16 build/XC16-EX16_MRF24WB/production/_ext/1954962658/ARP.o
 .bss               0x660c         0x16 build/XC16-EX16_MRF24WB/production/_ext/243675038/WFMac.o
                    0x6620                  _g_rxIndexSetBeyondBuffer
 .bss               0x6622         0x12 build/XC16-EX16_MRF24WB/production/_ext/243675038/WFDriverCom.o
                    0x6630                  _RawMoveState

.data               0x6634         0x10
 .data              0x6634         0x10 build/XC16-EX16_MRF24WB/production/_ext/1472/WiSteerLog.o
                    0x6634                  _g_logStarted
                    0x6636                  _m_cLogAppend
                    0x6638                  _m_logStartId
                    0x663c                  _m_cLogChanged
                    0x6640                  _g_wslogCheckPt

.bss                0x6644         0x1c
 .bss               0x6644          0xe build/XC16-EX16_MRF24WB/production/_ext/1954962658/SNTP.o
 .bss               0x6652          0xe build/XC16-EX16_MRF24WB/production/_ext/1954962658/StackTsk.o
                    0x6654                  _remoteNode

.data               0x6660         0x2a
 .data              0x6660          0xe build/XC16-EX16_MRF24WB/production/_ext/1472/WiSteerMain.o
                    0x6660                  _g_wisteerBoostMode
                    0x6662                  _g_tiNow
                    0x6666                  _g_deviceWithOpIdx
                    0x6668                  _g_cfgShareSourceDevId
                    0x666a                  _g_cfgShareSourceDate
 .data              0x666e          0xc build/XC16-EX16_MRF24WB/production/_ext/1472/WiSteerCom.o
                    0x6672                  _g_wiSteerCom_opOrder
                    0x6674                  _g_wiSteerCom_opOrderLast
                    0x6676                  _g_wiSteerAuthMd5Ok
                    0x6678                  _g_wiSteerComReqToDo
 .data              0x667a          0x8 build/XC16-EX16_MRF24WB/production/_ext/243675038/WFDriverCom.o
                    0x667a                  _g_DhcpSuccessful
                    0x667c                  _g_WiFiConnectionChanged
                    0x667e                  _g_WiFiConnection
                    0x6680                  _g_dhcpInProgress
 .data              0x6682          0x8 build/XC16-EX16_MRF24WB/production/_ext/1472/WF_Config.o
                    0x6682                  _g_prescan_adhoc_done
                    0x6684                  _g_tickConnectError
                    0x6688                  _g_bWifiConnectOk

.bss                0x668a          0x8
 .bss               0x668a          0x8 build/XC16-EX16_MRF24WB/production/_ext/1472/WiSteerHTTPtools.o
                    0x668a                  _g_httpTooMuchData

.data               0x6692          0xc
 .data              0x6692          0x6 build/XC16-EX16_MRF24WB/production/_ext/1954962658/DHCPs.o
                    0x6694                  _bDHCPServerEnabled
 .data              0x6698          0x6 build/XC16-EX16_MRF24WB/production/_ext/1954962658/StackTsk.o
                    0x6698                  _g_DhcpRenew
                    0x669a                  _g_DhcpRetryTimer

_04F3B4805461348c
                    0x669e          0x6
 _04F3B4805461348c
                    0x669e          0x6 build/XC16-EX16_MRF24WB/production/_ext/1954962658/Tick.o
                    0x669e                  _vTickReading

.bss                0x66a4         0x12
 .bss               0x66a4          0x6 build/XC16-EX16_MRF24WB/production/_ext/243675038/WFDriverRaw.o
                    0x66a4                  _RawWindowReady
                    0x66a8                  _RawWindowState
 .bss               0x66aa          0x6 build/XC16-EX16_MRF24WB/production/_ext/243675038/WFMgmtMsg.o
 .bss               0x66b0          0x6 c:/program files (x86)/microchip/xc16/v1.20/bin/bin/../../lib\libc-elf.a(_iob.epeo)
                    0x66b0                  __outdone
                    0x66b1                  __sibuf
                    0x66b3                  __sobuf

.data               0x66b6          0x8
 .data              0x66b6          0x4 build/XC16-EX16_MRF24WB/production/_ext/1954962658/DNS.o
 .data              0x66ba          0x4 build/XC16-EX16_MRF24WB/production/_ext/1954962658/Helpers.o

.bss                0x66be          0x8
 .bss               0x66be          0x4 build/XC16-EX16_MRF24WB/production/_ext/1954962658/IP.o
 .bss               0x66c2          0x4 build/XC16-EX16_MRF24WB/production/_ext/1954962658/NBNS.o

.data               0x66c6          0xe
 .data              0x66c6          0x4 build/XC16-EX16_MRF24WB/production/_ext/1954962658/Tick.o
                    0x66c6                  _dwInternalTicks
 .data              0x66ca          0x4 build/XC16-EX16_MRF24WB/production/_ext/1472/MPFS2.o
                    0x66ca                  _mpfsLastSeek
 .data              0x66ce          0x4 build/XC16-EX16_MRF24WB/production/_ext/1472/WiSteerTime.o
                    0x66ce                  _g_timeOffset
 .data              0x66d2          0x2 build/XC16-EX16_MRF24WB/production/_ext/1954962658/DHCP.o
                    0x66d2                  _DHCPClientInitializedOnce

.pbss               0x66d4          0x2
 .pbss              0x66d4          0x2 build/XC16-EX16_MRF24WB/production/_ext/1954962658/DNS.o

.data               0x66d6          0x6
 .data              0x66d6          0x2 build/XC16-EX16_MRF24WB/production/_ext/1954962658/DNSs.o
 .data              0x66d8          0x2 build/XC16-EX16_MRF24WB/production/_ext/1954962658/SNTP.o
 .data              0x66da          0x2 build/XC16-EX16_MRF24WB/production/_ext/1954962658/TCP.o

.pbss               0x66dc          0x2
 .pbss              0x66dc          0x2 build/XC16-EX16_MRF24WB/production/_ext/1954962658/TCP.o

.data               0x66de          0x2
 .data              0x66de          0x2 build/XC16-EX16_MRF24WB/production/_ext/1954962658/UDP.o

.pbss               0x66e0          0x2
 .pbss              0x66e0          0x2 build/XC16-EX16_MRF24WB/production/_ext/1954962658/UDP.o

.data               0x66e2          0x2
 .data              0x66e2          0x2 build/XC16-EX16_MRF24WB/production/_ext/243675038/WFConnectionAlgorithm.o

.bss                0x66e4          0x2
 .bss               0x66e4          0x2 build/XC16-EX16_MRF24WB/production/_ext/243675038/WFConnectionManager.o

.data               0x66e6          0xa
 .data              0x66e6          0x2 build/XC16-EX16_MRF24WB/production/_ext/243675038/WFDriverRaw.o
                    0x66e6                  _g_HostRAWDataPacketReceived
 .data              0x66e8          0x2 build/XC16-EX16_MRF24WB/production/_ext/243675038/WFEasyConfig.o
                    0x66e8                  _preScanResult_Count
 .data              0x66ea          0x2 build/XC16-EX16_MRF24WB/production/_ext/243675038/WFInit.o
                    0x66ea                  _gRFModuleVer1209orLater
 .data              0x66ec          0x2 build/XC16-EX16_MRF24WB/production/_ext/243675038/WFMgmtMsg.o
                    0x66ec                  _g_WaitingForMgmtResponse
 .data              0x66ee          0x2 build/XC16-EX16_MRF24WB/production/_ext/1472/WiSteerHTTP.o

.bss                0x66f0          0x2
 .bss               0x66f0          0x2 c:/program files (x86)/microchip/xc16/v1.20/bin/bin/../../lib\libc-elf.a(errno.epeo)
                    0x66f0                  _errno

.data.__C30_UART
                    0x66f2          0x2
 .data.__C30_UART
                    0x66f2          0x2 c:/program files (x86)/microchip/xc16/v1.20/bin/bin/../../lib\libpic30-elf.a(c30_uartep.eo)
                    0x66f2                  ___C30_UART

.heap               0x66f4        0x3e8
 .heap              0x66f4        0x3e8 heap

.const              0xcdde       0x2a12 load address 0x004dde  
 .const             0xcdde        0xadc build/XC16-EX16_MRF24WB/production/_ext/1472/WiSteerCom.o
 .const             0xd8ba        0x89e build/XC16-EX16_MRF24WB/production/_ext/1472/WiSteerHTTP.o
                    0xd8ba                  _c_formInput_nochg
                    0xd8bb                  _c_formInput_post
                    0xe151                  _HTML_UP_ARROW
                    0xe154                  _HTML_DOWN_ARROW
 .const             0xe158        0x5be build/XC16-EX16_MRF24WB/production/_ext/1472/HTTP2.o
                    0xe2e2                  _http2m_ContentTypes
 .const             0xe716        0x414 build/XC16-EX16_MRF24WB/production/_ext/243675038/WFDebugStrings.o
 .const             0xeb2a        0x3b0 build/XC16-EX16_MRF24WB/production/_ext/1472/WiSteerMain.o
 .const             0xeeda        0x228 build/XC16-EX16_MRF24WB/production/_ext/1472/WiSteerTime.o
                    0xef14                  _wstime_weekDay
                    0xef78                  _wstime_month
 .const             0xf102        0x16e build/XC16-EX16_MRF24WB/production/_ext/1472/WiSteerAction.o
 .const             0xf270        0x140 build/XC16-EX16_MRF24WB/production/_ext/1954962658/Hashes.o
 .const             0xf3b0        0x112 build/XC16-EX16_MRF24WB/production/_ext/1472/WF_Config.o
 .const             0xf4c2         0xd0 build/XC16-EX16_MRF24WB/production/_ext/1954962658/DHCP.o
 .const             0xf592         0xb0 build/XC16-EX16_MRF24WB/production/_ext/1472/WiSteerHTTPtools.o
 .const             0xf642         0xaa build/XC16-EX16_MRF24WB/production/_ext/243675038/WFConsoleMsgs.o
                    0xf642                  _helpCmd
                    0xf647                  _helpHelp
                    0xf65a                  _getwfverCmd
                    0xf663                  _getwfverHelp
                    0xf67c                  _resetCmd
                    0xf682                  _resetHelp
                    0xf691                  _clsCmd
                    0xf695                  _clsHelp
                    0xf6a3                  _seeDocHelp
                    0xf6b5                  _pingCmd
                    0xf6ba                  _pingHelp
                    0xf6cc                  _g_consoleCmd
                    0xf6ea                  _g_numCmds
 .const             0xf6ec         0x4a build/XC16-EX16_MRF24WB/production/_ext/1472/WiSteerLog.o
 .const             0xf736         0x34 build/XC16-EX16_MRF24WB/production/_ext/243675038/WFEasyConfig.o
 .const             0xf76a         0x2a build/XC16-EX16_MRF24WB/production/_ext/1954962658/StackTsk.o
 .const             0xf794         0x26 build/XC16-EX16_MRF24WB/production/_ext/1472/MPFS2.o
 .const             0xf7ba         0x18 build/XC16-EX16_MRF24WB/production/_ext/1954962658/TCP.o
                    0xf7ba                  _TCPSocketInitializer
 .const             0xf7d2          0x8 build/XC16-EX16_MRF24WB/production/_ext/1954962658/DNSs.o
 .const             0xf7da          0x6 build/XC16-EX16_MRF24WB/production/_ext/243675038/WFInit.o
 .const             0xf7e0          0x4 build/XC16-EX16_MRF24WB/production/_ext/243675038/WFConsoleMsgHandler.o
 .const             0xf7e4          0x4 build/XC16-EX16_MRF24WB/production/_ext/243675038/WFDriverRaw.o
 .const             0xf7e8          0x4 build/XC16-EX16_MRF24WB/production/_ext/243675038/WF_pbkdf2.o
 .const             0xf7ec          0x4 build/XC16-EX16_MRF24WB/production/_ext/1472/WiSteerMpfsSource.o
                    0xf7ec                  _MPFS_Start

MPFSData          0x0077f0      0x1c98e
 MPFSData         0x0077f0      0x1c98e build/XC16-EX16_MRF24WB/production/_ext/1472/WiSteerMpfsSource.o
                  0x0077f4                  BEGIN_MPFS

.text             0x02417e      0x1e694
 .text            0x02417e       0x7a18 build/XC16-EX16_MRF24WB/production/_ext/1472/WiSteerHTTP.o
                  0x02417e                  _HTTPNeedsAuth
                  0x02420e                  _HTTPCheckAuth
                  0x024244                  _HTTPPrint_postWifiConfig
                  0x0245da                  _HTTPPrint_postTcpIpConfig
                  0x0249ac                  _HTTPPrint_builddate
                  0x0249b8                  _HTTPPrint_tcpipVersion
                  0x0249c4                  _HTTPPrint_version
                  0x0249fe                  _HTTPPrint_led
                  0x024aa2                  _HTTPPrint_ledSelected
                  0x024b54                  _HTTPPrint_temp
                  0x024bec                  _HTTPPrint_pot
                  0x024c64                  _HTTPPrint_zcross
                  0x024c6a                  _HTTPQueryIf_zcrossOk
                  0x024c74                  _HTTPQueryIf_zcrossNotOk
                  0x024c7e                  _HTTPPrint_time
                  0x024cb0                  _HTTPPrint_timeBoot
                  0x024ce0                  _HTTPPrintIP
                  0x024d46                  _HTTPPrint_host
                  0x024d64                  _HTTPPrint_config_hostname
                  0x024d82                  _HTTPPrint_config_netbiosname
                  0x024da0                  _HTTPPrint_config_dhcpchecked
                  0x024dca                  _HTTPPrint_config_ip
                  0x024df8                  _HTTPPrint_config_gw
                  0x024e26                  _HTTPPrint_config_subnet
                  0x024e54                  _HTTPPrint_config_dns1
                  0x024e82                  _HTTPPrint_config_dns2
                  0x024eb0                  _HTTPPrint_config_mac
                  0x024f84                  _HTTPPrint_reboot
                  0x024f9c                  _HTTPPrint_rebootaddr
                  0x024fca                  _HTTPPrint_status_ok
                  0x025010                  _HTTPPrint_status_fail
                  0x025056                  _HTTPPrint_fwver
                  0x0250a8                  _HTTPPrint_ssid
                  0x0250da                  _HTTPPrint_nextSSID
                  0x0250f8                  _HTTPPrint_prevSSID
                  0x025116                  _getWlanStr
                  0x02513e                  _HTTPPrint_prevWLAN
                  0x025168                  _HTTPPrint_nextWLAN
                  0x025192                  _HTTPPrint_label
                  0x0251b0                  _HTTPQueryIf_wifiConfigured
                  0x0251be                  _HTTPQueryIf_devConfigured
                  0x02521e                  _HTTPQueryIf_wifiAndDevConfigured
                  0x025236                  _HTTPQueryIf_wifiNotConfigured
                  0x02524c                  _HTTPQueryIf_devNotConfigured
                  0x025260                  _HTTPQueryIf_logToGet
                  0x02527c                  _HTTPQueryIf_actionToGet
                  0x025298                  _HTTPQueryIf_actionToReload
                  0x0252ca                  _HTTPQueryWhile_logEnum
                  0x0253f8                  _HTTPPrint_logID
                  0x02543a                  _HTTPPrint_logTime
                  0x02547a                  _HTTPPrint_logLevel
                  0x0254b8                  _HTTPPrint_logDetails
                  0x0254de                  _HTTPPrint_actionsPost
                  0x02553e                  _HTTPPrint_actionsPostLed
                  0x025690                  _HTTPPrint_actionsPostCmd
                  0x0257d2                  _HTTPPrint_actionsPostInfo
                  0x025876                  _HTTPPrint_wifiScanPost
                  0x0259ce                  _HTTPPrint_wifiScanInProgress
                  0x025a34                  _HTTPPrint_bssCount
                  0x025a70                  _HTTPPrint_bssValid
                  0x025a9a                  _HTTPPrint_bssName
                  0x025aca                  _HTTPPrint_bssPrivacy
                  0x025b10                  _HTTPPrint_bssWlan
                  0x025b46                  _HTTPPrint_bssStrength
                  0x025b7c                  _HTTPQueryIf_pageIdIs
                  0x025ba4                  _HTTPQueryIf_pageIdIsNot
                  0x025bcc                  _HTTPPrint_pageId
                  0x025c06                  _HTTPPrint_wifiPowerMax
                  0x025c46                  _HTTPPrint_wifiFactoryPowerMax
                  0x025c82                  _HTTPPrint_postWifiPowerMax
                  0x025cf4                  _HTTPPrint_timeScanStartLow
                  0x025e4c                  _HTTPPrint_timeScanStart
                  0x025eac                  _HTTPPrint_timeDay
                  0x025eea                  _HTTPPrint_timeMonth
                  0x025f28                  _HTTPPrint_timeYear
                  0x025f64                  _HTTPPrint_timeHour
                  0x025fa2                  _HTTPPrint_timeMin
                  0x025fe0                  _HTTPPrint_timeSec
                  0x02601e                  _HTTPPrint_timeZoneId
                  0x026070                  _HTTPPrint_timeBias
                  0x0260ac                  _HTTPQueryIf_cfg_timeDlON
                  0x0260ee                  _HTTPPrint_timeDltWeekDayNo
                  0x026136                  _HTTPPrint_timeDltWeekDay
                  0x02617e                  _HTTPPrint_timeDltMonth
                  0x0261c6                  _HTTPPrint_timeDltHour
                  0x02620e                  _HTTPPrint_timeDltMin
                  0x026256                  _HTTPPrint_timeDltSec
                  0x02629e                  _HTTPPrint_timeDltBias
                  0x0262da                  _HTTPPrint_timeSdtWeekDayNo
                  0x026322                  _HTTPPrint_timeSdtWeekDay
                  0x02636a                  _HTTPPrint_timeSdtMonth
                  0x0263b2                  _HTTPPrint_timeSdtHour
                  0x0263fa                  _HTTPPrint_timeSdtMin
                  0x026442                  _HTTPPrint_timeSdtSec
                  0x02648a                  _HTTPPrint_timeSdtBias
                  0x0264c6                  _HTTPQueryWhile_catEnum
                  0x02652a                  _HTTPPrint_catEnumId
                  0x026566                  _HTTPPrint_catEnumLabel
                  0x02658e                  _HTTPPrint_cfg_label
                  0x0265b4                  _HTTPQueryIf_cfg_debugON
                  0x026638                  _HTTPQueryIf_cfg_testON
                  0x0266bc                  _MPFStestMode
                  0x026710                  _HTTPQueryIf_testON
                  0x026764                  _HTTPQueryIf_cfg_haltfON
                  0x0267e8                  _HTTPQueryIf_cfg_activityLedON
                  0x02686c                  _HTTPQueryIf_cfg_protectAllON
                  0x0268f0                  _HTTPQueryIf_cfg_homeActivityPanelON
                  0x026974                  _HTTPQueryIf_homeActivityPanelON
                  0x0269c8                  _HTTPQueryIf_cfg_boostModeON
                  0x026a4c                  _HTTPQueryIf_boostModeON
                  0x026aa0                  _HTTPQueryIf_cfg_wisteerNetBrowseON
                  0x026b24                  _HTTPQueryIf_cfg_wisteerAutoUpdateON
                  0x026b2e                  _HTTPQueryIf_cfg_mpfsUploadON
                  0x026b38                  _HTTPPrint_cfg_login
                  0x026b5e                  _HTTPPrint_cfg_pwd1
                  0x026b64                  _HTTPPrint_cfg_pwd2
                  0x026b6a                  _HTTPQueryIf_category_available
                  0x026b7c                  _HTTPQueryIf_cfg_timeServerSyncON
                  0x026c00                  _HTTPPrint_cfg_timeServer
                  0x026c26                  _HTTPPrint_cfg_catCountVal
                  0x026c62                  _HTTPPrint_cfg_catCount
                  0x026c8e                  _HTTPPrint_cfg_catCountMax
                  0x026cb4                  _HTTPPrint_cfg_catMainCatId
                  0x026d44                  _HTTPQueryWhile_cfg_catMainEnum
                  0x026dee                  _HTTPPrint_cfg_catMainEnumId
                  0x026e2c                  _HTTPPrint_cfg_catMainEnumNo
                  0x026e6c                  _HTTPPrint_cfg_catMainEnumExc
                  0x026f28                  _HTTPQueryWhile_cfg_catEnum
                  0x026f72                  _HTTPPrint_cfg_catEnumId
                  0x026fb2                  _HTTPPrint_cfg_catEnumLabel
                  0x027012                  _HTTPQueryWhile_ioPinEnum
                  0x0270b4                  _HTTPPrint_ioPinEnumId
                  0x0270f0                  _HTTPPrint_ioPinEnumLabel
                  0x02711a                  _HTTPPrint_ioPinEnumType
                  0x027182                  _HTTPQueryWhile_cmdOutEnum
                  0x0271ec                  _HTTPPrint_cmdOutEnumId
                  0x027228                  _HTTPPrint_cmdOutEnumLabel
                  0x027250                  _HTTPPrint_cfg_cmdCfgCountVal
                  0x02728c                  _HTTPPrint_cfg_cmdCfgCount
                  0x0272b8                  _HTTPPrint_cfg_cmdCfgCountMax
                  0x0272de                  _HTTPQueryWhile_cfg_cmdCfgEnum
                  0x027336                  _HTTPPrint_cfg_cmdCfgEnumId
                  0x027376                  _HTTPPrint_cfg_cmdCfgEnumLabel
                  0x027412                  _HTTPPrint_cfg_cmdCfgEnumPrior
                  0x027504                  _HTTPPrint_cfg_cmdCfgEnumImg
                  0x0275d8                  _HTTPPrint_cfg_cmdCfgEnumPin1s
                  0x0276ac                  _HTTPPrint_cfg_cmdCfgEnumPin0s
                  0x027780                  _HTTPPrint_cfg_cmdCfgEnumPinRs
                  0x027854                  _HTTPPrint_cfg_cmdCfgEnumCatId
                  0x027918                  _HTTPQueryWhile_cfg_cmdCfgEnumCatEnum
                  0x0279e6                  _HTTPPrint_cfg_cmdCfgEnumCatEnumId
                  0x027a42                  _HTTPPrint_cfg_cmdCfgEnumCatEnumNo
                  0x027a82                  _HTTPPrint_cfg_cmdCfgEnumCatEnumExc
                  0x027b46                  _HTTPPrint_cfg_cmdCfgEnumTypeVal
                  0x027c0e                  _HTTPPrint_cfg_cmdCfgEnumType
                  0x027c62                  _HTTPQueryIf_cfg_cmdCfgEnumTypeIs
                  0x027c7e                  _HTTPPrint_cfg_cmdCfgEnumPin
                  0x027d52                  _HTTPPrint_cfg_cmdCfgEnumIOtypeVal
                  0x027e3e                  _HTTPPrint_cfg_cmdCfgEnumIOtype
                  0x027e92                  _HTTPQueryIf_cfg_cmdCfgEnumIOtypeIs
                  0x027eae                  _HTTPPrint_cfg_cmdCfgEnumRact
                  0x027fa0                  _HTTPPrint_cfg_cmdCfgEnumPulse
                  0x028092                  _HTTPPrint_cfg_cmdCfgEnumTimeNext
                  0x028178                  _HTTPPrint_cfg_cmdCfgEnumTimeOff
                  0x02825e                  _HTTPPrint_cfg_cmdCfgEnumAct
                  0x028350                  _HTTPPrint_cfg_cmdCfgEnumAskTypeVal
                  0x028412                  _HTTPPrint_cfg_cmdCfgEnumAskType
                  0x028466                  _HTTPPrint_cfg_ioCountVal
                  0x0284a2                  _HTTPPrint_cfg_ioCount
                  0x0284ce                  _HTTPPrint_cfg_ioCountMax
                  0x0284f4                  _HTTPQueryWhile_cfg_ioEnum
                  0x02853e                  _HTTPPrint_cfg_ioEnumId
                  0x02857e                  _HTTPPrint_cfg_ioEnumLabel
                  0x0285e0                  _HTTPPrint_cfg_ioEnumTypeVal
                  0x028662                  _HTTPPrint_cfg_ioEnumType
                  0x028696                  _HTTPPrint_postDevIOconfig
                  0x0287fa                  _HTTPPrint_formFocus
                  0x02881e                  _HTTPPrint_postDevIOconfig_configMain
                  0x02951a                  _HTTPPrint_postDevIOconfig_configTime
                  0x029966                  _HTTPPrint_postDevIOconfig_configCmds
                  0x02a2ba                  _HTTPPrint_postDevIOconfig_configIOs
                  0x02a54a                  _HTTPPrint_postDevIOconfig_configCats
                  0x02a6a0                  _HTTPQueryWhile_actionEnum
                  0x02a740                  _HTTPPrint_actionEnumId
                  0x02a77c                  _HTTPPrint_actionEnumUnicId
                  0x02a7ee                  _HTTPPrint_actionEnumLabel
                  0x02a818                  _HTTPPrint_actionEnumImg
                  0x02a864                  _HTTPQueryIf_actionEnumON
                  0x02a898                  _HTTPQueryIf_actionEnumONavail
                  0x02a8ce                  _HTTPQueryIf_actionEnumRunning
                  0x02a904                  _HTTPQueryIf_actionEnumError
                  0x02a938                  _HTTPPrint_actionEnumStatus
                  0x02a9d8                  _HTTPPrint_actionEnumPriority
                  0x02aa46                  _HTTPPrint_actionEnumCats
                  0x02ab8c                  _HTTPPrint_actionEnumAskType
                  0x02abd6                  _HTTPQueryIf_formConfigured
                  0x02ac86                  _HTTPQueryIf_formExpanded
                  0x02acd6                  _HTTPQueryWhile_deviceEnum
                  0x02ad18                  _HTTPPrint_deviceID
                  0x02ad40                  _HTTPPrint_deviceLabel
                  0x02ad66                  _HTTPPrint_deviceMac
                  0x02add0                  _HTTPPrint_deviceIP
                  0x02ae2a                  _HTTPPrint_deviceStatus
                  0x02b156                  _HTTPPrint_deviceTime
                  0x02b1ca                  _HTTPPrint_deviceSentTime
                  0x02b23e                  _HTTPPrint_deviceFWver
                  0x02b29c                  _HTTPPrint_deviceMpfsDate
                  0x02b2e6                  _HTTPPrint_deviceBootDate
                  0x02b330                  _HTTPQueryIf_deviceLinked
                  0x02b342                  _HTTPPrint_cfg_gpsLat
                  0x02b400                  _HTTPPrint_cfg_gpsLon
                  0x02b4be                  _HTTPPrint_cfg_gpsDist
                  0x02b57c                  _HTTPPrint_gpsLatitude
                  0x02b638                  _HTTPPrint_gpsLongitude
                  0x02b6f4                  _HTTPPrint_gpsDistanceMax
                  0x02b7b0                  _HTTPQueryIf_wisteerMpfsDynamic
                  0x02b7ba                  _HTTPQueryIf_wisteerMpfsUploadON
                  0x02b7c4                  _HTTPPrint_postDevIOconfig_configTools
                  0x02b848                  _HTTPPrint_mpfsdate
                  0x02b898                  _HTTPPrint_postDevLst
                  0x02b8a2                  _HTTPPrint_actionVer
                  0x02b8e6                  _HTTPPrint_categoryMax
                  0x02b91c                  _HTTPQueryIf_actionPending
                  0x02b936                  _HTTPPrint_btnResetStatus
                  0x02b966                  _HTTPQueryWhile_btnEnum
                  0x02b9da                  _HTTPPrint_btnEnumId
                  0x02ba18                  _HTTPPrint_btnEnumLabel
                  0x02ba46                  _HTTPPrint_btnEnumStatus
                  0x02baa2                  _HTTPPrint_cfg_ioEnumDimLevel
                  0x02baf6                  _HTTPQueryIf_cfg_ioEnumTypeIs
                  0x02bb10                  _HTTPPrint_cfg_ioEnumDimLevelVal
 .text            0x02bb96       0x4a5e build/XC16-EX16_MRF24WB/production/_ext/243675038/WF_pbkdf2.o
                  0x02bb96                  _hmac_sha1_vector
                  0x02bcbe                  _hmac_sha1
                  0x02bcde                  _sha1_prf
                  0x02bd82                  _sha1_t_prf
                  0x02bf28                  _pbkdf2_sha1
                  0x02bf88                  _sha1_vector
                  0x02bfd4                  _sha1_transform
 .text            0x0305f4       0x332e build/XC16-EX16_MRF24WB/production/_ext/1472/WiSteerCom.o
                  0x0305f4                  _WiSteerCom_AnnounceIP
                  0x03067a                  _WiSteerCom_AnnounceModeToOpCode
                  0x0306a0                  _WiSteerCom_AnnounceTask
                  0x030836                  _WiSteerCom_init
                  0x03088e                  _WiSteerCom_AnnounceSend
                  0x030a20                  _WiSteerCom_DiscoveryTask
                  0x030be2                  _WiSteerCom_DiscoveryRecv
                  0x030d4c                  _WiSteerCom_DiscoveryReply
                  0x030e6e                  _WiSteerCom_AuthMd5
                  0x030ecc                  _WiSteerCom_AuthMd5Reset
                  0x030ed6                  _WiSteerCom_AnnounceProcess
                  0x031236                  _WiSteerCom_DiscoverySendTask
                  0x031492                  _WiSteerCom_DiscoverySendTaskCat
                  0x03169c                  _WiSteerCom_DiscoverySendTaskCmd
                  0x0318a0                  _WiSteerCom_RetrieveInfoSend
                  0x03192e                  _WiSteerCom_RetrieveInfoError
                  0x031986                  _WiSteerCom_RetrieveCatProcess
                  0x031a5c                  _WiSteerCom_RetrieveCmdProcess
                  0x031b60                  _WiSteerCom_deviceSource
                  0x031bee                  _WiSteerCom_RetrieveCatInfoProcess
                  0x031d28                  _WiSteerCom_RetrieveCatErrorProcess
                  0x031e42                  _WiSteerCom_RetrieveCmdInfoProcess
                  0x031fe4                  _WiSteerCom_RetrieveCmdErrorProcess
                  0x0320fe                  _WiSteerCom_actionProcessCmdCfgOutputId
                  0x032442                  _WiSteerCom_DiscoverySendTaskCmdAction
                  0x032726                  _WiSteerCom_CmdActionProcess
                  0x032888                  _WiSteerCom_CmdActionErrorSend
                  0x0328e4                  _WiSteerCom_CmdActionInfoProcess
                  0x0329e4                  _WiSteerCom_CmdActionErrorProcess
                  0x032b1a                  _WiSteerCom_CmdActionChanged
                  0x032bac                  _WiSteerCom_DiscoverySendTaskCmdChanged
                  0x032e90                  _WiSteerCom_CmdStatusProcess
                  0x033056                  _WiSteerCom_CmdLog
                  0x03317c                  _WiSteerCom_CmdStatusInfoProcess
                  0x033274                  _cmdModeRemoteRecv
                  0x0332b0                  _WiSteerCom_CatActionAsk
                  0x0333c8                  _WiSteerCom_DiscoverySendTaskCatAction
                  0x0336be                  _WiSteerCom_CatActionProcess
                  0x0337d8                  _WiSteerCom_CatActionInfoProcess
 .text            0x033922       0x3240 build/XC16-EX16_MRF24WB/production/_ext/1472/HTTP2.o
                  0x033922                  _HTTPPrint
                  0x033e9c                  _HTTPQueryIf
                  0x034122                  _HTTPQueryWhile
                  0x0341ea                  _HTTPQueryContentType
                  0x0341f6                  _HTTPInit
                  0x034274                  _HTTPServer
                  0x035c80                  _HTTPMPFS2mSendData
                  0x03615a                  _HTTPURLDecode
                  0x03622e                  _HTTPargGet
                  0x0362ce                  _HTTPargTrimGet
                  0x0363b4                  _HTTPargSet
                  0x0365c0                  _HTTPReadPostName
                  0x0365ec                  _HTTPReadPostValue
                  0x0368ce                  _HTTPIncFile
                  0x036a3e                  _CRC32_Init
                  0x036ada                  _CRC32_Push
                  0x036b50                  _CRC32_Get
 .text            0x036b62       0x273a build/XC16-EX16_MRF24WB/production/_ext/1472/WiSteerAction.o
                  0x036b62                  _actionPendingClear
                  0x036b8a                  _ioPinMode
                  0x036bf6                  _ioPinInitLow
                  0x036c00                  _ioPinInit
                  0x036c2c                  _cmdCfgIsValid
                  0x036cc0                  _cmdCfgDisplayIsValid
                  0x036ce6                  _cmdCfgHiddenIsValid
                  0x036d0c                  _cmdCfgOutIsValid
                  0x036d66                  _cmdCfgCatIsValid
                  0x036db4                  _actionInit
                  0x036e00                  _actionInputInit
                  0x036f24                  _actionInputReset
                  0x036f38                  _actionInputWatchAdd
                  0x036fea                  _actionInputWatch
                  0x037078                  _actionInputChanged
                  0x03710e                  _actionInputSignal
                  0x037188                  _actionInputPulse
                  0x037248                  _actionInputPulseChoose
                  0x0373bc                  _actionInputPulseProcess
                  0x037498                  _actionInputSignalProcess
                  0x03776c                  _cmdSumCalc
                  0x0378fc                  _actionSumFromCmdId
                  0x0379d2                  _actionPostCmd
                  0x037ac4                  _actionRunningRemoteUpdate
                  0x037b54                  _actionRunningTick
                  0x037b76                  _actionStatus
                  0x037be0                  _actionProcessMask
                  0x037c88                  _actionProcess
                  0x037cbe                  _actionProcessCmdSumId
                  0x037d90                  _actTypeFromInputMode
                  0x037dde                  _actTypeFromLinkMode
                  0x037e2c                  _actionProcessCmdSum
                  0x037e66                  _actionProcessCmdCfgId
                  0x03800a                  _actionProcessCmdCfgOutputId
                  0x03864a                  _actionProcessCmdCfgOutputPin
                  0x038698                  _actionProcessCmdCfgOutputPinLow
                  0x03872c                  _actionProcessCmdCfgOutputPinStatus
                  0x03878a                  __actionProcessCmdOrCatId
                  0x03880e                  _actionProcessCmdOrCatId
                  0x0388fe                  _actionAskerGet
                  0x038976                  _actionAskerFree
                  0x038a0c                  _actionAskerError
                  0x038a54                  _actionAskerLabel
                  0x038a9e                  _actionLocalInit
                  0x038aba                  _actionProcessCatId
                  0x038dc6                  _catInCatList
                  0x038df8                  _actionCatFilter
                  0x038e3c                  _actionProcessCatCom
                  0x038ede                  _actionProcessCmdCfgInputPinStatus
                  0x038f34                  _actionAutoOff
                  0x038fc4                  _actionAutoOffReset
                  0x039032                  _actionAutoOffWatch
                  0x039136                  _actionInitToOffForIO
                  0x039190                  _actionInitToOffForIOcmd
 .text            0x03929c       0x24cc build/XC16-EX16_MRF24WB/production/_ext/1954962658/TCP.o
                  0x039362                  _TCPInit
                  0x039452                  _TCPOpen
                  0x0395ae                  _TCPWasReset
                  0x0395dc                  _TCPIsConnected
                  0x039600                  _TCPDisconnect
                  0x0396a0                  _TCPClose
                  0x0396c0                  _TCPGetRemoteInfo
                  0x0396ea                  _TCPFlush
                  0x039710                  _TCPIsPutReady
                  0x03975e                  _TCPPut
                  0x039804                  _TCPPutArray
                  0x0398ea                  _TCPPutString
                  0x03990e                  _TCPGetTxFIFOFull
                  0x03993a                  _TCPDiscard
                  0x03995a                  _TCPIsGetReady
                  0x039992                  _TCPGet
                  0x039a0c                  _TCPGetArray
                  0x039ad8                  _TCPGetRxFIFOFree
                  0x039b02                  _TCPPeekArray
                  0x039bac                  _TCPPeek
                  0x039bc4                  _TCPFindArrayEx
                  0x039e34                  _TCPFindEx
                  0x039e58                  _TCPTick
                  0x03a348                  _TCPProcess
                  0x03b554                  _TCPAdjustFIFOSize
                  0x03b756                  _GetTcbInfo
 .text            0x03b768       0x10fc build/XC16-EX16_MRF24WB/production/_ext/1472/WiSteerTime.o
                  0x03b768                  _wstimeEncode
                  0x03b96e                  _wstimeDecode
                  0x03bb62                  _wstimeMonthLength
                  0x03bbe6                  _wstimeWeekDay
                  0x03bc16                  _wstimeStToStr
                  0x03bfa8                  _wstimeToStr
                  0x03bfdc                  _wstimeStr
                  0x03c00e                  _wstickStr
                  0x03c0c8                  _wstimeLowGet
                  0x03c0e2                  _wstimeSet
                  0x03c14c                  _wstimeGet
                  0x03c160                  _ntpServerPort
                  0x03c16c                  _ntpServer
                  0x03c1ca                  _ntpTimeRecv
                  0x03c214                  _tzInfoIsUtc
                  0x03c23c                  _tzInfoHasDayLight
                  0x03c25c                  _tzInfoMakeDate
                  0x03c3c0                  _wstimeStDiff
                  0x03c47c                  _tzInfoToLocalTime
                  0x03c634                  _tzInfoToUtcTime
                  0x03c73e                  _timeBiasStr
                  0x03c7ae                  _timeBiasFromStr
 .text            0x03c864        0xc60 build/XC16-EX16_MRF24WB/production/_ext/1954962658/DHCP.o
                  0x03c864                  _DHCPInit
                  0x03c8c0                  _DHCPDisable
                  0x03c8e4                  _DHCPEnable
                  0x03c904                  _DHCPIsEnabled
                  0x03c918                  _DHCPIsBound
                  0x03c928                  _DHCPStateChanged
                  0x03c946                  _DHCPIsServerDetected
                  0x03c958                  _DHCPTempIPAddr
                  0x03c99a                  _DHCPTask
 .text            0x03d4c4        0xc26 build/XC16-EX16_MRF24WB/production/_ext/1472/MPFS2.o
                  0x03d4c4                  _MPFSInit
                  0x03d4f8                  _MPFSOpen
                  0x03d64e                  _MPFSOpenID
                  0x03d6d8                  _MPFSClose
                  0x03d6fe                  _MPFSGet
                  0x03d88e                  _MPFSGetArray
                  0x03dab8                  _MPFSGetLong
                  0x03dada                  _MPFSSeek
                  0x03dcec                  _MPFSGetTimestamp
                  0x03dd32                  _MPFSGetContentTypeId
                  0x03ddb8                  _MPFSGetContentType
                  0x03de14                  _MPFSGetFlags
                  0x03de58                  _MPFSGetSize
                  0x03de9e                  _MPFSGetBytesRem
                  0x03dedc                  _MPFSGetPhysAddr
                  0x03df22                  _MPFSGetStartAddr
                  0x03df6a                  _MPFSGetEndAddr
                  0x03dfbc                  _MPFSGetFilename
                  0x03e020                  _MPFSGetPosition
                  0x03e05c                  _MPFSGetID
                  0x03e0cc                  _MPFSseekInit
                  0x03e0da                  _MPFSputHdrCorrect
                  0x03e0e0                  _MPFSLocked
 .text            0x03e0ea        0xb40 build/XC16-EX16_MRF24WB/production/_ext/1954962658/DHCPs.o
                  0x03e0ea                  _DHCPServerTask
                  0x03ebf8                  _DHCPServer_Disable
                  0x03ec1a                  _DHCPServer_Enable
 .text            0x03ec2a        0xa78 build/XC16-EX16_MRF24WB/production/_ext/243675038/WFMac.o
                  0x03ee32                  _MACProcess
                  0x03ee70                  _WFGetTCBSize
                  0x03ee7a                  _MACInit
                  0x03ee84                  _RawInit
                  0x03eed6                  _MACIsLinked
                  0x03eee4                  _MACIsTxReady
                  0x03ef3a                  _WFisTxMgmtReady
                  0x03ef74                  _WFFreeMgmtTx
                  0x03efa8                  _SendRAWManagementFrame
                  0x03efb8                  _RawGetMgmtRxBuffer
                  0x03effa                  _SetRawRxMgmtInProgress
                  0x03f012                  _isRawRxMgmtInProgress
                  0x03f01c                  _MACDiscardRx
                  0x03f026                  _MACGetFreeRxSize
                  0x03f0a0                  _MACGetHeader
                  0x03f194                  _MACPutHeader
                  0x03f1ec                  _MACFlush
                  0x03f252                  _MACSetReadPtrInRx
                  0x03f264                  _MACSetWritePtr
                  0x03f27c                  _MACSetReadPtr
                  0x03f294                  _MACCalcRxChecksum
                  0x03f2c2                  _MACMemCopyAsync
                  0x03f518                  _MACIsMemCopyDone
                  0x03f522                  _MACGet
                  0x03f54e                  _MACGetArray
                  0x03f5a8                  _MACPut
                  0x03f5d6                  _MACPutArray
                  0x03f604                  _CalcIPBufferChecksum
                  0x03f696                  _MACPowerDown
                  0x03f69c                  _MACPowerUp
 .text            0x03f6a2        0x8b4 build/XC16-EX16_MRF24WB/production/_ext/1954962658/Helpers.o
                  0x03f6a2                  _LFSRSeedRand
                  0x03f6e4                  _LFSRRand
                  0x03f754                  _GenerateRandomDWORD
                  0x03f85e                  _StringToIPAddress
                  0x03f9d0                  _Base64Decode
                  0x03fb38                  _uitoa
                  0x03fbc2                  _hexatob
                  0x03fc2c                  _btohexa_high
                  0x03fc4e                  _btohexa_low
                  0x03fc6c                  _stricmppgm2ram
                  0x03fd04                  _swaps
                  0x03fd20                  _swapl
                  0x03fd80                  _CalcIPChecksum
                  0x03fe02                  _strupr
                  0x03fe40                  _FormatNetBIOSName
                  0x03fe8a                  _strnchr
                  0x03fed8                  _strncpy_m
 .text            0x03ff56        0x896 build/XC16-EX16_MRF24WB/production/_ext/1954962658/DNS.o
                  0x03ff56                  _DNSBeginUsage
                  0x03ff76                  _DNSEndUsage
                  0x03ffae                  _DNSResolve
                  0x03ffee                  _DNSIsResolved
 .text            0x0407ec        0x86e build/XC16-EX16_MRF24WB/production/_ext/1472/WiSteerLog.o
                  0x0407ec                  _wslog
                  0x0409e6                  _wsvlogf
                  0x040a08                  _wslogf
                  0x040b3a                  _wslogReset
                  0x040b5a                  _wslogWrite
                  0x040f38                  _wslogEnum
                  0x040fcc                  _wslogSeekNext
                  0x04100a                  _wslogTimeAdjust
                  0x041034                  _wslogTimeAdjustRestart
                  0x041040                  _logFatalCheckPt
 .text            0x04105a        0x81a build/XC16-EX16_MRF24WB/production/_ext/1954962658/UDP.o
                  0x04105a                  _UDPInit
                  0x04107a                  _UDPOpenEx
                  0x041194                  _UDPTask
                  0x0413d4                  _UDPIsOpened
                  0x0413f6                  _UDPClose
                  0x04144e                  _UDPSetTxBuffer
                  0x041464                  _UDPSetRxBuffer
                  0x04147a                  _UDPIsPutReady
                  0x0414b0                  _UDPPut
                  0x0414e0                  _UDPPutArray
                  0x04151c                  _UDPPutString
                  0x04153a                  _UDPFlush
                  0x0415a8                  _UDPIsGetReady
                  0x0415de                  _UDPGet
                  0x041612                  _UDPGetArray
                  0x04165e                  _UDPDiscard
                  0x041684                  _UDPDiscardRxTx
                  0x041698                  _UDPProcess
 .text            0x041874        0x6d4 build/XC16-EX16_MRF24WB/production/_ext/1472/WiSteerHTTPtools.o
                  0x041874                  _HTTPExecuteGet
                  0x04187e                  _HTTPExecutePost
                  0x0418fc                  _HTTPPrint_tooMuchData
                  0x041922                  _HTTPPrint_out
                  0x04193c                  _HTTPPrint_outLen
                  0x041a8a                  _HTTPPrint_jsEscape
                  0x041aa4                  _HTTPPrint_jsEscapeLen
                  0x041c0a                  _HTTPPrint_htmlEscape
                  0x041c24                  _HTTPPrint_htmlEscapeLen
                  0x041dfa                  _HTTPPrint_postJSf
                  0x041e18                  _HTTPPrintTry_postJSf
                  0x041e3a                  _HTTPPrint_postJS
                  0x041e66                  _HTTPPrintTry_postJS
                  0x041eee                  _HTTPPrint_postErrorField
                  0x041f06                  _HTTPPrint_postErrorFieldArg1
                  0x041f24                  _HTTPPrint_postErrorFieldArg2
 .text            0x041f48        0x478 build/XC16-EX16_MRF24WB/production/_ext/1954962658/Hashes.o
                  0x041f48                  _HashAddData
                  0x041f64                  _MD5Initialize
                  0x041fa0                  _MD5AddData
                  0x042240                  _MD5Calculate
 .text            0x0423c0        0x452 build/XC16-EX16_MRF24WB/production/_ext/243675038/WFConnectionAlgorithm.o
                  0x0423c0                  _WF_CASetElements
                  0x04247e                  _WF_CASetElementsN
                  0x0424b6                  _WF_CAGetElements
                  0x042502                  _WF_CASetScanType
                  0x042512                  _WF_CAGetScanType
                  0x042524                  _WF_CASetMinChannelTime
                  0x042540                  _WF_CAGetMinChannelTime
                  0x042562                  _WF_CASetMaxChannelTime
                  0x04257e                  _WF_CAGetMaxChannelTime
                  0x0425a0                  _WF_CASetProbeDelay
                  0x0425bc                  _WF_CAGetProbeDelay
                  0x0425de                  _WF_CASetScanCount
                  0x0425ee                  _WF_CAGetScanCount
                  0x042600                  _WF_CASetRssi
                  0x042610                  _WF_CAGetRssi
                  0x042622                  _WF_CASetConnectionProfileList
                  0x042632                  _WF_CAGetConnectionProfileList
                  0x042642                  _WF_CASetListRetryCount
                  0x042652                  _WF_CAGetListRetryCount
                  0x042664                  _WF_CASetEventNotificationAction
                  0x042670                  _WF_CAGetEventNotificationAction
                  0x042680                  _WF_CASetBeaconTimeoutAction
                  0x042690                  _WF_CAGetBeaconTimeoutAction
                  0x0426a2                  _WF_CASetDeauthAction
                  0x0426b2                  _WF_CAGetDeauthAction
                  0x0426c4                  _WF_CASetChannelList
                  0x0426d6                  _WF_CAGetChannelList
                  0x042712                  _WF_CASetListenInterval
                  0x04272e                  _WF_CAGetListenInterval
                  0x042750                  _WF_CASetBeaconTimeout
                  0x042760                  _WF_CAGetBeaconTimeout
                  0x04277e                  _GetEventNotificationMask
                  0x042800                  _WF_DisableModuleConnectionManager

.dinit            0x042812        0x452
 .dinit           0x042812        0x452 data_init

.text             0x042c64       0x3bd4
 .text            0x042c64        0x44e build/XC16-EX16_MRF24WB/production/_ext/243675038/WFDriverCom.o
                  0x042c64                  _WiFiTask
                  0x042c74                  _SignalDHCPSuccessful
                  0x042c82                  _SetDhcpProgressState
                  0x042c8c                  _SignalWiFiConnectionChanged
                  0x042c9c                  _WFProcess
                  0x042d4e                  _Read8BitWFRegister
                  0x042d78                  _Write8BitWFRegister
                  0x042da0                  _Read16BitWFRegister
                  0x042dd6                  _Write16BitWFRegister
                  0x042e0a                  _WriteWFArray
                  0x042e3a                  _ReadWFArray
                  0x042f9e                  _WFEintHandler
                  0x04303e                  _ReenablePowerSaveMode
                  0x043044                  _WFHardwareInit
 .text            0x0430b2        0x448 build/XC16-EX16_MRF24WB/production/_ext/243675038/WFDriverRaw.o
                  0x0430b2                  _AllocateMgmtTxBuffer
                  0x0430f8                  _DeallocateMgmtRxBuffer
                  0x043112                  _AllocateDataTxBuffer
                  0x043158                  _DeallocateDataTxBuffer
                  0x043172                  _DeallocateDataRxBuffer
                  0x043182                  _RawSendTxBuffer
                  0x04319e                  _RawMountRxBuffer
                  0x0431c0                  _RawToRawCopy
                  0x0431d8                  _PushRawWindow
                  0x0431ee                  _PopRawWindow
                  0x04320c                  _ScratchMount
                  0x043246                  _ScratchUnmount
                  0x043270                  _RawRead
                  0x043294                  _RawWrite
                  0x043326                  _RawSetIndex
                  0x04339c                  _RawGetIndex
                  0x0433c0                  _RawGetByte
                  0x043406                  _RawSetByte
                  0x0434dc                  _SendRAWDataFrame
 .text            0x0434fa        0x3d6 build/XC16-EX16_MRF24WB/production/_ext/243675038/WFEasyConfig.o
                  0x0434fa                  _WFEasyConfigInit
                  0x043530                  _WFEasyConfigMgr
                  0x0436e2                  _WFInitScan
                  0x0436f6                  _WFStartScan
                  0x043734                  _WFRetrieveScanResult
                  0x043770                  _WFScanEventHandler
                  0x043792                  _WFGetScanResults
                  0x043806                  _WFDisplayScanMgr
 .text            0x0438d0        0x3ae build/XC16-EX16_MRF24WB/production/_ext/1954962658/NBNS.o
                  0x0438d0                  _NBNSTask
 .text            0x043c7e        0x3a8 build/XC16-EX16_MRF24WB/production/_ext/1954962658/ARP.o
                  0x043c7e                  _ARPSendPkt
                  0x043d52                  _ARPInit
                  0x043d84                  _ARPProcess
                  0x043e5c                  _ARPResolve
                  0x043f26                  _ARPIsResolved
                  0x043fee                  _SwapARPPacket
 .text            0x044026        0x398 build/XC16-EX16_MRF24WB/production/_ext/1954962658/StackTsk.o
                  0x044026                  _dhcpConnectOk
                  0x044052                  _StackInit
                  0x0440b2                  _StackTask
                  0x04438e                  _StackApplications
                  0x0443b0                  _RenewDhcp
 .text            0x0443be        0x38a build/XC16-EX16_MRF24WB/production/_ext/1954962658/SPIEEPROM.o
                  0x0443be                  _XEEInit
                  0x0443dc                  _XEEBeginRead
                  0x0443f4                  _XEERead
                  0x04443a                  _XEEEndRead
                  0x044444                  _XEEReadArray
                  0x044526                  _XEEBeginWrite
                  0x04453e                  _XEEWrite
                  0x044584                  _XEEWriteArray
                  0x0445b2                  _XEEEndWrite
                  0x0446d0                  _XEEIsBusy
 .text            0x044748        0x386 build/XC16-EX16_MRF24WB/production/_ext/243675038/WFConnectionProfile.o
                  0x044748                  _WF_CPCreate
                  0x044776                  _WF_CPDelete
                  0x04479c                  _WF_CPGetIds
                  0x0447c4                  _WF_CPSetElements
                  0x0447f8                  _WF_CPGetElements
                  0x044810                  _WF_CPSetSsidType
                  0x044826                  _WF_CPGetSsidType
                  0x04483c                  _WF_CPSetSsid
                  0x044862                  _WF_CPGetSsid
                  0x0448a2                  _WF_CPSetBssid
                  0x0448b6                  _WF_CPGetBssid
                  0x0448cc                  _WF_CPSetNetworkType
                  0x0448e2                  _WF_CPGetNetworkType
                  0x0448f8                  _WF_CPSetWepKeyType
                  0x04490e                  _WF_CPGetWepKeyType
                  0x044924                  _WF_CPSetSecurity
                  0x04498c                  _WF_CPGetSecurity
                  0x0449f8                  _WF_CPSetDefaultWepKeyIndex
                  0x044a0e                  _WF_CPGetDefaultWepKeyIndex
                  0x044a24                  _WF_CPSetAdHocBehavior
                  0x044a3a                  _WF_CPGetAdHocBehavior
 .text            0x044ace        0x2f2 build/XC16-EX16_MRF24WB/production/_ext/243675038/WFParamMsg.o
                  0x044ace                  _WFEnableMRF24WB0MMode
                  0x044ae0                  _WFEnableBroadcastProbeResponse
                  0x044af2                  _WF_SetLinkDownThreshold
                  0x044b02                  _WFEnableDeferredPowerSave
                  0x044b14                  _WF_GetDeviceInfo
                  0x044b36                  _WF_SetMacAddress
                  0x044b46                  _WF_GetMacAddress
                  0x044b56                  _WF_SetMultiCastFilter
                  0x044bc4                  _WF_GetMultiCastFilter
                  0x044c2a                  _WF_SetTxDataConfirm
                  0x044c3a                  _WF_GetTxDataConfirm
                  0x044c4a                  _WF_SetRegionalDomain
                  0x044c5a                  _WF_GetRegionalDomain
                  0x044c6a                  _WF_SetRtsThreshold
                  0x044c96                  _WF_GetRtsThreshold
                  0x044cb6                  _WF_GetMacStats
                  0x044d5c                  _SendSetParamMsg
                  0x044d8c                  _SendGetParamMsg
 .text            0x044dc0        0x2e0 build/XC16-EX16_MRF24WB/production/_ext/1472/WF_Config.o
                  0x044dc0                  _WF_ProcessEvent
                  0x044f14                  __wifiConnectOk
                  0x044f3a                  _wifiConnectOk
                  0x044f46                  _wifiDhcpOk
                  0x044f4e                  _wifiConnectError
                  0x044f80                  _wifiConnectCheck
                  0x044fe0                  _wifiConnectRetry
 .text            0x0450a0        0x2de build/XC16-EX16_MRF24WB/production/_ext/1954962658/DNSs.o
                  0x0450a0                  _DNSServerTask
 .text            0x04537e        0x26a build/XC16-EX16_MRF24WB/production/_ext/1954962658/SNTP.o
                  0x04537e                  _SNTPClientRestart
                  0x045398                  _SNTPClient
                  0x045596                  _SNTPGetUTCSeconds
 .text            0x0455e8        0x21a build/XC16-EX16_MRF24WB/production/_ext/1954962658/IP.o
                  0x0455e8                  _IPGetHeader
                  0x045702                  _IPPutHeader
                  0x0457b4                  _IPSetRxBuffer
 .text            0x045802        0x214 build/XC16-EX16_MRF24WB/production/_ext/243675038/WFEventHandler.o
                  0x045802                  _WFProcessMgmtIndicateMsg
 .text            0x045a16        0x1f6 build/XC16-EX16_MRF24WB/production/_ext/243675038/WFMgmtMsg.o
                  0x045a16                  _SendMgmtMsg
                  0x045aba                  _SignalMgmtConfirmReceivedEvent
                  0x045ac4                  _WaitForMgmtResponse
                  0x045b68                  _WaitForMgmtResponseAndReadData
                  0x045be2                  _WFSetFuncState
 .text            0x045c0c        0x1b6 build/XC16-EX16_MRF24WB/production/_ext/1954962658/LCDBlocking.o
                  0x045c54                  _LCDInit
                  0x045ce2                  _LCDUpdate
                  0x045da6                  _LCDErase
 .text            0x045dc2        0x186 build/XC16-EX16_MRF24WB/production/_ext/1954962658/Tick.o
                  0x045dc2                  _TickInit
                  0x045e6c                  _TickGet
                  0x045e9e                  _TickGetDiv256
                  0x045ed0                  _TickGetDiv64K
                  0x045f02                  _TickConvertToMilliseconds
                  0x045f30                  __T1Interrupt
 .text            0x045f48        0x160 build/XC16-EX16_MRF24WB/production/_ext/243675038/WFConnectionManager.o
                  0x045f48                  _WF_CMConnect
                  0x045f96                  _WF_CMDisconnect
                  0x045fcc                  _WF_CMGetConnectionState
                  0x04601e                  _WFisConnected
                  0x046028                  _SetLogicalConnectionState
                  0x046034                  _WF_CMCheckConnectionState
                  0x04606c                  _WF_ConvPassphrase2Key
 .text            0x0460a8        0x144 build/XC16-EX16_MRF24WB/production/_ext/243675038/WFDebugStrings.o
                  0x04610c                  _WF_OutputConnectionDebugMsg
                  0x0461b2                  _WF_OutputConnectionInfo
                  0x0461ba                  _WF_AssertionFailed
 .text            0x0461ec         0xde build/XC16-EX16_MRF24WB/production/_ext/243675038/WFTxPower.o
                  0x0461ec                  _WF_TxPowerSetMinMax
                  0x046250                  _WF_TxPowerGetMinMax
                  0x046292                  _WF_FixTxRateWithMaxPower
                  0x0462b2                  _WF_TxPowerGetFactoryMax
 .text            0x0462ca         0xca build/XC16-EX16_MRF24WB/production/_ext/243675038/WFConsoleMsgs.o
                  0x0462ca                  _ConvertASCIIHexToBinary
                  0x04635a                  _HexToBin
 .text            0x046394         0xc8 build/XC16-EX16_MRF24WB/production/_ext/243675038/WFScan.o
                  0x0463b8                  _WF_Scan
                  0x04640c                  _WF_ScanGetResult
 .text            0x04645c         0xac build/XC16-EX16_MRF24WB/production/_ext/243675038/WF_Spi.o
                  0x04645c                  _WF_SpiInit
                  0x04647c                  _WF_SpiEnableChipSelect
                  0x046484                  _WF_SpiDisableChipSelect
                  0x04648e                  _WFSpiTxRx
 .text            0x046508         0xa6 build/XC16-EX16_MRF24WB/production/_ext/243675038/WF_Eint.o
                  0x046508                  _WF_EintIsDisabled
                  0x04651e                  _WF_EintIsPending
                  0x046540                  __INT3Interrupt
                  0x046580                  _WF_EintEnable
                  0x046594                  _WF_EintDisable
                  0x04659c                  _WF_EintInit
 .text            0x0465ae         0x94 build/XC16-EX16_MRF24WB/production/_ext/1954962658/ICMP.o
                  0x0465ae                  _ICMPProcess
 .text            0x046642         0x8c build/XC16-EX16_MRF24WB/production/_ext/243675038/WFConsoleMsgHandler.o
                  0x046642                  _convertAsciiToHexInPlace
 .text            0x0466ce         0x7e build/XC16-EX16_MRF24WB/production/_ext/243675038/WFInit.o
                  0x0466ce                  _WF_Init
 .text            0x04674c         0x78 build/XC16-EX16_MRF24WB/production/_ext/1954962658/Delay.o
                  0x04674c                  _DelayMs
                  0x046788                  _Delay10us
 .text            0x0467c4         0x74 build/XC16-EX16_MRF24WB/production/WiSteerUpdateHlp.o
                  0x0467c4                  _WriteMem
                  0x0467e6                  _WriteLatch
                  0x0467ee                  _ReadLatchLo
                  0x0467fe                  _ReadLatchHi
                  0x04680e                  _ErasePage

MPFSHelpers       0x046838          0xe
 MPFSHelpers      0x046838          0xe build/XC16-EX16_MRF24WB/production/_ext/1472/WiSteerMpfsSource.o
                  0x046838                  _ReadProgramMemory

.text             0x046846          0x6
 .text            0x046846          0x6 build/XC16-EX16_MRF24WB/production/_ext/1472/WiSteerStructSizeCheck.o
                  0x046846                  _WiSteerStructCheck
